Archive member included because of file (symbol)

c:/program files/microchip/xc32/v1.33/bin/bin/../../lib/gcc/pic32mx/4.5.2/../../../../pic32mx/lib\libmchp_peripheral_32MX795F512H.a(soft_reset_lib.o)
                              build/ChaletDuinoV2_775F512H_/debug/Source/exceptions.o (SoftReset)
c:/program files/microchip/xc32/v1.33/bin/bin/../../lib/gcc/pic32mx/4.5.2/../../../../pic32mx/lib\libmchp_peripheral_32MX795F512H.a(pcache.o)
                              build/ChaletDuinoV2_775F512H_/debug/Source/main.o (CheKseg0CacheOn)
c:/program files/microchip/xc32/v1.33/bin/bin/../../lib/gcc/pic32mx/4.5.2/../../../../pic32mx/lib\libmchp_peripheral_32MX795F512H.a(int_configure_system_lib.o)
                              build/ChaletDuinoV2_775F512H_/debug/Source/main.o (INTConfigureSystem)
c:/program files/microchip/xc32/v1.33/bin/bin/../../lib/gcc/pic32mx/4.5.2/../../../../pic32mx/lib\libmchp_peripheral_32MX795F512H.a(int_enable_interrupts_lib.o)
                              build/ChaletDuinoV2_775F512H_/debug/Source/main.o (INTEnableInterrupts)
c:/program files/microchip/xc32/v1.33/bin/bin/../../lib/gcc/pic32mx/4.5.2/../../../../pic32mx/lib\libmchp_peripheral_32MX795F512H.a(int_disable_interrupts_lib.o)
                              build/ChaletDuinoV2_775F512H_/debug/Source/main.o (INTDisableInterrupts)
c:/program files/microchip/xc32/v1.33/bin/bin/../../lib/gcc/pic32mx/4.5.2/../../../../pic32mx/lib\libmchp_peripheral_32MX795F512H.a(int_restore_interrupts_lib.o)
                              build/ChaletDuinoV2_775F512H_/debug/Source/main.o (INTRestoreInterrupts)
c:/program files/microchip/xc32/v1.33/bin/bin/../../lib/gcc/pic32mx/4.5.2/../../../../pic32mx/lib\libpic32.a(memcpy.o)
                              build/ChaletDuinoV2_775F512H_/debug/Source/NetworkProtocol.o (memcpy)
c:/program files/microchip/xc32/v1.33/bin/bin/../../lib/gcc/pic32mx/4.5.2/../../../../pic32mx/lib\libpic32.a(memset.o)
                              build/ChaletDuinoV2_775F512H_/debug/Source/winc3400/winc_init.o (memset)
c:/program files/microchip/xc32/v1.33/bin/bin/../../lib/gcc/pic32mx/4.5.2/../../../../pic32mx/lib\libpic32.a(strcpy.o)
                              build/ChaletDuinoV2_775F512H_/debug/Source/Terminal.o (strcpy)
c:/program files/microchip/xc32/v1.33/bin/bin/../../lib/gcc/pic32mx/4.5.2/../../../../pic32mx/lib\libpic32.a(strlen.o)
                              build/ChaletDuinoV2_775F512H_/debug/Source/Terminal.o (strlen)
c:/program files/microchip/xc32/v1.33/bin/bin/../../lib/gcc/pic32mx/4.5.2/../../../../pic32mx/lib\libpic32.a(default-bootstrap-exception-handler.o)
                              c:/program files/microchip/xc32/v1.33/bin/bin/../../lib/gcc/pic32mx/4.5.2/../../../../pic32mx/lib/./proc/32MX795F512H/crt0_mips32r2.o (_bootstrap_exception_handler)
c:/program files/microchip/xc32/v1.33/bin/bin/../../lib/gcc/pic32mx/4.5.2/../../../../pic32mx/lib\libpic32.a(default-on-reset.o)
                              c:/program files/microchip/xc32/v1.33/bin/bin/../../lib/gcc/pic32mx/4.5.2/../../../../pic32mx/lib/./proc/32MX795F512H/crt0_mips32r2.o (_on_reset)
c:/program files/microchip/xc32/v1.33/bin/bin/../../lib/gcc/pic32mx/4.5.2/../../../../pic32mx/lib\libpic32.a(default-on-bootstrap.o)
                              c:/program files/microchip/xc32/v1.33/bin/bin/../../lib/gcc/pic32mx/4.5.2/../../../../pic32mx/lib/./proc/32MX795F512H/crt0_mips32r2.o (_on_bootstrap)
c:/program files/microchip/xc32/v1.33/bin/bin/../../lib/gcc/pic32mx/4.5.2/../../../../pic32mx/lib\libpic32.a(default-nmi-handler.o)
                              c:/program files/microchip/xc32/v1.33/bin/bin/../../lib/gcc/pic32mx/4.5.2/../../../../pic32mx/lib/./proc/32MX795F512H/crt0_mips32r2.o (_nmi_handler)
c:/program files/microchip/xc32/v1.33/bin/bin/../../lib/gcc/pic32mx/4.5.2/../../../../pic32mx/lib\libpic32.a(general-exception.o)
                              c:/program files/microchip/xc32/v1.33/bin/bin/../../lib/gcc/pic32mx/4.5.2/../../../../pic32mx/lib/./proc/32MX795F512H/crt0_mips32r2.o (_general_exception_context)
c:/program files/microchip/xc32/v1.33/bin/bin/../../lib/gcc/pic32mx/4.5.2/../../../../pic32mx/lib\libpic32.a(vector0.o)
                              c:/program files/microchip/xc32/v1.33/bin/bin/../../lib/gcc/pic32mx/4.5.2/../../../../pic32mx/lib/./proc/32MX795F512H\default_isr_vectors.o (__vector_dispatch_0)
c:/program files/microchip/xc32/v1.33/bin/bin/../../lib/gcc/pic32mx/4.5.2/../../../../pic32mx/lib\libpic32.a(vector1.o)
                              c:/program files/microchip/xc32/v1.33/bin/bin/../../lib/gcc/pic32mx/4.5.2/../../../../pic32mx/lib/./proc/32MX795F512H\default_isr_vectors.o (__vector_dispatch_1)
c:/program files/microchip/xc32/v1.33/bin/bin/../../lib/gcc/pic32mx/4.5.2/../../../../pic32mx/lib\libpic32.a(vector2.o)
                              c:/program files/microchip/xc32/v1.33/bin/bin/../../lib/gcc/pic32mx/4.5.2/../../../../pic32mx/lib/./proc/32MX795F512H\default_isr_vectors.o (__vector_dispatch_2)
c:/program files/microchip/xc32/v1.33/bin/bin/../../lib/gcc/pic32mx/4.5.2/../../../../pic32mx/lib\libpic32.a(vector5.o)
                              c:/program files/microchip/xc32/v1.33/bin/bin/../../lib/gcc/pic32mx/4.5.2/../../../../pic32mx/lib/./proc/32MX795F512H\default_isr_vectors.o (__vector_dispatch_5)
c:/program files/microchip/xc32/v1.33/bin/bin/../../lib/gcc/pic32mx/4.5.2/../../../../pic32mx/lib\libpic32.a(vector6.o)
                              c:/program files/microchip/xc32/v1.33/bin/bin/../../lib/gcc/pic32mx/4.5.2/../../../../pic32mx/lib/./proc/32MX795F512H\default_isr_vectors.o (__vector_dispatch_6)
c:/program files/microchip/xc32/v1.33/bin/bin/../../lib/gcc/pic32mx/4.5.2/../../../../pic32mx/lib\libpic32.a(vector7.o)
                              c:/program files/microchip/xc32/v1.33/bin/bin/../../lib/gcc/pic32mx/4.5.2/../../../../pic32mx/lib/./proc/32MX795F512H\default_isr_vectors.o (__vector_dispatch_7)
c:/program files/microchip/xc32/v1.33/bin/bin/../../lib/gcc/pic32mx/4.5.2/../../../../pic32mx/lib\libpic32.a(vector8.o)
                              c:/program files/microchip/xc32/v1.33/bin/bin/../../lib/gcc/pic32mx/4.5.2/../../../../pic32mx/lib/./proc/32MX795F512H\default_isr_vectors.o (__vector_dispatch_8)
c:/program files/microchip/xc32/v1.33/bin/bin/../../lib/gcc/pic32mx/4.5.2/../../../../pic32mx/lib\libpic32.a(vector9.o)
                              c:/program files/microchip/xc32/v1.33/bin/bin/../../lib/gcc/pic32mx/4.5.2/../../../../pic32mx/lib/./proc/32MX795F512H\default_isr_vectors.o (__vector_dispatch_9)
c:/program files/microchip/xc32/v1.33/bin/bin/../../lib/gcc/pic32mx/4.5.2/../../../../pic32mx/lib\libpic32.a(vector10.o)
                              c:/program files/microchip/xc32/v1.33/bin/bin/../../lib/gcc/pic32mx/4.5.2/../../../../pic32mx/lib/./proc/32MX795F512H\default_isr_vectors.o (__vector_dispatch_10)
c:/program files/microchip/xc32/v1.33/bin/bin/../../lib/gcc/pic32mx/4.5.2/../../../../pic32mx/lib\libpic32.a(vector11.o)
                              c:/program files/microchip/xc32/v1.33/bin/bin/../../lib/gcc/pic32mx/4.5.2/../../../../pic32mx/lib/./proc/32MX795F512H\default_isr_vectors.o (__vector_dispatch_11)
c:/program files/microchip/xc32/v1.33/bin/bin/../../lib/gcc/pic32mx/4.5.2/../../../../pic32mx/lib\libpic32.a(vector12.o)
                              c:/program files/microchip/xc32/v1.33/bin/bin/../../lib/gcc/pic32mx/4.5.2/../../../../pic32mx/lib/./proc/32MX795F512H\default_isr_vectors.o (__vector_dispatch_12)
c:/program files/microchip/xc32/v1.33/bin/bin/../../lib/gcc/pic32mx/4.5.2/../../../../pic32mx/lib\libpic32.a(vector13.o)
                              c:/program files/microchip/xc32/v1.33/bin/bin/../../lib/gcc/pic32mx/4.5.2/../../../../pic32mx/lib/./proc/32MX795F512H\default_isr_vectors.o (__vector_dispatch_13)
c:/program files/microchip/xc32/v1.33/bin/bin/../../lib/gcc/pic32mx/4.5.2/../../../../pic32mx/lib\libpic32.a(vector14.o)
                              c:/program files/microchip/xc32/v1.33/bin/bin/../../lib/gcc/pic32mx/4.5.2/../../../../pic32mx/lib/./proc/32MX795F512H\default_isr_vectors.o (__vector_dispatch_14)
c:/program files/microchip/xc32/v1.33/bin/bin/../../lib/gcc/pic32mx/4.5.2/../../../../pic32mx/lib\libpic32.a(vector15.o)
                              c:/program files/microchip/xc32/v1.33/bin/bin/../../lib/gcc/pic32mx/4.5.2/../../../../pic32mx/lib/./proc/32MX795F512H\default_isr_vectors.o (__vector_dispatch_15)
c:/program files/microchip/xc32/v1.33/bin/bin/../../lib/gcc/pic32mx/4.5.2/../../../../pic32mx/lib\libpic32.a(vector16.o)
                              c:/program files/microchip/xc32/v1.33/bin/bin/../../lib/gcc/pic32mx/4.5.2/../../../../pic32mx/lib/./proc/32MX795F512H\default_isr_vectors.o (__vector_dispatch_16)
c:/program files/microchip/xc32/v1.33/bin/bin/../../lib/gcc/pic32mx/4.5.2/../../../../pic32mx/lib\libpic32.a(vector17.o)
                              c:/program files/microchip/xc32/v1.33/bin/bin/../../lib/gcc/pic32mx/4.5.2/../../../../pic32mx/lib/./proc/32MX795F512H\default_isr_vectors.o (__vector_dispatch_17)
c:/program files/microchip/xc32/v1.33/bin/bin/../../lib/gcc/pic32mx/4.5.2/../../../../pic32mx/lib\libpic32.a(vector18.o)
                              c:/program files/microchip/xc32/v1.33/bin/bin/../../lib/gcc/pic32mx/4.5.2/../../../../pic32mx/lib/./proc/32MX795F512H\default_isr_vectors.o (__vector_dispatch_18)
c:/program files/microchip/xc32/v1.33/bin/bin/../../lib/gcc/pic32mx/4.5.2/../../../../pic32mx/lib\libpic32.a(vector19.o)
                              c:/program files/microchip/xc32/v1.33/bin/bin/../../lib/gcc/pic32mx/4.5.2/../../../../pic32mx/lib/./proc/32MX795F512H\default_isr_vectors.o (__vector_dispatch_19)
c:/program files/microchip/xc32/v1.33/bin/bin/../../lib/gcc/pic32mx/4.5.2/../../../../pic32mx/lib\libpic32.a(vector20.o)
                              c:/program files/microchip/xc32/v1.33/bin/bin/../../lib/gcc/pic32mx/4.5.2/../../../../pic32mx/lib/./proc/32MX795F512H\default_isr_vectors.o (__vector_dispatch_20)
c:/program files/microchip/xc32/v1.33/bin/bin/../../lib/gcc/pic32mx/4.5.2/../../../../pic32mx/lib\libpic32.a(vector21.o)
                              c:/program files/microchip/xc32/v1.33/bin/bin/../../lib/gcc/pic32mx/4.5.2/../../../../pic32mx/lib/./proc/32MX795F512H\default_isr_vectors.o (__vector_dispatch_21)
c:/program files/microchip/xc32/v1.33/bin/bin/../../lib/gcc/pic32mx/4.5.2/../../../../pic32mx/lib\libpic32.a(vector22.o)
                              c:/program files/microchip/xc32/v1.33/bin/bin/../../lib/gcc/pic32mx/4.5.2/../../../../pic32mx/lib/./proc/32MX795F512H\default_isr_vectors.o (__vector_dispatch_22)
c:/program files/microchip/xc32/v1.33/bin/bin/../../lib/gcc/pic32mx/4.5.2/../../../../pic32mx/lib\libpic32.a(vector23.o)
                              c:/program files/microchip/xc32/v1.33/bin/bin/../../lib/gcc/pic32mx/4.5.2/../../../../pic32mx/lib/./proc/32MX795F512H\default_isr_vectors.o (__vector_dispatch_23)
c:/program files/microchip/xc32/v1.33/bin/bin/../../lib/gcc/pic32mx/4.5.2/../../../../pic32mx/lib\libpic32.a(vector25.o)
                              c:/program files/microchip/xc32/v1.33/bin/bin/../../lib/gcc/pic32mx/4.5.2/../../../../pic32mx/lib/./proc/32MX795F512H\default_isr_vectors.o (__vector_dispatch_25)
c:/program files/microchip/xc32/v1.33/bin/bin/../../lib/gcc/pic32mx/4.5.2/../../../../pic32mx/lib\libpic32.a(vector26.o)
                              c:/program files/microchip/xc32/v1.33/bin/bin/../../lib/gcc/pic32mx/4.5.2/../../../../pic32mx/lib/./proc/32MX795F512H\default_isr_vectors.o (__vector_dispatch_26)
c:/program files/microchip/xc32/v1.33/bin/bin/../../lib/gcc/pic32mx/4.5.2/../../../../pic32mx/lib\libpic32.a(vector27.o)
                              c:/program files/microchip/xc32/v1.33/bin/bin/../../lib/gcc/pic32mx/4.5.2/../../../../pic32mx/lib/./proc/32MX795F512H\default_isr_vectors.o (__vector_dispatch_27)
c:/program files/microchip/xc32/v1.33/bin/bin/../../lib/gcc/pic32mx/4.5.2/../../../../pic32mx/lib\libpic32.a(vector28.o)
                              c:/program files/microchip/xc32/v1.33/bin/bin/../../lib/gcc/pic32mx/4.5.2/../../../../pic32mx/lib/./proc/32MX795F512H\default_isr_vectors.o (__vector_dispatch_28)
c:/program files/microchip/xc32/v1.33/bin/bin/../../lib/gcc/pic32mx/4.5.2/../../../../pic32mx/lib\libpic32.a(vector29.o)
                              c:/program files/microchip/xc32/v1.33/bin/bin/../../lib/gcc/pic32mx/4.5.2/../../../../pic32mx/lib/./proc/32MX795F512H\default_isr_vectors.o (__vector_dispatch_29)
c:/program files/microchip/xc32/v1.33/bin/bin/../../lib/gcc/pic32mx/4.5.2/../../../../pic32mx/lib\libpic32.a(vector30.o)
                              c:/program files/microchip/xc32/v1.33/bin/bin/../../lib/gcc/pic32mx/4.5.2/../../../../pic32mx/lib/./proc/32MX795F512H\default_isr_vectors.o (__vector_dispatch_30)
c:/program files/microchip/xc32/v1.33/bin/bin/../../lib/gcc/pic32mx/4.5.2/../../../../pic32mx/lib\libpic32.a(vector31.o)
                              c:/program files/microchip/xc32/v1.33/bin/bin/../../lib/gcc/pic32mx/4.5.2/../../../../pic32mx/lib/./proc/32MX795F512H\default_isr_vectors.o (__vector_dispatch_31)
c:/program files/microchip/xc32/v1.33/bin/bin/../../lib/gcc/pic32mx/4.5.2/../../../../pic32mx/lib\libpic32.a(vector33.o)
                              c:/program files/microchip/xc32/v1.33/bin/bin/../../lib/gcc/pic32mx/4.5.2/../../../../pic32mx/lib/./proc/32MX795F512H\default_isr_vectors.o (__vector_dispatch_33)
c:/program files/microchip/xc32/v1.33/bin/bin/../../lib/gcc/pic32mx/4.5.2/../../../../pic32mx/lib\libpic32.a(vector34.o)
                              c:/program files/microchip/xc32/v1.33/bin/bin/../../lib/gcc/pic32mx/4.5.2/../../../../pic32mx/lib/./proc/32MX795F512H\default_isr_vectors.o (__vector_dispatch_34)
c:/program files/microchip/xc32/v1.33/bin/bin/../../lib/gcc/pic32mx/4.5.2/../../../../pic32mx/lib\libpic32.a(vector35.o)
                              c:/program files/microchip/xc32/v1.33/bin/bin/../../lib/gcc/pic32mx/4.5.2/../../../../pic32mx/lib/./proc/32MX795F512H\default_isr_vectors.o (__vector_dispatch_35)
c:/program files/microchip/xc32/v1.33/bin/bin/../../lib/gcc/pic32mx/4.5.2/../../../../pic32mx/lib\libpic32.a(vector36.o)
                              c:/program files/microchip/xc32/v1.33/bin/bin/../../lib/gcc/pic32mx/4.5.2/../../../../pic32mx/lib/./proc/32MX795F512H\default_isr_vectors.o (__vector_dispatch_36)
c:/program files/microchip/xc32/v1.33/bin/bin/../../lib/gcc/pic32mx/4.5.2/../../../../pic32mx/lib\libpic32.a(vector37.o)
                              c:/program files/microchip/xc32/v1.33/bin/bin/../../lib/gcc/pic32mx/4.5.2/../../../../pic32mx/lib/./proc/32MX795F512H\default_isr_vectors.o (__vector_dispatch_37)
c:/program files/microchip/xc32/v1.33/bin/bin/../../lib/gcc/pic32mx/4.5.2/../../../../pic32mx/lib\libpic32.a(vector38.o)
                              c:/program files/microchip/xc32/v1.33/bin/bin/../../lib/gcc/pic32mx/4.5.2/../../../../pic32mx/lib/./proc/32MX795F512H\default_isr_vectors.o (__vector_dispatch_38)
c:/program files/microchip/xc32/v1.33/bin/bin/../../lib/gcc/pic32mx/4.5.2/../../../../pic32mx/lib\libpic32.a(vector39.o)
                              c:/program files/microchip/xc32/v1.33/bin/bin/../../lib/gcc/pic32mx/4.5.2/../../../../pic32mx/lib/./proc/32MX795F512H\default_isr_vectors.o (__vector_dispatch_39)
c:/program files/microchip/xc32/v1.33/bin/bin/../../lib/gcc/pic32mx/4.5.2/../../../../pic32mx/lib\libpic32.a(vector40.o)
                              c:/program files/microchip/xc32/v1.33/bin/bin/../../lib/gcc/pic32mx/4.5.2/../../../../pic32mx/lib/./proc/32MX795F512H\default_isr_vectors.o (__vector_dispatch_40)
c:/program files/microchip/xc32/v1.33/bin/bin/../../lib/gcc/pic32mx/4.5.2/../../../../pic32mx/lib\libpic32.a(vector41.o)
                              c:/program files/microchip/xc32/v1.33/bin/bin/../../lib/gcc/pic32mx/4.5.2/../../../../pic32mx/lib/./proc/32MX795F512H\default_isr_vectors.o (__vector_dispatch_41)
c:/program files/microchip/xc32/v1.33/bin/bin/../../lib/gcc/pic32mx/4.5.2/../../../../pic32mx/lib\libpic32.a(vector42.o)
                              c:/program files/microchip/xc32/v1.33/bin/bin/../../lib/gcc/pic32mx/4.5.2/../../../../pic32mx/lib/./proc/32MX795F512H\default_isr_vectors.o (__vector_dispatch_42)
c:/program files/microchip/xc32/v1.33/bin/bin/../../lib/gcc/pic32mx/4.5.2/../../../../pic32mx/lib\libpic32.a(vector43.o)
                              c:/program files/microchip/xc32/v1.33/bin/bin/../../lib/gcc/pic32mx/4.5.2/../../../../pic32mx/lib/./proc/32MX795F512H\default_isr_vectors.o (__vector_dispatch_43)
c:/program files/microchip/xc32/v1.33/bin/bin/../../lib/gcc/pic32mx/4.5.2/../../../../pic32mx/lib\libpic32.a(vector44.o)
                              c:/program files/microchip/xc32/v1.33/bin/bin/../../lib/gcc/pic32mx/4.5.2/../../../../pic32mx/lib/./proc/32MX795F512H\default_isr_vectors.o (__vector_dispatch_44)
c:/program files/microchip/xc32/v1.33/bin/bin/../../lib/gcc/pic32mx/4.5.2/../../../../pic32mx/lib\libpic32.a(vector45.o)
                              c:/program files/microchip/xc32/v1.33/bin/bin/../../lib/gcc/pic32mx/4.5.2/../../../../pic32mx/lib/./proc/32MX795F512H\default_isr_vectors.o (__vector_dispatch_45)
c:/program files/microchip/xc32/v1.33/bin/bin/../../lib/gcc/pic32mx/4.5.2/../../../../pic32mx/lib\libpic32.a(vector46.o)
                              c:/program files/microchip/xc32/v1.33/bin/bin/../../lib/gcc/pic32mx/4.5.2/../../../../pic32mx/lib/./proc/32MX795F512H\default_isr_vectors.o (__vector_dispatch_46)
c:/program files/microchip/xc32/v1.33/bin/bin/../../lib/gcc/pic32mx/4.5.2/../../../../pic32mx/lib\libpic32.a(vector47.o)
                              c:/program files/microchip/xc32/v1.33/bin/bin/../../lib/gcc/pic32mx/4.5.2/../../../../pic32mx/lib/./proc/32MX795F512H\default_isr_vectors.o (__vector_dispatch_47)
c:/program files/microchip/xc32/v1.33/bin/bin/../../lib/gcc/pic32mx/4.5.2/../../../../pic32mx/lib\libpic32.a(vector48.o)
                              c:/program files/microchip/xc32/v1.33/bin/bin/../../lib/gcc/pic32mx/4.5.2/../../../../pic32mx/lib/./proc/32MX795F512H\default_isr_vectors.o (__vector_dispatch_48)
c:/program files/microchip/xc32/v1.33/bin/bin/../../lib/gcc/pic32mx/4.5.2/../../../../pic32mx/lib\libpic32.a(vector49.o)
                              c:/program files/microchip/xc32/v1.33/bin/bin/../../lib/gcc/pic32mx/4.5.2/../../../../pic32mx/lib/./proc/32MX795F512H\default_isr_vectors.o (__vector_dispatch_49)
c:/program files/microchip/xc32/v1.33/bin/bin/../../lib/gcc/pic32mx/4.5.2/../../../../pic32mx/lib\libpic32.a(vector50.o)
                              c:/program files/microchip/xc32/v1.33/bin/bin/../../lib/gcc/pic32mx/4.5.2/../../../../pic32mx/lib/./proc/32MX795F512H\default_isr_vectors.o (__vector_dispatch_50)
c:/program files/microchip/xc32/v1.33/bin/bin/../../lib/gcc/pic32mx/4.5.2/../../../../pic32mx/lib\libpic32.a(vector51.o)
                              c:/program files/microchip/xc32/v1.33/bin/bin/../../lib/gcc/pic32mx/4.5.2/../../../../pic32mx/lib/./proc/32MX795F512H\default_isr_vectors.o (__vector_dispatch_51)
c:/program files/microchip/xc32/v1.33/bin/bin/../../lib/gcc/pic32mx/4.5.2/../../../../pic32mx/lib\libpic32.a(vector52.o)
                              c:/program files/microchip/xc32/v1.33/bin/bin/../../lib/gcc/pic32mx/4.5.2/../../../../pic32mx/lib/./proc/32MX795F512H\default_isr_vectors.o (__vector_dispatch_52)
c:/program files/microchip/xc32/v1.33/bin/bin/../../lib/gcc/pic32mx/4.5.2/../../../../pic32mx/lib\libpic32.a(vector53.o)
                              c:/program files/microchip/xc32/v1.33/bin/bin/../../lib/gcc/pic32mx/4.5.2/../../../../pic32mx/lib/./proc/32MX795F512H\default_isr_vectors.o (__vector_dispatch_53)
c:/program files/microchip/xc32/v1.33/bin/bin/../../lib/gcc/pic32mx/4.5.2/../../../../pic32mx/lib\libpic32.a(vector54.o)
                              c:/program files/microchip/xc32/v1.33/bin/bin/../../lib/gcc/pic32mx/4.5.2/../../../../pic32mx/lib/./proc/32MX795F512H\default_isr_vectors.o (__vector_dispatch_54)
c:/program files/microchip/xc32/v1.33/bin/bin/../../lib/gcc/pic32mx/4.5.2/../../../../pic32mx/lib\libpic32.a(vector55.o)
                              c:/program files/microchip/xc32/v1.33/bin/bin/../../lib/gcc/pic32mx/4.5.2/../../../../pic32mx/lib/./proc/32MX795F512H\default_isr_vectors.o (__vector_dispatch_55)
c:/program files/microchip/xc32/v1.33/bin/bin/../../lib/gcc/pic32mx/4.5.2/../../../../pic32mx/lib\libpic32.a(vector56.o)
                              c:/program files/microchip/xc32/v1.33/bin/bin/../../lib/gcc/pic32mx/4.5.2/../../../../pic32mx/lib/./proc/32MX795F512H\default_isr_vectors.o (__vector_dispatch_56)
c:/program files/microchip/xc32/v1.33/bin/bin/../../lib/gcc/pic32mx/4.5.2/../../../../pic32mx/lib\libpic32.a(vector57.o)
                              c:/program files/microchip/xc32/v1.33/bin/bin/../../lib/gcc/pic32mx/4.5.2/../../../../pic32mx/lib/./proc/32MX795F512H\default_isr_vectors.o (__vector_dispatch_57)
c:/program files/microchip/xc32/v1.33/bin/bin/../../lib/gcc/pic32mx/4.5.2/../../../../pic32mx/lib\libpic32.a(vector58.o)
                              c:/program files/microchip/xc32/v1.33/bin/bin/../../lib/gcc/pic32mx/4.5.2/../../../../pic32mx/lib/./proc/32MX795F512H\default_isr_vectors.o (__vector_dispatch_58)
c:/program files/microchip/xc32/v1.33/bin/bin/../../lib/gcc/pic32mx/4.5.2/../../../../pic32mx/lib\libpic32.a(vector59.o)
                              c:/program files/microchip/xc32/v1.33/bin/bin/../../lib/gcc/pic32mx/4.5.2/../../../../pic32mx/lib/./proc/32MX795F512H\default_isr_vectors.o (__vector_dispatch_59)
c:/program files/microchip/xc32/v1.33/bin/bin/../../lib/gcc/pic32mx/4.5.2/../../../../pic32mx/lib\libpic32.a(vector60.o)
                              c:/program files/microchip/xc32/v1.33/bin/bin/../../lib/gcc/pic32mx/4.5.2/../../../../pic32mx/lib/./proc/32MX795F512H\default_isr_vectors.o (__vector_dispatch_60)
c:/program files/microchip/xc32/v1.33/bin/bin/../../lib/gcc/pic32mx/4.5.2/../../../../pic32mx/lib\libpic32.a(vector61.o)
                              c:/program files/microchip/xc32/v1.33/bin/bin/../../lib/gcc/pic32mx/4.5.2/../../../../pic32mx/lib/./proc/32MX795F512H\default_isr_vectors.o (__vector_dispatch_61)
c:/program files/microchip/xc32/v1.33/bin/bin/../../lib/gcc/pic32mx/4.5.2/../../../../pic32mx/lib\libpic32.a(vector62.o)
                              c:/program files/microchip/xc32/v1.33/bin/bin/../../lib/gcc/pic32mx/4.5.2/../../../../pic32mx/lib/./proc/32MX795F512H\default_isr_vectors.o (__vector_dispatch_62)
c:/program files/microchip/xc32/v1.33/bin/bin/../../lib/gcc/pic32mx/4.5.2/../../../../pic32mx/lib\libpic32.a(vector63.o)
                              c:/program files/microchip/xc32/v1.33/bin/bin/../../lib/gcc/pic32mx/4.5.2/../../../../pic32mx/lib/./proc/32MX795F512H\default_isr_vectors.o (__vector_dispatch_63)
c:/program files/microchip/xc32/v1.33/bin/bin/../../lib/gcc/pic32mx/4.5.2/../../../../pic32mx/lib\libpic32.a(defaultinterrupt.o)
                              c:/program files/microchip/xc32/v1.33/bin/bin/../../lib/gcc/pic32mx/4.5.2/../../../../pic32mx/lib\libpic32.a(vector0.o) (_DefaultInterrupt)
c:/program files/microchip/xc32/v1.33/bin/bin/../../lib/gcc/pic32mx/4.5.2/../../../../pic32mx/lib\libm.a(fp32div.o)
                              build/ChaletDuinoV2_775F512H_/debug/Source/BatteryMonitor.o (fpdiv)
c:/program files/microchip/xc32/v1.33/bin/bin/../../lib/gcc/pic32mx/4.5.2/../../../../pic32mx/lib\libm.a(fp32mul.o)
                              build/ChaletDuinoV2_775F512H_/debug/Source/BatteryMonitor.o (fpmul)
c:/program files/microchip/xc32/v1.33/bin/bin/../../lib/gcc/pic32mx/4.5.2/../../../../pic32mx/lib\libm.a(fp32subadd.o)
                              build/ChaletDuinoV2_775F512H_/debug/Source/BatteryMonitor.o (fpadd)
c:/program files/microchip/xc32/v1.33/bin/bin/../../lib/gcc/pic32mx/4.5.2/../../../../pic32mx/lib\libm.a(sitofp.o)
                              build/ChaletDuinoV2_775F512H_/debug/Source/BatteryMonitor.o (sitofp)
c:/program files/microchip/xc32/v1.33/bin/bin/../../lib/gcc/pic32mx/4.5.2/../../../../pic32mx/lib\libc.a(_iob.o)
                              build/ChaletDuinoV2_775F512H_/debug/Source/Uart.o (_iob)
c:/program files/microchip/xc32/v1.33/bin/bin/../../lib/gcc/pic32mx/4.5.2/../../../../pic32mx/lib\libc.a(fflush.o)
                              build/ChaletDuinoV2_775F512H_/debug/Source/Uart.o (fflush)
c:/program files/microchip/xc32/v1.33/bin/bin/../../lib/gcc/pic32mx/4.5.2/../../../../pic32mx/lib\libc.a(malloc.o)
                              build/ChaletDuinoV2_775F512H_/debug/Source/winc3400/driver/source/m2m_wifi.o (malloc)
c:/program files/microchip/xc32/v1.33/bin/bin/../../lib/gcc/pic32mx/4.5.2/../../../../pic32mx/lib\libc.a(puts.o)
                              build/ChaletDuinoV2_775F512H_/debug/Source/InternalUart.o (puts)
c:/program files/microchip/xc32/v1.33/bin/bin/../../lib/gcc/pic32mx/4.5.2/../../../../pic32mx/lib\libc.a(setbuf.o)
                              build/ChaletDuinoV2_775F512H_/debug/Source/Uart.o (setbuf)
c:/program files/microchip/xc32/v1.33/bin/bin/../../lib/gcc/pic32mx/4.5.2/../../../../pic32mx/lib\libc.a(strncmp.o)
                              build/ChaletDuinoV2_775F512H_/debug/Source/Terminal.o (strncmp)
c:/program files/microchip/xc32/v1.33/bin/bin/../../lib/gcc/pic32mx/4.5.2/../../../../pic32mx/lib\libc.a(printf_cdfFnopsuxX.eo)
                              (_printf_cdfFnopsuxX)
c:/program files/microchip/xc32/v1.33/bin/bin/../../lib/gcc/pic32mx/4.5.2/../../../../pic32mx/lib\libc.a(printf_cdnopsuxX.eo)
                              build/ChaletDuinoV2_775F512H_/debug/Source/WiFiCtrl.o (_printf_cdnopsuxX)
c:/program files/microchip/xc32/v1.33/bin/bin/../../lib/gcc/pic32mx/4.5.2/../../../../pic32mx/lib\libc.a(printf_cdnopuxX.eo)
                              build/ChaletDuinoV2_775F512H_/debug/Source/main.o (_printf_cdnopuxX)
c:/program files/microchip/xc32/v1.33/bin/bin/../../lib/gcc/pic32mx/4.5.2/../../../../pic32mx/lib\libc.a(printf_fF.eo)
                              build/ChaletDuinoV2_775F512H_/debug/Source/BatteryMonitor.o (_printf_fF)
c:/program files/microchip/xc32/v1.33/bin/bin/../../lib/gcc/pic32mx/4.5.2/../../../../pic32mx/lib\libc.a(sprintf_cdfFnopuxX.eo)
                              build/ChaletDuinoV2_775F512H_/debug/Source/Terminal.o (_sprintf_cdfFnopuxX)
c:/program files/microchip/xc32/v1.33/bin/bin/../../lib/gcc/pic32mx/4.5.2/../../../../pic32mx/lib\libc.a(sprintf_cdnopuxX.eo)
                              build/ChaletDuinoV2_775F512H_/debug/Source/Util.o (_sprintf_cdnopuxX)
c:/program files/microchip/xc32/v1.33/bin/bin/../../lib/gcc/pic32mx/4.5.2/../../../../pic32mx/lib\libc.a(sscanf_s.eo)
                              build/ChaletDuinoV2_775F512H_/debug/Source/Terminal.o (_sscanf_s)
c:/program files/microchip/xc32/v1.33/bin/bin/../../lib/gcc/pic32mx/4.5.2/../../../../pic32mx/lib\libc.a(_fputc_simple.o)
                              c:/program files/microchip/xc32/v1.33/bin/bin/../../lib/gcc/pic32mx/4.5.2/../../../../pic32mx/lib\libc.a(puts.o) (fputc)
c:/program files/microchip/xc32/v1.33/bin/bin/../../lib/gcc/pic32mx/4.5.2/../../../../pic32mx/lib\libc.a(buf.o)
                              c:/program files/microchip/xc32/v1.33/bin/bin/../../lib/gcc/pic32mx/4.5.2/../../../../pic32mx/lib\libc.a(setbuf.o) (_bufallo)
c:/program files/microchip/xc32/v1.33/bin/bin/../../lib/gcc/pic32mx/4.5.2/../../../../pic32mx/lib\libc.a(errno.o)
                              c:/program files/microchip/xc32/v1.33/bin/bin/../../lib/gcc/pic32mx/4.5.2/../../../../pic32mx/lib\libc.a(buf.o) (errno)
c:/program files/microchip/xc32/v1.33/bin/bin/../../lib/gcc/pic32mx/4.5.2/../../../../pic32mx/lib\libc.a(doprnt_cdfFnopsuxX.eo)
                              c:/program files/microchip/xc32/v1.33/bin/bin/../../lib/gcc/pic32mx/4.5.2/../../../../pic32mx/lib\libc.a(printf_cdfFnopsuxX.eo) (_vfprintf_cdfFnopsuxX)
c:/program files/microchip/xc32/v1.33/bin/bin/../../lib/gcc/pic32mx/4.5.2/../../../../pic32mx/lib\libc.a(doprnt_cdfFnopuxX.eo)
                              c:/program files/microchip/xc32/v1.33/bin/bin/../../lib/gcc/pic32mx/4.5.2/../../../../pic32mx/lib\libc.a(sprintf_cdfFnopuxX.eo) (_vfprintf_cdfFnopuxX)
c:/program files/microchip/xc32/v1.33/bin/bin/../../lib/gcc/pic32mx/4.5.2/../../../../pic32mx/lib\libc.a(doprnt_cdnopsuxX.eo)
                              c:/program files/microchip/xc32/v1.33/bin/bin/../../lib/gcc/pic32mx/4.5.2/../../../../pic32mx/lib\libc.a(printf_cdnopsuxX.eo) (_vfprintf_cdnopsuxX)
c:/program files/microchip/xc32/v1.33/bin/bin/../../lib/gcc/pic32mx/4.5.2/../../../../pic32mx/lib\libc.a(doprnt_cdnopuxX.eo)
                              c:/program files/microchip/xc32/v1.33/bin/bin/../../lib/gcc/pic32mx/4.5.2/../../../../pic32mx/lib\libc.a(printf_cdnopuxX.eo) (_vfprintf_cdnopuxX)
c:/program files/microchip/xc32/v1.33/bin/bin/../../lib/gcc/pic32mx/4.5.2/../../../../pic32mx/lib\libc.a(doprnt_fF.eo)
                              c:/program files/microchip/xc32/v1.33/bin/bin/../../lib/gcc/pic32mx/4.5.2/../../../../pic32mx/lib\libc.a(printf_fF.eo) (_vfprintf_fF)
c:/program files/microchip/xc32/v1.33/bin/bin/../../lib/gcc/pic32mx/4.5.2/../../../../pic32mx/lib\libc.a(doscan_s.eo)
                              c:/program files/microchip/xc32/v1.33/bin/bin/../../lib/gcc/pic32mx/4.5.2/../../../../pic32mx/lib\libc.a(sscanf_s.eo) (_vfscanf_s)
c:/program files/microchip/xc32/v1.33/bin/bin/../../lib/gcc/pic32mx/4.5.2/../../../../pic32mx/lib\libc.a(_flsbuf_simple.o)
                              c:/program files/microchip/xc32/v1.33/bin/bin/../../lib/gcc/pic32mx/4.5.2/../../../../pic32mx/lib\libc.a(_fputc_simple.o) (_flsbuf)
c:/program files/microchip/xc32/v1.33/bin/bin/../../lib/gcc/pic32mx/4.5.2/../../../../pic32mx/lib\libc.a(fgetc.o)
                              c:/program files/microchip/xc32/v1.33/bin/bin/../../lib/gcc/pic32mx/4.5.2/../../../../pic32mx/lib\libc.a(doscan_s.eo) (fgetc)
c:/program files/microchip/xc32/v1.33/bin/bin/../../lib/gcc/pic32mx/4.5.2/../../../../pic32mx/lib\libc.a(atoi.o)
                              c:/program files/microchip/xc32/v1.33/bin/bin/../../lib/gcc/pic32mx/4.5.2/../../../../pic32mx/lib\libc.a(doscan_s.eo) (atoi)
c:/program files/microchip/xc32/v1.33/bin/bin/../../lib/gcc/pic32mx/4.5.2/../../../../pic32mx/lib\libc.a(ctype.o)
                              c:/program files/microchip/xc32/v1.33/bin/bin/../../lib/gcc/pic32mx/4.5.2/../../../../pic32mx/lib\libc.a(doprnt_cdfFnopsuxX.eo) (_ctype)
c:/program files/microchip/xc32/v1.33/bin/bin/../../lib/gcc/pic32mx/4.5.2/../../../../pic32mx/lib\libc.a(ctypef.o)
                              c:/program files/microchip/xc32/v1.33/bin/bin/../../lib/gcc/pic32mx/4.5.2/../../../../pic32mx/lib\libc.a(doscan_s.eo) (tolower)
c:/program files/microchip/xc32/v1.33/bin/bin/../../lib/gcc/pic32mx/4.5.2/../../../../pic32mx/lib\libc.a(powersf.o)
                              c:/program files/microchip/xc32/v1.33/bin/bin/../../lib/gcc/pic32mx/4.5.2/../../../../pic32mx/lib\libc.a(doprnt_cdfFnopsuxX.eo) (_powers_f)
c:/program files/microchip/xc32/v1.33/bin/bin/../../lib/gcc/pic32mx/4.5.2/../../../../pic32mx/lib\libc.a(ungetc.o)
                              c:/program files/microchip/xc32/v1.33/bin/bin/../../lib/gcc/pic32mx/4.5.2/../../../../pic32mx/lib\libc.a(doscan_s.eo) (ungetc)
c:/program files/microchip/xc32/v1.33/bin/bin/../../lib/gcc/pic32mx/4.5.2/../../../../pic32mx/lib\libc.a(filbuf.o)
                              c:/program files/microchip/xc32/v1.33/bin/bin/../../lib/gcc/pic32mx/4.5.2/../../../../pic32mx/lib\libc.a(fgetc.o) (_filbuf)
c:/program files/microchip/xc32/v1.33/bin/bin/../../lib/gcc/pic32mx/4.5.2/../../../../pic32mx/lib\libpic32.a(sbrk.o)
                              c:/program files/microchip/xc32/v1.33/bin/bin/../../lib/gcc/pic32mx/4.5.2/../../../../pic32mx/lib\libc.a(malloc.o) (sbrk)
c:/program files/microchip/xc32/v1.33/bin/bin/../../lib/gcc/pic32mx/4.5.2/../../../../pic32mx/lib\libpic32.a(read.o)
                              c:/program files/microchip/xc32/v1.33/bin/bin/../../lib/gcc/pic32mx/4.5.2/../../../../pic32mx/lib\libc.a(filbuf.o) (read)
c:/program files/microchip/xc32/v1.33/bin/bin/../../lib/gcc/pic32mx/4.5.2/../../../../pic32mx/lib\libpic32.a(write.o)
                              c:/program files/microchip/xc32/v1.33/bin/bin/../../lib/gcc/pic32mx/4.5.2/../../../../pic32mx/lib\libc.a(fflush.o) (write)
c:/program files/microchip/xc32/v1.33/bin/bin/../../lib/gcc/pic32mx/4.5.2/../../../../pic32mx/lib\libpic32.a(xc32_uart.o)
                              c:/program files/microchip/xc32/v1.33/bin/bin/../../lib/gcc/pic32mx/4.5.2/../../../../pic32mx/lib\libpic32.a(read.o) (__XC_UART)
c:/program files/microchip/xc32/v1.33/bin/bin/../../lib/gcc/pic32mx/4.5.2/../../../../pic32mx/lib\libm.a(fpcmp.o)
                              c:/program files/microchip/xc32/v1.33/bin/bin/../../lib/gcc/pic32mx/4.5.2/../../../../pic32mx/lib\libc.a(doprnt_cdfFnopsuxX.eo) (fpcmp)
c:/program files/microchip/xc32/v1.33/bin/bin/../../lib/gcc/pic32mx/4.5.2/../../../../pic32mx/lib\libm.a(fpfrexp.o)
                              c:/program files/microchip/xc32/v1.33/bin/bin/../../lib/gcc/pic32mx/4.5.2/../../../../pic32mx/lib\libc.a(doprnt_cdfFnopsuxX.eo) (frexpf)
c:/program files/microchip/xc32/v1.33/bin/bin/../../lib/gcc/pic32mx/4.5.2/../../../../pic32mx/lib\libm.a(fptoul.o)
                              c:/program files/microchip/xc32/v1.33/bin/bin/../../lib/gcc/pic32mx/4.5.2/../../../../pic32mx/lib\libc.a(doprnt_cdfFnopsuxX.eo) (fptoui)
c:/program files/microchip/xc32/v1.33/bin/bin/../../lib/gcc/pic32mx/4.5.2/../../../../pic32mx/lib\libe.a(_floatdisf.o)
                              c:/program files/microchip/xc32/v1.33/bin/bin/../../lib/gcc/pic32mx/4.5.2/../../../../pic32mx/lib\libc.a(doprnt_cdfFnopsuxX.eo) (__floatdisf)
c:/program files/microchip/xc32/v1.33/bin/bin/../../lib/gcc/pic32mx/4.5.2\libgcc.a(_floatundisf.o)
                              c:/program files/microchip/xc32/v1.33/bin/bin/../../lib/gcc/pic32mx/4.5.2/../../../../pic32mx/lib\libc.a(doprnt_cdfFnopsuxX.eo) (__floatundisf)
c:/program files/microchip/xc32/v1.33/bin/bin/../../lib/gcc/pic32mx/4.5.2\libgcc.a(_udivdi3.o)
                              c:/program files/microchip/xc32/v1.33/bin/bin/../../lib/gcc/pic32mx/4.5.2/../../../../pic32mx/lib\libc.a(doprnt_cdfFnopsuxX.eo) (__udivdi3)
c:/program files/microchip/xc32/v1.33/bin/bin/../../lib/gcc/pic32mx/4.5.2\libgcc.a(_umoddi3.o)
                              c:/program files/microchip/xc32/v1.33/bin/bin/../../lib/gcc/pic32mx/4.5.2/../../../../pic32mx/lib\libc.a(doprnt_cdfFnopsuxX.eo) (__umoddi3)
c:/program files/microchip/xc32/v1.33/bin/bin/../../lib/gcc/pic32mx/4.5.2\libgcc.a(floatunsisf.o)
                              c:/program files/microchip/xc32/v1.33/bin/bin/../../lib/gcc/pic32mx/4.5.2\libgcc.a(_floatundisf.o) (__floatunsisf)

Allocating common symbols
Common symbol       size              file

mSyslogBufPtr       0x4               build/ChaletDuinoV2_775F512H_/debug/Source/Syslog.o
BootloaderRxPtr     0x4               build/ChaletDuinoV2_775F512H_/debug/Source/BootloaderProtocol.o
u8IsMacAddrValid    0x1               build/ChaletDuinoV2_775F512H_/debug/Source/WiFiCtrl.o
CurDataChunkSize    0x4               build/ChaletDuinoV2_775F512H_/debug/Source/BootloaderInterface.o
mTerminalOpened     0x4               build/ChaletDuinoV2_775F512H_/debug/Source/Terminal.o
TerminalDataPtr     0x4               build/ChaletDuinoV2_775F512H_/debug/Source/Terminal.o
gpfAppResolveCb     0x4               build/ChaletDuinoV2_775F512H_/debug/Source/winc3400/socket/source/socket.o
BootloaderFirmwareChunkWriteCount
                    0x4               build/ChaletDuinoV2_775F512H_/debug/Source/BootloaderInterface.o
BootloaderFlashWriteDataPtr
                    0x4               build/ChaletDuinoV2_775F512H_/debug/Source/BootloaderInterface.o
mTerminalPendingAction
                    0x4               build/ChaletDuinoV2_775F512H_/debug/Source/Terminal.o
acIntUartRxBuff     0x2               build/ChaletDuinoV2_775F512H_/debug/Source/InternalUart.o
mBatteryCurrent     0x4               build/ChaletDuinoV2_775F512H_/debug/Source/BatteryMonitor.o
mVoltageMeanSum     0x4               build/ChaletDuinoV2_775F512H_/debug/Source/BatteryMonitor.o
mSPIFlashHighSpeedBaudrate
                    0x1               build/ChaletDuinoV2_775F512H_/debug/Source/SPI_Flash.o
NetworkRxBuf        0x400             build/ChaletDuinoV2_775F512H_/debug/Source/WiFiCtrl.o
TerminalRxBuf       0x400             build/ChaletDuinoV2_775F512H_/debug/Source/WiFiCtrl.o
TerminalWorkString  0x12c             build/ChaletDuinoV2_775F512H_/debug/Source/Terminal.o
gu16BufferSize      0x2               build/ChaletDuinoV2_775F512H_/debug/Source/winc3400/socket/source/socket.o
mWifiSPIBaudrate    0x1               build/ChaletDuinoV2_775F512H_/debug/Source/winc3400/bus_wrapper/source/nm_bus_wrapper.o
BootloaderRxBuf     0x400             build/ChaletDuinoV2_775F512H_/debug/Source/WiFiCtrl.o
mVoltageMeanCount   0x4               build/ChaletDuinoV2_775F512H_/debug/Source/BatteryMonitor.o
mBatterySOC         0x4               build/ChaletDuinoV2_775F512H_/debug/Source/BatteryMonitor.o
BootloaderFlashErased
                    0x4               build/ChaletDuinoV2_775F512H_/debug/Source/BootloaderInterface.o
gpfAppSocketCb      0x4               build/ChaletDuinoV2_775F512H_/debug/Source/winc3400/socket/source/socket.o
BootloaderFlashWriteState
                    0x4               build/ChaletDuinoV2_775F512H_/debug/Source/BootloaderInterface.o
mac_addr            0x6               build/ChaletDuinoV2_775F512H_/debug/Source/WiFiCtrl.o
BootloaderCurFlashWriteAddress
                    0x4               build/ChaletDuinoV2_775F512H_/debug/Source/BootloaderInterface.o
mRxData             0x136             build/ChaletDuinoV2_775F512H_/debug/Source/NetworkProtocol.o
mHelpStringPtr      0x4               build/ChaletDuinoV2_775F512H_/debug/Source/Terminal.o
mSyslogBuffer       0x1f4             build/ChaletDuinoV2_775F512H_/debug/Source/Syslog.o
mDeviceID           0x2               build/ChaletDuinoV2_775F512H_/debug/Source/TC77.o
ActualTemp          0x4               build/ChaletDuinoV2_775F512H_/debug/Source/main.o
addr_in             0x10              build/ChaletDuinoV2_775F512H_/debug/Source/WiFiCtrl.o
BooloaderFlashEraseState
                    0x4               build/ChaletDuinoV2_775F512H_/debug/Source/BootloaderInterface.o
PowerRelayState     0x4               build/ChaletDuinoV2_775F512H_/debug/Source/ChaletPowerRelay.o
param               0x1c              build/ChaletDuinoV2_775F512H_/debug/Source/WiFiCtrl.o
mModuleIPConfig     0x10              build/ChaletDuinoV2_775F512H_/debug/Source/WiFiCtrl.o
gsockerrno          0x1               build/ChaletDuinoV2_775F512H_/debug/Source/winc3400/socket/source/socket.o
astUartData         0x620             build/ChaletDuinoV2_775F512H_/debug/Source/Uart.o
mLastTransactionOK  0x4               build/ChaletDuinoV2_775F512H_/debug/Source/I2C.o
BootloaderBuffer    0x12c             build/ChaletDuinoV2_775F512H_/debug/Source/BootloaderInterface.o
I2CSlaveBuffer      0xa               build/ChaletDuinoV2_775F512H_/debug/Source/ina219.o
mSPIFlashBaudrate   0x1               build/ChaletDuinoV2_775F512H_/debug/Source/SPI_Flash.o
BootloaderCurFlashEraseAddress
                    0x4               build/ChaletDuinoV2_775F512H_/debug/Source/BootloaderInterface.o
TerminalPrevDataBuf
                    0x12c             build/ChaletDuinoV2_775F512H_/debug/Source/Terminal.o
BootloaderFlashWritePollCount
                    0x4               build/ChaletDuinoV2_775F512H_/debug/Source/BootloaderInterface.o
BootloaderInterfaceState
                    0x4               build/ChaletDuinoV2_775F512H_/debug/Source/BootloaderInterface.o
DataChunkWritten    0x4               build/ChaletDuinoV2_775F512H_/debug/Source/BootloaderInterface.o
mTxData             0x136             build/ChaletDuinoV2_775F512H_/debug/Source/NetworkProtocol.o
mBatteryVoltage     0x4               build/ChaletDuinoV2_775F512H_/debug/Source/BatteryMonitor.o
mI2CWaitCounter     0x4               build/ChaletDuinoV2_775F512H_/debug/Source/I2C.o
gastrSockets        0xb0              build/ChaletDuinoV2_775F512H_/debug/Source/winc3400/socket/source/socket.o
mCurrentModuleOK    0x4               build/ChaletDuinoV2_775F512H_/debug/Source/BatteryMonitor.o
at_sb_printf        0x4               build/ChaletDuinoV2_775F512H_/debug/Source/winc3400/bsp/source/nm_bsp.o
mTerminalTickState  0x4               build/ChaletDuinoV2_775F512H_/debug/Source/Terminal.o
I2CMasterBuffer     0xa               build/ChaletDuinoV2_775F512H_/debug/Source/ina219.o
BooloaderFlashErasePollCount
                    0x4               build/ChaletDuinoV2_775F512H_/debug/Source/BootloaderInterface.o
FirmwareUploaded    0x4               build/ChaletDuinoV2_775F512H_/debug/Source/BootloaderInterface.o
gfpPingCb           0x4               build/ChaletDuinoV2_775F512H_/debug/Source/winc3400/socket/source/socket.o
mFlashSectorBuffer  0x1000            build/ChaletDuinoV2_775F512H_/debug/Source/SPI_Flash.o
CurDataChunkIndex   0x4               build/ChaletDuinoV2_775F512H_/debug/Source/BootloaderInterface.o
gu8OpCode           0x1               build/ChaletDuinoV2_775F512H_/debug/Source/winc3400/socket/source/socket.o
astTimer            0xf0              build/ChaletDuinoV2_775F512H_/debug/Source/timer.o
TerminalDataBuf     0x12c             build/ChaletDuinoV2_775F512H_/debug/Source/Terminal.o
astInternalUartData
                    0x40              build/ChaletDuinoV2_775F512H_/debug/Source/InternalUart.o
SyslogRxBuf         0xc8              build/ChaletDuinoV2_775F512H_/debug/Source/WiFiCtrl.o

Microchip PIC32 Memory-Usage Report

kseg0 Program-Memory Usage
section                    address  length [bytes]      (dec)  Description
-------                 ----------  -------------------------  -----------
.text                   0x9d003800         0xbcd4       48340  App's exec code 
.text._vfprintf_cdfFnop 0x9d00f4d4         0x13d4        5076   
.text                   0x9d0108a8         0x7248       29256  App's exec code 
.dinit                  0x9d017af0          0xb50        2896   
.text                   0x9d018640          0xb04        2820  App's exec code 
.rodata                 0x9d019144          0x990        2448  Read-only const 
.text                   0x9d019ad4          0x974        2420  App's exec code 
.text._vfscanf_s        0x9d01a448          0x868        2152   
.text                   0x9d01acb0         0x2a84       10884  App's exec code 
.rodata                 0x9d01d734          0x494        1172  Read-only const 
.text                   0x9d01dbc8         0x1108        4360  App's exec code 
.rodata                 0x9d01ecd0          0x404        1028  Read-only const 
.text                   0x9d01f0d4         0x1048        4168  App's exec code 
.text.scale             0x9d02011c          0x2a0         672   
.text.fpsubadd          0x9d0203bc          0x278         632   
.text.malloc            0x9d020634          0x278         632   
.text                   0x9d0208ac          0x26c         620  App's exec code 
.rodata                 0x9d020b18          0x268         616  Read-only const 
.text                   0x9d020d80          0x4a8        1192  App's exec code 
.text.fp32div           0x9d021228          0x230         560   
.text.__floatdisf       0x9d021458          0x220         544   
.text.fp32mul           0x9d021678          0x1bc         444   
.text                   0x9d021834          0x1a0         416  App's exec code 
.text.realloc           0x9d0219d4          0x194         404   
.text._sbrk_init        0x9d021b68          0x194         404   
.text._filbuf           0x9d021cfc          0x188         392   
.text.read              0x9d021e84          0x174         372   
.text                   0x9d021ff8          0x2d0         720  App's exec code 
.text.fputc             0x9d0222c8          0x15c         348   
.text._flsbuf           0x9d022424          0x12c         300   
.text                   0x9d022550          0x11c         284  App's exec code 
.text.fgetc             0x9d02266c          0x108         264   
.rodata                 0x9d022774          0x204         516  Read-only const 
.text.setvbuf           0x9d022978           0xfc         252   
.rodata                 0x9d022a74            0x4           4  Read-only const 
.rodata                 0x9d022a78           0xe0         224  Read-only const 
.text.general_exception 0x9d022b58           0xdc         220   
.text                   0x9d022c34          0x1ac         428  App's exec code 
.rodata                 0x9d022de0           0xc8         200  Read-only const 
.text._sbrk             0x9d022ea8           0xc4         196   
.text                   0x9d022f6c           0xa8         168  App's exec code 
.text.atoi              0x9d023014           0xa8         168   
.text.range             0x9d0230bc           0xa0         160   
.text.fpcmp             0x9d02315c           0x9c         156   
.text.fflush            0x9d0231f8           0x94         148   
.text.write             0x9d02328c           0x94         148   
.text.libm              0x9d023320           0x88         136   
.text                   0x9d0233a8           0x80         128  App's exec code 
.text.fptoul            0x9d023428           0x7c         124   
.text.SoftReset         0x9d0234a4           0x78         120   
.text.fputs             0x9d02351c           0x78         120   
.text.strncmp           0x9d023594           0x78         120   
.text.ungetc            0x9d02360c           0x74         116   
.text                   0x9d023680           0xd8         216  App's exec code 
.text._sprintf_cdfFnopu 0x9d023758           0x68         104   
.rodata                 0x9d0237c0           0x68         104  Read-only const 
.text.sitofp            0x9d023828           0x60          96   
.text.wspace            0x9d023888           0x60          96   
.text                   0x9d0238e8           0x58          88  App's exec code 
.text._sscanf_s         0x9d023940           0x54          84   
.text._bufallo          0x9d023994           0x54          84   
.text.sbrk              0x9d0239e8           0x50          80   
.text.main_entry        0x9d023a38           0x4c          76   
.text                   0x9d023a84           0x4c          76  App's exec code 
.text._bootstrap_except 0x9d023ad0           0x48          72   
.text                   0x9d023b18           0x44          68  App's exec code 
.text.puts              0x9d023b5c           0x44          68   
.text._printf_cdfFnopsu 0x9d023ba0           0x40          64   
.vector_default         0x9d023be0           0x38          56   
.rodata                 0x9d023c18           0x30          48  Read-only const 
.text.INTConfigureSyste 0x9d023c48           0x30          48   
.text.free              0x9d023c78           0x30          48   
.rodata                 0x9d023ca8           0x2c          44  Read-only const 
.text._stub_sbd_memlayo 0x9d023cd4           0x2c          44   
.rodata                 0x9d023d00           0x28          40  Read-only const 
.text.tolower           0x9d023d28           0x24          36   
.text.toupper           0x9d023d4c           0x24          36   
.text                   0x9d023d70           0x20          32  App's exec code 
.rodata                 0x9d023d90           0x1c          28  Read-only const 
.text.INTRestoreInterru 0x9d023dac           0x1c          28   
.text.setbuf            0x9d023dc8           0x1c          28   
.rodata                 0x9d023de4           0x18          24  Read-only const 
.text.CheKseg0CacheOff  0x9d023dfc           0x18          24   
.text.CheKseg0CacheOn   0x9d023e14           0x18          24   
.text                   0x9d023e2c           0x18          24  App's exec code 
.text.isalnum           0x9d023e44           0x18          24   
.text.isalpha           0x9d023e5c           0x18          24   
.text.iscntrl           0x9d023e74           0x18          24   
.text.isdigit           0x9d023e8c           0x18          24   
.text.isgraph           0x9d023ea4           0x18          24   
.text.islower           0x9d023ebc           0x18          24   
.text.isprint           0x9d023ed4           0x18          24   
.text.ispunct           0x9d023eec           0x18          24   
.text.isspace           0x9d023f04           0x18          24   
.text.isupper           0x9d023f1c           0x18          24   
.text.isxdigit          0x9d023f34           0x18          24   
.text._buffree          0x9d023f4c           0x14          20   
.text.__exception_handl 0x9d023f60            0xc          12   
.rodata                 0x9d023f6c           0x1c          28  Read-only const 
.text.INTEnableInterrup 0x9d023f88            0x8           8   
.text.INTDisableInterru 0x9d023f90            0x8           8   
.text._on_reset         0x9d023f98            0x8           8   
.text._on_bootstrap     0x9d023fa0            0x8           8   
.text.isascii           0x9d023fa8            0x8           8   
.text.toascii           0x9d023fb0            0x8           8   
.text._tolower          0x9d023fb8            0x8           8   
.text._toupper          0x9d023fc0            0x8           8   
.text.getpagesize       0x9d023fc8            0x8           8   
.rodata                 0x9d023fd0            0x8           8  Read-only const 
.rodata                 0x9d023fd8            0x4           4  Read-only const 
      Total kseg0_program_mem used  :     0x207dc      133084  26.1% of 0x7c7ff

kseg0 Boot-Memory Usage
section                    address  length [bytes]      (dec)  Description
-------                 ----------  -------------------------  -----------
         Total kseg0_boot_mem used  :           0           0  <1% of 0x7f0

Exception-Memory Usage 
section                    address  length [bytes]      (dec)  Description
-------                 ----------  -------------------------  -----------
.app_excpt              0x9d002180           0x10          16  General-Exception 
.vector_0               0x9d002200            0x8           8  Interrupt Vector 0 
.vector_1               0x9d002220            0x8           8  Interrupt Vector 1 
.vector_2               0x9d002240            0x8           8  Interrupt Vector 2 
.vector_3               0x9d002260            0x8           8  Interrupt Vector 3 
.vector_4               0x9d002280            0x8           8  Interrupt Vector 4 
.vector_5               0x9d0022a0            0x8           8  Interrupt Vector 5 
.vector_6               0x9d0022c0            0x8           8  Interrupt Vector 6 
.vector_7               0x9d0022e0            0x8           8  Interrupt Vector 7 
.vector_8               0x9d002300            0x8           8  Interrupt Vector 8 
.vector_9               0x9d002320            0x8           8  Interrupt Vector 9 
.vector_10              0x9d002340            0x8           8  Interrupt Vector 10 
.vector_11              0x9d002360            0x8           8  Interrupt Vector 11 
.vector_12              0x9d002380            0x8           8  Interrupt Vector 12 
.vector_13              0x9d0023a0            0x8           8  Interrupt Vector 13 
.vector_14              0x9d0023c0            0x8           8  Interrupt Vector 14 
.vector_15              0x9d0023e0            0x8           8  Interrupt Vector 15 
.vector_16              0x9d002400            0x8           8  Interrupt Vector 16 
.vector_17              0x9d002420            0x8           8  Interrupt Vector 17 
.vector_18              0x9d002440            0x8           8  Interrupt Vector 18 
.vector_19              0x9d002460            0x8           8  Interrupt Vector 19 
.vector_20              0x9d002480            0x8           8  Interrupt Vector 20 
.vector_21              0x9d0024a0            0x8           8  Interrupt Vector 21 
.vector_22              0x9d0024c0            0x8           8  Interrupt Vector 22 
.vector_23              0x9d0024e0            0x8           8  Interrupt Vector 23 
.vector_24              0x9d002500            0x8           8  Interrupt Vector 24 
.vector_25              0x9d002520            0x8           8  Interrupt Vector 25 
.vector_26              0x9d002540            0x8           8  Interrupt Vector 26 
.vector_27              0x9d002560            0x8           8  Interrupt Vector 27 
.vector_28              0x9d002580            0x8           8  Interrupt Vector 28 
.vector_29              0x9d0025a0            0x8           8  Interrupt Vector 29 
.vector_30              0x9d0025c0            0x8           8  Interrupt Vector 30 
.vector_31              0x9d0025e0            0x8           8  Interrupt Vector 31 
.vector_32              0x9d002600            0x8           8  Interrupt Vector 32 
.vector_33              0x9d002620            0x8           8  Interrupt Vector 33 
.vector_34              0x9d002640            0x8           8  Interrupt Vector 34 
.vector_35              0x9d002660            0x8           8  Interrupt Vector 35 
.vector_36              0x9d002680            0x8           8  Interrupt Vector 36 
.vector_37              0x9d0026a0            0x8           8  Interrupt Vector 37 
.vector_38              0x9d0026c0            0x8           8  Interrupt Vector 38 
.vector_39              0x9d0026e0            0x8           8  Interrupt Vector 39 
.vector_40              0x9d002700            0x8           8  Interrupt Vector 40 
.vector_41              0x9d002720            0x8           8  Interrupt Vector 41 
.vector_42              0x9d002740            0x8           8  Interrupt Vector 42 
.vector_43              0x9d002760            0x8           8  Interrupt Vector 43 
.vector_44              0x9d002780            0x8           8  Interrupt Vector 44 
.vector_45              0x9d0027a0            0x8           8  Interrupt Vector 45 
.vector_46              0x9d0027c0            0x8           8  Interrupt Vector 46 
.vector_47              0x9d0027e0            0x8           8  Interrupt Vector 47 
.vector_48              0x9d002800            0x8           8  Interrupt Vector 48 
.vector_49              0x9d002820            0x8           8  Interrupt Vector 49 
.vector_50              0x9d002840            0x8           8  Interrupt Vector 50 
.vector_51              0x9d002860            0x8           8  Interrupt Vector 51 
.vector_52              0x9d002880            0x8           8  Interrupt Vector 52 
.vector_53              0x9d0028a0            0x8           8  Interrupt Vector 53 
.vector_54              0x9d0028c0            0x8           8  Interrupt Vector 54 
.vector_55              0x9d0028e0            0x8           8  Interrupt Vector 55 
.vector_56              0x9d002900            0x8           8  Interrupt Vector 56 
.vector_57              0x9d002920            0x8           8  Interrupt Vector 57 
.vector_58              0x9d002940            0x8           8  Interrupt Vector 58 
.vector_59              0x9d002960            0x8           8  Interrupt Vector 59 
.vector_60              0x9d002980            0x8           8  Interrupt Vector 60 
.vector_61              0x9d0029a0            0x8           8  Interrupt Vector 61 
.vector_62              0x9d0029c0            0x8           8  Interrupt Vector 62 
.vector_63              0x9d0029e0            0x8           8  Interrupt Vector 63 
          Total exception_mem used  :       0x210         528  12.9% of 0x1000

kseg1 Boot-Memory Usage
section                    address  length [bytes]      (dec)  Description
-------                 ----------  -------------------------  -----------
.reset                  0xbfc00000          0x1f0         496  Reset handler 
.bev_excpt              0xbfc00380           0x10          16  BEV-Exception 
         Total kseg1_boot_mem used  :       0x200         512  43.8% of 0x490
        --------------------------------------------------------------------------
         Total Program Memory used  :     0x20bec      134124  25.9% of 0x7e47f
        --------------------------------------------------------------------------


kseg0 Data-Memory Usage
section                    address  length [bytes]      (dec)  Description
-------                 ----------  -------------------------  -----------
reserve_data_0_kseg0    0x80000000          0x200         512   
         Total kseg0_data_mem used  :       0x200         512  100.0% of 0x200

kseg1 Data-Memory Usage
section                    address  length [bytes]      (dec)  Description
-------                 ----------  -------------------------  -----------
reserve_data_0_kseg1    0xa0000000          0x200         512   
.eh_frame               0xa0000200           0x30          48   
.sdata                  0xa0000230           0x74         116  Small init data 
.sbss                   0xa00002a4          0x194         404  Small uninit data 
.bss                    0xa0000438         0x2e30       11824  Uninitialized data 
.data                   0xa0003268          0x4bc        1212  Initialized data 
.bss                    0xa0003724          0x800        2048  Uninitialized data 
.data                   0xa0003f24          0x2c4         708  Initialized data 
.bss                    0xa00041e8           0x74         116  Uninitialized data 
         Total kseg1_data_mem used  :      0x425c       16988  25.9% of 0x10000
        --------------------------------------------------------------------------
            Total Data Memory used  :      0x445c       17500  26.5% of 0x10200
        --------------------------------------------------------------------------


Dynamic Data-Memory Reservation
section                    address  length [bytes]      (dec)  Description
-------                 ----------  -------------------------  -----------
heap                    0xa0004260          0x200         512  Reserved for heap 
stack                   0xa0004478         0xbb78       47992  Reserved for stack 

        --------------------------------------------------------------------------

Discarded input sections

 .reginfo       0x00000000       0x18 c:/program files/microchip/xc32/v1.33/bin/bin/../../lib/gcc/pic32mx/4.5.2/../../../../pic32mx/lib\software-debug-break.o
 .reginfo       0x00000000       0x18 build/ChaletDuinoV2_775F512H_/debug/Source/ChaletduinoV2Board.o
 .reginfo       0x00000000       0x18 build/ChaletDuinoV2_775F512H_/debug/Source/winc3400/bsp/source/nm_bsp.o
 .reginfo       0x00000000       0x18 build/ChaletDuinoV2_775F512H_/debug/Source/winc3400/bus_wrapper/source/nm_bus_wrapper.o
 .reginfo       0x00000000       0x18 build/ChaletDuinoV2_775F512H_/debug/Source/winc3400/common/source/nm_common.o
 .reginfo       0x00000000       0x18 build/ChaletDuinoV2_775F512H_/debug/Source/winc3400/driver/source/m2m_ate_mode.o
 .reginfo       0x00000000       0x18 build/ChaletDuinoV2_775F512H_/debug/Source/winc3400/driver/source/m2m_crypto.o
 .reginfo       0x00000000       0x18 build/ChaletDuinoV2_775F512H_/debug/Source/winc3400/driver/source/m2m_hif.o
 .reginfo       0x00000000       0x18 build/ChaletDuinoV2_775F512H_/debug/Source/winc3400/driver/source/m2m_ota.o
 .reginfo       0x00000000       0x18 build/ChaletDuinoV2_775F512H_/debug/Source/winc3400/driver/source/m2m_periph.o
 .reginfo       0x00000000       0x18 build/ChaletDuinoV2_775F512H_/debug/Source/winc3400/driver/source/m2m_ssl.o
 .reginfo       0x00000000       0x18 build/ChaletDuinoV2_775F512H_/debug/Source/winc3400/driver/source/m2m_wifi.o
 .reginfo       0x00000000       0x18 build/ChaletDuinoV2_775F512H_/debug/Source/winc3400/driver/source/nmasic.o
 .reginfo       0x00000000       0x18 build/ChaletDuinoV2_775F512H_/debug/Source/winc3400/driver/source/nmbus.o
 .reginfo       0x00000000       0x18 build/ChaletDuinoV2_775F512H_/debug/Source/winc3400/driver/source/nmdrv.o
 .reginfo       0x00000000       0x18 build/ChaletDuinoV2_775F512H_/debug/Source/winc3400/driver/source/nmi2c.o
 .reginfo       0x00000000       0x18 build/ChaletDuinoV2_775F512H_/debug/Source/winc3400/driver/source/nmspi.o
 .reginfo       0x00000000       0x18 build/ChaletDuinoV2_775F512H_/debug/Source/winc3400/driver/source/nmuart.o
 .reginfo       0x00000000       0x18 build/ChaletDuinoV2_775F512H_/debug/Source/winc3400/socket/source/socket.o
 .reginfo       0x00000000       0x18 build/ChaletDuinoV2_775F512H_/debug/Source/winc3400/spi_flash/source/spi_flash.o
 .reginfo       0x00000000       0x18 build/ChaletDuinoV2_775F512H_/debug/Source/winc3400/winc_init.o
 .reginfo       0x00000000       0x18 build/ChaletDuinoV2_775F512H_/debug/Source/DigitalIO.o
 .reginfo       0x00000000       0x18 build/ChaletDuinoV2_775F512H_/debug/Source/InternalUart.o
 .reginfo       0x00000000       0x18 build/ChaletDuinoV2_775F512H_/debug/Source/NetworkProtocol.o
 .reginfo       0x00000000       0x18 build/ChaletDuinoV2_775F512H_/debug/Source/Terminal.o
 .reginfo       0x00000000       0x18 build/ChaletDuinoV2_775F512H_/debug/Source/Uart.o
 .reginfo       0x00000000       0x18 build/ChaletDuinoV2_775F512H_/debug/Source/Util.o
 .reginfo       0x00000000       0x18 build/ChaletDuinoV2_775F512H_/debug/Source/exceptions.o
 .reginfo       0x00000000       0x18 build/ChaletDuinoV2_775F512H_/debug/Source/interrupts.o
 .reginfo       0x00000000       0x18 build/ChaletDuinoV2_775F512H_/debug/Source/main.o
 .reginfo       0x00000000       0x18 build/ChaletDuinoV2_775F512H_/debug/Source/system.o
 .reginfo       0x00000000       0x18 build/ChaletDuinoV2_775F512H_/debug/Source/template.o
 .reginfo       0x00000000       0x18 build/ChaletDuinoV2_775F512H_/debug/Source/timer.o
 .reginfo       0x00000000       0x18 build/ChaletDuinoV2_775F512H_/debug/Source/WiFiCtrl.o
 .reginfo       0x00000000       0x18 build/ChaletDuinoV2_775F512H_/debug/Source/SPI.o
 .reginfo       0x00000000       0x18 build/ChaletDuinoV2_775F512H_/debug/Source/LoraNetworkInterface.o
 .reginfo       0x00000000       0x18 build/ChaletDuinoV2_775F512H_/debug/Source/ChaletPowerRelay.o
 .reginfo       0x00000000       0x18 build/ChaletDuinoV2_775F512H_/debug/Source/HarakiriRelay.o
 .reginfo       0x00000000       0x18 build/ChaletDuinoV2_775F512H_/debug/Source/BatteryMonitor.o
 .reginfo       0x00000000       0x18 build/ChaletDuinoV2_775F512H_/debug/Source/ina219.o
 .reginfo       0x00000000       0x18 build/ChaletDuinoV2_775F512H_/debug/Source/I2C.o
 .reginfo       0x00000000       0x18 build/ChaletDuinoV2_775F512H_/debug/Source/SPI_Flash.o
 .reginfo       0x00000000       0x18 build/ChaletDuinoV2_775F512H_/debug/Source/Syslog.o
 .reginfo       0x00000000       0x18 build/ChaletDuinoV2_775F512H_/debug/Source/Watchdog.o
 .reginfo       0x00000000       0x18 build/ChaletDuinoV2_775F512H_/debug/Source/BootloaderInterface.o
 .reginfo       0x00000000       0x18 build/ChaletDuinoV2_775F512H_/debug/Source/TemperatureSensor.o
 .reginfo       0x00000000       0x18 build/ChaletDuinoV2_775F512H_/debug/Source/TC77.o
 .reginfo       0x00000000       0x18 build/ChaletDuinoV2_775F512H_/debug/Source/BootloaderProtocol.o
 .reginfo       0x00000000       0x18 build/ChaletDuinoV2_775F512H_/debug/Source/crc32.o
 .reginfo       0x00000000       0x18 c:/program files/microchip/xc32/v1.33/bin/bin/../../lib/gcc/pic32mx/4.5.2/../../../../pic32mx/lib/./proc/32MX795F512H\default_isr_vectors.o
 .discard       0x00000000      0x100 c:/program files/microchip/xc32/v1.33/bin/bin/../../lib/gcc/pic32mx/4.5.2/../../../../pic32mx/lib/./proc/32MX795F512H\default_isr_vectors.o
 .reginfo       0x00000000       0x18 c:/program files/microchip/xc32/v1.33/bin/bin/../../lib/gcc/pic32mx/4.5.2/../../../../pic32mx/lib\pic32_software_reset.o
 .reginfo       0x00000000       0x18 c:/program files/microchip/xc32/v1.33/bin/bin/../../lib/gcc/pic32mx/4.5.2/../../../../pic32mx/lib/./proc/32MX795F512H\processor.o
 .reginfo       0x00000000       0x18 c:/program files/microchip/xc32/v1.33/bin/bin/../../lib/gcc/pic32mx/4.5.2/../../../../pic32mx/lib\libmchp_peripheral_32MX795F512H.a(soft_reset_lib.o)
 .reginfo       0x00000000       0x18 c:/program files/microchip/xc32/v1.33/bin/bin/../../lib/gcc/pic32mx/4.5.2/../../../../pic32mx/lib\libmchp_peripheral_32MX795F512H.a(pcache.o)
 .reginfo       0x00000000       0x18 c:/program files/microchip/xc32/v1.33/bin/bin/../../lib/gcc/pic32mx/4.5.2/../../../../pic32mx/lib\libmchp_peripheral_32MX795F512H.a(int_configure_system_lib.o)
 .reginfo       0x00000000       0x18 c:/program files/microchip/xc32/v1.33/bin/bin/../../lib/gcc/pic32mx/4.5.2/../../../../pic32mx/lib\libmchp_peripheral_32MX795F512H.a(int_enable_interrupts_lib.o)
 .reginfo       0x00000000       0x18 c:/program files/microchip/xc32/v1.33/bin/bin/../../lib/gcc/pic32mx/4.5.2/../../../../pic32mx/lib\libmchp_peripheral_32MX795F512H.a(int_disable_interrupts_lib.o)
 .reginfo       0x00000000       0x18 c:/program files/microchip/xc32/v1.33/bin/bin/../../lib/gcc/pic32mx/4.5.2/../../../../pic32mx/lib\libmchp_peripheral_32MX795F512H.a(int_restore_interrupts_lib.o)
 .reginfo       0x00000000       0x18 c:/program files/microchip/xc32/v1.33/bin/bin/../../lib/gcc/pic32mx/4.5.2/../../../../pic32mx/lib\libpic32.a(memcpy.o)
 .reginfo       0x00000000       0x18 c:/program files/microchip/xc32/v1.33/bin/bin/../../lib/gcc/pic32mx/4.5.2/../../../../pic32mx/lib\libpic32.a(memset.o)
 .reginfo       0x00000000       0x18 c:/program files/microchip/xc32/v1.33/bin/bin/../../lib/gcc/pic32mx/4.5.2/../../../../pic32mx/lib\libpic32.a(strcpy.o)
 .reginfo       0x00000000       0x18 c:/program files/microchip/xc32/v1.33/bin/bin/../../lib/gcc/pic32mx/4.5.2/../../../../pic32mx/lib\libpic32.a(strlen.o)
 .reginfo       0x00000000       0x18 c:/program files/microchip/xc32/v1.33/bin/bin/../../lib/gcc/pic32mx/4.5.2/../../../../pic32mx/lib\libpic32.a(default-bootstrap-exception-handler.o)
 .reginfo       0x00000000       0x18 c:/program files/microchip/xc32/v1.33/bin/bin/../../lib/gcc/pic32mx/4.5.2/../../../../pic32mx/lib\libpic32.a(default-on-reset.o)
 .reginfo       0x00000000       0x18 c:/program files/microchip/xc32/v1.33/bin/bin/../../lib/gcc/pic32mx/4.5.2/../../../../pic32mx/lib\libpic32.a(default-on-bootstrap.o)
 .reginfo       0x00000000       0x18 c:/program files/microchip/xc32/v1.33/bin/bin/../../lib/gcc/pic32mx/4.5.2/../../../../pic32mx/lib\libpic32.a(default-nmi-handler.o)
 .reginfo       0x00000000       0x18 c:/program files/microchip/xc32/v1.33/bin/bin/../../lib/gcc/pic32mx/4.5.2/../../../../pic32mx/lib\libpic32.a(general-exception.o)
 .reginfo       0x00000000       0x18 c:/program files/microchip/xc32/v1.33/bin/bin/../../lib/gcc/pic32mx/4.5.2/../../../../pic32mx/lib\libpic32.a(vector0.o)
 .reginfo       0x00000000       0x18 c:/program files/microchip/xc32/v1.33/bin/bin/../../lib/gcc/pic32mx/4.5.2/../../../../pic32mx/lib\libpic32.a(vector1.o)
 .reginfo       0x00000000       0x18 c:/program files/microchip/xc32/v1.33/bin/bin/../../lib/gcc/pic32mx/4.5.2/../../../../pic32mx/lib\libpic32.a(vector2.o)
 .reginfo       0x00000000       0x18 c:/program files/microchip/xc32/v1.33/bin/bin/../../lib/gcc/pic32mx/4.5.2/../../../../pic32mx/lib\libpic32.a(vector5.o)
 .reginfo       0x00000000       0x18 c:/program files/microchip/xc32/v1.33/bin/bin/../../lib/gcc/pic32mx/4.5.2/../../../../pic32mx/lib\libpic32.a(vector6.o)
 .reginfo       0x00000000       0x18 c:/program files/microchip/xc32/v1.33/bin/bin/../../lib/gcc/pic32mx/4.5.2/../../../../pic32mx/lib\libpic32.a(vector7.o)
 .reginfo       0x00000000       0x18 c:/program files/microchip/xc32/v1.33/bin/bin/../../lib/gcc/pic32mx/4.5.2/../../../../pic32mx/lib\libpic32.a(vector8.o)
 .reginfo       0x00000000       0x18 c:/program files/microchip/xc32/v1.33/bin/bin/../../lib/gcc/pic32mx/4.5.2/../../../../pic32mx/lib\libpic32.a(vector9.o)
 .reginfo       0x00000000       0x18 c:/program files/microchip/xc32/v1.33/bin/bin/../../lib/gcc/pic32mx/4.5.2/../../../../pic32mx/lib\libpic32.a(vector10.o)
 .reginfo       0x00000000       0x18 c:/program files/microchip/xc32/v1.33/bin/bin/../../lib/gcc/pic32mx/4.5.2/../../../../pic32mx/lib\libpic32.a(vector11.o)
 .reginfo       0x00000000       0x18 c:/program files/microchip/xc32/v1.33/bin/bin/../../lib/gcc/pic32mx/4.5.2/../../../../pic32mx/lib\libpic32.a(vector12.o)
 .reginfo       0x00000000       0x18 c:/program files/microchip/xc32/v1.33/bin/bin/../../lib/gcc/pic32mx/4.5.2/../../../../pic32mx/lib\libpic32.a(vector13.o)
 .reginfo       0x00000000       0x18 c:/program files/microchip/xc32/v1.33/bin/bin/../../lib/gcc/pic32mx/4.5.2/../../../../pic32mx/lib\libpic32.a(vector14.o)
 .reginfo       0x00000000       0x18 c:/program files/microchip/xc32/v1.33/bin/bin/../../lib/gcc/pic32mx/4.5.2/../../../../pic32mx/lib\libpic32.a(vector15.o)
 .reginfo       0x00000000       0x18 c:/program files/microchip/xc32/v1.33/bin/bin/../../lib/gcc/pic32mx/4.5.2/../../../../pic32mx/lib\libpic32.a(vector16.o)
 .reginfo       0x00000000       0x18 c:/program files/microchip/xc32/v1.33/bin/bin/../../lib/gcc/pic32mx/4.5.2/../../../../pic32mx/lib\libpic32.a(vector17.o)
 .reginfo       0x00000000       0x18 c:/program files/microchip/xc32/v1.33/bin/bin/../../lib/gcc/pic32mx/4.5.2/../../../../pic32mx/lib\libpic32.a(vector18.o)
 .reginfo       0x00000000       0x18 c:/program files/microchip/xc32/v1.33/bin/bin/../../lib/gcc/pic32mx/4.5.2/../../../../pic32mx/lib\libpic32.a(vector19.o)
 .reginfo       0x00000000       0x18 c:/program files/microchip/xc32/v1.33/bin/bin/../../lib/gcc/pic32mx/4.5.2/../../../../pic32mx/lib\libpic32.a(vector20.o)
 .reginfo       0x00000000       0x18 c:/program files/microchip/xc32/v1.33/bin/bin/../../lib/gcc/pic32mx/4.5.2/../../../../pic32mx/lib\libpic32.a(vector21.o)
 .reginfo       0x00000000       0x18 c:/program files/microchip/xc32/v1.33/bin/bin/../../lib/gcc/pic32mx/4.5.2/../../../../pic32mx/lib\libpic32.a(vector22.o)
 .reginfo       0x00000000       0x18 c:/program files/microchip/xc32/v1.33/bin/bin/../../lib/gcc/pic32mx/4.5.2/../../../../pic32mx/lib\libpic32.a(vector23.o)
 .reginfo       0x00000000       0x18 c:/program files/microchip/xc32/v1.33/bin/bin/../../lib/gcc/pic32mx/4.5.2/../../../../pic32mx/lib\libpic32.a(vector25.o)
 .reginfo       0x00000000       0x18 c:/program files/microchip/xc32/v1.33/bin/bin/../../lib/gcc/pic32mx/4.5.2/../../../../pic32mx/lib\libpic32.a(vector26.o)
 .reginfo       0x00000000       0x18 c:/program files/microchip/xc32/v1.33/bin/bin/../../lib/gcc/pic32mx/4.5.2/../../../../pic32mx/lib\libpic32.a(vector27.o)
 .reginfo       0x00000000       0x18 c:/program files/microchip/xc32/v1.33/bin/bin/../../lib/gcc/pic32mx/4.5.2/../../../../pic32mx/lib\libpic32.a(vector28.o)
 .reginfo       0x00000000       0x18 c:/program files/microchip/xc32/v1.33/bin/bin/../../lib/gcc/pic32mx/4.5.2/../../../../pic32mx/lib\libpic32.a(vector29.o)
 .reginfo       0x00000000       0x18 c:/program files/microchip/xc32/v1.33/bin/bin/../../lib/gcc/pic32mx/4.5.2/../../../../pic32mx/lib\libpic32.a(vector30.o)
 .reginfo       0x00000000       0x18 c:/program files/microchip/xc32/v1.33/bin/bin/../../lib/gcc/pic32mx/4.5.2/../../../../pic32mx/lib\libpic32.a(vector31.o)
 .reginfo       0x00000000       0x18 c:/program files/microchip/xc32/v1.33/bin/bin/../../lib/gcc/pic32mx/4.5.2/../../../../pic32mx/lib\libpic32.a(vector33.o)
 .reginfo       0x00000000       0x18 c:/program files/microchip/xc32/v1.33/bin/bin/../../lib/gcc/pic32mx/4.5.2/../../../../pic32mx/lib\libpic32.a(vector34.o)
 .reginfo       0x00000000       0x18 c:/program files/microchip/xc32/v1.33/bin/bin/../../lib/gcc/pic32mx/4.5.2/../../../../pic32mx/lib\libpic32.a(vector35.o)
 .reginfo       0x00000000       0x18 c:/program files/microchip/xc32/v1.33/bin/bin/../../lib/gcc/pic32mx/4.5.2/../../../../pic32mx/lib\libpic32.a(vector36.o)
 .reginfo       0x00000000       0x18 c:/program files/microchip/xc32/v1.33/bin/bin/../../lib/gcc/pic32mx/4.5.2/../../../../pic32mx/lib\libpic32.a(vector37.o)
 .reginfo       0x00000000       0x18 c:/program files/microchip/xc32/v1.33/bin/bin/../../lib/gcc/pic32mx/4.5.2/../../../../pic32mx/lib\libpic32.a(vector38.o)
 .reginfo       0x00000000       0x18 c:/program files/microchip/xc32/v1.33/bin/bin/../../lib/gcc/pic32mx/4.5.2/../../../../pic32mx/lib\libpic32.a(vector39.o)
 .reginfo       0x00000000       0x18 c:/program files/microchip/xc32/v1.33/bin/bin/../../lib/gcc/pic32mx/4.5.2/../../../../pic32mx/lib\libpic32.a(vector40.o)
 .reginfo       0x00000000       0x18 c:/program files/microchip/xc32/v1.33/bin/bin/../../lib/gcc/pic32mx/4.5.2/../../../../pic32mx/lib\libpic32.a(vector41.o)
 .reginfo       0x00000000       0x18 c:/program files/microchip/xc32/v1.33/bin/bin/../../lib/gcc/pic32mx/4.5.2/../../../../pic32mx/lib\libpic32.a(vector42.o)
 .reginfo       0x00000000       0x18 c:/program files/microchip/xc32/v1.33/bin/bin/../../lib/gcc/pic32mx/4.5.2/../../../../pic32mx/lib\libpic32.a(vector43.o)
 .reginfo       0x00000000       0x18 c:/program files/microchip/xc32/v1.33/bin/bin/../../lib/gcc/pic32mx/4.5.2/../../../../pic32mx/lib\libpic32.a(vector44.o)
 .reginfo       0x00000000       0x18 c:/program files/microchip/xc32/v1.33/bin/bin/../../lib/gcc/pic32mx/4.5.2/../../../../pic32mx/lib\libpic32.a(vector45.o)
 .reginfo       0x00000000       0x18 c:/program files/microchip/xc32/v1.33/bin/bin/../../lib/gcc/pic32mx/4.5.2/../../../../pic32mx/lib\libpic32.a(vector46.o)
 .reginfo       0x00000000       0x18 c:/program files/microchip/xc32/v1.33/bin/bin/../../lib/gcc/pic32mx/4.5.2/../../../../pic32mx/lib\libpic32.a(vector47.o)
 .reginfo       0x00000000       0x18 c:/program files/microchip/xc32/v1.33/bin/bin/../../lib/gcc/pic32mx/4.5.2/../../../../pic32mx/lib\libpic32.a(vector48.o)
 .reginfo       0x00000000       0x18 c:/program files/microchip/xc32/v1.33/bin/bin/../../lib/gcc/pic32mx/4.5.2/../../../../pic32mx/lib\libpic32.a(vector49.o)
 .reginfo       0x00000000       0x18 c:/program files/microchip/xc32/v1.33/bin/bin/../../lib/gcc/pic32mx/4.5.2/../../../../pic32mx/lib\libpic32.a(vector50.o)
 .reginfo       0x00000000       0x18 c:/program files/microchip/xc32/v1.33/bin/bin/../../lib/gcc/pic32mx/4.5.2/../../../../pic32mx/lib\libpic32.a(vector51.o)
 .reginfo       0x00000000       0x18 c:/program files/microchip/xc32/v1.33/bin/bin/../../lib/gcc/pic32mx/4.5.2/../../../../pic32mx/lib\libpic32.a(vector52.o)
 .reginfo       0x00000000       0x18 c:/program files/microchip/xc32/v1.33/bin/bin/../../lib/gcc/pic32mx/4.5.2/../../../../pic32mx/lib\libpic32.a(vector53.o)
 .reginfo       0x00000000       0x18 c:/program files/microchip/xc32/v1.33/bin/bin/../../lib/gcc/pic32mx/4.5.2/../../../../pic32mx/lib\libpic32.a(vector54.o)
 .reginfo       0x00000000       0x18 c:/program files/microchip/xc32/v1.33/bin/bin/../../lib/gcc/pic32mx/4.5.2/../../../../pic32mx/lib\libpic32.a(vector55.o)
 .reginfo       0x00000000       0x18 c:/program files/microchip/xc32/v1.33/bin/bin/../../lib/gcc/pic32mx/4.5.2/../../../../pic32mx/lib\libpic32.a(vector56.o)
 .reginfo       0x00000000       0x18 c:/program files/microchip/xc32/v1.33/bin/bin/../../lib/gcc/pic32mx/4.5.2/../../../../pic32mx/lib\libpic32.a(vector57.o)
 .reginfo       0x00000000       0x18 c:/program files/microchip/xc32/v1.33/bin/bin/../../lib/gcc/pic32mx/4.5.2/../../../../pic32mx/lib\libpic32.a(vector58.o)
 .reginfo       0x00000000       0x18 c:/program files/microchip/xc32/v1.33/bin/bin/../../lib/gcc/pic32mx/4.5.2/../../../../pic32mx/lib\libpic32.a(vector59.o)
 .reginfo       0x00000000       0x18 c:/program files/microchip/xc32/v1.33/bin/bin/../../lib/gcc/pic32mx/4.5.2/../../../../pic32mx/lib\libpic32.a(vector60.o)
 .reginfo       0x00000000       0x18 c:/program files/microchip/xc32/v1.33/bin/bin/../../lib/gcc/pic32mx/4.5.2/../../../../pic32mx/lib\libpic32.a(vector61.o)
 .reginfo       0x00000000       0x18 c:/program files/microchip/xc32/v1.33/bin/bin/../../lib/gcc/pic32mx/4.5.2/../../../../pic32mx/lib\libpic32.a(vector62.o)
 .reginfo       0x00000000       0x18 c:/program files/microchip/xc32/v1.33/bin/bin/../../lib/gcc/pic32mx/4.5.2/../../../../pic32mx/lib\libpic32.a(vector63.o)
 .reginfo       0x00000000       0x18 c:/program files/microchip/xc32/v1.33/bin/bin/../../lib/gcc/pic32mx/4.5.2/../../../../pic32mx/lib\libpic32.a(defaultinterrupt.o)
 .reginfo       0x00000000       0x18 c:/program files/microchip/xc32/v1.33/bin/bin/../../lib/gcc/pic32mx/4.5.2/../../../../pic32mx/lib\libm.a(fp32div.o)
 .reginfo       0x00000000       0x18 c:/program files/microchip/xc32/v1.33/bin/bin/../../lib/gcc/pic32mx/4.5.2/../../../../pic32mx/lib\libm.a(fp32mul.o)
 .reginfo       0x00000000       0x18 c:/program files/microchip/xc32/v1.33/bin/bin/../../lib/gcc/pic32mx/4.5.2/../../../../pic32mx/lib\libm.a(fp32subadd.o)
 .reginfo       0x00000000       0x18 c:/program files/microchip/xc32/v1.33/bin/bin/../../lib/gcc/pic32mx/4.5.2/../../../../pic32mx/lib\libm.a(sitofp.o)
 .reginfo       0x00000000       0x18 c:/program files/microchip/xc32/v1.33/bin/bin/../../lib/gcc/pic32mx/4.5.2/../../../../pic32mx/lib\libc.a(_iob.o)
 .reginfo       0x00000000       0x18 c:/program files/microchip/xc32/v1.33/bin/bin/../../lib/gcc/pic32mx/4.5.2/../../../../pic32mx/lib\libc.a(fflush.o)
 .reginfo       0x00000000       0x18 c:/program files/microchip/xc32/v1.33/bin/bin/../../lib/gcc/pic32mx/4.5.2/../../../../pic32mx/lib\libc.a(malloc.o)
 .reginfo       0x00000000       0x18 c:/program files/microchip/xc32/v1.33/bin/bin/../../lib/gcc/pic32mx/4.5.2/../../../../pic32mx/lib\libc.a(puts.o)
 .reginfo       0x00000000       0x18 c:/program files/microchip/xc32/v1.33/bin/bin/../../lib/gcc/pic32mx/4.5.2/../../../../pic32mx/lib\libc.a(setbuf.o)
 .reginfo       0x00000000       0x18 c:/program files/microchip/xc32/v1.33/bin/bin/../../lib/gcc/pic32mx/4.5.2/../../../../pic32mx/lib\libc.a(strncmp.o)
 .reginfo       0x00000000       0x18 c:/program files/microchip/xc32/v1.33/bin/bin/../../lib/gcc/pic32mx/4.5.2/../../../../pic32mx/lib\libc.a(printf_cdfFnopsuxX.eo)
 .reginfo       0x00000000       0x18 c:/program files/microchip/xc32/v1.33/bin/bin/../../lib/gcc/pic32mx/4.5.2/../../../../pic32mx/lib\libc.a(sprintf_cdfFnopuxX.eo)
 .reginfo       0x00000000       0x18 c:/program files/microchip/xc32/v1.33/bin/bin/../../lib/gcc/pic32mx/4.5.2/../../../../pic32mx/lib\libc.a(sscanf_s.eo)
 .reginfo       0x00000000       0x18 c:/program files/microchip/xc32/v1.33/bin/bin/../../lib/gcc/pic32mx/4.5.2/../../../../pic32mx/lib\libc.a(_fputc_simple.o)
 .reginfo       0x00000000       0x18 c:/program files/microchip/xc32/v1.33/bin/bin/../../lib/gcc/pic32mx/4.5.2/../../../../pic32mx/lib\libc.a(buf.o)
 .reginfo       0x00000000       0x18 c:/program files/microchip/xc32/v1.33/bin/bin/../../lib/gcc/pic32mx/4.5.2/../../../../pic32mx/lib\libc.a(errno.o)
 .reginfo       0x00000000       0x18 c:/program files/microchip/xc32/v1.33/bin/bin/../../lib/gcc/pic32mx/4.5.2/../../../../pic32mx/lib\libc.a(doprnt_cdfFnopsuxX.eo)
 .reginfo       0x00000000       0x18 c:/program files/microchip/xc32/v1.33/bin/bin/../../lib/gcc/pic32mx/4.5.2/../../../../pic32mx/lib\libc.a(doscan_s.eo)
 .reginfo       0x00000000       0x18 c:/program files/microchip/xc32/v1.33/bin/bin/../../lib/gcc/pic32mx/4.5.2/../../../../pic32mx/lib\libc.a(_flsbuf_simple.o)
 .reginfo       0x00000000       0x18 c:/program files/microchip/xc32/v1.33/bin/bin/../../lib/gcc/pic32mx/4.5.2/../../../../pic32mx/lib\libc.a(fgetc.o)
 .reginfo       0x00000000       0x18 c:/program files/microchip/xc32/v1.33/bin/bin/../../lib/gcc/pic32mx/4.5.2/../../../../pic32mx/lib\libc.a(atoi.o)
 .reginfo       0x00000000       0x18 c:/program files/microchip/xc32/v1.33/bin/bin/../../lib/gcc/pic32mx/4.5.2/../../../../pic32mx/lib\libc.a(ctype.o)
 .reginfo       0x00000000       0x18 c:/program files/microchip/xc32/v1.33/bin/bin/../../lib/gcc/pic32mx/4.5.2/../../../../pic32mx/lib\libc.a(ctypef.o)
 .reginfo       0x00000000       0x18 c:/program files/microchip/xc32/v1.33/bin/bin/../../lib/gcc/pic32mx/4.5.2/../../../../pic32mx/lib\libc.a(powersf.o)
 .reginfo       0x00000000       0x18 c:/program files/microchip/xc32/v1.33/bin/bin/../../lib/gcc/pic32mx/4.5.2/../../../../pic32mx/lib\libc.a(ungetc.o)
 .reginfo       0x00000000       0x18 c:/program files/microchip/xc32/v1.33/bin/bin/../../lib/gcc/pic32mx/4.5.2/../../../../pic32mx/lib\libc.a(filbuf.o)
 .reginfo       0x00000000       0x18 c:/program files/microchip/xc32/v1.33/bin/bin/../../lib/gcc/pic32mx/4.5.2/../../../../pic32mx/lib\libpic32.a(sbrk.o)
 .reginfo       0x00000000       0x18 c:/program files/microchip/xc32/v1.33/bin/bin/../../lib/gcc/pic32mx/4.5.2/../../../../pic32mx/lib\libpic32.a(read.o)
 .reginfo       0x00000000       0x18 c:/program files/microchip/xc32/v1.33/bin/bin/../../lib/gcc/pic32mx/4.5.2/../../../../pic32mx/lib\libpic32.a(write.o)
 .reginfo       0x00000000       0x18 c:/program files/microchip/xc32/v1.33/bin/bin/../../lib/gcc/pic32mx/4.5.2/../../../../pic32mx/lib\libpic32.a(xc32_uart.o)
 .reginfo       0x00000000       0x18 c:/program files/microchip/xc32/v1.33/bin/bin/../../lib/gcc/pic32mx/4.5.2/../../../../pic32mx/lib\libm.a(fpcmp.o)
 .reginfo       0x00000000       0x18 c:/program files/microchip/xc32/v1.33/bin/bin/../../lib/gcc/pic32mx/4.5.2/../../../../pic32mx/lib\libm.a(fpfrexp.o)
 .reginfo       0x00000000       0x18 c:/program files/microchip/xc32/v1.33/bin/bin/../../lib/gcc/pic32mx/4.5.2/../../../../pic32mx/lib\libm.a(fptoul.o)
 .reginfo       0x00000000       0x18 c:/program files/microchip/xc32/v1.33/bin/bin/../../lib/gcc/pic32mx/4.5.2/../../../../pic32mx/lib\libe.a(_floatdisf.o)
 .reginfo       0x00000000       0x18 c:/program files/microchip/xc32/v1.33/bin/bin/../../lib/gcc/pic32mx/4.5.2\libgcc.a(_floatundisf.o)
 .reginfo       0x00000000       0x18 c:/program files/microchip/xc32/v1.33/bin/bin/../../lib/gcc/pic32mx/4.5.2\libgcc.a(_udivdi3.o)
 .reginfo       0x00000000       0x18 c:/program files/microchip/xc32/v1.33/bin/bin/../../lib/gcc/pic32mx/4.5.2\libgcc.a(_umoddi3.o)
 .reginfo       0x00000000       0x18 c:/program files/microchip/xc32/v1.33/bin/bin/../../lib/gcc/pic32mx/4.5.2\libgcc.a(floatunsisf.o)

Memory Configuration

Name             Origin             Length             Attributes
kseg0_data_mem   0x80000000         0x00000200
kseg1_data_mem   0xa0000000         0x00010000         w !x
kseg0_boot_mem   0x9d003000         0x000007f0
kseg1_boot_mem   0xbfc00000         0x00000490
kseg0_program_mem 0x9d003800         0x0007c7ff         xr
exception_mem    0x9d002000         0x00001000
debug_exec_mem   0xbfc02000         0x00000ff0
config3          0xbfc02ff0         0x00000004
config2          0xbfc02ff4         0x00000004
config1          0xbfc02ff8         0x00000004
config0          0xbfc02ffc         0x00000004
sfrs             0xbf800000         0x00100000
configsfrs       0xbfc02ff0         0x00000010
*default*        0x00000000         0xffffffff

Linker script and memory map


reserve_data_0_kseg0
                0x80000000      0x200
                0x80000000        0x2 SHORT 0x0
                0x000001fd                . = 0x1fd
 *fill*         0x80000002      0x1fb 
                0x80000200                . = ALIGN (0x4)
 *fill*         0x800001fd        0x3 

reserve_data_0_kseg1
                0xa0000000      0x200
                0xa0000000        0x2 SHORT 0x0
                0x000001fd                . = 0x1fd
 *fill*         0xa0000002      0x1fb 
                0xa0000200                . = ALIGN (0x4)
 *fill*         0xa00001fd        0x3 

reserve_boot_0x1fc02000_kseg0
                0x9fc02000      0xff0
                0x9fc02000        0x2 SHORT 0x0
                0x00000500                . = 0x500
 *fill*         0x9fc02002      0x4fe 
                0x9fc02500                . = ALIGN (0x4)
                0x9fc02500        0x2 SHORT 0x0
                0x00000ff0                . = 0xff0
 *fill*         0x9fc02502      0xaee 
                0x9fc02ff0                . = ALIGN (0x4)

reserve_boot_0x1fc02000_kseg1
                0xbfc02000      0xff0
                0xbfc02000        0x2 SHORT 0x0
                0x00000500                . = 0x500
 *fill*         0xbfc02002      0x4fe 
                0xbfc02500                . = ALIGN (0x4)
                0xbfc02500        0x2 SHORT 0x0
                0x00000ff0                . = 0xff0
 *fill*         0xbfc02502      0xaee 
                0xbfc02ff0                . = ALIGN (0x4)
LOAD c:/program files/microchip/xc32/v1.33/bin/bin/../../lib/gcc/pic32mx/4.5.2/../../../../pic32mx/lib/./proc/32MX795F512H/crt0_mips32r2.o
LOAD c:/program files/microchip/xc32/v1.33/bin/bin/../../lib/gcc/pic32mx/4.5.2/../../../../pic32mx/lib\software-debug-break.o
LOAD build/ChaletDuinoV2_775F512H_/debug/Source/ChaletduinoV2Board.o
LOAD build/ChaletDuinoV2_775F512H_/debug/Source/winc3400/bsp/source/nm_bsp.o
LOAD build/ChaletDuinoV2_775F512H_/debug/Source/winc3400/bus_wrapper/source/nm_bus_wrapper.o
LOAD build/ChaletDuinoV2_775F512H_/debug/Source/winc3400/common/source/nm_common.o
LOAD build/ChaletDuinoV2_775F512H_/debug/Source/winc3400/driver/source/m2m_ate_mode.o
LOAD build/ChaletDuinoV2_775F512H_/debug/Source/winc3400/driver/source/m2m_crypto.o
LOAD build/ChaletDuinoV2_775F512H_/debug/Source/winc3400/driver/source/m2m_hif.o
LOAD build/ChaletDuinoV2_775F512H_/debug/Source/winc3400/driver/source/m2m_ota.o
LOAD build/ChaletDuinoV2_775F512H_/debug/Source/winc3400/driver/source/m2m_periph.o
LOAD build/ChaletDuinoV2_775F512H_/debug/Source/winc3400/driver/source/m2m_ssl.o
LOAD build/ChaletDuinoV2_775F512H_/debug/Source/winc3400/driver/source/m2m_wifi.o
LOAD build/ChaletDuinoV2_775F512H_/debug/Source/winc3400/driver/source/nmasic.o
LOAD build/ChaletDuinoV2_775F512H_/debug/Source/winc3400/driver/source/nmbus.o
LOAD build/ChaletDuinoV2_775F512H_/debug/Source/winc3400/driver/source/nmdrv.o
LOAD build/ChaletDuinoV2_775F512H_/debug/Source/winc3400/driver/source/nmi2c.o
LOAD build/ChaletDuinoV2_775F512H_/debug/Source/winc3400/driver/source/nmspi.o
LOAD build/ChaletDuinoV2_775F512H_/debug/Source/winc3400/driver/source/nmuart.o
LOAD build/ChaletDuinoV2_775F512H_/debug/Source/winc3400/socket/source/socket.o
LOAD build/ChaletDuinoV2_775F512H_/debug/Source/winc3400/spi_flash/source/spi_flash.o
LOAD build/ChaletDuinoV2_775F512H_/debug/Source/winc3400/winc_init.o
LOAD build/ChaletDuinoV2_775F512H_/debug/Source/DigitalIO.o
LOAD build/ChaletDuinoV2_775F512H_/debug/Source/InternalUart.o
LOAD build/ChaletDuinoV2_775F512H_/debug/Source/NetworkProtocol.o
LOAD build/ChaletDuinoV2_775F512H_/debug/Source/Terminal.o
LOAD build/ChaletDuinoV2_775F512H_/debug/Source/Uart.o
LOAD build/ChaletDuinoV2_775F512H_/debug/Source/Util.o
LOAD build/ChaletDuinoV2_775F512H_/debug/Source/exceptions.o
LOAD build/ChaletDuinoV2_775F512H_/debug/Source/interrupts.o
LOAD build/ChaletDuinoV2_775F512H_/debug/Source/main.o
LOAD build/ChaletDuinoV2_775F512H_/debug/Source/system.o
LOAD build/ChaletDuinoV2_775F512H_/debug/Source/template.o
LOAD build/ChaletDuinoV2_775F512H_/debug/Source/timer.o
LOAD build/ChaletDuinoV2_775F512H_/debug/Source/WiFiCtrl.o
LOAD build/ChaletDuinoV2_775F512H_/debug/Source/SPI.o
LOAD build/ChaletDuinoV2_775F512H_/debug/Source/LoraNetworkInterface.o
LOAD build/ChaletDuinoV2_775F512H_/debug/Source/ChaletPowerRelay.o
LOAD build/ChaletDuinoV2_775F512H_/debug/Source/HarakiriRelay.o
LOAD build/ChaletDuinoV2_775F512H_/debug/Source/BatteryMonitor.o
LOAD build/ChaletDuinoV2_775F512H_/debug/Source/ina219.o
LOAD build/ChaletDuinoV2_775F512H_/debug/Source/I2C.o
LOAD build/ChaletDuinoV2_775F512H_/debug/Source/SPI_Flash.o
LOAD build/ChaletDuinoV2_775F512H_/debug/Source/Syslog.o
LOAD build/ChaletDuinoV2_775F512H_/debug/Source/Watchdog.o
LOAD build/ChaletDuinoV2_775F512H_/debug/Source/BootloaderInterface.o
LOAD build/ChaletDuinoV2_775F512H_/debug/Source/TemperatureSensor.o
LOAD build/ChaletDuinoV2_775F512H_/debug/Source/TC77.o
LOAD build/ChaletDuinoV2_775F512H_/debug/Source/BootloaderProtocol.o
LOAD build/ChaletDuinoV2_775F512H_/debug/Source/crc32.o
                0x00000001                __MPLAB_BUILD = 0x1
                0x00000001                __MPLAB_DEBUG = 0x1
                0x00000001                __DEBUG = 0x1
                0x00000001                __MPLAB_DEBUGGER_ICD3 = 0x1
                0x00000200                _min_heap_size = 0x200
LOAD c:/program files/microchip/xc32/v1.33/bin/bin/../../lib/gcc/pic32mx/4.5.2/../../../../pic32mx/lib/./proc/32MX795F512H\default_isr_vectors.o
LOAD c:/program files/microchip/xc32/v1.33/bin/bin/../../lib/gcc/pic32mx/4.5.2/../../../../pic32mx/lib\pic32_software_reset.o
                0x00000400                PROVIDE (_min_stack_size, 0x400)
LOAD c:/program files/microchip/xc32/v1.33/bin/bin/../../lib/gcc/pic32mx/4.5.2/../../../../pic32mx/lib/./proc/32MX795F512H\processor.o
START GROUP
LOAD c:/program files/microchip/xc32/v1.33/bin/bin/../../lib/gcc/pic32mx/4.5.2/../../../../pic32mx/lib\libmchp_peripheral.a
END GROUP
START GROUP
LOAD c:/program files/microchip/xc32/v1.33/bin/bin/../../lib/gcc/pic32mx/4.5.2/../../../../pic32mx/lib\libmchp_peripheral_32MX795F512H.a
END GROUP
                0x00000001                PROVIDE (_vector_spacing, 0x1)
                0x9d002000                _ebase_address = 0x9d002000
                0xbfc00000                _RESET_ADDR = 0xbfc00000
                0xbfc00380                _BEV_EXCPT_ADDR = 0xbfc00380
                0xbfc00480                _DBG_EXCPT_ADDR = 0xbfc00480
                0xbfc02000                _DBG_CODE_ADDR = 0xbfc02000
                0x00000ff0                _DBG_CODE_SIZE = 0xff0
                0x9d002180                _GEN_EXCPT_ADDR = (_ebase_address + 0x180)

.config_BFC02FF0
 *(.config_BFC02FF0)

.config_BFC02FF4
                0xbfc02ff4        0x4
 *(.config_BFC02FF4)
 .config_BFC02FF4
                0xbfc02ff4        0x4 build/ChaletDuinoV2_775F512H_/debug/Source/main.o

.config_BFC02FF8
                0xbfc02ff8        0x4
 *(.config_BFC02FF8)
 .config_BFC02FF8
                0xbfc02ff8        0x4 build/ChaletDuinoV2_775F512H_/debug/Source/main.o

.config_BFC02FFC
                0xbfc02ffc        0x4
 *(.config_BFC02FFC)
 .config_BFC02FFC
                0xbfc02ffc        0x4 build/ChaletDuinoV2_775F512H_/debug/Source/main.o
                0xbfc02000                PROVIDE (_DBG_CODE_ADDR, 0xbfc02000)
                0x00000ff0                PROVIDE (_DBG_CODE_SIZE, 0xff0)

.reset          0xbfc00000      0x1f0
 *(.reset)
 .reset         0xbfc00000        0x8 c:/program files/microchip/xc32/v1.33/bin/bin/../../lib/gcc/pic32mx/4.5.2/../../../../pic32mx/lib/./proc/32MX795F512H/crt0_mips32r2.o
                0xbfc00000                _reset
 *(.reset.startup)
 .reset.startup
                0xbfc00008      0x1e8 c:/program files/microchip/xc32/v1.33/bin/bin/../../lib/gcc/pic32mx/4.5.2/../../../../pic32mx/lib/./proc/32MX795F512H/crt0_mips32r2.o

.bev_excpt      0xbfc00380       0x10
 *(.bev_handler)
 .bev_handler   0xbfc00380       0x10 c:/program files/microchip/xc32/v1.33/bin/bin/../../lib/gcc/pic32mx/4.5.2/../../../../pic32mx/lib/./proc/32MX795F512H/crt0_mips32r2.o

.dbg_excpt      0xbfc00480        0x0
                0xbfc00480                . = (. + DEFINED (_DEBUGGER)?0x8:0x0)

.dbg_code       0xbfc02000        0x0
                0xbfc02000                . = (. + DEFINED (_DEBUGGER)?_DBG_CODE_SIZE:0x0)

.app_excpt      0x9d002180       0x10
 *(.gen_handler)
 .gen_handler   0x9d002180       0x10 c:/program files/microchip/xc32/v1.33/bin/bin/../../lib/gcc/pic32mx/4.5.2/../../../../pic32mx/lib/./proc/32MX795F512H/crt0_mips32r2.o

.vector_0       0x9d002200        0x8
 *(.vector_0)
 .vector_0      0x9d002200        0x8 c:/program files/microchip/xc32/v1.33/bin/bin/../../lib/gcc/pic32mx/4.5.2/../../../../pic32mx/lib\libpic32.a(vector0.o)
                0x9d002200                __vector_dispatch_0
                0x00000001                ASSERT (((_vector_spacing == 0x0) || (SIZEOF (.vector_0) <= (_vector_spacing << 0x5))), function at exception vector 0 too large)

.vector_1       0x9d002220        0x8
 *(.vector_1)
 .vector_1      0x9d002220        0x8 c:/program files/microchip/xc32/v1.33/bin/bin/../../lib/gcc/pic32mx/4.5.2/../../../../pic32mx/lib\libpic32.a(vector1.o)
                0x9d002220                __vector_dispatch_1
                0x00000001                ASSERT (((_vector_spacing == 0x0) || (SIZEOF (.vector_1) <= (_vector_spacing << 0x5))), function at exception vector 1 too large)

.vector_2       0x9d002240        0x8
 *(.vector_2)
 .vector_2      0x9d002240        0x8 c:/program files/microchip/xc32/v1.33/bin/bin/../../lib/gcc/pic32mx/4.5.2/../../../../pic32mx/lib\libpic32.a(vector2.o)
                0x9d002240                __vector_dispatch_2
                0x00000001                ASSERT (((_vector_spacing == 0x0) || (SIZEOF (.vector_2) <= (_vector_spacing << 0x5))), function at exception vector 2 too large)

.vector_3       0x9d002260        0x8
 *(.vector_3)
 .vector_3      0x9d002260        0x8 build/ChaletDuinoV2_775F512H_/debug/Source/winc3400/bsp/source/nm_bsp.o
                0x9d002260                __vector_dispatch_3
                0x00000001                ASSERT (((_vector_spacing == 0x0) || (SIZEOF (.vector_3) <= (_vector_spacing << 0x5))), function at exception vector 3 too large)

.vector_4       0x9d002280        0x8
 *(.vector_4)
 .vector_4      0x9d002280        0x8 build/ChaletDuinoV2_775F512H_/debug/Source/timer.o
                0x9d002280                __vector_dispatch_4
                0x00000001                ASSERT (((_vector_spacing == 0x0) || (SIZEOF (.vector_4) <= (_vector_spacing << 0x5))), function at exception vector 4 too large)

.vector_5       0x9d0022a0        0x8
 *(.vector_5)
 .vector_5      0x9d0022a0        0x8 c:/program files/microchip/xc32/v1.33/bin/bin/../../lib/gcc/pic32mx/4.5.2/../../../../pic32mx/lib\libpic32.a(vector5.o)
                0x9d0022a0                __vector_dispatch_5
                0x00000001                ASSERT (((_vector_spacing == 0x0) || (SIZEOF (.vector_5) <= (_vector_spacing << 0x5))), function at exception vector 5 too large)

.vector_6       0x9d0022c0        0x8
 *(.vector_6)
 .vector_6      0x9d0022c0        0x8 c:/program files/microchip/xc32/v1.33/bin/bin/../../lib/gcc/pic32mx/4.5.2/../../../../pic32mx/lib\libpic32.a(vector6.o)
                0x9d0022c0                __vector_dispatch_6
                0x00000001                ASSERT (((_vector_spacing == 0x0) || (SIZEOF (.vector_6) <= (_vector_spacing << 0x5))), function at exception vector 6 too large)

.vector_7       0x9d0022e0        0x8
 *(.vector_7)
 .vector_7      0x9d0022e0        0x8 c:/program files/microchip/xc32/v1.33/bin/bin/../../lib/gcc/pic32mx/4.5.2/../../../../pic32mx/lib\libpic32.a(vector7.o)
                0x9d0022e0                __vector_dispatch_7
                0x00000001                ASSERT (((_vector_spacing == 0x0) || (SIZEOF (.vector_7) <= (_vector_spacing << 0x5))), function at exception vector 7 too large)

.vector_8       0x9d002300        0x8
 *(.vector_8)
 .vector_8      0x9d002300        0x8 c:/program files/microchip/xc32/v1.33/bin/bin/../../lib/gcc/pic32mx/4.5.2/../../../../pic32mx/lib\libpic32.a(vector8.o)
                0x9d002300                __vector_dispatch_8
                0x00000001                ASSERT (((_vector_spacing == 0x0) || (SIZEOF (.vector_8) <= (_vector_spacing << 0x5))), function at exception vector 8 too large)

.vector_9       0x9d002320        0x8
 *(.vector_9)
 .vector_9      0x9d002320        0x8 c:/program files/microchip/xc32/v1.33/bin/bin/../../lib/gcc/pic32mx/4.5.2/../../../../pic32mx/lib\libpic32.a(vector9.o)
                0x9d002320                __vector_dispatch_9
                0x00000001                ASSERT (((_vector_spacing == 0x0) || (SIZEOF (.vector_9) <= (_vector_spacing << 0x5))), function at exception vector 9 too large)

.vector_10      0x9d002340        0x8
 *(.vector_10)
 .vector_10     0x9d002340        0x8 c:/program files/microchip/xc32/v1.33/bin/bin/../../lib/gcc/pic32mx/4.5.2/../../../../pic32mx/lib\libpic32.a(vector10.o)
                0x9d002340                __vector_dispatch_10
                0x00000001                ASSERT (((_vector_spacing == 0x0) || (SIZEOF (.vector_10) <= (_vector_spacing << 0x5))), function at exception vector 10 too large)

.vector_11      0x9d002360        0x8
 *(.vector_11)
 .vector_11     0x9d002360        0x8 c:/program files/microchip/xc32/v1.33/bin/bin/../../lib/gcc/pic32mx/4.5.2/../../../../pic32mx/lib\libpic32.a(vector11.o)
                0x9d002360                __vector_dispatch_11
                0x00000001                ASSERT (((_vector_spacing == 0x0) || (SIZEOF (.vector_11) <= (_vector_spacing << 0x5))), function at exception vector 11 too large)

.vector_12      0x9d002380        0x8
 *(.vector_12)
 .vector_12     0x9d002380        0x8 c:/program files/microchip/xc32/v1.33/bin/bin/../../lib/gcc/pic32mx/4.5.2/../../../../pic32mx/lib\libpic32.a(vector12.o)
                0x9d002380                __vector_dispatch_12
                0x00000001                ASSERT (((_vector_spacing == 0x0) || (SIZEOF (.vector_12) <= (_vector_spacing << 0x5))), function at exception vector 12 too large)

.vector_13      0x9d0023a0        0x8
 *(.vector_13)
 .vector_13     0x9d0023a0        0x8 c:/program files/microchip/xc32/v1.33/bin/bin/../../lib/gcc/pic32mx/4.5.2/../../../../pic32mx/lib\libpic32.a(vector13.o)
                0x9d0023a0                __vector_dispatch_13
                0x00000001                ASSERT (((_vector_spacing == 0x0) || (SIZEOF (.vector_13) <= (_vector_spacing << 0x5))), function at exception vector 13 too large)

.vector_14      0x9d0023c0        0x8
 *(.vector_14)
 .vector_14     0x9d0023c0        0x8 c:/program files/microchip/xc32/v1.33/bin/bin/../../lib/gcc/pic32mx/4.5.2/../../../../pic32mx/lib\libpic32.a(vector14.o)
                0x9d0023c0                __vector_dispatch_14
                0x00000001                ASSERT (((_vector_spacing == 0x0) || (SIZEOF (.vector_14) <= (_vector_spacing << 0x5))), function at exception vector 14 too large)

.vector_15      0x9d0023e0        0x8
 *(.vector_15)
 .vector_15     0x9d0023e0        0x8 c:/program files/microchip/xc32/v1.33/bin/bin/../../lib/gcc/pic32mx/4.5.2/../../../../pic32mx/lib\libpic32.a(vector15.o)
                0x9d0023e0                __vector_dispatch_15
                0x00000001                ASSERT (((_vector_spacing == 0x0) || (SIZEOF (.vector_15) <= (_vector_spacing << 0x5))), function at exception vector 15 too large)

.vector_16      0x9d002400        0x8
 *(.vector_16)
 .vector_16     0x9d002400        0x8 c:/program files/microchip/xc32/v1.33/bin/bin/../../lib/gcc/pic32mx/4.5.2/../../../../pic32mx/lib\libpic32.a(vector16.o)
                0x9d002400                __vector_dispatch_16
                0x00000001                ASSERT (((_vector_spacing == 0x0) || (SIZEOF (.vector_16) <= (_vector_spacing << 0x5))), function at exception vector 16 too large)

.vector_17      0x9d002420        0x8
 *(.vector_17)
 .vector_17     0x9d002420        0x8 c:/program files/microchip/xc32/v1.33/bin/bin/../../lib/gcc/pic32mx/4.5.2/../../../../pic32mx/lib\libpic32.a(vector17.o)
                0x9d002420                __vector_dispatch_17
                0x00000001                ASSERT (((_vector_spacing == 0x0) || (SIZEOF (.vector_17) <= (_vector_spacing << 0x5))), function at exception vector 17 too large)

.vector_18      0x9d002440        0x8
 *(.vector_18)
 .vector_18     0x9d002440        0x8 c:/program files/microchip/xc32/v1.33/bin/bin/../../lib/gcc/pic32mx/4.5.2/../../../../pic32mx/lib\libpic32.a(vector18.o)
                0x9d002440                __vector_dispatch_18
                0x00000001                ASSERT (((_vector_spacing == 0x0) || (SIZEOF (.vector_18) <= (_vector_spacing << 0x5))), function at exception vector 18 too large)

.vector_19      0x9d002460        0x8
 *(.vector_19)
 .vector_19     0x9d002460        0x8 c:/program files/microchip/xc32/v1.33/bin/bin/../../lib/gcc/pic32mx/4.5.2/../../../../pic32mx/lib\libpic32.a(vector19.o)
                0x9d002460                __vector_dispatch_19
                0x00000001                ASSERT (((_vector_spacing == 0x0) || (SIZEOF (.vector_19) <= (_vector_spacing << 0x5))), function at exception vector 19 too large)

.vector_20      0x9d002480        0x8
 *(.vector_20)
 .vector_20     0x9d002480        0x8 c:/program files/microchip/xc32/v1.33/bin/bin/../../lib/gcc/pic32mx/4.5.2/../../../../pic32mx/lib\libpic32.a(vector20.o)
                0x9d002480                __vector_dispatch_20
                0x00000001                ASSERT (((_vector_spacing == 0x0) || (SIZEOF (.vector_20) <= (_vector_spacing << 0x5))), function at exception vector 20 too large)

.vector_21      0x9d0024a0        0x8
 *(.vector_21)
 .vector_21     0x9d0024a0        0x8 c:/program files/microchip/xc32/v1.33/bin/bin/../../lib/gcc/pic32mx/4.5.2/../../../../pic32mx/lib\libpic32.a(vector21.o)
                0x9d0024a0                __vector_dispatch_21
                0x00000001                ASSERT (((_vector_spacing == 0x0) || (SIZEOF (.vector_21) <= (_vector_spacing << 0x5))), function at exception vector 21 too large)

.vector_22      0x9d0024c0        0x8
 *(.vector_22)
 .vector_22     0x9d0024c0        0x8 c:/program files/microchip/xc32/v1.33/bin/bin/../../lib/gcc/pic32mx/4.5.2/../../../../pic32mx/lib\libpic32.a(vector22.o)
                0x9d0024c0                __vector_dispatch_22
                0x00000001                ASSERT (((_vector_spacing == 0x0) || (SIZEOF (.vector_22) <= (_vector_spacing << 0x5))), function at exception vector 22 too large)

.vector_23      0x9d0024e0        0x8
 *(.vector_23)
 .vector_23     0x9d0024e0        0x8 c:/program files/microchip/xc32/v1.33/bin/bin/../../lib/gcc/pic32mx/4.5.2/../../../../pic32mx/lib\libpic32.a(vector23.o)
                0x9d0024e0                __vector_dispatch_23
                0x00000001                ASSERT (((_vector_spacing == 0x0) || (SIZEOF (.vector_23) <= (_vector_spacing << 0x5))), function at exception vector 23 too large)

.vector_24      0x9d002500        0x8
 *(.vector_24)
 .vector_24     0x9d002500        0x8 build/ChaletDuinoV2_775F512H_/debug/Source/InternalUart.o
                0x9d002500                __vector_dispatch_24
                0x00000001                ASSERT (((_vector_spacing == 0x0) || (SIZEOF (.vector_24) <= (_vector_spacing << 0x5))), function at exception vector 24 too large)

.vector_25      0x9d002520        0x8
 *(.vector_25)
 .vector_25     0x9d002520        0x8 c:/program files/microchip/xc32/v1.33/bin/bin/../../lib/gcc/pic32mx/4.5.2/../../../../pic32mx/lib\libpic32.a(vector25.o)
                0x9d002520                __vector_dispatch_25
                0x00000001                ASSERT (((_vector_spacing == 0x0) || (SIZEOF (.vector_25) <= (_vector_spacing << 0x5))), function at exception vector 25 too large)

.vector_26      0x9d002540        0x8
 *(.vector_26)
 .vector_26     0x9d002540        0x8 c:/program files/microchip/xc32/v1.33/bin/bin/../../lib/gcc/pic32mx/4.5.2/../../../../pic32mx/lib\libpic32.a(vector26.o)
                0x9d002540                __vector_dispatch_26
                0x00000001                ASSERT (((_vector_spacing == 0x0) || (SIZEOF (.vector_26) <= (_vector_spacing << 0x5))), function at exception vector 26 too large)

.vector_27      0x9d002560        0x8
 *(.vector_27)
 .vector_27     0x9d002560        0x8 c:/program files/microchip/xc32/v1.33/bin/bin/../../lib/gcc/pic32mx/4.5.2/../../../../pic32mx/lib\libpic32.a(vector27.o)
                0x9d002560                __vector_dispatch_27
                0x00000001                ASSERT (((_vector_spacing == 0x0) || (SIZEOF (.vector_27) <= (_vector_spacing << 0x5))), function at exception vector 27 too large)

.vector_28      0x9d002580        0x8
 *(.vector_28)
 .vector_28     0x9d002580        0x8 c:/program files/microchip/xc32/v1.33/bin/bin/../../lib/gcc/pic32mx/4.5.2/../../../../pic32mx/lib\libpic32.a(vector28.o)
                0x9d002580                __vector_dispatch_28
                0x00000001                ASSERT (((_vector_spacing == 0x0) || (SIZEOF (.vector_28) <= (_vector_spacing << 0x5))), function at exception vector 28 too large)

.vector_29      0x9d0025a0        0x8
 *(.vector_29)
 .vector_29     0x9d0025a0        0x8 c:/program files/microchip/xc32/v1.33/bin/bin/../../lib/gcc/pic32mx/4.5.2/../../../../pic32mx/lib\libpic32.a(vector29.o)
                0x9d0025a0                __vector_dispatch_29
                0x00000001                ASSERT (((_vector_spacing == 0x0) || (SIZEOF (.vector_29) <= (_vector_spacing << 0x5))), function at exception vector 29 too large)

.vector_30      0x9d0025c0        0x8
 *(.vector_30)
 .vector_30     0x9d0025c0        0x8 c:/program files/microchip/xc32/v1.33/bin/bin/../../lib/gcc/pic32mx/4.5.2/../../../../pic32mx/lib\libpic32.a(vector30.o)
                0x9d0025c0                __vector_dispatch_30
                0x00000001                ASSERT (((_vector_spacing == 0x0) || (SIZEOF (.vector_30) <= (_vector_spacing << 0x5))), function at exception vector 30 too large)

.vector_31      0x9d0025e0        0x8
 *(.vector_31)
 .vector_31     0x9d0025e0        0x8 c:/program files/microchip/xc32/v1.33/bin/bin/../../lib/gcc/pic32mx/4.5.2/../../../../pic32mx/lib\libpic32.a(vector31.o)
                0x9d0025e0                __vector_dispatch_31
                0x00000001                ASSERT (((_vector_spacing == 0x0) || (SIZEOF (.vector_31) <= (_vector_spacing << 0x5))), function at exception vector 31 too large)

.vector_32      0x9d002600        0x8
 *(.vector_32)
 .vector_32     0x9d002600        0x8 build/ChaletDuinoV2_775F512H_/debug/Source/InternalUart.o
                0x9d002600                __vector_dispatch_32
                0x00000001                ASSERT (((_vector_spacing == 0x0) || (SIZEOF (.vector_32) <= (_vector_spacing << 0x5))), function at exception vector 32 too large)

.vector_33      0x9d002620        0x8
 *(.vector_33)
 .vector_33     0x9d002620        0x8 c:/program files/microchip/xc32/v1.33/bin/bin/../../lib/gcc/pic32mx/4.5.2/../../../../pic32mx/lib\libpic32.a(vector33.o)
                0x9d002620                __vector_dispatch_33
                0x00000001                ASSERT (((_vector_spacing == 0x0) || (SIZEOF (.vector_33) <= (_vector_spacing << 0x5))), function at exception vector 33 too large)

.vector_34      0x9d002640        0x8
 *(.vector_34)
 .vector_34     0x9d002640        0x8 c:/program files/microchip/xc32/v1.33/bin/bin/../../lib/gcc/pic32mx/4.5.2/../../../../pic32mx/lib\libpic32.a(vector34.o)
                0x9d002640                __vector_dispatch_34
                0x00000001                ASSERT (((_vector_spacing == 0x0) || (SIZEOF (.vector_34) <= (_vector_spacing << 0x5))), function at exception vector 34 too large)

.vector_35      0x9d002660        0x8
 *(.vector_35)
 .vector_35     0x9d002660        0x8 c:/program files/microchip/xc32/v1.33/bin/bin/../../lib/gcc/pic32mx/4.5.2/../../../../pic32mx/lib\libpic32.a(vector35.o)
                0x9d002660                __vector_dispatch_35
                0x00000001                ASSERT (((_vector_spacing == 0x0) || (SIZEOF (.vector_35) <= (_vector_spacing << 0x5))), function at exception vector 35 too large)

.vector_36      0x9d002680        0x8
 *(.vector_36)
 .vector_36     0x9d002680        0x8 c:/program files/microchip/xc32/v1.33/bin/bin/../../lib/gcc/pic32mx/4.5.2/../../../../pic32mx/lib\libpic32.a(vector36.o)
                0x9d002680                __vector_dispatch_36
                0x00000001                ASSERT (((_vector_spacing == 0x0) || (SIZEOF (.vector_36) <= (_vector_spacing << 0x5))), function at exception vector 36 too large)

.vector_37      0x9d0026a0        0x8
 *(.vector_37)
 .vector_37     0x9d0026a0        0x8 c:/program files/microchip/xc32/v1.33/bin/bin/../../lib/gcc/pic32mx/4.5.2/../../../../pic32mx/lib\libpic32.a(vector37.o)
                0x9d0026a0                __vector_dispatch_37
                0x00000001                ASSERT (((_vector_spacing == 0x0) || (SIZEOF (.vector_37) <= (_vector_spacing << 0x5))), function at exception vector 37 too large)

.vector_38      0x9d0026c0        0x8
 *(.vector_38)
 .vector_38     0x9d0026c0        0x8 c:/program files/microchip/xc32/v1.33/bin/bin/../../lib/gcc/pic32mx/4.5.2/../../../../pic32mx/lib\libpic32.a(vector38.o)
                0x9d0026c0                __vector_dispatch_38
                0x00000001                ASSERT (((_vector_spacing == 0x0) || (SIZEOF (.vector_38) <= (_vector_spacing << 0x5))), function at exception vector 38 too large)

.vector_39      0x9d0026e0        0x8
 *(.vector_39)
 .vector_39     0x9d0026e0        0x8 c:/program files/microchip/xc32/v1.33/bin/bin/../../lib/gcc/pic32mx/4.5.2/../../../../pic32mx/lib\libpic32.a(vector39.o)
                0x9d0026e0                __vector_dispatch_39
                0x00000001                ASSERT (((_vector_spacing == 0x0) || (SIZEOF (.vector_39) <= (_vector_spacing << 0x5))), function at exception vector 39 too large)

.vector_40      0x9d002700        0x8
 *(.vector_40)
 .vector_40     0x9d002700        0x8 c:/program files/microchip/xc32/v1.33/bin/bin/../../lib/gcc/pic32mx/4.5.2/../../../../pic32mx/lib\libpic32.a(vector40.o)
                0x9d002700                __vector_dispatch_40
                0x00000001                ASSERT (((_vector_spacing == 0x0) || (SIZEOF (.vector_40) <= (_vector_spacing << 0x5))), function at exception vector 40 too large)

.vector_41      0x9d002720        0x8
 *(.vector_41)
 .vector_41     0x9d002720        0x8 c:/program files/microchip/xc32/v1.33/bin/bin/../../lib/gcc/pic32mx/4.5.2/../../../../pic32mx/lib\libpic32.a(vector41.o)
                0x9d002720                __vector_dispatch_41
                0x00000001                ASSERT (((_vector_spacing == 0x0) || (SIZEOF (.vector_41) <= (_vector_spacing << 0x5))), function at exception vector 41 too large)

.vector_42      0x9d002740        0x8
 *(.vector_42)
 .vector_42     0x9d002740        0x8 c:/program files/microchip/xc32/v1.33/bin/bin/../../lib/gcc/pic32mx/4.5.2/../../../../pic32mx/lib\libpic32.a(vector42.o)
                0x9d002740                __vector_dispatch_42
                0x00000001                ASSERT (((_vector_spacing == 0x0) || (SIZEOF (.vector_42) <= (_vector_spacing << 0x5))), function at exception vector 42 too large)

.vector_43      0x9d002760        0x8
 *(.vector_43)
 .vector_43     0x9d002760        0x8 c:/program files/microchip/xc32/v1.33/bin/bin/../../lib/gcc/pic32mx/4.5.2/../../../../pic32mx/lib\libpic32.a(vector43.o)
                0x9d002760                __vector_dispatch_43
                0x00000001                ASSERT (((_vector_spacing == 0x0) || (SIZEOF (.vector_43) <= (_vector_spacing << 0x5))), function at exception vector 43 too large)

.vector_44      0x9d002780        0x8
 *(.vector_44)
 .vector_44     0x9d002780        0x8 c:/program files/microchip/xc32/v1.33/bin/bin/../../lib/gcc/pic32mx/4.5.2/../../../../pic32mx/lib\libpic32.a(vector44.o)
                0x9d002780                __vector_dispatch_44
                0x00000001                ASSERT (((_vector_spacing == 0x0) || (SIZEOF (.vector_44) <= (_vector_spacing << 0x5))), function at exception vector 44 too large)

.vector_45      0x9d0027a0        0x8
 *(.vector_45)
 .vector_45     0x9d0027a0        0x8 c:/program files/microchip/xc32/v1.33/bin/bin/../../lib/gcc/pic32mx/4.5.2/../../../../pic32mx/lib\libpic32.a(vector45.o)
                0x9d0027a0                __vector_dispatch_45
                0x00000001                ASSERT (((_vector_spacing == 0x0) || (SIZEOF (.vector_45) <= (_vector_spacing << 0x5))), function at exception vector 45 too large)

.vector_46      0x9d0027c0        0x8
 *(.vector_46)
 .vector_46     0x9d0027c0        0x8 c:/program files/microchip/xc32/v1.33/bin/bin/../../lib/gcc/pic32mx/4.5.2/../../../../pic32mx/lib\libpic32.a(vector46.o)
                0x9d0027c0                __vector_dispatch_46
                0x00000001                ASSERT (((_vector_spacing == 0x0) || (SIZEOF (.vector_46) <= (_vector_spacing << 0x5))), function at exception vector 46 too large)

.vector_47      0x9d0027e0        0x8
 *(.vector_47)
 .vector_47     0x9d0027e0        0x8 c:/program files/microchip/xc32/v1.33/bin/bin/../../lib/gcc/pic32mx/4.5.2/../../../../pic32mx/lib\libpic32.a(vector47.o)
                0x9d0027e0                __vector_dispatch_47
                0x00000001                ASSERT (((_vector_spacing == 0x0) || (SIZEOF (.vector_47) <= (_vector_spacing << 0x5))), function at exception vector 47 too large)

.vector_48      0x9d002800        0x8
 *(.vector_48)
 .vector_48     0x9d002800        0x8 c:/program files/microchip/xc32/v1.33/bin/bin/../../lib/gcc/pic32mx/4.5.2/../../../../pic32mx/lib\libpic32.a(vector48.o)
                0x9d002800                __vector_dispatch_48
                0x00000001                ASSERT (((_vector_spacing == 0x0) || (SIZEOF (.vector_48) <= (_vector_spacing << 0x5))), function at exception vector 48 too large)

.vector_49      0x9d002820        0x8
 *(.vector_49)
 .vector_49     0x9d002820        0x8 c:/program files/microchip/xc32/v1.33/bin/bin/../../lib/gcc/pic32mx/4.5.2/../../../../pic32mx/lib\libpic32.a(vector49.o)
                0x9d002820                __vector_dispatch_49
                0x00000001                ASSERT (((_vector_spacing == 0x0) || (SIZEOF (.vector_49) <= (_vector_spacing << 0x5))), function at exception vector 49 too large)

.vector_50      0x9d002840        0x8
 *(.vector_50)
 .vector_50     0x9d002840        0x8 c:/program files/microchip/xc32/v1.33/bin/bin/../../lib/gcc/pic32mx/4.5.2/../../../../pic32mx/lib\libpic32.a(vector50.o)
                0x9d002840                __vector_dispatch_50
                0x00000001                ASSERT (((_vector_spacing == 0x0) || (SIZEOF (.vector_50) <= (_vector_spacing << 0x5))), function at exception vector 50 too large)

.vector_51      0x9d002860        0x8
 *(.vector_51)
 .vector_51     0x9d002860        0x8 c:/program files/microchip/xc32/v1.33/bin/bin/../../lib/gcc/pic32mx/4.5.2/../../../../pic32mx/lib\libpic32.a(vector51.o)
                0x9d002860                __vector_dispatch_51
                0x00000001                ASSERT (((_vector_spacing == 0x0) || (SIZEOF (.vector_51) <= (_vector_spacing << 0x5))), function at exception vector 51 too large)

.vector_52      0x9d002880        0x8
 *(.vector_52)
 .vector_52     0x9d002880        0x8 c:/program files/microchip/xc32/v1.33/bin/bin/../../lib/gcc/pic32mx/4.5.2/../../../../pic32mx/lib\libpic32.a(vector52.o)
                0x9d002880                __vector_dispatch_52
                0x00000001                ASSERT (((_vector_spacing == 0x0) || (SIZEOF (.vector_52) <= (_vector_spacing << 0x5))), function at exception vector 52 too large)

.vector_53      0x9d0028a0        0x8
 *(.vector_53)
 .vector_53     0x9d0028a0        0x8 c:/program files/microchip/xc32/v1.33/bin/bin/../../lib/gcc/pic32mx/4.5.2/../../../../pic32mx/lib\libpic32.a(vector53.o)
                0x9d0028a0                __vector_dispatch_53
                0x00000001                ASSERT (((_vector_spacing == 0x0) || (SIZEOF (.vector_53) <= (_vector_spacing << 0x5))), function at exception vector 53 too large)

.vector_54      0x9d0028c0        0x8
 *(.vector_54)
 .vector_54     0x9d0028c0        0x8 c:/program files/microchip/xc32/v1.33/bin/bin/../../lib/gcc/pic32mx/4.5.2/../../../../pic32mx/lib\libpic32.a(vector54.o)
                0x9d0028c0                __vector_dispatch_54
                0x00000001                ASSERT (((_vector_spacing == 0x0) || (SIZEOF (.vector_54) <= (_vector_spacing << 0x5))), function at exception vector 54 too large)

.vector_55      0x9d0028e0        0x8
 *(.vector_55)
 .vector_55     0x9d0028e0        0x8 c:/program files/microchip/xc32/v1.33/bin/bin/../../lib/gcc/pic32mx/4.5.2/../../../../pic32mx/lib\libpic32.a(vector55.o)
                0x9d0028e0                __vector_dispatch_55
                0x00000001                ASSERT (((_vector_spacing == 0x0) || (SIZEOF (.vector_55) <= (_vector_spacing << 0x5))), function at exception vector 55 too large)

.vector_56      0x9d002900        0x8
 *(.vector_56)
 .vector_56     0x9d002900        0x8 c:/program files/microchip/xc32/v1.33/bin/bin/../../lib/gcc/pic32mx/4.5.2/../../../../pic32mx/lib\libpic32.a(vector56.o)
                0x9d002900                __vector_dispatch_56
                0x00000001                ASSERT (((_vector_spacing == 0x0) || (SIZEOF (.vector_56) <= (_vector_spacing << 0x5))), function at exception vector 56 too large)

.vector_57      0x9d002920        0x8
 *(.vector_57)
 .vector_57     0x9d002920        0x8 c:/program files/microchip/xc32/v1.33/bin/bin/../../lib/gcc/pic32mx/4.5.2/../../../../pic32mx/lib\libpic32.a(vector57.o)
                0x9d002920                __vector_dispatch_57
                0x00000001                ASSERT (((_vector_spacing == 0x0) || (SIZEOF (.vector_57) <= (_vector_spacing << 0x5))), function at exception vector 57 too large)

.vector_58      0x9d002940        0x8
 *(.vector_58)
 .vector_58     0x9d002940        0x8 c:/program files/microchip/xc32/v1.33/bin/bin/../../lib/gcc/pic32mx/4.5.2/../../../../pic32mx/lib\libpic32.a(vector58.o)
                0x9d002940                __vector_dispatch_58
                0x00000001                ASSERT (((_vector_spacing == 0x0) || (SIZEOF (.vector_58) <= (_vector_spacing << 0x5))), function at exception vector 58 too large)

.vector_59      0x9d002960        0x8
 *(.vector_59)
 .vector_59     0x9d002960        0x8 c:/program files/microchip/xc32/v1.33/bin/bin/../../lib/gcc/pic32mx/4.5.2/../../../../pic32mx/lib\libpic32.a(vector59.o)
                0x9d002960                __vector_dispatch_59
                0x00000001                ASSERT (((_vector_spacing == 0x0) || (SIZEOF (.vector_59) <= (_vector_spacing << 0x5))), function at exception vector 59 too large)

.vector_60      0x9d002980        0x8
 *(.vector_60)
 .vector_60     0x9d002980        0x8 c:/program files/microchip/xc32/v1.33/bin/bin/../../lib/gcc/pic32mx/4.5.2/../../../../pic32mx/lib\libpic32.a(vector60.o)
                0x9d002980                __vector_dispatch_60
                0x00000001                ASSERT (((_vector_spacing == 0x0) || (SIZEOF (.vector_60) <= (_vector_spacing << 0x5))), function at exception vector 60 too large)

.vector_61      0x9d0029a0        0x8
 *(.vector_61)
 .vector_61     0x9d0029a0        0x8 c:/program files/microchip/xc32/v1.33/bin/bin/../../lib/gcc/pic32mx/4.5.2/../../../../pic32mx/lib\libpic32.a(vector61.o)
                0x9d0029a0                __vector_dispatch_61
                0x00000001                ASSERT (((_vector_spacing == 0x0) || (SIZEOF (.vector_61) <= (_vector_spacing << 0x5))), function at exception vector 61 too large)

.vector_62      0x9d0029c0        0x8
 *(.vector_62)
 .vector_62     0x9d0029c0        0x8 c:/program files/microchip/xc32/v1.33/bin/bin/../../lib/gcc/pic32mx/4.5.2/../../../../pic32mx/lib\libpic32.a(vector62.o)
                0x9d0029c0                __vector_dispatch_62
                0x00000001                ASSERT (((_vector_spacing == 0x0) || (SIZEOF (.vector_62) <= (_vector_spacing << 0x5))), function at exception vector 62 too large)

.vector_63      0x9d0029e0        0x8
 *(.vector_63)
 .vector_63     0x9d0029e0        0x8 c:/program files/microchip/xc32/v1.33/bin/bin/../../lib/gcc/pic32mx/4.5.2/../../../../pic32mx/lib\libpic32.a(vector63.o)
                0x9d0029e0                __vector_dispatch_63
                0x00000001                ASSERT (((_vector_spacing == 0x0) || (SIZEOF (.vector_63) <= (_vector_spacing << 0x5))), function at exception vector 63 too large)

.startup
 *(.startup)

.text           0x9d003800        0x0
 *(.stub .gnu.linkonce.t.*)
 *(.text.*personality*)
 *(.mips16.fn.*)
 *(.mips16.call.*)
 *(.gnu.warning)
                0x9d003800                . = ALIGN (0x4)

.init           0x9d003800        0x0
 *crti.o(.init)
 *crtbegin.o(.init)
 *(EXCLUDE_FILE(*crtn.o *crtend?.o *crtend.o) .init)
 *crtend.o(.init)
 *crtn.o(.init)
                0x9d003800                . = ALIGN (0x4)

.fini           0x9d003800        0x0
 *(.fini)
                0x9d003800                . = ALIGN (0x4)

.preinit_array  0x9d003800        0x0
                0x9d003800                PROVIDE (__preinit_array_start, .)
 *(.preinit_array)
                0x9d003800                PROVIDE (__preinit_array_end, .)
                0x9d003800                . = ALIGN (0x4)

.init_array     0x9d003800        0x0
                0x9d003800                PROVIDE (__init_array_start, .)
 *(SORT(.init_array.*))
 *(.init_array)
                0x9d003800                PROVIDE (__init_array_end, .)
                0x9d003800                . = ALIGN (0x4)

.fini_array     0x9d003800        0x0
                0x9d003800                PROVIDE (__fini_array_start, .)
 *(SORT(.fini_array.*))
 *(.fini_array)
                0x9d003800                PROVIDE (__fini_array_end, .)
                0x9d003800                . = ALIGN (0x4)

.ctors          0x9d003800        0x0
 *crtbegin.o(.ctors)
 *crtbegin?.o(.ctors)
 *(EXCLUDE_FILE(*crtend?.o *crtend.o) .ctors)
 *(SORT(.ctors.*))
 *(.ctors)
                0x9d003800                . = ALIGN (0x4)

.dtors          0x9d003800        0x0
 *crtbegin.o(.dtors)
 *crtbegin?.o(.dtors)
 *(EXCLUDE_FILE(*crtend?.o *crtend.o) .dtors)
 *(SORT(.dtors.*))
 *(.dtors)
                0x9d003800                . = ALIGN (0x4)

.rodata         0x9d003800        0x0
 *(.gnu.linkonce.r.*)
 *(.rodata1)
                0x9d003800                . = ALIGN (0x4)

.sdata2         0x9d003000        0x0
 *(.sdata2 .sdata2.* .gnu.linkonce.s2.*)
                0x9d003000                . = ALIGN (0x4)

.sbss2          0x9d003000        0x0
 *(.sbss2 .sbss2.* .gnu.linkonce.sb2.*)
                0x9d003000                . = ALIGN (0x4)

.eh_frame_hdr
 *(.eh_frame_hdr)
                0x9d003000                . = ALIGN (0x4)

.eh_frame
 *(.eh_frame)
                0x9d003000                . = ALIGN (0x4)

.gcc_except_table
 *(.gcc_except_table .gcc_except_table.*)
                0x9d003000                . = ALIGN (0x4)

.dbg_data       0xa0000200        0x0
                0xa0000200                . = (. + DEFINED (_DEBUGGER)?0x200:0x0)

.jcr            0xa0000200        0x0
 *(.jcr)
                0xa0000200                . = ALIGN (0x4)

.eh_frame       0xa0000200       0x30
 *(.eh_frame)
 .eh_frame      0xa0000200       0x20 c:/program files/microchip/xc32/v1.33/bin/bin/../../lib/gcc/pic32mx/4.5.2\libgcc.a(_udivdi3.o)
 .eh_frame      0xa0000220       0x10 c:/program files/microchip/xc32/v1.33/bin/bin/../../lib/gcc/pic32mx/4.5.2\libgcc.a(_umoddi3.o)
                0xa0000230                . = ALIGN (0x4)

.gcc_except_table
 *(.gcc_except_table .gcc_except_table.*)
                0xa0000230                . = ALIGN (0x4)

.persist        0xa0000230        0x0
                0xa0000230                _persist_begin = .
 *(.persist .persist.*)
 *(.pbss .pbss.*)
                0xa0000230                . = ALIGN (0x4)
                0xa0000230                _persist_end = .

.data           0xa0000230        0x0
 *(.gnu.linkonce.d.*)
 *(.data1)
                0xa0000230                . = ALIGN (0x4)
                0xa0000230                . = .
                0xa0008220                _gp = (ALIGN (0x10) + 0x7ff0)

.got            0xa0000230        0x0
 *(.got.plt)
 *(.got)
                0xa0000230                . = ALIGN (0x4)

.sdata          0xa0000230       0x74
                0xa0000230                _sdata_begin = .
 *(.sdata .sdata.* .gnu.linkonce.s.*)
 .sdata         0xa0000230        0x4 build/ChaletDuinoV2_775F512H_/debug/Source/winc3400/bus_wrapper/source/nm_bus_wrapper.o
                0xa0000230                egstrNmBusCapabilities
 .sdata         0xa0000234        0x8 build/ChaletDuinoV2_775F512H_/debug/Source/winc3400/driver/source/m2m_hif.o
 .sdata         0xa000023c        0x4 build/ChaletDuinoV2_775F512H_/debug/Source/winc3400/driver/source/m2m_ssl.o
 .sdata         0xa0000240        0x4 build/ChaletDuinoV2_775F512H_/debug/Source/winc3400/driver/source/nmasic.o
 .sdata         0xa0000244        0x2 build/ChaletDuinoV2_775F512H_/debug/Source/NetworkProtocol.o
                0xa0000244                State
 *fill*         0xa0000246        0x2 
 .sdata         0xa0000248        0xc build/ChaletDuinoV2_775F512H_/debug/Source/Terminal.o
 .sdata         0xa0000254        0x4 build/ChaletDuinoV2_775F512H_/debug/Source/Uart.o
                0xa0000254                gUartStrings
 .sdata         0xa0000258        0x8 build/ChaletDuinoV2_775F512H_/debug/Source/main.o
 .sdata         0xa0000260       0x10 build/ChaletDuinoV2_775F512H_/debug/Source/WiFiCtrl.o
                0xa0000267                TerminalSocket
                0xa0000268                TerminalServerSocket
                0xa0000269                SyslogSocket
                0xa000026a                SyslogServerSocket
                0xa000026b                NetworkSocket
                0xa000026c                NetworkServerSocket
                0xa000026d                BootloaderSocket
                0xa000026e                BootloaderServerSocket
                0xa000026f                mWiFiState
 .sdata         0xa0000270        0x4 build/ChaletDuinoV2_775F512H_/debug/Source/LoraNetworkInterface.o
                0xa0000270                mLoraPreamble
 .sdata         0xa0000274        0x8 build/ChaletDuinoV2_775F512H_/debug/Source/BatteryMonitor.o
 .sdata         0xa000027c        0x8 build/ChaletDuinoV2_775F512H_/debug/Source/Syslog.o
 .sdata         0xa0000284        0x8 build/ChaletDuinoV2_775F512H_/debug/Source/BootloaderInterface.o
 .sdata         0xa000028c       0x10 build/ChaletDuinoV2_775F512H_/debug/Source/BootloaderProtocol.o
                0xa0000292                BootloaderState
                0xa0000294                BootloaderDataStartPtr
 .sdata         0xa000029c        0x4 c:/program files/microchip/xc32/v1.33/bin/bin/../../lib/gcc/pic32mx/4.5.2/../../../../pic32mx/lib\libc.a(_iob.o)
                0xa000029c                _Files
 .sdata         0xa00002a0        0x4 c:/program files/microchip/xc32/v1.33/bin/bin/../../lib/gcc/pic32mx/4.5.2/../../../../pic32mx/lib\libpic32.a(xc32_uart.o)
                0xa00002a0                __XC_UART
                0xa00002a4                . = ALIGN (0x4)
                0xa00002a4                _sdata_end = .

.lit8
 *(.lit8)

.lit4
 *(.lit4)
                0xa00002a4                . = ALIGN (0x4)
                0xa00002a4                _data_end = .
                0xa00002a4                _bss_begin = .

.sbss           0xa00002a4      0x194
                0xa00002a4                _sbss_begin = .
 *(.dynsbss)
 *(.sbss .sbss.* .gnu.linkonce.sb.*)
 .sbss          0xa00002a4        0x4 build/ChaletDuinoV2_775F512H_/debug/Source/winc3400/bsp/source/nm_bsp.o
 .sbss          0xa00002a8       0x20 build/ChaletDuinoV2_775F512H_/debug/Source/winc3400/driver/source/m2m_hif.o
                0xa00002b0                pfWifiCb
                0xa00002b4                pfIpCb
                0xa00002b8                pfOtaCb
                0xa00002bc                pfSigmaCb
                0xa00002c0                pfHifCb
                0xa00002c4                pfSSLCb
 .sbss          0xa00002c8        0x8 build/ChaletDuinoV2_775F512H_/debug/Source/winc3400/driver/source/m2m_ota.o
 .sbss          0xa00002d0        0x8 build/ChaletDuinoV2_775F512H_/debug/Source/winc3400/driver/source/m2m_ssl.o
 .sbss          0xa00002d8       0x14 build/ChaletDuinoV2_775F512H_/debug/Source/winc3400/driver/source/m2m_wifi.o
 .sbss          0xa00002ec        0x4 build/ChaletDuinoV2_775F512H_/debug/Source/winc3400/driver/source/nmasic.o
 .sbss          0xa00002f0        0x1 build/ChaletDuinoV2_775F512H_/debug/Source/winc3400/driver/source/nmspi.o
 *fill*         0xa00002f1        0x1 
 .sbss          0xa00002f2        0x6 build/ChaletDuinoV2_775F512H_/debug/Source/winc3400/socket/source/socket.o
                0xa00002f2                gu16SessionID
                0xa00002f4                gbSocketInit
 .sbss          0xa00002f8        0x4 build/ChaletDuinoV2_775F512H_/debug/Source/winc3400/spi_flash/source/spi_flash.o
 .sbss          0xa00002fc        0x4 build/ChaletDuinoV2_775F512H_/debug/Source/InternalUart.o
                0xa00002fc                LoraData
 .sbss          0xa0000300       0x18 build/ChaletDuinoV2_775F512H_/debug/Source/NetworkProtocol.o
                0xa0000300                DataSize
                0xa0000304                DataCtr
                0xa0000308                BufPtr
                0xa000030c                RxPtr
                0xa000030d                Command
                0xa000030e                CRC
                0xa000030f                SenderID
                0xa0000310                SenderAddress
                0xa0000311                Flags
                0xa0000312                IsUpdating
                0xa0000314                BmpDataPtr
 .sbss          0xa0000318        0xc build/ChaletDuinoV2_775F512H_/debug/Source/exceptions.o
 .sbss          0xa0000324       0x18 build/ChaletDuinoV2_775F512H_/debug/Source/WiFiCtrl.o
                0xa0000324                gu32HostIp
                0xa0000328                gu8RetryCount
                0xa0000338                mWiFiInitOK
 .sbss          0xa000033c        0x4 build/ChaletDuinoV2_775F512H_/debug/Source/BatteryMonitor.o
 .sbss          0xa0000340        0x8 build/ChaletDuinoV2_775F512H_/debug/Source/ina219.o
                0xa0000340                ina219_currentDivider_mA
                0xa0000344                ina219_powerDivider_mW
 .sbss          0xa0000348        0x4 build/ChaletDuinoV2_775F512H_/debug/Source/Watchdog.o
                0xa0000348                WatchdogTriggered
 .sbss          0xa000034c       0x18 build/ChaletDuinoV2_775F512H_/debug/Source/BootloaderProtocol.o
                0xa000034c                BootloaderHeader
                0xa0000350                BootloaderDataSize
                0xa0000354                BootloaderDataCtr
                0xa0000358                BootloaderBufPtr
                0xa000035c                BootloaderCRC
                0xa0000360                BootloaderCommand
 .sbss          0xa0000364        0x1 build/ChaletDuinoV2_775F512H_/debug/Source/crc32.o
 .sbss          0xa0000365        0x1 c:/program files/microchip/xc32/v1.33/bin/bin/../../lib/gcc/pic32mx/4.5.2/../../../../pic32mx/lib\libc.a(_iob.o)
                0xa0000365                _outdone
 *fill*         0xa0000366        0x2 
 .sbss          0xa0000368       0x10 c:/program files/microchip/xc32/v1.33/bin/bin/../../lib/gcc/pic32mx/4.5.2/../../../../pic32mx/lib\libc.a(malloc.o)
                0xa0000368                __allocp
                0xa000036c                __alloct
                0xa0000370                __allocx
 .sbss          0xa0000378        0x4 c:/program files/microchip/xc32/v1.33/bin/bin/../../lib/gcc/pic32mx/4.5.2/../../../../pic32mx/lib\libc.a(errno.o)
                0xa0000378                errno
 .sbss          0xa000037c        0x8 c:/program files/microchip/xc32/v1.33/bin/bin/../../lib/gcc/pic32mx/4.5.2/../../../../pic32mx/lib\libpic32.a(sbrk.o)
                0xa000037c                _minbrk
                0xa0000380                _maxbrk
 *(.scommon)
 .scommon       0xa0000384        0x4 build/ChaletDuinoV2_775F512H_/debug/Source/winc3400/bsp/source/nm_bsp.o
                0xa0000384                at_sb_printf
 .scommon       0xa0000388        0x1 build/ChaletDuinoV2_775F512H_/debug/Source/winc3400/bus_wrapper/source/nm_bus_wrapper.o
                0xa0000388                mWifiSPIBaudrate
 .scommon       0xa0000389        0x0 build/ChaletDuinoV2_775F512H_/debug/Source/winc3400/common/source/nm_common.o
 .scommon       0xa0000389        0x0 build/ChaletDuinoV2_775F512H_/debug/Source/winc3400/driver/source/m2m_crypto.o
 .scommon       0xa0000389        0x0 build/ChaletDuinoV2_775F512H_/debug/Source/winc3400/driver/source/m2m_hif.o
 .scommon       0xa0000389        0x0 build/ChaletDuinoV2_775F512H_/debug/Source/winc3400/driver/source/m2m_ota.o
 .scommon       0xa0000389        0x0 build/ChaletDuinoV2_775F512H_/debug/Source/winc3400/driver/source/m2m_periph.o
 .scommon       0xa0000389        0x0 build/ChaletDuinoV2_775F512H_/debug/Source/winc3400/driver/source/m2m_ssl.o
 .scommon       0xa0000389        0x0 build/ChaletDuinoV2_775F512H_/debug/Source/winc3400/driver/source/m2m_wifi.o
 .scommon       0xa0000389        0x0 build/ChaletDuinoV2_775F512H_/debug/Source/winc3400/driver/source/nmasic.o
 .scommon       0xa0000389        0x0 build/ChaletDuinoV2_775F512H_/debug/Source/winc3400/driver/source/nmbus.o
 .scommon       0xa0000389        0x0 build/ChaletDuinoV2_775F512H_/debug/Source/winc3400/driver/source/nmdrv.o
 .scommon       0xa0000389        0x0 build/ChaletDuinoV2_775F512H_/debug/Source/winc3400/driver/source/nmi2c.o
 .scommon       0xa0000389        0x0 build/ChaletDuinoV2_775F512H_/debug/Source/winc3400/driver/source/nmspi.o
 .scommon       0xa0000389        0x0 build/ChaletDuinoV2_775F512H_/debug/Source/winc3400/driver/source/nmuart.o
 *fill*         0xa0000389        0x3 
 .scommon       0xa000038c       0x15 build/ChaletDuinoV2_775F512H_/debug/Source/winc3400/socket/source/socket.o
                0xa000038c                gpfAppResolveCb
                0xa0000390                gu16BufferSize
                0xa0000394                gpfAppSocketCb
                0xa0000398                gsockerrno
                0xa000039c                gfpPingCb
                0xa00003a0                gu8OpCode
 .scommon       0xa00003a1        0x0 build/ChaletDuinoV2_775F512H_/debug/Source/winc3400/spi_flash/source/spi_flash.o
 .scommon       0xa00003a1        0x0 build/ChaletDuinoV2_775F512H_/debug/Source/winc3400/winc_init.o
 *fill*         0xa00003a1        0x3 
 .scommon       0xa00003a4        0x2 build/ChaletDuinoV2_775F512H_/debug/Source/InternalUart.o
                0xa00003a4                acIntUartRxBuff
 *fill*         0xa00003a6        0x2 
 .scommon       0xa00003a8       0x14 build/ChaletDuinoV2_775F512H_/debug/Source/Terminal.o
                0xa00003a8                mTerminalOpened
                0xa00003ac                TerminalDataPtr
                0xa00003b0                mTerminalPendingAction
                0xa00003b4                mHelpStringPtr
                0xa00003b8                mTerminalTickState
 .scommon       0xa00003bc        0x4 build/ChaletDuinoV2_775F512H_/debug/Source/main.o
                0xa00003bc                ActualTemp
 .scommon       0xa00003c0        0xa build/ChaletDuinoV2_775F512H_/debug/Source/WiFiCtrl.o
                0xa00003c0                u8IsMacAddrValid
                0xa00003c4                mac_addr
 .scommon       0xa00003ca        0x0 build/ChaletDuinoV2_775F512H_/debug/Source/LoraNetworkInterface.o
 *fill*         0xa00003ca        0x2 
 .scommon       0xa00003cc        0x4 build/ChaletDuinoV2_775F512H_/debug/Source/ChaletPowerRelay.o
                0xa00003cc                PowerRelayState
 .scommon       0xa00003d0       0x18 build/ChaletDuinoV2_775F512H_/debug/Source/BatteryMonitor.o
                0xa00003d0                mBatteryCurrent
                0xa00003d4                mVoltageMeanSum
                0xa00003d8                mVoltageMeanCount
                0xa00003dc                mBatterySOC
                0xa00003e0                mBatteryVoltage
                0xa00003e4                mCurrentModuleOK
 .scommon       0xa00003e8        0x8 build/ChaletDuinoV2_775F512H_/debug/Source/I2C.o
                0xa00003e8                mLastTransactionOK
                0xa00003ec                mI2CWaitCounter
 .scommon       0xa00003f0        0x2 build/ChaletDuinoV2_775F512H_/debug/Source/SPI_Flash.o
                0xa00003f0                mSPIFlashHighSpeedBaudrate
                0xa00003f1                mSPIFlashBaudrate
 *fill*         0xa00003f2        0x2 
 .scommon       0xa00003f4        0x4 build/ChaletDuinoV2_775F512H_/debug/Source/Syslog.o
                0xa00003f4                mSyslogBufPtr
 .scommon       0xa00003f8       0x38 build/ChaletDuinoV2_775F512H_/debug/Source/BootloaderInterface.o
                0xa00003f8                CurDataChunkSize
                0xa00003fc                BootloaderFirmwareChunkWriteCount
                0xa0000400                BootloaderFlashWriteDataPtr
                0xa0000404                BootloaderFlashErased
                0xa0000408                BootloaderFlashWriteState
                0xa000040c                BootloaderCurFlashWriteAddress
                0xa0000410                BooloaderFlashEraseState
                0xa0000414                BootloaderCurFlashEraseAddress
                0xa0000418                BootloaderFlashWritePollCount
                0xa000041c                BootloaderInterfaceState
                0xa0000420                DataChunkWritten
                0xa0000424                BooloaderFlashErasePollCount
                0xa0000428                FirmwareUploaded
                0xa000042c                CurDataChunkIndex
 .scommon       0xa0000430        0x0 build/ChaletDuinoV2_775F512H_/debug/Source/TemperatureSensor.o
 .scommon       0xa0000430        0x2 build/ChaletDuinoV2_775F512H_/debug/Source/TC77.o
                0xa0000430                mDeviceID
 *fill*         0xa0000432        0x2 
 .scommon       0xa0000434        0x4 build/ChaletDuinoV2_775F512H_/debug/Source/BootloaderProtocol.o
                0xa0000434                BootloaderRxPtr
                0xa0000438                _sbss_end = .
                0xa0000438                . = ALIGN (0x4)

.bss            0xa0000438     0x2e30
 *(.dynbss)
 *(COMMON)
 COMMON         0xa0000438       0xb0 build/ChaletDuinoV2_775F512H_/debug/Source/winc3400/socket/source/socket.o
                0xa0000438                gastrSockets
 COMMON         0xa00004e8       0x40 build/ChaletDuinoV2_775F512H_/debug/Source/InternalUart.o
                0xa00004e8                astInternalUartData
 COMMON         0xa0000528      0x26e build/ChaletDuinoV2_775F512H_/debug/Source/NetworkProtocol.o
                0xa0000528                mRxData
                0xa0000660                mTxData
 *fill*         0xa0000796        0x2 
 COMMON         0xa0000798      0x384 build/ChaletDuinoV2_775F512H_/debug/Source/Terminal.o
                0xa0000798                TerminalWorkString
                0xa00008c4                TerminalPrevDataBuf
                0xa00009f0                TerminalDataBuf
 COMMON         0xa0000b1c      0x620 build/ChaletDuinoV2_775F512H_/debug/Source/Uart.o
                0xa0000b1c                astUartData
 COMMON         0xa000113c       0xf0 build/ChaletDuinoV2_775F512H_/debug/Source/timer.o
                0xa000113c                astTimer
 COMMON         0xa000122c      0xd04 build/ChaletDuinoV2_775F512H_/debug/Source/WiFiCtrl.o
                0xa000122c                NetworkRxBuf
                0xa000162c                TerminalRxBuf
                0xa0001a2c                BootloaderRxBuf
                0xa0001e2c                addr_in
                0xa0001e3c                param
                0xa0001e58                mModuleIPConfig
                0xa0001e68                SyslogRxBuf
 COMMON         0xa0001f30       0x16 build/ChaletDuinoV2_775F512H_/debug/Source/ina219.o
                0xa0001f30                I2CSlaveBuffer
                0xa0001f3c                I2CMasterBuffer
 *fill*         0xa0001f46        0x2 
 COMMON         0xa0001f48     0x1000 build/ChaletDuinoV2_775F512H_/debug/Source/SPI_Flash.o
                0xa0001f48                mFlashSectorBuffer
 COMMON         0xa0002f48      0x1f4 build/ChaletDuinoV2_775F512H_/debug/Source/Syslog.o
                0xa0002f48                mSyslogBuffer
 COMMON         0xa000313c      0x12c build/ChaletDuinoV2_775F512H_/debug/Source/BootloaderInterface.o
                0xa000313c                BootloaderBuffer
                0xa0003268                . = ALIGN ((. != 0x0)?0x4:0x1)
                0xa0003268                . = ALIGN (0x4)
                0xa0003268                _end = .
                0xa0003268                _bss_end = .
                0x00010000                _bmxdudba_address = 0x10000
                0x00010000                _bmxdupba_address = 0x10000

/DISCARD/
 *(.pdr)
 *(.rel.dyn)
 *(.note.GNU-stack)
 *(.note.GNU-stack)
 *(.gnu_debuglink)
 *(.gnu.lto_*)
 *(.discard)

.gptab.sdata
 *(.gptab.data)
 *(.gptab.sdata)

.gptab.sbss
 *(.gptab.bss)
 *(.gptab.sbss)

.mdebug.abi32   0xa0003268        0x0
 *(.mdebug.abi32)
 .mdebug.abi32  0xa0003268        0x0 c:/program files/microchip/xc32/v1.33/bin/bin/../../lib/gcc/pic32mx/4.5.2/../../../../pic32mx/lib\software-debug-break.o
 .mdebug.abi32  0xa0003268        0x0 build/ChaletDuinoV2_775F512H_/debug/Source/ChaletduinoV2Board.o
 .mdebug.abi32  0xa0003268        0x0 build/ChaletDuinoV2_775F512H_/debug/Source/winc3400/bsp/source/nm_bsp.o
 .mdebug.abi32  0xa0003268        0x0 build/ChaletDuinoV2_775F512H_/debug/Source/winc3400/bus_wrapper/source/nm_bus_wrapper.o
 .mdebug.abi32  0xa0003268        0x0 build/ChaletDuinoV2_775F512H_/debug/Source/winc3400/common/source/nm_common.o
 .mdebug.abi32  0xa0003268        0x0 build/ChaletDuinoV2_775F512H_/debug/Source/winc3400/driver/source/m2m_ate_mode.o
 .mdebug.abi32  0xa0003268        0x0 build/ChaletDuinoV2_775F512H_/debug/Source/winc3400/driver/source/m2m_crypto.o
 .mdebug.abi32  0xa0003268        0x0 build/ChaletDuinoV2_775F512H_/debug/Source/winc3400/driver/source/m2m_hif.o
 .mdebug.abi32  0xa0003268        0x0 build/ChaletDuinoV2_775F512H_/debug/Source/winc3400/driver/source/m2m_ota.o
 .mdebug.abi32  0xa0003268        0x0 build/ChaletDuinoV2_775F512H_/debug/Source/winc3400/driver/source/m2m_periph.o
 .mdebug.abi32  0xa0003268        0x0 build/ChaletDuinoV2_775F512H_/debug/Source/winc3400/driver/source/m2m_ssl.o
 .mdebug.abi32  0xa0003268        0x0 build/ChaletDuinoV2_775F512H_/debug/Source/winc3400/driver/source/m2m_wifi.o
 .mdebug.abi32  0xa0003268        0x0 build/ChaletDuinoV2_775F512H_/debug/Source/winc3400/driver/source/nmasic.o
 .mdebug.abi32  0xa0003268        0x0 build/ChaletDuinoV2_775F512H_/debug/Source/winc3400/driver/source/nmbus.o
 .mdebug.abi32  0xa0003268        0x0 build/ChaletDuinoV2_775F512H_/debug/Source/winc3400/driver/source/nmdrv.o
 .mdebug.abi32  0xa0003268        0x0 build/ChaletDuinoV2_775F512H_/debug/Source/winc3400/driver/source/nmi2c.o
 .mdebug.abi32  0xa0003268        0x0 build/ChaletDuinoV2_775F512H_/debug/Source/winc3400/driver/source/nmspi.o
 .mdebug.abi32  0xa0003268        0x0 build/ChaletDuinoV2_775F512H_/debug/Source/winc3400/driver/source/nmuart.o
 .mdebug.abi32  0xa0003268        0x0 build/ChaletDuinoV2_775F512H_/debug/Source/winc3400/socket/source/socket.o
 .mdebug.abi32  0xa0003268        0x0 build/ChaletDuinoV2_775F512H_/debug/Source/winc3400/spi_flash/source/spi_flash.o
 .mdebug.abi32  0xa0003268        0x0 build/ChaletDuinoV2_775F512H_/debug/Source/winc3400/winc_init.o
 .mdebug.abi32  0xa0003268        0x0 build/ChaletDuinoV2_775F512H_/debug/Source/DigitalIO.o
 .mdebug.abi32  0xa0003268        0x0 build/ChaletDuinoV2_775F512H_/debug/Source/InternalUart.o
 .mdebug.abi32  0xa0003268        0x0 build/ChaletDuinoV2_775F512H_/debug/Source/NetworkProtocol.o
 .mdebug.abi32  0xa0003268        0x0 build/ChaletDuinoV2_775F512H_/debug/Source/Terminal.o
 .mdebug.abi32  0xa0003268        0x0 build/ChaletDuinoV2_775F512H_/debug/Source/Uart.o
 .mdebug.abi32  0xa0003268        0x0 build/ChaletDuinoV2_775F512H_/debug/Source/Util.o
 .mdebug.abi32  0xa0003268        0x0 build/ChaletDuinoV2_775F512H_/debug/Source/exceptions.o
 .mdebug.abi32  0xa0003268        0x0 build/ChaletDuinoV2_775F512H_/debug/Source/interrupts.o
 .mdebug.abi32  0xa0003268        0x0 build/ChaletDuinoV2_775F512H_/debug/Source/main.o
 .mdebug.abi32  0xa0003268        0x0 build/ChaletDuinoV2_775F512H_/debug/Source/system.o
 .mdebug.abi32  0xa0003268        0x0 build/ChaletDuinoV2_775F512H_/debug/Source/template.o
 .mdebug.abi32  0xa0003268        0x0 build/ChaletDuinoV2_775F512H_/debug/Source/timer.o
 .mdebug.abi32  0xa0003268        0x0 build/ChaletDuinoV2_775F512H_/debug/Source/WiFiCtrl.o
 .mdebug.abi32  0xa0003268        0x0 build/ChaletDuinoV2_775F512H_/debug/Source/SPI.o
 .mdebug.abi32  0xa0003268        0x0 build/ChaletDuinoV2_775F512H_/debug/Source/LoraNetworkInterface.o
 .mdebug.abi32  0xa0003268        0x0 build/ChaletDuinoV2_775F512H_/debug/Source/ChaletPowerRelay.o
 .mdebug.abi32  0xa0003268        0x0 build/ChaletDuinoV2_775F512H_/debug/Source/HarakiriRelay.o
 .mdebug.abi32  0xa0003268        0x0 build/ChaletDuinoV2_775F512H_/debug/Source/BatteryMonitor.o
 .mdebug.abi32  0xa0003268        0x0 build/ChaletDuinoV2_775F512H_/debug/Source/ina219.o
 .mdebug.abi32  0xa0003268        0x0 build/ChaletDuinoV2_775F512H_/debug/Source/I2C.o
 .mdebug.abi32  0xa0003268        0x0 build/ChaletDuinoV2_775F512H_/debug/Source/SPI_Flash.o
 .mdebug.abi32  0xa0003268        0x0 build/ChaletDuinoV2_775F512H_/debug/Source/Syslog.o
 .mdebug.abi32  0xa0003268        0x0 build/ChaletDuinoV2_775F512H_/debug/Source/Watchdog.o
 .mdebug.abi32  0xa0003268        0x0 build/ChaletDuinoV2_775F512H_/debug/Source/BootloaderInterface.o
 .mdebug.abi32  0xa0003268        0x0 build/ChaletDuinoV2_775F512H_/debug/Source/TemperatureSensor.o
 .mdebug.abi32  0xa0003268        0x0 build/ChaletDuinoV2_775F512H_/debug/Source/TC77.o
 .mdebug.abi32  0xa0003268        0x0 build/ChaletDuinoV2_775F512H_/debug/Source/BootloaderProtocol.o
 .mdebug.abi32  0xa0003268        0x0 build/ChaletDuinoV2_775F512H_/debug/Source/crc32.o
 .mdebug.abi32  0xa0003268        0x0 c:/program files/microchip/xc32/v1.33/bin/bin/../../lib/gcc/pic32mx/4.5.2/../../../../pic32mx/lib\libmchp_peripheral_32MX795F512H.a(soft_reset_lib.o)
 .mdebug.abi32  0xa0003268        0x0 c:/program files/microchip/xc32/v1.33/bin/bin/../../lib/gcc/pic32mx/4.5.2/../../../../pic32mx/lib\libmchp_peripheral_32MX795F512H.a(pcache.o)
 .mdebug.abi32  0xa0003268        0x0 c:/program files/microchip/xc32/v1.33/bin/bin/../../lib/gcc/pic32mx/4.5.2/../../../../pic32mx/lib\libmchp_peripheral_32MX795F512H.a(int_configure_system_lib.o)
 .mdebug.abi32  0xa0003268        0x0 c:/program files/microchip/xc32/v1.33/bin/bin/../../lib/gcc/pic32mx/4.5.2/../../../../pic32mx/lib\libmchp_peripheral_32MX795F512H.a(int_enable_interrupts_lib.o)
 .mdebug.abi32  0xa0003268        0x0 c:/program files/microchip/xc32/v1.33/bin/bin/../../lib/gcc/pic32mx/4.5.2/../../../../pic32mx/lib\libmchp_peripheral_32MX795F512H.a(int_disable_interrupts_lib.o)
 .mdebug.abi32  0xa0003268        0x0 c:/program files/microchip/xc32/v1.33/bin/bin/../../lib/gcc/pic32mx/4.5.2/../../../../pic32mx/lib\libmchp_peripheral_32MX795F512H.a(int_restore_interrupts_lib.o)
 .mdebug.abi32  0xa0003268        0x0 c:/program files/microchip/xc32/v1.33/bin/bin/../../lib/gcc/pic32mx/4.5.2/../../../../pic32mx/lib\libpic32.a(default-bootstrap-exception-handler.o)
 .mdebug.abi32  0xa0003268        0x0 c:/program files/microchip/xc32/v1.33/bin/bin/../../lib/gcc/pic32mx/4.5.2/../../../../pic32mx/lib\libpic32.a(default-on-reset.o)
 .mdebug.abi32  0xa0003268        0x0 c:/program files/microchip/xc32/v1.33/bin/bin/../../lib/gcc/pic32mx/4.5.2/../../../../pic32mx/lib\libpic32.a(default-on-bootstrap.o)
 .mdebug.abi32  0xa0003268        0x0 c:/program files/microchip/xc32/v1.33/bin/bin/../../lib/gcc/pic32mx/4.5.2/../../../../pic32mx/lib\libpic32.a(defaultinterrupt.o)
 .mdebug.abi32  0xa0003268        0x0 c:/program files/microchip/xc32/v1.33/bin/bin/../../lib/gcc/pic32mx/4.5.2/../../../../pic32mx/lib\libc.a(_iob.o)
 .mdebug.abi32  0xa0003268        0x0 c:/program files/microchip/xc32/v1.33/bin/bin/../../lib/gcc/pic32mx/4.5.2/../../../../pic32mx/lib\libc.a(fflush.o)
 .mdebug.abi32  0xa0003268        0x0 c:/program files/microchip/xc32/v1.33/bin/bin/../../lib/gcc/pic32mx/4.5.2/../../../../pic32mx/lib\libc.a(malloc.o)
 .mdebug.abi32  0xa0003268        0x0 c:/program files/microchip/xc32/v1.33/bin/bin/../../lib/gcc/pic32mx/4.5.2/../../../../pic32mx/lib\libc.a(puts.o)
 .mdebug.abi32  0xa0003268        0x0 c:/program files/microchip/xc32/v1.33/bin/bin/../../lib/gcc/pic32mx/4.5.2/../../../../pic32mx/lib\libc.a(setbuf.o)
 .mdebug.abi32  0xa0003268        0x0 c:/program files/microchip/xc32/v1.33/bin/bin/../../lib/gcc/pic32mx/4.5.2/../../../../pic32mx/lib\libc.a(strncmp.o)
 .mdebug.abi32  0xa0003268        0x0 c:/program files/microchip/xc32/v1.33/bin/bin/../../lib/gcc/pic32mx/4.5.2/../../../../pic32mx/lib\libc.a(printf_cdfFnopsuxX.eo)
 .mdebug.abi32  0xa0003268        0x0 c:/program files/microchip/xc32/v1.33/bin/bin/../../lib/gcc/pic32mx/4.5.2/../../../../pic32mx/lib\libc.a(sprintf_cdfFnopuxX.eo)
 .mdebug.abi32  0xa0003268        0x0 c:/program files/microchip/xc32/v1.33/bin/bin/../../lib/gcc/pic32mx/4.5.2/../../../../pic32mx/lib\libc.a(sscanf_s.eo)
 .mdebug.abi32  0xa0003268        0x0 c:/program files/microchip/xc32/v1.33/bin/bin/../../lib/gcc/pic32mx/4.5.2/../../../../pic32mx/lib\libc.a(_fputc_simple.o)
 .mdebug.abi32  0xa0003268        0x0 c:/program files/microchip/xc32/v1.33/bin/bin/../../lib/gcc/pic32mx/4.5.2/../../../../pic32mx/lib\libc.a(buf.o)
 .mdebug.abi32  0xa0003268        0x0 c:/program files/microchip/xc32/v1.33/bin/bin/../../lib/gcc/pic32mx/4.5.2/../../../../pic32mx/lib\libc.a(errno.o)
 .mdebug.abi32  0xa0003268        0x0 c:/program files/microchip/xc32/v1.33/bin/bin/../../lib/gcc/pic32mx/4.5.2/../../../../pic32mx/lib\libc.a(doprnt_cdfFnopsuxX.eo)
 .mdebug.abi32  0xa0003268        0x0 c:/program files/microchip/xc32/v1.33/bin/bin/../../lib/gcc/pic32mx/4.5.2/../../../../pic32mx/lib\libc.a(doscan_s.eo)
 .mdebug.abi32  0xa0003268        0x0 c:/program files/microchip/xc32/v1.33/bin/bin/../../lib/gcc/pic32mx/4.5.2/../../../../pic32mx/lib\libc.a(_flsbuf_simple.o)
 .mdebug.abi32  0xa0003268        0x0 c:/program files/microchip/xc32/v1.33/bin/bin/../../lib/gcc/pic32mx/4.5.2/../../../../pic32mx/lib\libc.a(fgetc.o)
 .mdebug.abi32  0xa0003268        0x0 c:/program files/microchip/xc32/v1.33/bin/bin/../../lib/gcc/pic32mx/4.5.2/../../../../pic32mx/lib\libc.a(atoi.o)
 .mdebug.abi32  0xa0003268        0x0 c:/program files/microchip/xc32/v1.33/bin/bin/../../lib/gcc/pic32mx/4.5.2/../../../../pic32mx/lib\libc.a(ctype.o)
 .mdebug.abi32  0xa0003268        0x0 c:/program files/microchip/xc32/v1.33/bin/bin/../../lib/gcc/pic32mx/4.5.2/../../../../pic32mx/lib\libc.a(ctypef.o)
 .mdebug.abi32  0xa0003268        0x0 c:/program files/microchip/xc32/v1.33/bin/bin/../../lib/gcc/pic32mx/4.5.2/../../../../pic32mx/lib\libc.a(powersf.o)
 .mdebug.abi32  0xa0003268        0x0 c:/program files/microchip/xc32/v1.33/bin/bin/../../lib/gcc/pic32mx/4.5.2/../../../../pic32mx/lib\libc.a(ungetc.o)
 .mdebug.abi32  0xa0003268        0x0 c:/program files/microchip/xc32/v1.33/bin/bin/../../lib/gcc/pic32mx/4.5.2/../../../../pic32mx/lib\libc.a(filbuf.o)
 .mdebug.abi32  0xa0003268        0x0 c:/program files/microchip/xc32/v1.33/bin/bin/../../lib/gcc/pic32mx/4.5.2/../../../../pic32mx/lib\libpic32.a(sbrk.o)
 .mdebug.abi32  0xa0003268        0x0 c:/program files/microchip/xc32/v1.33/bin/bin/../../lib/gcc/pic32mx/4.5.2/../../../../pic32mx/lib\libpic32.a(read.o)
 .mdebug.abi32  0xa0003268        0x0 c:/program files/microchip/xc32/v1.33/bin/bin/../../lib/gcc/pic32mx/4.5.2/../../../../pic32mx/lib\libpic32.a(write.o)
 .mdebug.abi32  0xa0003268        0x0 c:/program files/microchip/xc32/v1.33/bin/bin/../../lib/gcc/pic32mx/4.5.2/../../../../pic32mx/lib\libpic32.a(xc32_uart.o)
 .mdebug.abi32  0xa0003268        0x0 c:/program files/microchip/xc32/v1.33/bin/bin/../../lib/gcc/pic32mx/4.5.2/../../../../pic32mx/lib\libe.a(_floatdisf.o)
 .mdebug.abi32  0xa0003268        0x0 c:/program files/microchip/xc32/v1.33/bin/bin/../../lib/gcc/pic32mx/4.5.2\libgcc.a(_floatundisf.o)
 .mdebug.abi32  0xa0003268        0x0 c:/program files/microchip/xc32/v1.33/bin/bin/../../lib/gcc/pic32mx/4.5.2\libgcc.a(_udivdi3.o)
 .mdebug.abi32  0xa0003268        0x0 c:/program files/microchip/xc32/v1.33/bin/bin/../../lib/gcc/pic32mx/4.5.2\libgcc.a(_umoddi3.o)
 .mdebug.abi32  0xa0003268        0x0 c:/program files/microchip/xc32/v1.33/bin/bin/../../lib/gcc/pic32mx/4.5.2\libgcc.a(floatunsisf.o)

.mdebug.abiN32
 *(.mdebug.abiN32)

.mdebug.abi64
 *(.mdebug.abi64)

.mdebug.abiO64
 *(.mdebug.abiO64)

.mdebug.eabi32
 *(.mdebug.eabi32)

.mdebug.eabi64
 *(.mdebug.eabi64)

.gcc_compiled_long32
 *(.gcc_compiled_long32)

.gcc_compiled_long64
 *(.gcc_compiled_long64)

.stab
 *(.stab)

.stabstr
 *(.stabstr)

.stab.excl
 *(.stab.excl)

.stab.exclstr
 *(.stab.exclstr)

.stab.index
 *(.stab.index)

.stab.indexstr
 *(.stab.indexstr)

.comment        0x00000000      0x248
 *(.comment)
 .comment       0x00000000       0x3c c:/program files/microchip/xc32/v1.33/bin/bin/../../lib/gcc/pic32mx/4.5.2/../../../../pic32mx/lib\software-debug-break.o
                                 0x3d (size before relaxing)
 .comment       0x00000000       0x3d build/ChaletDuinoV2_775F512H_/debug/Source/ChaletduinoV2Board.o
 .comment       0x00000000       0x3d build/ChaletDuinoV2_775F512H_/debug/Source/winc3400/bsp/source/nm_bsp.o
 .comment       0x00000000       0x3d build/ChaletDuinoV2_775F512H_/debug/Source/winc3400/bus_wrapper/source/nm_bus_wrapper.o
 .comment       0x00000000       0x3d build/ChaletDuinoV2_775F512H_/debug/Source/winc3400/common/source/nm_common.o
 .comment       0x00000000       0x3d build/ChaletDuinoV2_775F512H_/debug/Source/winc3400/driver/source/m2m_ate_mode.o
 .comment       0x00000000       0x3d build/ChaletDuinoV2_775F512H_/debug/Source/winc3400/driver/source/m2m_crypto.o
 .comment       0x00000000       0x3d build/ChaletDuinoV2_775F512H_/debug/Source/winc3400/driver/source/m2m_hif.o
 .comment       0x00000000       0x3d build/ChaletDuinoV2_775F512H_/debug/Source/winc3400/driver/source/m2m_ota.o
 .comment       0x00000000       0x3d build/ChaletDuinoV2_775F512H_/debug/Source/winc3400/driver/source/m2m_periph.o
 .comment       0x00000000       0x3d build/ChaletDuinoV2_775F512H_/debug/Source/winc3400/driver/source/m2m_ssl.o
 .comment       0x00000000       0x3d build/ChaletDuinoV2_775F512H_/debug/Source/winc3400/driver/source/m2m_wifi.o
 .comment       0x00000000       0x3d build/ChaletDuinoV2_775F512H_/debug/Source/winc3400/driver/source/nmasic.o
 .comment       0x00000000       0x3d build/ChaletDuinoV2_775F512H_/debug/Source/winc3400/driver/source/nmbus.o
 .comment       0x00000000       0x3d build/ChaletDuinoV2_775F512H_/debug/Source/winc3400/driver/source/nmdrv.o
 .comment       0x00000000       0x3d build/ChaletDuinoV2_775F512H_/debug/Source/winc3400/driver/source/nmi2c.o
 .comment       0x00000000       0x3d build/ChaletDuinoV2_775F512H_/debug/Source/winc3400/driver/source/nmspi.o
 .comment       0x00000000       0x3d build/ChaletDuinoV2_775F512H_/debug/Source/winc3400/driver/source/nmuart.o
 .comment       0x00000000       0x3d build/ChaletDuinoV2_775F512H_/debug/Source/winc3400/socket/source/socket.o
 .comment       0x00000000       0x3d build/ChaletDuinoV2_775F512H_/debug/Source/winc3400/spi_flash/source/spi_flash.o
 .comment       0x00000000       0x3d build/ChaletDuinoV2_775F512H_/debug/Source/winc3400/winc_init.o
 .comment       0x00000000       0x3d build/ChaletDuinoV2_775F512H_/debug/Source/DigitalIO.o
 .comment       0x00000000       0x3d build/ChaletDuinoV2_775F512H_/debug/Source/InternalUart.o
 .comment       0x00000000       0x3d build/ChaletDuinoV2_775F512H_/debug/Source/NetworkProtocol.o
 .comment       0x00000000       0x3d build/ChaletDuinoV2_775F512H_/debug/Source/Terminal.o
 .comment       0x00000000       0x3d build/ChaletDuinoV2_775F512H_/debug/Source/Uart.o
 .comment       0x00000000       0x3d build/ChaletDuinoV2_775F512H_/debug/Source/Util.o
 .comment       0x00000000       0x3d build/ChaletDuinoV2_775F512H_/debug/Source/exceptions.o
 .comment       0x00000000       0x3d build/ChaletDuinoV2_775F512H_/debug/Source/interrupts.o
 .comment       0x00000000       0x3d build/ChaletDuinoV2_775F512H_/debug/Source/main.o
 .comment       0x00000000       0x3d build/ChaletDuinoV2_775F512H_/debug/Source/system.o
 .comment       0x00000000       0x3d build/ChaletDuinoV2_775F512H_/debug/Source/template.o
 .comment       0x00000000       0x3d build/ChaletDuinoV2_775F512H_/debug/Source/timer.o
 .comment       0x00000000       0x3d build/ChaletDuinoV2_775F512H_/debug/Source/WiFiCtrl.o
 .comment       0x00000000       0x3d build/ChaletDuinoV2_775F512H_/debug/Source/SPI.o
 .comment       0x00000000       0x3d build/ChaletDuinoV2_775F512H_/debug/Source/LoraNetworkInterface.o
 .comment       0x00000000       0x3d build/ChaletDuinoV2_775F512H_/debug/Source/ChaletPowerRelay.o
 .comment       0x00000000       0x3d build/ChaletDuinoV2_775F512H_/debug/Source/HarakiriRelay.o
 .comment       0x00000000       0x3d build/ChaletDuinoV2_775F512H_/debug/Source/BatteryMonitor.o
 .comment       0x00000000       0x3d build/ChaletDuinoV2_775F512H_/debug/Source/ina219.o
 .comment       0x00000000       0x3d build/ChaletDuinoV2_775F512H_/debug/Source/I2C.o
 .comment       0x00000000       0x3d build/ChaletDuinoV2_775F512H_/debug/Source/SPI_Flash.o
 .comment       0x00000000       0x3d build/ChaletDuinoV2_775F512H_/debug/Source/Syslog.o
 .comment       0x00000000       0x3d build/ChaletDuinoV2_775F512H_/debug/Source/Watchdog.o
 .comment       0x00000000       0x3d build/ChaletDuinoV2_775F512H_/debug/Source/BootloaderInterface.o
 .comment       0x00000000       0x3d build/ChaletDuinoV2_775F512H_/debug/Source/TemperatureSensor.o
 .comment       0x00000000       0x3d build/ChaletDuinoV2_775F512H_/debug/Source/TC77.o
 .comment       0x00000000       0x3d build/ChaletDuinoV2_775F512H_/debug/Source/BootloaderProtocol.o
 .comment       0x00000000       0x3d build/ChaletDuinoV2_775F512H_/debug/Source/crc32.o
 .comment       0x0000003c       0x3c c:/program files/microchip/xc32/v1.33/bin/bin/../../lib/gcc/pic32mx/4.5.2/../../../../pic32mx/lib\libmchp_peripheral_32MX795F512H.a(soft_reset_lib.o)
                                 0x3d (size before relaxing)
 .comment       0x00000000       0x3d c:/program files/microchip/xc32/v1.33/bin/bin/../../lib/gcc/pic32mx/4.5.2/../../../../pic32mx/lib\libmchp_peripheral_32MX795F512H.a(pcache.o)
 .comment       0x00000000       0x3d c:/program files/microchip/xc32/v1.33/bin/bin/../../lib/gcc/pic32mx/4.5.2/../../../../pic32mx/lib\libmchp_peripheral_32MX795F512H.a(int_configure_system_lib.o)
 .comment       0x00000000       0x3d c:/program files/microchip/xc32/v1.33/bin/bin/../../lib/gcc/pic32mx/4.5.2/../../../../pic32mx/lib\libmchp_peripheral_32MX795F512H.a(int_enable_interrupts_lib.o)
 .comment       0x00000000       0x3d c:/program files/microchip/xc32/v1.33/bin/bin/../../lib/gcc/pic32mx/4.5.2/../../../../pic32mx/lib\libmchp_peripheral_32MX795F512H.a(int_disable_interrupts_lib.o)
 .comment       0x00000000       0x3d c:/program files/microchip/xc32/v1.33/bin/bin/../../lib/gcc/pic32mx/4.5.2/../../../../pic32mx/lib\libmchp_peripheral_32MX795F512H.a(int_restore_interrupts_lib.o)
 .comment       0x00000078       0x18 c:/program files/microchip/xc32/v1.33/bin/bin/../../lib/gcc/pic32mx/4.5.2/../../../../pic32mx/lib\libpic32.a(memset.o)
                                 0x19 (size before relaxing)
 .comment       0x00000090       0x19 c:/program files/microchip/xc32/v1.33/bin/bin/../../lib/gcc/pic32mx/4.5.2/../../../../pic32mx/lib\libpic32.a(strcpy.o)
                                 0x1a (size before relaxing)
 .comment       0x000000a9       0x19 c:/program files/microchip/xc32/v1.33/bin/bin/../../lib/gcc/pic32mx/4.5.2/../../../../pic32mx/lib\libpic32.a(strlen.o)
                                 0x1a (size before relaxing)
 .comment       0x00000000       0x3d c:/program files/microchip/xc32/v1.33/bin/bin/../../lib/gcc/pic32mx/4.5.2/../../../../pic32mx/lib\libpic32.a(default-bootstrap-exception-handler.o)
 .comment       0x00000000       0x3d c:/program files/microchip/xc32/v1.33/bin/bin/../../lib/gcc/pic32mx/4.5.2/../../../../pic32mx/lib\libpic32.a(default-on-reset.o)
 .comment       0x00000000       0x3d c:/program files/microchip/xc32/v1.33/bin/bin/../../lib/gcc/pic32mx/4.5.2/../../../../pic32mx/lib\libpic32.a(default-on-bootstrap.o)
 .comment       0x00000000       0x3d c:/program files/microchip/xc32/v1.33/bin/bin/../../lib/gcc/pic32mx/4.5.2/../../../../pic32mx/lib\libpic32.a(defaultinterrupt.o)
 .comment       0x00000000       0x3d c:/program files/microchip/xc32/v1.33/bin/bin/../../lib/gcc/pic32mx/4.5.2/../../../../pic32mx/lib\libc.a(_iob.o)
 .comment       0x00000000       0x3d c:/program files/microchip/xc32/v1.33/bin/bin/../../lib/gcc/pic32mx/4.5.2/../../../../pic32mx/lib\libc.a(fflush.o)
 .comment       0x00000000       0x3d c:/program files/microchip/xc32/v1.33/bin/bin/../../lib/gcc/pic32mx/4.5.2/../../../../pic32mx/lib\libc.a(malloc.o)
 .comment       0x00000000       0x3d c:/program files/microchip/xc32/v1.33/bin/bin/../../lib/gcc/pic32mx/4.5.2/../../../../pic32mx/lib\libc.a(puts.o)
 .comment       0x00000000       0x3d c:/program files/microchip/xc32/v1.33/bin/bin/../../lib/gcc/pic32mx/4.5.2/../../../../pic32mx/lib\libc.a(setbuf.o)
 .comment       0x00000000       0x3d c:/program files/microchip/xc32/v1.33/bin/bin/../../lib/gcc/pic32mx/4.5.2/../../../../pic32mx/lib\libc.a(strncmp.o)
 .comment       0x00000000       0x3d c:/program files/microchip/xc32/v1.33/bin/bin/../../lib/gcc/pic32mx/4.5.2/../../../../pic32mx/lib\libc.a(printf_cdfFnopsuxX.eo)
 .comment       0x00000000       0x3d c:/program files/microchip/xc32/v1.33/bin/bin/../../lib/gcc/pic32mx/4.5.2/../../../../pic32mx/lib\libc.a(sprintf_cdfFnopuxX.eo)
 .comment       0x00000000       0x3d c:/program files/microchip/xc32/v1.33/bin/bin/../../lib/gcc/pic32mx/4.5.2/../../../../pic32mx/lib\libc.a(sscanf_s.eo)
 .comment       0x00000000       0x3d c:/program files/microchip/xc32/v1.33/bin/bin/../../lib/gcc/pic32mx/4.5.2/../../../../pic32mx/lib\libc.a(_fputc_simple.o)
 .comment       0x00000000       0x3d c:/program files/microchip/xc32/v1.33/bin/bin/../../lib/gcc/pic32mx/4.5.2/../../../../pic32mx/lib\libc.a(buf.o)
 .comment       0x00000000       0x3d c:/program files/microchip/xc32/v1.33/bin/bin/../../lib/gcc/pic32mx/4.5.2/../../../../pic32mx/lib\libc.a(errno.o)
 .comment       0x00000000       0x3d c:/program files/microchip/xc32/v1.33/bin/bin/../../lib/gcc/pic32mx/4.5.2/../../../../pic32mx/lib\libc.a(doprnt_cdfFnopsuxX.eo)
 .comment       0x00000000       0x3d c:/program files/microchip/xc32/v1.33/bin/bin/../../lib/gcc/pic32mx/4.5.2/../../../../pic32mx/lib\libc.a(doscan_s.eo)
 .comment       0x00000000       0x3d c:/program files/microchip/xc32/v1.33/bin/bin/../../lib/gcc/pic32mx/4.5.2/../../../../pic32mx/lib\libc.a(_flsbuf_simple.o)
 .comment       0x00000000       0x3d c:/program files/microchip/xc32/v1.33/bin/bin/../../lib/gcc/pic32mx/4.5.2/../../../../pic32mx/lib\libc.a(fgetc.o)
 .comment       0x00000000       0x3d c:/program files/microchip/xc32/v1.33/bin/bin/../../lib/gcc/pic32mx/4.5.2/../../../../pic32mx/lib\libc.a(atoi.o)
 .comment       0x000000c2       0x4e c:/program files/microchip/xc32/v1.33/bin/bin/../../lib/gcc/pic32mx/4.5.2/../../../../pic32mx/lib\libc.a(ctype.o)
                                 0x8b (size before relaxing)
 .comment       0x00000110       0x4f c:/program files/microchip/xc32/v1.33/bin/bin/../../lib/gcc/pic32mx/4.5.2/../../../../pic32mx/lib\libc.a(ctypef.o)
                                 0x8c (size before relaxing)
 .comment       0x00000000       0x3d c:/program files/microchip/xc32/v1.33/bin/bin/../../lib/gcc/pic32mx/4.5.2/../../../../pic32mx/lib\libc.a(powersf.o)
 .comment       0x00000000       0x3d c:/program files/microchip/xc32/v1.33/bin/bin/../../lib/gcc/pic32mx/4.5.2/../../../../pic32mx/lib\libc.a(ungetc.o)
 .comment       0x00000000       0x3d c:/program files/microchip/xc32/v1.33/bin/bin/../../lib/gcc/pic32mx/4.5.2/../../../../pic32mx/lib\libc.a(filbuf.o)
 .comment       0x0000015f       0x4b c:/program files/microchip/xc32/v1.33/bin/bin/../../lib/gcc/pic32mx/4.5.2/../../../../pic32mx/lib\libpic32.a(sbrk.o)
                                 0x88 (size before relaxing)
 .comment       0x00000000       0x3d c:/program files/microchip/xc32/v1.33/bin/bin/../../lib/gcc/pic32mx/4.5.2/../../../../pic32mx/lib\libpic32.a(read.o)
 .comment       0x00000000       0x3d c:/program files/microchip/xc32/v1.33/bin/bin/../../lib/gcc/pic32mx/4.5.2/../../../../pic32mx/lib\libpic32.a(write.o)
 .comment       0x00000000       0x3d c:/program files/microchip/xc32/v1.33/bin/bin/../../lib/gcc/pic32mx/4.5.2/../../../../pic32mx/lib\libpic32.a(xc32_uart.o)
 .comment       0x000001aa       0x9e c:/program files/microchip/xc32/v1.33/bin/bin/../../lib/gcc/pic32mx/4.5.2/../../../../pic32mx/lib\libe.a(_floatdisf.o)
                                 0xdb (size before relaxing)
 .comment       0x00000000       0x3d c:/program files/microchip/xc32/v1.33/bin/bin/../../lib/gcc/pic32mx/4.5.2\libgcc.a(_floatundisf.o)
 .comment       0x00000000       0x3d c:/program files/microchip/xc32/v1.33/bin/bin/../../lib/gcc/pic32mx/4.5.2\libgcc.a(_udivdi3.o)
 .comment       0x00000000       0x3d c:/program files/microchip/xc32/v1.33/bin/bin/../../lib/gcc/pic32mx/4.5.2\libgcc.a(_umoddi3.o)
 .comment       0x00000000       0x3d c:/program files/microchip/xc32/v1.33/bin/bin/../../lib/gcc/pic32mx/4.5.2\libgcc.a(floatunsisf.o)

.debug
 *(.debug)

.line
 *(.line)

.debug_srcinfo
 *(.debug_srcinfo)

.debug_sfnames
 *(.debug_sfnames)

.debug_aranges  0x00000000      0xaa8
 *(.debug_aranges)
 .debug_aranges
                0x00000000       0x20 c:/program files/microchip/xc32/v1.33/bin/bin/../../lib/gcc/pic32mx/4.5.2/../../../../pic32mx/lib\software-debug-break.o
 .debug_aranges
                0x00000020       0x20 build/ChaletDuinoV2_775F512H_/debug/Source/ChaletduinoV2Board.o
 .debug_aranges
                0x00000040       0x20 build/ChaletDuinoV2_775F512H_/debug/Source/winc3400/bsp/source/nm_bsp.o
 .debug_aranges
                0x00000060       0x20 build/ChaletDuinoV2_775F512H_/debug/Source/winc3400/bus_wrapper/source/nm_bus_wrapper.o
 .debug_aranges
                0x00000080       0x20 build/ChaletDuinoV2_775F512H_/debug/Source/winc3400/common/source/nm_common.o
 .debug_aranges
                0x000000a0       0x20 build/ChaletDuinoV2_775F512H_/debug/Source/winc3400/driver/source/m2m_hif.o
 .debug_aranges
                0x000000c0       0x20 build/ChaletDuinoV2_775F512H_/debug/Source/winc3400/driver/source/m2m_ota.o
 .debug_aranges
                0x000000e0       0x20 build/ChaletDuinoV2_775F512H_/debug/Source/winc3400/driver/source/m2m_periph.o
 .debug_aranges
                0x00000100       0x20 build/ChaletDuinoV2_775F512H_/debug/Source/winc3400/driver/source/m2m_ssl.o
 .debug_aranges
                0x00000120       0x20 build/ChaletDuinoV2_775F512H_/debug/Source/winc3400/driver/source/m2m_wifi.o
 .debug_aranges
                0x00000140       0x20 build/ChaletDuinoV2_775F512H_/debug/Source/winc3400/driver/source/nmasic.o
 .debug_aranges
                0x00000160       0x20 build/ChaletDuinoV2_775F512H_/debug/Source/winc3400/driver/source/nmbus.o
 .debug_aranges
                0x00000180       0x20 build/ChaletDuinoV2_775F512H_/debug/Source/winc3400/driver/source/nmdrv.o
 .debug_aranges
                0x000001a0       0x20 build/ChaletDuinoV2_775F512H_/debug/Source/winc3400/driver/source/nmspi.o
 .debug_aranges
                0x000001c0       0x20 build/ChaletDuinoV2_775F512H_/debug/Source/winc3400/socket/source/socket.o
 .debug_aranges
                0x000001e0       0x20 build/ChaletDuinoV2_775F512H_/debug/Source/winc3400/spi_flash/source/spi_flash.o
 .debug_aranges
                0x00000200       0x20 build/ChaletDuinoV2_775F512H_/debug/Source/winc3400/winc_init.o
 .debug_aranges
                0x00000220       0x20 build/ChaletDuinoV2_775F512H_/debug/Source/DigitalIO.o
 .debug_aranges
                0x00000240       0x20 build/ChaletDuinoV2_775F512H_/debug/Source/InternalUart.o
 .debug_aranges
                0x00000260       0x20 build/ChaletDuinoV2_775F512H_/debug/Source/NetworkProtocol.o
 .debug_aranges
                0x00000280       0x20 build/ChaletDuinoV2_775F512H_/debug/Source/Terminal.o
 .debug_aranges
                0x000002a0       0x20 build/ChaletDuinoV2_775F512H_/debug/Source/Uart.o
 .debug_aranges
                0x000002c0       0x20 build/ChaletDuinoV2_775F512H_/debug/Source/Util.o
 .debug_aranges
                0x000002e0       0x20 build/ChaletDuinoV2_775F512H_/debug/Source/exceptions.o
 .debug_aranges
                0x00000300       0x20 build/ChaletDuinoV2_775F512H_/debug/Source/main.o
 .debug_aranges
                0x00000320       0x20 build/ChaletDuinoV2_775F512H_/debug/Source/timer.o
 .debug_aranges
                0x00000340       0x20 build/ChaletDuinoV2_775F512H_/debug/Source/WiFiCtrl.o
 .debug_aranges
                0x00000360       0x20 build/ChaletDuinoV2_775F512H_/debug/Source/SPI.o
 .debug_aranges
                0x00000380       0x20 build/ChaletDuinoV2_775F512H_/debug/Source/LoraNetworkInterface.o
 .debug_aranges
                0x000003a0       0x20 build/ChaletDuinoV2_775F512H_/debug/Source/ChaletPowerRelay.o
 .debug_aranges
                0x000003c0       0x20 build/ChaletDuinoV2_775F512H_/debug/Source/HarakiriRelay.o
 .debug_aranges
                0x000003e0       0x20 build/ChaletDuinoV2_775F512H_/debug/Source/BatteryMonitor.o
 .debug_aranges
                0x00000400       0x20 build/ChaletDuinoV2_775F512H_/debug/Source/ina219.o
 .debug_aranges
                0x00000420       0x20 build/ChaletDuinoV2_775F512H_/debug/Source/I2C.o
 .debug_aranges
                0x00000440       0x20 build/ChaletDuinoV2_775F512H_/debug/Source/SPI_Flash.o
 .debug_aranges
                0x00000460       0x20 build/ChaletDuinoV2_775F512H_/debug/Source/Syslog.o
 .debug_aranges
                0x00000480       0x20 build/ChaletDuinoV2_775F512H_/debug/Source/Watchdog.o
 .debug_aranges
                0x000004a0       0x20 build/ChaletDuinoV2_775F512H_/debug/Source/BootloaderInterface.o
 .debug_aranges
                0x000004c0       0x20 build/ChaletDuinoV2_775F512H_/debug/Source/TemperatureSensor.o
 .debug_aranges
                0x000004e0       0x20 build/ChaletDuinoV2_775F512H_/debug/Source/TC77.o
 .debug_aranges
                0x00000500       0x20 build/ChaletDuinoV2_775F512H_/debug/Source/BootloaderProtocol.o
 .debug_aranges
                0x00000520       0x20 build/ChaletDuinoV2_775F512H_/debug/Source/crc32.o
 .debug_aranges
                0x00000540       0x20 c:/program files/microchip/xc32/v1.33/bin/bin/../../lib/gcc/pic32mx/4.5.2/../../../../pic32mx/lib\libmchp_peripheral_32MX795F512H.a(soft_reset_lib.o)
 .debug_aranges
                0x00000560       0x28 c:/program files/microchip/xc32/v1.33/bin/bin/../../lib/gcc/pic32mx/4.5.2/../../../../pic32mx/lib\libmchp_peripheral_32MX795F512H.a(pcache.o)
 .debug_aranges
                0x00000588       0x20 c:/program files/microchip/xc32/v1.33/bin/bin/../../lib/gcc/pic32mx/4.5.2/../../../../pic32mx/lib\libmchp_peripheral_32MX795F512H.a(int_configure_system_lib.o)
 .debug_aranges
                0x000005a8       0x20 c:/program files/microchip/xc32/v1.33/bin/bin/../../lib/gcc/pic32mx/4.5.2/../../../../pic32mx/lib\libmchp_peripheral_32MX795F512H.a(int_enable_interrupts_lib.o)
 .debug_aranges
                0x000005c8       0x20 c:/program files/microchip/xc32/v1.33/bin/bin/../../lib/gcc/pic32mx/4.5.2/../../../../pic32mx/lib\libmchp_peripheral_32MX795F512H.a(int_disable_interrupts_lib.o)
 .debug_aranges
                0x000005e8       0x20 c:/program files/microchip/xc32/v1.33/bin/bin/../../lib/gcc/pic32mx/4.5.2/../../../../pic32mx/lib\libmchp_peripheral_32MX795F512H.a(int_restore_interrupts_lib.o)
 .debug_aranges
                0x00000608       0x20 c:/program files/microchip/xc32/v1.33/bin/bin/../../lib/gcc/pic32mx/4.5.2/../../../../pic32mx/lib\libpic32.a(default-bootstrap-exception-handler.o)
 .debug_aranges
                0x00000628       0x20 c:/program files/microchip/xc32/v1.33/bin/bin/../../lib/gcc/pic32mx/4.5.2/../../../../pic32mx/lib\libpic32.a(default-on-reset.o)
 .debug_aranges
                0x00000648       0x20 c:/program files/microchip/xc32/v1.33/bin/bin/../../lib/gcc/pic32mx/4.5.2/../../../../pic32mx/lib\libpic32.a(default-on-bootstrap.o)
 .debug_aranges
                0x00000668       0x20 c:/program files/microchip/xc32/v1.33/bin/bin/../../lib/gcc/pic32mx/4.5.2/../../../../pic32mx/lib\libpic32.a(defaultinterrupt.o)
 .debug_aranges
                0x00000688       0x20 c:/program files/microchip/xc32/v1.33/bin/bin/../../lib/gcc/pic32mx/4.5.2/../../../../pic32mx/lib\libc.a(fflush.o)
 .debug_aranges
                0x000006a8       0x30 c:/program files/microchip/xc32/v1.33/bin/bin/../../lib/gcc/pic32mx/4.5.2/../../../../pic32mx/lib\libc.a(malloc.o)
 .debug_aranges
                0x000006d8       0x28 c:/program files/microchip/xc32/v1.33/bin/bin/../../lib/gcc/pic32mx/4.5.2/../../../../pic32mx/lib\libc.a(puts.o)
 .debug_aranges
                0x00000700       0x28 c:/program files/microchip/xc32/v1.33/bin/bin/../../lib/gcc/pic32mx/4.5.2/../../../../pic32mx/lib\libc.a(setbuf.o)
 .debug_aranges
                0x00000728       0x20 c:/program files/microchip/xc32/v1.33/bin/bin/../../lib/gcc/pic32mx/4.5.2/../../../../pic32mx/lib\libc.a(strncmp.o)
 .debug_aranges
                0x00000748       0x20 c:/program files/microchip/xc32/v1.33/bin/bin/../../lib/gcc/pic32mx/4.5.2/../../../../pic32mx/lib\libc.a(printf_cdfFnopsuxX.eo)
 .debug_aranges
                0x00000768       0x20 c:/program files/microchip/xc32/v1.33/bin/bin/../../lib/gcc/pic32mx/4.5.2/../../../../pic32mx/lib\libc.a(sprintf_cdfFnopuxX.eo)
 .debug_aranges
                0x00000788       0x20 c:/program files/microchip/xc32/v1.33/bin/bin/../../lib/gcc/pic32mx/4.5.2/../../../../pic32mx/lib\libc.a(sscanf_s.eo)
 .debug_aranges
                0x000007a8       0x20 c:/program files/microchip/xc32/v1.33/bin/bin/../../lib/gcc/pic32mx/4.5.2/../../../../pic32mx/lib\libc.a(_fputc_simple.o)
 .debug_aranges
                0x000007c8       0x28 c:/program files/microchip/xc32/v1.33/bin/bin/../../lib/gcc/pic32mx/4.5.2/../../../../pic32mx/lib\libc.a(buf.o)
 .debug_aranges
                0x000007f0       0x28 c:/program files/microchip/xc32/v1.33/bin/bin/../../lib/gcc/pic32mx/4.5.2/../../../../pic32mx/lib\libc.a(doprnt_cdfFnopsuxX.eo)
 .debug_aranges
                0x00000818       0x30 c:/program files/microchip/xc32/v1.33/bin/bin/../../lib/gcc/pic32mx/4.5.2/../../../../pic32mx/lib\libc.a(doscan_s.eo)
 .debug_aranges
                0x00000848       0x20 c:/program files/microchip/xc32/v1.33/bin/bin/../../lib/gcc/pic32mx/4.5.2/../../../../pic32mx/lib\libc.a(_flsbuf_simple.o)
 .debug_aranges
                0x00000868       0x20 c:/program files/microchip/xc32/v1.33/bin/bin/../../lib/gcc/pic32mx/4.5.2/../../../../pic32mx/lib\libc.a(fgetc.o)
 .debug_aranges
                0x00000888       0x20 c:/program files/microchip/xc32/v1.33/bin/bin/../../lib/gcc/pic32mx/4.5.2/../../../../pic32mx/lib\libc.a(atoi.o)
 .debug_aranges
                0x000008a8       0xa0 c:/program files/microchip/xc32/v1.33/bin/bin/../../lib/gcc/pic32mx/4.5.2/../../../../pic32mx/lib\libc.a(ctypef.o)
 .debug_aranges
                0x00000948       0x20 c:/program files/microchip/xc32/v1.33/bin/bin/../../lib/gcc/pic32mx/4.5.2/../../../../pic32mx/lib\libc.a(ungetc.o)
 .debug_aranges
                0x00000968       0x20 c:/program files/microchip/xc32/v1.33/bin/bin/../../lib/gcc/pic32mx/4.5.2/../../../../pic32mx/lib\libc.a(filbuf.o)
 .debug_aranges
                0x00000988       0x40 c:/program files/microchip/xc32/v1.33/bin/bin/../../lib/gcc/pic32mx/4.5.2/../../../../pic32mx/lib\libpic32.a(sbrk.o)
 .debug_aranges
                0x000009c8       0x20 c:/program files/microchip/xc32/v1.33/bin/bin/../../lib/gcc/pic32mx/4.5.2/../../../../pic32mx/lib\libpic32.a(read.o)
 .debug_aranges
                0x000009e8       0x20 c:/program files/microchip/xc32/v1.33/bin/bin/../../lib/gcc/pic32mx/4.5.2/../../../../pic32mx/lib\libpic32.a(write.o)
 .debug_aranges
                0x00000a08       0x20 c:/program files/microchip/xc32/v1.33/bin/bin/../../lib/gcc/pic32mx/4.5.2/../../../../pic32mx/lib\libe.a(_floatdisf.o)
 .debug_aranges
                0x00000a28       0x20 c:/program files/microchip/xc32/v1.33/bin/bin/../../lib/gcc/pic32mx/4.5.2\libgcc.a(_floatundisf.o)
 .debug_aranges
                0x00000a48       0x20 c:/program files/microchip/xc32/v1.33/bin/bin/../../lib/gcc/pic32mx/4.5.2\libgcc.a(_udivdi3.o)
 .debug_aranges
                0x00000a68       0x20 c:/program files/microchip/xc32/v1.33/bin/bin/../../lib/gcc/pic32mx/4.5.2\libgcc.a(_umoddi3.o)
 .debug_aranges
                0x00000a88       0x20 c:/program files/microchip/xc32/v1.33/bin/bin/../../lib/gcc/pic32mx/4.5.2\libgcc.a(floatunsisf.o)

.debug_pubnames
                0x00000000     0x34e5
 *(.debug_pubnames)
 .debug_pubnames
                0x00000000       0x30 c:/program files/microchip/xc32/v1.33/bin/bin/../../lib/gcc/pic32mx/4.5.2/../../../../pic32mx/lib\software-debug-break.o
 .debug_pubnames
                0x00000030       0x20 build/ChaletDuinoV2_775F512H_/debug/Source/ChaletduinoV2Board.o
 .debug_pubnames
                0x00000050       0xa6 build/ChaletDuinoV2_775F512H_/debug/Source/winc3400/bsp/source/nm_bsp.o
 .debug_pubnames
                0x000000f6       0xa6 build/ChaletDuinoV2_775F512H_/debug/Source/winc3400/bus_wrapper/source/nm_bus_wrapper.o
 .debug_pubnames
                0x0000019c       0x8f build/ChaletDuinoV2_775F512H_/debug/Source/winc3400/common/source/nm_common.o
 .debug_pubnames
                0x0000022b       0x23 build/ChaletDuinoV2_775F512H_/debug/Source/winc3400/driver/source/m2m_crypto.o
 .debug_pubnames
                0x0000024e      0x173 build/ChaletDuinoV2_775F512H_/debug/Source/winc3400/driver/source/m2m_hif.o
 .debug_pubnames
                0x000003c1       0xe5 build/ChaletDuinoV2_775F512H_/debug/Source/winc3400/driver/source/m2m_ota.o
 .debug_pubnames
                0x000004a6       0xa6 build/ChaletDuinoV2_775F512H_/debug/Source/winc3400/driver/source/m2m_periph.o
 .debug_pubnames
                0x0000054c      0x104 build/ChaletDuinoV2_775F512H_/debug/Source/winc3400/driver/source/m2m_ssl.o
 .debug_pubnames
                0x00000650      0x6fd build/ChaletDuinoV2_775F512H_/debug/Source/winc3400/driver/source/m2m_wifi.o
 .debug_pubnames
                0x00000d4d      0x207 build/ChaletDuinoV2_775F512H_/debug/Source/winc3400/driver/source/nmasic.o
 .debug_pubnames
                0x00000f54       0xcd build/ChaletDuinoV2_775F512H_/debug/Source/winc3400/driver/source/nmbus.o
 .debug_pubnames
                0x00001021       0xee build/ChaletDuinoV2_775F512H_/debug/Source/winc3400/driver/source/nmdrv.o
 .debug_pubnames
                0x0000110f       0x23 build/ChaletDuinoV2_775F512H_/debug/Source/winc3400/driver/source/nmi2c.o
 .debug_pubnames
                0x00001132       0xb8 build/ChaletDuinoV2_775F512H_/debug/Source/winc3400/driver/source/nmspi.o
 .debug_pubnames
                0x000011ea       0x23 build/ChaletDuinoV2_775F512H_/debug/Source/winc3400/driver/source/nmuart.o
 .debug_pubnames
                0x0000120d      0x1ce build/ChaletDuinoV2_775F512H_/debug/Source/winc3400/socket/source/socket.o
 .debug_pubnames
                0x000013db       0x75 build/ChaletDuinoV2_775F512H_/debug/Source/winc3400/spi_flash/source/spi_flash.o
 .debug_pubnames
                0x00001450       0x31 build/ChaletDuinoV2_775F512H_/debug/Source/winc3400/winc_init.o
 .debug_pubnames
                0x00001481       0x24 build/ChaletDuinoV2_775F512H_/debug/Source/DigitalIO.o
 .debug_pubnames
                0x000014a5      0x125 build/ChaletDuinoV2_775F512H_/debug/Source/InternalUart.o
 .debug_pubnames
                0x000015ca      0x194 build/ChaletDuinoV2_775F512H_/debug/Source/NetworkProtocol.o
 .debug_pubnames
                0x0000175e      0x174 build/ChaletDuinoV2_775F512H_/debug/Source/Terminal.o
 .debug_pubnames
                0x000018d2      0x101 build/ChaletDuinoV2_775F512H_/debug/Source/Uart.o
 .debug_pubnames
                0x000019d3       0xd8 build/ChaletDuinoV2_775F512H_/debug/Source/Util.o
 .debug_pubnames
                0x00001aab       0x31 build/ChaletDuinoV2_775F512H_/debug/Source/exceptions.o
 .debug_pubnames
                0x00001adc       0x49 build/ChaletDuinoV2_775F512H_/debug/Source/main.o
 .debug_pubnames
                0x00001b25       0xec build/ChaletDuinoV2_775F512H_/debug/Source/timer.o
 .debug_pubnames
                0x00001c11      0x347 build/ChaletDuinoV2_775F512H_/debug/Source/WiFiCtrl.o
 .debug_pubnames
                0x00001f58       0x25 build/ChaletDuinoV2_775F512H_/debug/Source/SPI.o
 .debug_pubnames
                0x00001f7d       0x72 build/ChaletDuinoV2_775F512H_/debug/Source/LoraNetworkInterface.o
 .debug_pubnames
                0x00001fef       0xca build/ChaletDuinoV2_775F512H_/debug/Source/ChaletPowerRelay.o
 .debug_pubnames
                0x000020b9       0x41 build/ChaletDuinoV2_775F512H_/debug/Source/HarakiriRelay.o
 .debug_pubnames
                0x000020fa      0x13b build/ChaletDuinoV2_775F512H_/debug/Source/BatteryMonitor.o
 .debug_pubnames
                0x00002235      0x1af build/ChaletDuinoV2_775F512H_/debug/Source/ina219.o
 .debug_pubnames
                0x000023e4       0x92 build/ChaletDuinoV2_775F512H_/debug/Source/I2C.o
 .debug_pubnames
                0x00002476      0x18a build/ChaletDuinoV2_775F512H_/debug/Source/SPI_Flash.o
 .debug_pubnames
                0x00002600       0xa3 build/ChaletDuinoV2_775F512H_/debug/Source/Syslog.o
 .debug_pubnames
                0x000026a3       0x71 build/ChaletDuinoV2_775F512H_/debug/Source/Watchdog.o
 .debug_pubnames
                0x00002714      0x3b9 build/ChaletDuinoV2_775F512H_/debug/Source/BootloaderInterface.o
 .debug_pubnames
                0x00002acd       0x7d build/ChaletDuinoV2_775F512H_/debug/Source/TemperatureSensor.o
 .debug_pubnames
                0x00002b4a       0x5c build/ChaletDuinoV2_775F512H_/debug/Source/TC77.o
 .debug_pubnames
                0x00002ba6      0x2fb build/ChaletDuinoV2_775F512H_/debug/Source/BootloaderProtocol.o
 .debug_pubnames
                0x00002ea1       0x2f build/ChaletDuinoV2_775F512H_/debug/Source/crc32.o
 .debug_pubnames
                0x00002ed0       0x20 c:/program files/microchip/xc32/v1.33/bin/bin/../../lib/gcc/pic32mx/4.5.2/../../../../pic32mx/lib\libmchp_peripheral_32MX795F512H.a(soft_reset_lib.o)
 .debug_pubnames
                0x00002ef0       0x3b c:/program files/microchip/xc32/v1.33/bin/bin/../../lib/gcc/pic32mx/4.5.2/../../../../pic32mx/lib\libmchp_peripheral_32MX795F512H.a(pcache.o)
 .debug_pubnames
                0x00002f2b       0x29 c:/program files/microchip/xc32/v1.33/bin/bin/../../lib/gcc/pic32mx/4.5.2/../../../../pic32mx/lib\libmchp_peripheral_32MX795F512H.a(int_configure_system_lib.o)
 .debug_pubnames
                0x00002f54       0x2a c:/program files/microchip/xc32/v1.33/bin/bin/../../lib/gcc/pic32mx/4.5.2/../../../../pic32mx/lib\libmchp_peripheral_32MX795F512H.a(int_enable_interrupts_lib.o)
 .debug_pubnames
                0x00002f7e       0x2b c:/program files/microchip/xc32/v1.33/bin/bin/../../lib/gcc/pic32mx/4.5.2/../../../../pic32mx/lib\libmchp_peripheral_32MX795F512H.a(int_disable_interrupts_lib.o)
 .debug_pubnames
                0x00002fa9       0x2b c:/program files/microchip/xc32/v1.33/bin/bin/../../lib/gcc/pic32mx/4.5.2/../../../../pic32mx/lib\libmchp_peripheral_32MX795F512H.a(int_restore_interrupts_lib.o)
 .debug_pubnames
                0x00002fd4       0x33 c:/program files/microchip/xc32/v1.33/bin/bin/../../lib/gcc/pic32mx/4.5.2/../../../../pic32mx/lib\libpic32.a(default-bootstrap-exception-handler.o)
 .debug_pubnames
                0x00003007       0x20 c:/program files/microchip/xc32/v1.33/bin/bin/../../lib/gcc/pic32mx/4.5.2/../../../../pic32mx/lib\libpic32.a(default-on-reset.o)
 .debug_pubnames
                0x00003027       0x24 c:/program files/microchip/xc32/v1.33/bin/bin/../../lib/gcc/pic32mx/4.5.2/../../../../pic32mx/lib\libpic32.a(default-on-bootstrap.o)
 .debug_pubnames
                0x0000304b       0x28 c:/program files/microchip/xc32/v1.33/bin/bin/../../lib/gcc/pic32mx/4.5.2/../../../../pic32mx/lib\libpic32.a(defaultinterrupt.o)
 .debug_pubnames
                0x00003073       0x1d c:/program files/microchip/xc32/v1.33/bin/bin/../../lib/gcc/pic32mx/4.5.2/../../../../pic32mx/lib\libc.a(fflush.o)
 .debug_pubnames
                0x00003090       0x32 c:/program files/microchip/xc32/v1.33/bin/bin/../../lib/gcc/pic32mx/4.5.2/../../../../pic32mx/lib\libc.a(malloc.o)
 .debug_pubnames
                0x000030c2       0x25 c:/program files/microchip/xc32/v1.33/bin/bin/../../lib/gcc/pic32mx/4.5.2/../../../../pic32mx/lib\libc.a(puts.o)
 .debug_pubnames
                0x000030e7       0x29 c:/program files/microchip/xc32/v1.33/bin/bin/../../lib/gcc/pic32mx/4.5.2/../../../../pic32mx/lib\libc.a(setbuf.o)
 .debug_pubnames
                0x00003110       0x1e c:/program files/microchip/xc32/v1.33/bin/bin/../../lib/gcc/pic32mx/4.5.2/../../../../pic32mx/lib\libc.a(strncmp.o)
 .debug_pubnames
                0x0000312e       0x2a c:/program files/microchip/xc32/v1.33/bin/bin/../../lib/gcc/pic32mx/4.5.2/../../../../pic32mx/lib\libc.a(printf_cdfFnopsuxX.eo)
 .debug_pubnames
                0x00003158       0x2a c:/program files/microchip/xc32/v1.33/bin/bin/../../lib/gcc/pic32mx/4.5.2/../../../../pic32mx/lib\libc.a(sprintf_cdfFnopuxX.eo)
 .debug_pubnames
                0x00003182       0x20 c:/program files/microchip/xc32/v1.33/bin/bin/../../lib/gcc/pic32mx/4.5.2/../../../../pic32mx/lib\libc.a(sscanf_s.eo)
 .debug_pubnames
                0x000031a2       0x1c c:/program files/microchip/xc32/v1.33/bin/bin/../../lib/gcc/pic32mx/4.5.2/../../../../pic32mx/lib\libc.a(_fputc_simple.o)
 .debug_pubnames
                0x000031be       0x2c c:/program files/microchip/xc32/v1.33/bin/bin/../../lib/gcc/pic32mx/4.5.2/../../../../pic32mx/lib\libc.a(buf.o)
 .debug_pubnames
                0x000031ea       0x2c c:/program files/microchip/xc32/v1.33/bin/bin/../../lib/gcc/pic32mx/4.5.2/../../../../pic32mx/lib\libc.a(doprnt_cdfFnopsuxX.eo)
 .debug_pubnames
                0x00003216       0x21 c:/program files/microchip/xc32/v1.33/bin/bin/../../lib/gcc/pic32mx/4.5.2/../../../../pic32mx/lib\libc.a(doscan_s.eo)
 .debug_pubnames
                0x00003237       0x1e c:/program files/microchip/xc32/v1.33/bin/bin/../../lib/gcc/pic32mx/4.5.2/../../../../pic32mx/lib\libc.a(_flsbuf_simple.o)
 .debug_pubnames
                0x00003255       0x1c c:/program files/microchip/xc32/v1.33/bin/bin/../../lib/gcc/pic32mx/4.5.2/../../../../pic32mx/lib\libc.a(fgetc.o)
 .debug_pubnames
                0x00003271       0x1b c:/program files/microchip/xc32/v1.33/bin/bin/../../lib/gcc/pic32mx/4.5.2/../../../../pic32mx/lib\libc.a(atoi.o)
 .debug_pubnames
                0x0000328c       0xe1 c:/program files/microchip/xc32/v1.33/bin/bin/../../lib/gcc/pic32mx/4.5.2/../../../../pic32mx/lib\libc.a(ctypef.o)
 .debug_pubnames
                0x0000336d       0x1d c:/program files/microchip/xc32/v1.33/bin/bin/../../lib/gcc/pic32mx/4.5.2/../../../../pic32mx/lib\libc.a(ungetc.o)
 .debug_pubnames
                0x0000338a       0x1e c:/program files/microchip/xc32/v1.33/bin/bin/../../lib/gcc/pic32mx/4.5.2/../../../../pic32mx/lib\libc.a(filbuf.o)
 .debug_pubnames
                0x000033a8       0x5c c:/program files/microchip/xc32/v1.33/bin/bin/../../lib/gcc/pic32mx/4.5.2/../../../../pic32mx/lib\libpic32.a(sbrk.o)
 .debug_pubnames
                0x00003404       0x1b c:/program files/microchip/xc32/v1.33/bin/bin/../../lib/gcc/pic32mx/4.5.2/../../../../pic32mx/lib\libpic32.a(read.o)
 .debug_pubnames
                0x0000341f       0x1c c:/program files/microchip/xc32/v1.33/bin/bin/../../lib/gcc/pic32mx/4.5.2/../../../../pic32mx/lib\libpic32.a(write.o)
 .debug_pubnames
                0x0000343b       0x22 c:/program files/microchip/xc32/v1.33/bin/bin/../../lib/gcc/pic32mx/4.5.2/../../../../pic32mx/lib\libe.a(_floatdisf.o)
 .debug_pubnames
                0x0000345d       0x24 c:/program files/microchip/xc32/v1.33/bin/bin/../../lib/gcc/pic32mx/4.5.2\libgcc.a(_floatundisf.o)
 .debug_pubnames
                0x00003481       0x20 c:/program files/microchip/xc32/v1.33/bin/bin/../../lib/gcc/pic32mx/4.5.2\libgcc.a(_udivdi3.o)
 .debug_pubnames
                0x000034a1       0x20 c:/program files/microchip/xc32/v1.33/bin/bin/../../lib/gcc/pic32mx/4.5.2\libgcc.a(_umoddi3.o)
 .debug_pubnames
                0x000034c1       0x24 c:/program files/microchip/xc32/v1.33/bin/bin/../../lib/gcc/pic32mx/4.5.2\libgcc.a(floatunsisf.o)

.debug_info     0x00000000    0x40fc7
 *(.debug_info .gnu.linkonce.wi.*)
 .debug_info    0x00000000       0xd2 c:/program files/microchip/xc32/v1.33/bin/bin/../../lib/gcc/pic32mx/4.5.2/../../../../pic32mx/lib\software-debug-break.o
 .debug_info    0x000000d2     0x37b0 build/ChaletDuinoV2_775F512H_/debug/Source/ChaletduinoV2Board.o
 .debug_info    0x00003882     0x1cee build/ChaletDuinoV2_775F512H_/debug/Source/winc3400/bsp/source/nm_bsp.o
 .debug_info    0x00005570     0x166e build/ChaletDuinoV2_775F512H_/debug/Source/winc3400/bus_wrapper/source/nm_bus_wrapper.o
 .debug_info    0x00006bde      0x406 build/ChaletDuinoV2_775F512H_/debug/Source/winc3400/common/source/nm_common.o
 .debug_info    0x00006fe4        0x0 build/ChaletDuinoV2_775F512H_/debug/Source/winc3400/driver/source/m2m_ate_mode.o
 .debug_info    0x00006fe4      0x146 build/ChaletDuinoV2_775F512H_/debug/Source/winc3400/driver/source/m2m_crypto.o
 .debug_info    0x0000712a     0x11ca build/ChaletDuinoV2_775F512H_/debug/Source/winc3400/driver/source/m2m_hif.o
 .debug_info    0x000082f4      0x9b1 build/ChaletDuinoV2_775F512H_/debug/Source/winc3400/driver/source/m2m_ota.o
 .debug_info    0x00008ca5      0x496 build/ChaletDuinoV2_775F512H_/debug/Source/winc3400/driver/source/m2m_periph.o
 .debug_info    0x0000913b      0xc4d build/ChaletDuinoV2_775F512H_/debug/Source/winc3400/driver/source/m2m_ssl.o
 .debug_info    0x00009d88     0x3b2f build/ChaletDuinoV2_775F512H_/debug/Source/winc3400/driver/source/m2m_wifi.o
 .debug_info    0x0000d8b7      0xa67 build/ChaletDuinoV2_775F512H_/debug/Source/winc3400/driver/source/nmasic.o
 .debug_info    0x0000e31e      0x55b build/ChaletDuinoV2_775F512H_/debug/Source/winc3400/driver/source/nmbus.o
 .debug_info    0x0000e879      0x6a8 build/ChaletDuinoV2_775F512H_/debug/Source/winc3400/driver/source/nmdrv.o
 .debug_info    0x0000ef21      0x141 build/ChaletDuinoV2_775F512H_/debug/Source/winc3400/driver/source/nmi2c.o
 .debug_info    0x0000f062      0x986 build/ChaletDuinoV2_775F512H_/debug/Source/winc3400/driver/source/nmspi.o
 .debug_info    0x0000f9e8      0x142 build/ChaletDuinoV2_775F512H_/debug/Source/winc3400/driver/source/nmuart.o
 .debug_info    0x0000fb2a     0x1e42 build/ChaletDuinoV2_775F512H_/debug/Source/winc3400/socket/source/socket.o
 .debug_info    0x0001196c      0x825 build/ChaletDuinoV2_775F512H_/debug/Source/winc3400/spi_flash/source/spi_flash.o
 .debug_info    0x00012191      0x55b build/ChaletDuinoV2_775F512H_/debug/Source/winc3400/winc_init.o
 .debug_info    0x000126ec     0x115d build/ChaletDuinoV2_775F512H_/debug/Source/DigitalIO.o
 .debug_info    0x00013849     0x3b5e build/ChaletDuinoV2_775F512H_/debug/Source/InternalUart.o
 .debug_info    0x000173a7     0x1aba build/ChaletDuinoV2_775F512H_/debug/Source/NetworkProtocol.o
 .debug_info    0x00018e61     0x1977 build/ChaletDuinoV2_775F512H_/debug/Source/Terminal.o
 .debug_info    0x0001a7d8     0x1a1a build/ChaletDuinoV2_775F512H_/debug/Source/Uart.o
 .debug_info    0x0001c1f2     0x151d build/ChaletDuinoV2_775F512H_/debug/Source/Util.o
 .debug_info    0x0001d70f     0x127e build/ChaletDuinoV2_775F512H_/debug/Source/exceptions.o
 .debug_info    0x0001e98d     0x113f build/ChaletDuinoV2_775F512H_/debug/Source/interrupts.o
 .debug_info    0x0001facc     0x1a49 build/ChaletDuinoV2_775F512H_/debug/Source/main.o
 .debug_info    0x00021515     0x113b build/ChaletDuinoV2_775F512H_/debug/Source/system.o
 .debug_info    0x00022650     0x113d build/ChaletDuinoV2_775F512H_/debug/Source/template.o
 .debug_info    0x0002378d     0x217b build/ChaletDuinoV2_775F512H_/debug/Source/timer.o
 .debug_info    0x00025908     0x3219 build/ChaletDuinoV2_775F512H_/debug/Source/WiFiCtrl.o
 .debug_info    0x00028b21     0x131c build/ChaletDuinoV2_775F512H_/debug/Source/SPI.o
 .debug_info    0x00029e3d     0x1d7d build/ChaletDuinoV2_775F512H_/debug/Source/LoraNetworkInterface.o
 .debug_info    0x0002bbba     0x17a9 build/ChaletDuinoV2_775F512H_/debug/Source/ChaletPowerRelay.o
 .debug_info    0x0002d363     0x1305 build/ChaletDuinoV2_775F512H_/debug/Source/HarakiriRelay.o
 .debug_info    0x0002e668     0x18a8 build/ChaletDuinoV2_775F512H_/debug/Source/BatteryMonitor.o
 .debug_info    0x0002ff10     0x15d0 build/ChaletDuinoV2_775F512H_/debug/Source/ina219.o
 .debug_info    0x000314e0     0x1710 build/ChaletDuinoV2_775F512H_/debug/Source/I2C.o
 .debug_info    0x00032bf0     0x185c build/ChaletDuinoV2_775F512H_/debug/Source/SPI_Flash.o
 .debug_info    0x0003444c     0x15aa build/ChaletDuinoV2_775F512H_/debug/Source/Syslog.o
 .debug_info    0x000359f6     0x1330 build/ChaletDuinoV2_775F512H_/debug/Source/Watchdog.o
 .debug_info    0x00036d26     0x2b79 build/ChaletDuinoV2_775F512H_/debug/Source/BootloaderInterface.o
 .debug_info    0x0003989f     0x1314 build/ChaletDuinoV2_775F512H_/debug/Source/TemperatureSensor.o
 .debug_info    0x0003abb3     0x14d2 build/ChaletDuinoV2_775F512H_/debug/Source/TC77.o
 .debug_info    0x0003c085     0x1f95 build/ChaletDuinoV2_775F512H_/debug/Source/BootloaderProtocol.o
 .debug_info    0x0003e01a      0x2e4 build/ChaletDuinoV2_775F512H_/debug/Source/crc32.o
 .debug_info    0x0003e2fe       0xae c:/program files/microchip/xc32/v1.33/bin/bin/../../lib/gcc/pic32mx/4.5.2/../../../../pic32mx/lib\libmchp_peripheral_32MX795F512H.a(soft_reset_lib.o)
 .debug_info    0x0003e3ac       0xbb c:/program files/microchip/xc32/v1.33/bin/bin/../../lib/gcc/pic32mx/4.5.2/../../../../pic32mx/lib\libmchp_peripheral_32MX795F512H.a(pcache.o)
 .debug_info    0x0003e467       0xae c:/program files/microchip/xc32/v1.33/bin/bin/../../lib/gcc/pic32mx/4.5.2/../../../../pic32mx/lib\libmchp_peripheral_32MX795F512H.a(int_configure_system_lib.o)
 .debug_info    0x0003e515       0xb0 c:/program files/microchip/xc32/v1.33/bin/bin/../../lib/gcc/pic32mx/4.5.2/../../../../pic32mx/lib\libmchp_peripheral_32MX795F512H.a(int_enable_interrupts_lib.o)
 .debug_info    0x0003e5c5       0xb2 c:/program files/microchip/xc32/v1.33/bin/bin/../../lib/gcc/pic32mx/4.5.2/../../../../pic32mx/lib\libmchp_peripheral_32MX795F512H.a(int_disable_interrupts_lib.o)
 .debug_info    0x0003e677       0xb2 c:/program files/microchip/xc32/v1.33/bin/bin/../../lib/gcc/pic32mx/4.5.2/../../../../pic32mx/lib\libmchp_peripheral_32MX795F512H.a(int_restore_interrupts_lib.o)
 .debug_info    0x0003e729       0xe2 c:/program files/microchip/xc32/v1.33/bin/bin/../../lib/gcc/pic32mx/4.5.2/../../../../pic32mx/lib\libpic32.a(default-bootstrap-exception-handler.o)
 .debug_info    0x0003e80b       0xbc c:/program files/microchip/xc32/v1.33/bin/bin/../../lib/gcc/pic32mx/4.5.2/../../../../pic32mx/lib\libpic32.a(default-on-reset.o)
 .debug_info    0x0003e8c7       0xc4 c:/program files/microchip/xc32/v1.33/bin/bin/../../lib/gcc/pic32mx/4.5.2/../../../../pic32mx/lib\libpic32.a(default-on-bootstrap.o)
 .debug_info    0x0003e98b       0xd6 c:/program files/microchip/xc32/v1.33/bin/bin/../../lib/gcc/pic32mx/4.5.2/../../../../pic32mx/lib\libpic32.a(defaultinterrupt.o)
 .debug_info    0x0003ea61        0x0 c:/program files/microchip/xc32/v1.33/bin/bin/../../lib/gcc/pic32mx/4.5.2/../../../../pic32mx/lib\libc.a(_iob.o)
 .debug_info    0x0003ea61       0xb5 c:/program files/microchip/xc32/v1.33/bin/bin/../../lib/gcc/pic32mx/4.5.2/../../../../pic32mx/lib\libc.a(fflush.o)
 .debug_info    0x0003eb16       0xe4 c:/program files/microchip/xc32/v1.33/bin/bin/../../lib/gcc/pic32mx/4.5.2/../../../../pic32mx/lib\libc.a(malloc.o)
 .debug_info    0x0003ebfa       0xc5 c:/program files/microchip/xc32/v1.33/bin/bin/../../lib/gcc/pic32mx/4.5.2/../../../../pic32mx/lib\libc.a(puts.o)
 .debug_info    0x0003ecbf       0xcb c:/program files/microchip/xc32/v1.33/bin/bin/../../lib/gcc/pic32mx/4.5.2/../../../../pic32mx/lib\libc.a(setbuf.o)
 .debug_info    0x0003ed8a       0xb7 c:/program files/microchip/xc32/v1.33/bin/bin/../../lib/gcc/pic32mx/4.5.2/../../../../pic32mx/lib\libc.a(strncmp.o)
 .debug_info    0x0003ee41       0xc2 c:/program files/microchip/xc32/v1.33/bin/bin/../../lib/gcc/pic32mx/4.5.2/../../../../pic32mx/lib\libc.a(printf_cdfFnopsuxX.eo)
 .debug_info    0x0003ef03       0xc3 c:/program files/microchip/xc32/v1.33/bin/bin/../../lib/gcc/pic32mx/4.5.2/../../../../pic32mx/lib\libc.a(sprintf_cdfFnopuxX.eo)
 .debug_info    0x0003efc6       0xb8 c:/program files/microchip/xc32/v1.33/bin/bin/../../lib/gcc/pic32mx/4.5.2/../../../../pic32mx/lib\libc.a(sscanf_s.eo)
 .debug_info    0x0003f07e       0xb3 c:/program files/microchip/xc32/v1.33/bin/bin/../../lib/gcc/pic32mx/4.5.2/../../../../pic32mx/lib\libc.a(_fputc_simple.o)
 .debug_info    0x0003f131       0xda c:/program files/microchip/xc32/v1.33/bin/bin/../../lib/gcc/pic32mx/4.5.2/../../../../pic32mx/lib\libc.a(buf.o)
 .debug_info    0x0003f20b        0x0 c:/program files/microchip/xc32/v1.33/bin/bin/../../lib/gcc/pic32mx/4.5.2/../../../../pic32mx/lib\libc.a(errno.o)
 .debug_info    0x0003f20b       0xe5 c:/program files/microchip/xc32/v1.33/bin/bin/../../lib/gcc/pic32mx/4.5.2/../../../../pic32mx/lib\libc.a(doprnt_cdfFnopsuxX.eo)
 .debug_info    0x0003f2f0       0xe0 c:/program files/microchip/xc32/v1.33/bin/bin/../../lib/gcc/pic32mx/4.5.2/../../../../pic32mx/lib\libc.a(doscan_s.eo)
 .debug_info    0x0003f3d0       0xb6 c:/program files/microchip/xc32/v1.33/bin/bin/../../lib/gcc/pic32mx/4.5.2/../../../../pic32mx/lib\libc.a(_flsbuf_simple.o)
 .debug_info    0x0003f486       0xb3 c:/program files/microchip/xc32/v1.33/bin/bin/../../lib/gcc/pic32mx/4.5.2/../../../../pic32mx/lib\libc.a(fgetc.o)
 .debug_info    0x0003f539       0xb1 c:/program files/microchip/xc32/v1.33/bin/bin/../../lib/gcc/pic32mx/4.5.2/../../../../pic32mx/lib\libc.a(atoi.o)
 .debug_info    0x0003f5ea        0x0 c:/program files/microchip/xc32/v1.33/bin/bin/../../lib/gcc/pic32mx/4.5.2/../../../../pic32mx/lib\libc.a(ctype.o)
 .debug_info    0x0003f5ea      0x219 c:/program files/microchip/xc32/v1.33/bin/bin/../../lib/gcc/pic32mx/4.5.2/../../../../pic32mx/lib\libc.a(ctypef.o)
 .debug_info    0x0003f803        0x0 c:/program files/microchip/xc32/v1.33/bin/bin/../../lib/gcc/pic32mx/4.5.2/../../../../pic32mx/lib\libc.a(powersf.o)
 .debug_info    0x0003f803       0xb5 c:/program files/microchip/xc32/v1.33/bin/bin/../../lib/gcc/pic32mx/4.5.2/../../../../pic32mx/lib\libc.a(ungetc.o)
 .debug_info    0x0003f8b8       0xb6 c:/program files/microchip/xc32/v1.33/bin/bin/../../lib/gcc/pic32mx/4.5.2/../../../../pic32mx/lib\libc.a(filbuf.o)
 .debug_info    0x0003f96e      0x115 c:/program files/microchip/xc32/v1.33/bin/bin/../../lib/gcc/pic32mx/4.5.2/../../../../pic32mx/lib\libpic32.a(sbrk.o)
 .debug_info    0x0003fa83       0xab c:/program files/microchip/xc32/v1.33/bin/bin/../../lib/gcc/pic32mx/4.5.2/../../../../pic32mx/lib\libpic32.a(read.o)
 .debug_info    0x0003fb2e       0xad c:/program files/microchip/xc32/v1.33/bin/bin/../../lib/gcc/pic32mx/4.5.2/../../../../pic32mx/lib\libpic32.a(write.o)
 .debug_info    0x0003fbdb        0x0 c:/program files/microchip/xc32/v1.33/bin/bin/../../lib/gcc/pic32mx/4.5.2/../../../../pic32mx/lib\libpic32.a(xc32_uart.o)
 .debug_info    0x0003fbdb       0xcb c:/program files/microchip/xc32/v1.33/bin/bin/../../lib/gcc/pic32mx/4.5.2/../../../../pic32mx/lib\libe.a(_floatdisf.o)
 .debug_info    0x0003fca6      0x2c2 c:/program files/microchip/xc32/v1.33/bin/bin/../../lib/gcc/pic32mx/4.5.2\libgcc.a(_floatundisf.o)
 .debug_info    0x0003ff68      0x782 c:/program files/microchip/xc32/v1.33/bin/bin/../../lib/gcc/pic32mx/4.5.2\libgcc.a(_udivdi3.o)
 .debug_info    0x000406ea      0x7b8 c:/program files/microchip/xc32/v1.33/bin/bin/../../lib/gcc/pic32mx/4.5.2\libgcc.a(_umoddi3.o)
 .debug_info    0x00040ea2      0x125 c:/program files/microchip/xc32/v1.33/bin/bin/../../lib/gcc/pic32mx/4.5.2\libgcc.a(floatunsisf.o)

.debug_abbrev   0x00000000     0x60e2
 *(.debug_abbrev)
 .debug_abbrev  0x00000000       0x25 c:/program files/microchip/xc32/v1.33/bin/bin/../../lib/gcc/pic32mx/4.5.2/../../../../pic32mx/lib\software-debug-break.o
 .debug_abbrev  0x00000025      0x1f2 build/ChaletDuinoV2_775F512H_/debug/Source/ChaletduinoV2Board.o
 .debug_abbrev  0x00000217      0x203 build/ChaletDuinoV2_775F512H_/debug/Source/winc3400/bsp/source/nm_bsp.o
 .debug_abbrev  0x0000041a      0x257 build/ChaletDuinoV2_775F512H_/debug/Source/winc3400/bus_wrapper/source/nm_bus_wrapper.o
 .debug_abbrev  0x00000671       0xd7 build/ChaletDuinoV2_775F512H_/debug/Source/winc3400/common/source/nm_common.o
 .debug_abbrev  0x00000748        0x1 build/ChaletDuinoV2_775F512H_/debug/Source/winc3400/driver/source/m2m_ate_mode.o
 .debug_abbrev  0x00000749       0x55 build/ChaletDuinoV2_775F512H_/debug/Source/winc3400/driver/source/m2m_crypto.o
 .debug_abbrev  0x0000079e      0x27a build/ChaletDuinoV2_775F512H_/debug/Source/winc3400/driver/source/m2m_hif.o
 .debug_abbrev  0x00000a18      0x175 build/ChaletDuinoV2_775F512H_/debug/Source/winc3400/driver/source/m2m_ota.o
 .debug_abbrev  0x00000b8d      0x123 build/ChaletDuinoV2_775F512H_/debug/Source/winc3400/driver/source/m2m_periph.o
 .debug_abbrev  0x00000cb0      0x22a build/ChaletDuinoV2_775F512H_/debug/Source/winc3400/driver/source/m2m_ssl.o
 .debug_abbrev  0x00000eda      0x26f build/ChaletDuinoV2_775F512H_/debug/Source/winc3400/driver/source/m2m_wifi.o
 .debug_abbrev  0x00001149      0x1cb build/ChaletDuinoV2_775F512H_/debug/Source/winc3400/driver/source/nmasic.o
 .debug_abbrev  0x00001314      0x111 build/ChaletDuinoV2_775F512H_/debug/Source/winc3400/driver/source/nmbus.o
 .debug_abbrev  0x00001425      0x162 build/ChaletDuinoV2_775F512H_/debug/Source/winc3400/driver/source/nmdrv.o
 .debug_abbrev  0x00001587       0x55 build/ChaletDuinoV2_775F512H_/debug/Source/winc3400/driver/source/nmi2c.o
 .debug_abbrev  0x000015dc      0x1b1 build/ChaletDuinoV2_775F512H_/debug/Source/winc3400/driver/source/nmspi.o
 .debug_abbrev  0x0000178d       0x55 build/ChaletDuinoV2_775F512H_/debug/Source/winc3400/driver/source/nmuart.o
 .debug_abbrev  0x000017e2      0x2ae build/ChaletDuinoV2_775F512H_/debug/Source/winc3400/socket/source/socket.o
 .debug_abbrev  0x00001a90      0x140 build/ChaletDuinoV2_775F512H_/debug/Source/winc3400/spi_flash/source/spi_flash.o
 .debug_abbrev  0x00001bd0       0xf7 build/ChaletDuinoV2_775F512H_/debug/Source/winc3400/winc_init.o
 .debug_abbrev  0x00001cc7      0x17b build/ChaletDuinoV2_775F512H_/debug/Source/DigitalIO.o
 .debug_abbrev  0x00001e42      0x2d9 build/ChaletDuinoV2_775F512H_/debug/Source/InternalUart.o
 .debug_abbrev  0x0000211b      0x295 build/ChaletDuinoV2_775F512H_/debug/Source/NetworkProtocol.o
 .debug_abbrev  0x000023b0      0x2af build/ChaletDuinoV2_775F512H_/debug/Source/Terminal.o
 .debug_abbrev  0x0000265f      0x2e5 build/ChaletDuinoV2_775F512H_/debug/Source/Uart.o
 .debug_abbrev  0x00002944      0x26e build/ChaletDuinoV2_775F512H_/debug/Source/Util.o
 .debug_abbrev  0x00002bb2      0x1b1 build/ChaletDuinoV2_775F512H_/debug/Source/exceptions.o
 .debug_abbrev  0x00002d63      0x166 build/ChaletDuinoV2_775F512H_/debug/Source/interrupts.o
 .debug_abbrev  0x00002ec9      0x351 build/ChaletDuinoV2_775F512H_/debug/Source/main.o
 .debug_abbrev  0x0000321a      0x166 build/ChaletDuinoV2_775F512H_/debug/Source/system.o
 .debug_abbrev  0x00003380      0x166 build/ChaletDuinoV2_775F512H_/debug/Source/template.o
 .debug_abbrev  0x000034e6      0x226 build/ChaletDuinoV2_775F512H_/debug/Source/timer.o
 .debug_abbrev  0x0000370c      0x343 build/ChaletDuinoV2_775F512H_/debug/Source/WiFiCtrl.o
 .debug_abbrev  0x00003a4f      0x19d build/ChaletDuinoV2_775F512H_/debug/Source/SPI.o
 .debug_abbrev  0x00003bec      0x281 build/ChaletDuinoV2_775F512H_/debug/Source/LoraNetworkInterface.o
 .debug_abbrev  0x00003e6d      0x1c4 build/ChaletDuinoV2_775F512H_/debug/Source/ChaletPowerRelay.o
 .debug_abbrev  0x00004031      0x18e build/ChaletDuinoV2_775F512H_/debug/Source/HarakiriRelay.o
 .debug_abbrev  0x000041bf      0x22f build/ChaletDuinoV2_775F512H_/debug/Source/BatteryMonitor.o
 .debug_abbrev  0x000043ee      0x26b build/ChaletDuinoV2_775F512H_/debug/Source/ina219.o
 .debug_abbrev  0x00004659      0x1e9 build/ChaletDuinoV2_775F512H_/debug/Source/I2C.o
 .debug_abbrev  0x00004842      0x298 build/ChaletDuinoV2_775F512H_/debug/Source/SPI_Flash.o
 .debug_abbrev  0x00004ada      0x233 build/ChaletDuinoV2_775F512H_/debug/Source/Syslog.o
 .debug_abbrev  0x00004d0d      0x18c build/ChaletDuinoV2_775F512H_/debug/Source/Watchdog.o
 .debug_abbrev  0x00004e99      0x2f7 build/ChaletDuinoV2_775F512H_/debug/Source/BootloaderInterface.o
 .debug_abbrev  0x00005190      0x1b5 build/ChaletDuinoV2_775F512H_/debug/Source/TemperatureSensor.o
 .debug_abbrev  0x00005345      0x1c1 build/ChaletDuinoV2_775F512H_/debug/Source/TC77.o
 .debug_abbrev  0x00005506      0x2b3 build/ChaletDuinoV2_775F512H_/debug/Source/BootloaderProtocol.o
 .debug_abbrev  0x000057b9       0xa9 build/ChaletDuinoV2_775F512H_/debug/Source/crc32.o
 .debug_abbrev  0x00005862       0x32 c:/program files/microchip/xc32/v1.33/bin/bin/../../lib/gcc/pic32mx/4.5.2/../../../../pic32mx/lib\libmchp_peripheral_32MX795F512H.a(soft_reset_lib.o)
 .debug_abbrev  0x00005894       0x23 c:/program files/microchip/xc32/v1.33/bin/bin/../../lib/gcc/pic32mx/4.5.2/../../../../pic32mx/lib\libmchp_peripheral_32MX795F512H.a(pcache.o)
 .debug_abbrev  0x000058b7       0x23 c:/program files/microchip/xc32/v1.33/bin/bin/../../lib/gcc/pic32mx/4.5.2/../../../../pic32mx/lib\libmchp_peripheral_32MX795F512H.a(int_configure_system_lib.o)
 .debug_abbrev  0x000058da       0x23 c:/program files/microchip/xc32/v1.33/bin/bin/../../lib/gcc/pic32mx/4.5.2/../../../../pic32mx/lib\libmchp_peripheral_32MX795F512H.a(int_enable_interrupts_lib.o)
 .debug_abbrev  0x000058fd       0x23 c:/program files/microchip/xc32/v1.33/bin/bin/../../lib/gcc/pic32mx/4.5.2/../../../../pic32mx/lib\libmchp_peripheral_32MX795F512H.a(int_disable_interrupts_lib.o)
 .debug_abbrev  0x00005920       0x23 c:/program files/microchip/xc32/v1.33/bin/bin/../../lib/gcc/pic32mx/4.5.2/../../../../pic32mx/lib\libmchp_peripheral_32MX795F512H.a(int_restore_interrupts_lib.o)
 .debug_abbrev  0x00005943       0x25 c:/program files/microchip/xc32/v1.33/bin/bin/../../lib/gcc/pic32mx/4.5.2/../../../../pic32mx/lib\libpic32.a(default-bootstrap-exception-handler.o)
 .debug_abbrev  0x00005968       0x25 c:/program files/microchip/xc32/v1.33/bin/bin/../../lib/gcc/pic32mx/4.5.2/../../../../pic32mx/lib\libpic32.a(default-on-reset.o)
 .debug_abbrev  0x0000598d       0x25 c:/program files/microchip/xc32/v1.33/bin/bin/../../lib/gcc/pic32mx/4.5.2/../../../../pic32mx/lib\libpic32.a(default-on-bootstrap.o)
 .debug_abbrev  0x000059b2       0x25 c:/program files/microchip/xc32/v1.33/bin/bin/../../lib/gcc/pic32mx/4.5.2/../../../../pic32mx/lib\libpic32.a(defaultinterrupt.o)
 .debug_abbrev  0x000059d7        0x1 c:/program files/microchip/xc32/v1.33/bin/bin/../../lib/gcc/pic32mx/4.5.2/../../../../pic32mx/lib\libc.a(_iob.o)
 .debug_abbrev  0x000059d8       0x25 c:/program files/microchip/xc32/v1.33/bin/bin/../../lib/gcc/pic32mx/4.5.2/../../../../pic32mx/lib\libc.a(fflush.o)
 .debug_abbrev  0x000059fd       0x41 c:/program files/microchip/xc32/v1.33/bin/bin/../../lib/gcc/pic32mx/4.5.2/../../../../pic32mx/lib\libc.a(malloc.o)
 .debug_abbrev  0x00005a3e       0x25 c:/program files/microchip/xc32/v1.33/bin/bin/../../lib/gcc/pic32mx/4.5.2/../../../../pic32mx/lib\libc.a(puts.o)
 .debug_abbrev  0x00005a63       0x25 c:/program files/microchip/xc32/v1.33/bin/bin/../../lib/gcc/pic32mx/4.5.2/../../../../pic32mx/lib\libc.a(setbuf.o)
 .debug_abbrev  0x00005a88       0x25 c:/program files/microchip/xc32/v1.33/bin/bin/../../lib/gcc/pic32mx/4.5.2/../../../../pic32mx/lib\libc.a(strncmp.o)
 .debug_abbrev  0x00005aad       0x25 c:/program files/microchip/xc32/v1.33/bin/bin/../../lib/gcc/pic32mx/4.5.2/../../../../pic32mx/lib\libc.a(printf_cdfFnopsuxX.eo)
 .debug_abbrev  0x00005ad2       0x25 c:/program files/microchip/xc32/v1.33/bin/bin/../../lib/gcc/pic32mx/4.5.2/../../../../pic32mx/lib\libc.a(sprintf_cdfFnopuxX.eo)
 .debug_abbrev  0x00005af7       0x25 c:/program files/microchip/xc32/v1.33/bin/bin/../../lib/gcc/pic32mx/4.5.2/../../../../pic32mx/lib\libc.a(sscanf_s.eo)
 .debug_abbrev  0x00005b1c       0x25 c:/program files/microchip/xc32/v1.33/bin/bin/../../lib/gcc/pic32mx/4.5.2/../../../../pic32mx/lib\libc.a(_fputc_simple.o)
 .debug_abbrev  0x00005b41       0x49 c:/program files/microchip/xc32/v1.33/bin/bin/../../lib/gcc/pic32mx/4.5.2/../../../../pic32mx/lib\libc.a(buf.o)
 .debug_abbrev  0x00005b8a        0x1 c:/program files/microchip/xc32/v1.33/bin/bin/../../lib/gcc/pic32mx/4.5.2/../../../../pic32mx/lib\libc.a(errno.o)
 .debug_abbrev  0x00005b8b       0x43 c:/program files/microchip/xc32/v1.33/bin/bin/../../lib/gcc/pic32mx/4.5.2/../../../../pic32mx/lib\libc.a(doprnt_cdfFnopsuxX.eo)
 .debug_abbrev  0x00005bce       0x36 c:/program files/microchip/xc32/v1.33/bin/bin/../../lib/gcc/pic32mx/4.5.2/../../../../pic32mx/lib\libc.a(doscan_s.eo)
 .debug_abbrev  0x00005c04       0x25 c:/program files/microchip/xc32/v1.33/bin/bin/../../lib/gcc/pic32mx/4.5.2/../../../../pic32mx/lib\libc.a(_flsbuf_simple.o)
 .debug_abbrev  0x00005c29       0x25 c:/program files/microchip/xc32/v1.33/bin/bin/../../lib/gcc/pic32mx/4.5.2/../../../../pic32mx/lib\libc.a(fgetc.o)
 .debug_abbrev  0x00005c4e       0x25 c:/program files/microchip/xc32/v1.33/bin/bin/../../lib/gcc/pic32mx/4.5.2/../../../../pic32mx/lib\libc.a(atoi.o)
 .debug_abbrev  0x00005c73        0x1 c:/program files/microchip/xc32/v1.33/bin/bin/../../lib/gcc/pic32mx/4.5.2/../../../../pic32mx/lib\libc.a(ctype.o)
 .debug_abbrev  0x00005c74       0x25 c:/program files/microchip/xc32/v1.33/bin/bin/../../lib/gcc/pic32mx/4.5.2/../../../../pic32mx/lib\libc.a(ctypef.o)
 .debug_abbrev  0x00005c99        0x1 c:/program files/microchip/xc32/v1.33/bin/bin/../../lib/gcc/pic32mx/4.5.2/../../../../pic32mx/lib\libc.a(powersf.o)
 .debug_abbrev  0x00005c9a       0x25 c:/program files/microchip/xc32/v1.33/bin/bin/../../lib/gcc/pic32mx/4.5.2/../../../../pic32mx/lib\libc.a(ungetc.o)
 .debug_abbrev  0x00005cbf       0x25 c:/program files/microchip/xc32/v1.33/bin/bin/../../lib/gcc/pic32mx/4.5.2/../../../../pic32mx/lib\libc.a(filbuf.o)
 .debug_abbrev  0x00005ce4       0x38 c:/program files/microchip/xc32/v1.33/bin/bin/../../lib/gcc/pic32mx/4.5.2/../../../../pic32mx/lib\libpic32.a(sbrk.o)
 .debug_abbrev  0x00005d1c       0x25 c:/program files/microchip/xc32/v1.33/bin/bin/../../lib/gcc/pic32mx/4.5.2/../../../../pic32mx/lib\libpic32.a(read.o)
 .debug_abbrev  0x00005d41       0x25 c:/program files/microchip/xc32/v1.33/bin/bin/../../lib/gcc/pic32mx/4.5.2/../../../../pic32mx/lib\libpic32.a(write.o)
 .debug_abbrev  0x00005d66        0x1 c:/program files/microchip/xc32/v1.33/bin/bin/../../lib/gcc/pic32mx/4.5.2/../../../../pic32mx/lib\libpic32.a(xc32_uart.o)
 .debug_abbrev  0x00005d67       0x32 c:/program files/microchip/xc32/v1.33/bin/bin/../../lib/gcc/pic32mx/4.5.2/../../../../pic32mx/lib\libe.a(_floatdisf.o)
 .debug_abbrev  0x00005d99       0x79 c:/program files/microchip/xc32/v1.33/bin/bin/../../lib/gcc/pic32mx/4.5.2\libgcc.a(_floatundisf.o)
 .debug_abbrev  0x00005e12      0x132 c:/program files/microchip/xc32/v1.33/bin/bin/../../lib/gcc/pic32mx/4.5.2\libgcc.a(_udivdi3.o)
 .debug_abbrev  0x00005f44      0x13f c:/program files/microchip/xc32/v1.33/bin/bin/../../lib/gcc/pic32mx/4.5.2\libgcc.a(_umoddi3.o)
 .debug_abbrev  0x00006083       0x5f c:/program files/microchip/xc32/v1.33/bin/bin/../../lib/gcc/pic32mx/4.5.2\libgcc.a(floatunsisf.o)

.debug_line     0x00000000     0x835d
 *(.debug_line)
 .debug_line    0x00000000       0x8a c:/program files/microchip/xc32/v1.33/bin/bin/../../lib/gcc/pic32mx/4.5.2/../../../../pic32mx/lib\software-debug-break.o
 .debug_line    0x0000008a      0x20d build/ChaletDuinoV2_775F512H_/debug/Source/ChaletduinoV2Board.o
 .debug_line    0x00000297      0x251 build/ChaletDuinoV2_775F512H_/debug/Source/winc3400/bsp/source/nm_bsp.o
 .debug_line    0x000004e8      0x339 build/ChaletDuinoV2_775F512H_/debug/Source/winc3400/bus_wrapper/source/nm_bus_wrapper.o
 .debug_line    0x00000821      0x195 build/ChaletDuinoV2_775F512H_/debug/Source/winc3400/common/source/nm_common.o
 .debug_line    0x000009b6        0x0 build/ChaletDuinoV2_775F512H_/debug/Source/winc3400/driver/source/m2m_ate_mode.o
 .debug_line    0x000009b6       0x7a build/ChaletDuinoV2_775F512H_/debug/Source/winc3400/driver/source/m2m_crypto.o
 .debug_line    0x00000a30      0x3b2 build/ChaletDuinoV2_775F512H_/debug/Source/winc3400/driver/source/m2m_hif.o
 .debug_line    0x00000de2      0x22d build/ChaletDuinoV2_775F512H_/debug/Source/winc3400/driver/source/m2m_ota.o
 .debug_line    0x0000100f      0x1e8 build/ChaletDuinoV2_775F512H_/debug/Source/winc3400/driver/source/m2m_periph.o
 .debug_line    0x000011f7      0x2cd build/ChaletDuinoV2_775F512H_/debug/Source/winc3400/driver/source/m2m_ssl.o
 .debug_line    0x000014c4      0x568 build/ChaletDuinoV2_775F512H_/debug/Source/winc3400/driver/source/m2m_wifi.o
 .debug_line    0x00001a2c      0x34b build/ChaletDuinoV2_775F512H_/debug/Source/winc3400/driver/source/nmasic.o
 .debug_line    0x00001d77      0x207 build/ChaletDuinoV2_775F512H_/debug/Source/winc3400/driver/source/nmbus.o
 .debug_line    0x00001f7e      0x27e build/ChaletDuinoV2_775F512H_/debug/Source/winc3400/driver/source/nmdrv.o
 .debug_line    0x000021fc       0x7a build/ChaletDuinoV2_775F512H_/debug/Source/winc3400/driver/source/nmi2c.o
 .debug_line    0x00002276      0x2db build/ChaletDuinoV2_775F512H_/debug/Source/winc3400/driver/source/nmspi.o
 .debug_line    0x00002551       0x7a build/ChaletDuinoV2_775F512H_/debug/Source/winc3400/driver/source/nmuart.o
 .debug_line    0x000025cb      0x4ef build/ChaletDuinoV2_775F512H_/debug/Source/winc3400/socket/source/socket.o
 .debug_line    0x00002aba      0x2d3 build/ChaletDuinoV2_775F512H_/debug/Source/winc3400/spi_flash/source/spi_flash.o
 .debug_line    0x00002d8d      0x1f0 build/ChaletDuinoV2_775F512H_/debug/Source/winc3400/winc_init.o
 .debug_line    0x00002f7d      0x156 build/ChaletDuinoV2_775F512H_/debug/Source/DigitalIO.o
 .debug_line    0x000030d3      0x2c6 build/ChaletDuinoV2_775F512H_/debug/Source/InternalUart.o
 .debug_line    0x00003399      0x262 build/ChaletDuinoV2_775F512H_/debug/Source/NetworkProtocol.o
 .debug_line    0x000035fb      0x3c5 build/ChaletDuinoV2_775F512H_/debug/Source/Terminal.o
 .debug_line    0x000039c0      0x2ef build/ChaletDuinoV2_775F512H_/debug/Source/Uart.o
 .debug_line    0x00003caf      0x25b build/ChaletDuinoV2_775F512H_/debug/Source/Util.o
 .debug_line    0x00003f0a      0x161 build/ChaletDuinoV2_775F512H_/debug/Source/exceptions.o
 .debug_line    0x0000406b      0x101 build/ChaletDuinoV2_775F512H_/debug/Source/interrupts.o
 .debug_line    0x0000416c      0x38e build/ChaletDuinoV2_775F512H_/debug/Source/main.o
 .debug_line    0x000044fa      0x101 build/ChaletDuinoV2_775F512H_/debug/Source/system.o
 .debug_line    0x000045fb      0x101 build/ChaletDuinoV2_775F512H_/debug/Source/template.o
 .debug_line    0x000046fc      0x23b build/ChaletDuinoV2_775F512H_/debug/Source/timer.o
 .debug_line    0x00004937      0x574 build/ChaletDuinoV2_775F512H_/debug/Source/WiFiCtrl.o
 .debug_line    0x00004eab      0x155 build/ChaletDuinoV2_775F512H_/debug/Source/SPI.o
 .debug_line    0x00005000      0x23d build/ChaletDuinoV2_775F512H_/debug/Source/LoraNetworkInterface.o
 .debug_line    0x0000523d      0x1b9 build/ChaletDuinoV2_775F512H_/debug/Source/ChaletPowerRelay.o
 .debug_line    0x000053f6      0x16d build/ChaletDuinoV2_775F512H_/debug/Source/HarakiriRelay.o
 .debug_line    0x00005563      0x2d8 build/ChaletDuinoV2_775F512H_/debug/Source/BatteryMonitor.o
 .debug_line    0x0000583b      0x23e build/ChaletDuinoV2_775F512H_/debug/Source/ina219.o
 .debug_line    0x00005a79      0x1f5 build/ChaletDuinoV2_775F512H_/debug/Source/I2C.o
 .debug_line    0x00005c6e      0x29a build/ChaletDuinoV2_775F512H_/debug/Source/SPI_Flash.o
 .debug_line    0x00005f08      0x2af build/ChaletDuinoV2_775F512H_/debug/Source/Syslog.o
 .debug_line    0x000061b7      0x165 build/ChaletDuinoV2_775F512H_/debug/Source/Watchdog.o
 .debug_line    0x0000631c      0x4ed build/ChaletDuinoV2_775F512H_/debug/Source/BootloaderInterface.o
 .debug_line    0x00006809      0x193 build/ChaletDuinoV2_775F512H_/debug/Source/TemperatureSensor.o
 .debug_line    0x0000699c      0x19a build/ChaletDuinoV2_775F512H_/debug/Source/TC77.o
 .debug_line    0x00006b36      0x3b6 build/ChaletDuinoV2_775F512H_/debug/Source/BootloaderProtocol.o
 .debug_line    0x00006eec      0x137 build/ChaletDuinoV2_775F512H_/debug/Source/crc32.o
 .debug_line    0x00007023       0xb1 c:/program files/microchip/xc32/v1.33/bin/bin/../../lib/gcc/pic32mx/4.5.2/../../../../pic32mx/lib\libmchp_peripheral_32MX795F512H.a(soft_reset_lib.o)
 .debug_line    0x000070d4       0x62 c:/program files/microchip/xc32/v1.33/bin/bin/../../lib/gcc/pic32mx/4.5.2/../../../../pic32mx/lib\libmchp_peripheral_32MX795F512H.a(pcache.o)
 .debug_line    0x00007136       0x71 c:/program files/microchip/xc32/v1.33/bin/bin/../../lib/gcc/pic32mx/4.5.2/../../../../pic32mx/lib\libmchp_peripheral_32MX795F512H.a(int_configure_system_lib.o)
 .debug_line    0x000071a7       0x72 c:/program files/microchip/xc32/v1.33/bin/bin/../../lib/gcc/pic32mx/4.5.2/../../../../pic32mx/lib\libmchp_peripheral_32MX795F512H.a(int_enable_interrupts_lib.o)
 .debug_line    0x00007219       0x73 c:/program files/microchip/xc32/v1.33/bin/bin/../../lib/gcc/pic32mx/4.5.2/../../../../pic32mx/lib\libmchp_peripheral_32MX795F512H.a(int_disable_interrupts_lib.o)
 .debug_line    0x0000728c       0x73 c:/program files/microchip/xc32/v1.33/bin/bin/../../lib/gcc/pic32mx/4.5.2/../../../../pic32mx/lib\libmchp_peripheral_32MX795F512H.a(int_restore_interrupts_lib.o)
 .debug_line    0x000072ff       0x97 c:/program files/microchip/xc32/v1.33/bin/bin/../../lib/gcc/pic32mx/4.5.2/../../../../pic32mx/lib\libpic32.a(default-bootstrap-exception-handler.o)
 .debug_line    0x00007396       0x84 c:/program files/microchip/xc32/v1.33/bin/bin/../../lib/gcc/pic32mx/4.5.2/../../../../pic32mx/lib\libpic32.a(default-on-reset.o)
 .debug_line    0x0000741a       0x88 c:/program files/microchip/xc32/v1.33/bin/bin/../../lib/gcc/pic32mx/4.5.2/../../../../pic32mx/lib\libpic32.a(default-on-bootstrap.o)
 .debug_line    0x000074a2       0x96 c:/program files/microchip/xc32/v1.33/bin/bin/../../lib/gcc/pic32mx/4.5.2/../../../../pic32mx/lib\libpic32.a(defaultinterrupt.o)
 .debug_line    0x00007538        0x0 c:/program files/microchip/xc32/v1.33/bin/bin/../../lib/gcc/pic32mx/4.5.2/../../../../pic32mx/lib\libc.a(_iob.o)
 .debug_line    0x00007538       0x70 c:/program files/microchip/xc32/v1.33/bin/bin/../../lib/gcc/pic32mx/4.5.2/../../../../pic32mx/lib\libc.a(fflush.o)
 .debug_line    0x000075a8       0x70 c:/program files/microchip/xc32/v1.33/bin/bin/../../lib/gcc/pic32mx/4.5.2/../../../../pic32mx/lib\libc.a(malloc.o)
 .debug_line    0x00007618       0x6e c:/program files/microchip/xc32/v1.33/bin/bin/../../lib/gcc/pic32mx/4.5.2/../../../../pic32mx/lib\libc.a(puts.o)
 .debug_line    0x00007686       0x70 c:/program files/microchip/xc32/v1.33/bin/bin/../../lib/gcc/pic32mx/4.5.2/../../../../pic32mx/lib\libc.a(setbuf.o)
 .debug_line    0x000076f6       0x71 c:/program files/microchip/xc32/v1.33/bin/bin/../../lib/gcc/pic32mx/4.5.2/../../../../pic32mx/lib\libc.a(strncmp.o)
 .debug_line    0x00007767       0x70 c:/program files/microchip/xc32/v1.33/bin/bin/../../lib/gcc/pic32mx/4.5.2/../../../../pic32mx/lib\libc.a(printf_cdfFnopsuxX.eo)
 .debug_line    0x000077d7       0x71 c:/program files/microchip/xc32/v1.33/bin/bin/../../lib/gcc/pic32mx/4.5.2/../../../../pic32mx/lib\libc.a(sprintf_cdfFnopuxX.eo)
 .debug_line    0x00007848       0x70 c:/program files/microchip/xc32/v1.33/bin/bin/../../lib/gcc/pic32mx/4.5.2/../../../../pic32mx/lib\libc.a(sscanf_s.eo)
 .debug_line    0x000078b8       0x6f c:/program files/microchip/xc32/v1.33/bin/bin/../../lib/gcc/pic32mx/4.5.2/../../../../pic32mx/lib\libc.a(_fputc_simple.o)
 .debug_line    0x00007927       0x6d c:/program files/microchip/xc32/v1.33/bin/bin/../../lib/gcc/pic32mx/4.5.2/../../../../pic32mx/lib\libc.a(buf.o)
 .debug_line    0x00007994        0x0 c:/program files/microchip/xc32/v1.33/bin/bin/../../lib/gcc/pic32mx/4.5.2/../../../../pic32mx/lib\libc.a(errno.o)
 .debug_line    0x00007994       0x70 c:/program files/microchip/xc32/v1.33/bin/bin/../../lib/gcc/pic32mx/4.5.2/../../../../pic32mx/lib\libc.a(doprnt_cdfFnopsuxX.eo)
 .debug_line    0x00007a04       0x70 c:/program files/microchip/xc32/v1.33/bin/bin/../../lib/gcc/pic32mx/4.5.2/../../../../pic32mx/lib\libc.a(doscan_s.eo)
 .debug_line    0x00007a74       0x70 c:/program files/microchip/xc32/v1.33/bin/bin/../../lib/gcc/pic32mx/4.5.2/../../../../pic32mx/lib\libc.a(_flsbuf_simple.o)
 .debug_line    0x00007ae4       0x6f c:/program files/microchip/xc32/v1.33/bin/bin/../../lib/gcc/pic32mx/4.5.2/../../../../pic32mx/lib\libc.a(fgetc.o)
 .debug_line    0x00007b53       0x6e c:/program files/microchip/xc32/v1.33/bin/bin/../../lib/gcc/pic32mx/4.5.2/../../../../pic32mx/lib\libc.a(atoi.o)
 .debug_line    0x00007bc1        0x0 c:/program files/microchip/xc32/v1.33/bin/bin/../../lib/gcc/pic32mx/4.5.2/../../../../pic32mx/lib\libc.a(ctype.o)
 .debug_line    0x00007bc1       0x70 c:/program files/microchip/xc32/v1.33/bin/bin/../../lib/gcc/pic32mx/4.5.2/../../../../pic32mx/lib\libc.a(ctypef.o)
 .debug_line    0x00007c31        0x0 c:/program files/microchip/xc32/v1.33/bin/bin/../../lib/gcc/pic32mx/4.5.2/../../../../pic32mx/lib\libc.a(powersf.o)
 .debug_line    0x00007c31       0x70 c:/program files/microchip/xc32/v1.33/bin/bin/../../lib/gcc/pic32mx/4.5.2/../../../../pic32mx/lib\libc.a(ungetc.o)
 .debug_line    0x00007ca1       0x70 c:/program files/microchip/xc32/v1.33/bin/bin/../../lib/gcc/pic32mx/4.5.2/../../../../pic32mx/lib\libc.a(filbuf.o)
 .debug_line    0x00007d11       0x78 c:/program files/microchip/xc32/v1.33/bin/bin/../../lib/gcc/pic32mx/4.5.2/../../../../pic32mx/lib\libpic32.a(sbrk.o)
 .debug_line    0x00007d89       0x78 c:/program files/microchip/xc32/v1.33/bin/bin/../../lib/gcc/pic32mx/4.5.2/../../../../pic32mx/lib\libpic32.a(read.o)
 .debug_line    0x00007e01       0x79 c:/program files/microchip/xc32/v1.33/bin/bin/../../lib/gcc/pic32mx/4.5.2/../../../../pic32mx/lib\libpic32.a(write.o)
 .debug_line    0x00007e7a        0x0 c:/program files/microchip/xc32/v1.33/bin/bin/../../lib/gcc/pic32mx/4.5.2/../../../../pic32mx/lib\libpic32.a(xc32_uart.o)
 .debug_line    0x00007e7a       0x93 c:/program files/microchip/xc32/v1.33/bin/bin/../../lib/gcc/pic32mx/4.5.2/../../../../pic32mx/lib\libe.a(_floatdisf.o)
 .debug_line    0x00007f0d      0x105 c:/program files/microchip/xc32/v1.33/bin/bin/../../lib/gcc/pic32mx/4.5.2\libgcc.a(_floatundisf.o)
 .debug_line    0x00008012      0x168 c:/program files/microchip/xc32/v1.33/bin/bin/../../lib/gcc/pic32mx/4.5.2\libgcc.a(_udivdi3.o)
 .debug_line    0x0000817a      0x155 c:/program files/microchip/xc32/v1.33/bin/bin/../../lib/gcc/pic32mx/4.5.2\libgcc.a(_umoddi3.o)
 .debug_line    0x000082cf       0x8e c:/program files/microchip/xc32/v1.33/bin/bin/../../lib/gcc/pic32mx/4.5.2\libgcc.a(floatunsisf.o)

.debug_frame    0x00000000     0x3788
 *(.debug_frame)
 .debug_frame   0x00000000       0x20 c:/program files/microchip/xc32/v1.33/bin/bin/../../lib/gcc/pic32mx/4.5.2/../../../../pic32mx/lib\software-debug-break.o
 .debug_frame   0x00000020       0x2c build/ChaletDuinoV2_775F512H_/debug/Source/ChaletduinoV2Board.o
 .debug_frame   0x0000004c       0xfc build/ChaletDuinoV2_775F512H_/debug/Source/winc3400/bsp/source/nm_bsp.o
 .debug_frame   0x00000148       0x9c build/ChaletDuinoV2_775F512H_/debug/Source/winc3400/bus_wrapper/source/nm_bus_wrapper.o
 .debug_frame   0x000001e4       0xd4 build/ChaletDuinoV2_775F512H_/debug/Source/winc3400/common/source/nm_common.o
 .debug_frame   0x000002b8      0x208 build/ChaletDuinoV2_775F512H_/debug/Source/winc3400/driver/source/m2m_hif.o
 .debug_frame   0x000004c0      0x10c build/ChaletDuinoV2_775F512H_/debug/Source/winc3400/driver/source/m2m_ota.o
 .debug_frame   0x000005cc       0xd4 build/ChaletDuinoV2_775F512H_/debug/Source/winc3400/driver/source/m2m_periph.o
 .debug_frame   0x000006a0      0x10c build/ChaletDuinoV2_775F512H_/debug/Source/winc3400/driver/source/m2m_ssl.o
 .debug_frame   0x000007ac      0x748 build/ChaletDuinoV2_775F512H_/debug/Source/winc3400/driver/source/m2m_wifi.o
 .debug_frame   0x00000ef4      0x294 build/ChaletDuinoV2_775F512H_/debug/Source/winc3400/driver/source/nmasic.o
 .debug_frame   0x00001188      0x128 build/ChaletDuinoV2_775F512H_/debug/Source/winc3400/driver/source/nmbus.o
 .debug_frame   0x000012b0      0x10c build/ChaletDuinoV2_775F512H_/debug/Source/winc3400/driver/source/nmdrv.o
 .debug_frame   0x000013bc      0x20c build/ChaletDuinoV2_775F512H_/debug/Source/winc3400/driver/source/nmspi.o
 .debug_frame   0x000015c8      0x25c build/ChaletDuinoV2_775F512H_/debug/Source/winc3400/socket/source/socket.o
 .debug_frame   0x00001824      0x17c build/ChaletDuinoV2_775F512H_/debug/Source/winc3400/spi_flash/source/spi_flash.o
 .debug_frame   0x000019a0       0x2c build/ChaletDuinoV2_775F512H_/debug/Source/winc3400/winc_init.o
 .debug_frame   0x000019cc       0x2c build/ChaletDuinoV2_775F512H_/debug/Source/DigitalIO.o
 .debug_frame   0x000019f8      0x138 build/ChaletDuinoV2_775F512H_/debug/Source/InternalUart.o
 .debug_frame   0x00001b30      0x130 build/ChaletDuinoV2_775F512H_/debug/Source/NetworkProtocol.o
 .debug_frame   0x00001c60       0xf4 build/ChaletDuinoV2_775F512H_/debug/Source/Terminal.o
 .debug_frame   0x00001d54      0x128 build/ChaletDuinoV2_775F512H_/debug/Source/Uart.o
 .debug_frame   0x00001e7c      0x10c build/ChaletDuinoV2_775F512H_/debug/Source/Util.o
 .debug_frame   0x00001f88       0x2c build/ChaletDuinoV2_775F512H_/debug/Source/exceptions.o
 .debug_frame   0x00001fb4       0x64 build/ChaletDuinoV2_775F512H_/debug/Source/main.o
 .debug_frame   0x00002018      0x148 build/ChaletDuinoV2_775F512H_/debug/Source/timer.o
 .debug_frame   0x00002160      0x2b8 build/ChaletDuinoV2_775F512H_/debug/Source/WiFiCtrl.o
 .debug_frame   0x00002418       0x2c build/ChaletDuinoV2_775F512H_/debug/Source/SPI.o
 .debug_frame   0x00002444       0x64 build/ChaletDuinoV2_775F512H_/debug/Source/LoraNetworkInterface.o
 .debug_frame   0x000024a8       0xb8 build/ChaletDuinoV2_775F512H_/debug/Source/ChaletPowerRelay.o
 .debug_frame   0x00002560       0x48 build/ChaletDuinoV2_775F512H_/debug/Source/HarakiriRelay.o
 .debug_frame   0x000025a8       0xd8 build/ChaletDuinoV2_775F512H_/debug/Source/BatteryMonitor.o
 .debug_frame   0x00002680      0x198 build/ChaletDuinoV2_775F512H_/debug/Source/ina219.o
 .debug_frame   0x00002818       0x9c build/ChaletDuinoV2_775F512H_/debug/Source/I2C.o
 .debug_frame   0x000028b4      0x160 build/ChaletDuinoV2_775F512H_/debug/Source/SPI_Flash.o
 .debug_frame   0x00002a14       0xa0 build/ChaletDuinoV2_775F512H_/debug/Source/Syslog.o
 .debug_frame   0x00002ab4       0x80 build/ChaletDuinoV2_775F512H_/debug/Source/Watchdog.o
 .debug_frame   0x00002b34      0x1b4 build/ChaletDuinoV2_775F512H_/debug/Source/BootloaderInterface.o
 .debug_frame   0x00002ce8       0x80 build/ChaletDuinoV2_775F512H_/debug/Source/TemperatureSensor.o
 .debug_frame   0x00002d68       0x64 build/ChaletDuinoV2_775F512H_/debug/Source/TC77.o
 .debug_frame   0x00002dcc      0x198 build/ChaletDuinoV2_775F512H_/debug/Source/BootloaderProtocol.o
 .debug_frame   0x00002f64       0x64 build/ChaletDuinoV2_775F512H_/debug/Source/crc32.o
 .debug_frame   0x00002fc8       0x28 c:/program files/microchip/xc32/v1.33/bin/bin/../../lib/gcc/pic32mx/4.5.2/../../../../pic32mx/lib\libmchp_peripheral_32MX795F512H.a(soft_reset_lib.o)
 .debug_frame   0x00002ff0       0x30 c:/program files/microchip/xc32/v1.33/bin/bin/../../lib/gcc/pic32mx/4.5.2/../../../../pic32mx/lib\libmchp_peripheral_32MX795F512H.a(pcache.o)
 .debug_frame   0x00003020       0x20 c:/program files/microchip/xc32/v1.33/bin/bin/../../lib/gcc/pic32mx/4.5.2/../../../../pic32mx/lib\libmchp_peripheral_32MX795F512H.a(int_configure_system_lib.o)
 .debug_frame   0x00003040       0x20 c:/program files/microchip/xc32/v1.33/bin/bin/../../lib/gcc/pic32mx/4.5.2/../../../../pic32mx/lib\libmchp_peripheral_32MX795F512H.a(int_enable_interrupts_lib.o)
 .debug_frame   0x00003060       0x20 c:/program files/microchip/xc32/v1.33/bin/bin/../../lib/gcc/pic32mx/4.5.2/../../../../pic32mx/lib\libmchp_peripheral_32MX795F512H.a(int_disable_interrupts_lib.o)
 .debug_frame   0x00003080       0x20 c:/program files/microchip/xc32/v1.33/bin/bin/../../lib/gcc/pic32mx/4.5.2/../../../../pic32mx/lib\libmchp_peripheral_32MX795F512H.a(int_restore_interrupts_lib.o)
 .debug_frame   0x000030a0       0x28 c:/program files/microchip/xc32/v1.33/bin/bin/../../lib/gcc/pic32mx/4.5.2/../../../../pic32mx/lib\libpic32.a(default-bootstrap-exception-handler.o)
 .debug_frame   0x000030c8       0x20 c:/program files/microchip/xc32/v1.33/bin/bin/../../lib/gcc/pic32mx/4.5.2/../../../../pic32mx/lib\libpic32.a(default-on-reset.o)
 .debug_frame   0x000030e8       0x20 c:/program files/microchip/xc32/v1.33/bin/bin/../../lib/gcc/pic32mx/4.5.2/../../../../pic32mx/lib\libpic32.a(default-on-bootstrap.o)
 .debug_frame   0x00003108       0x20 c:/program files/microchip/xc32/v1.33/bin/bin/../../lib/gcc/pic32mx/4.5.2/../../../../pic32mx/lib\libpic32.a(defaultinterrupt.o)
 .debug_frame   0x00003128       0x2c c:/program files/microchip/xc32/v1.33/bin/bin/../../lib/gcc/pic32mx/4.5.2/../../../../pic32mx/lib\libc.a(fflush.o)
 .debug_frame   0x00003154       0x6c c:/program files/microchip/xc32/v1.33/bin/bin/../../lib/gcc/pic32mx/4.5.2/../../../../pic32mx/lib\libc.a(malloc.o)
 .debug_frame   0x000031c0       0x48 c:/program files/microchip/xc32/v1.33/bin/bin/../../lib/gcc/pic32mx/4.5.2/../../../../pic32mx/lib\libc.a(puts.o)
 .debug_frame   0x00003208       0x38 c:/program files/microchip/xc32/v1.33/bin/bin/../../lib/gcc/pic32mx/4.5.2/../../../../pic32mx/lib\libc.a(setbuf.o)
 .debug_frame   0x00003240       0x20 c:/program files/microchip/xc32/v1.33/bin/bin/../../lib/gcc/pic32mx/4.5.2/../../../../pic32mx/lib\libc.a(strncmp.o)
 .debug_frame   0x00003260       0x28 c:/program files/microchip/xc32/v1.33/bin/bin/../../lib/gcc/pic32mx/4.5.2/../../../../pic32mx/lib\libc.a(printf_cdfFnopsuxX.eo)
 .debug_frame   0x00003288       0x2c c:/program files/microchip/xc32/v1.33/bin/bin/../../lib/gcc/pic32mx/4.5.2/../../../../pic32mx/lib\libc.a(sprintf_cdfFnopuxX.eo)
 .debug_frame   0x000032b4       0x28 c:/program files/microchip/xc32/v1.33/bin/bin/../../lib/gcc/pic32mx/4.5.2/../../../../pic32mx/lib\libc.a(sscanf_s.eo)
 .debug_frame   0x000032dc       0x2c c:/program files/microchip/xc32/v1.33/bin/bin/../../lib/gcc/pic32mx/4.5.2/../../../../pic32mx/lib\libc.a(_fputc_simple.o)
 .debug_frame   0x00003308       0x38 c:/program files/microchip/xc32/v1.33/bin/bin/../../lib/gcc/pic32mx/4.5.2/../../../../pic32mx/lib\libc.a(buf.o)
 .debug_frame   0x00003340       0x58 c:/program files/microchip/xc32/v1.33/bin/bin/../../lib/gcc/pic32mx/4.5.2/../../../../pic32mx/lib\libc.a(doprnt_cdfFnopsuxX.eo)
 .debug_frame   0x00003398       0x74 c:/program files/microchip/xc32/v1.33/bin/bin/../../lib/gcc/pic32mx/4.5.2/../../../../pic32mx/lib\libc.a(doscan_s.eo)
 .debug_frame   0x0000340c       0x28 c:/program files/microchip/xc32/v1.33/bin/bin/../../lib/gcc/pic32mx/4.5.2/../../../../pic32mx/lib\libc.a(_flsbuf_simple.o)
 .debug_frame   0x00003434       0x30 c:/program files/microchip/xc32/v1.33/bin/bin/../../lib/gcc/pic32mx/4.5.2/../../../../pic32mx/lib\libc.a(fgetc.o)
 .debug_frame   0x00003464       0x20 c:/program files/microchip/xc32/v1.33/bin/bin/../../lib/gcc/pic32mx/4.5.2/../../../../pic32mx/lib\libc.a(atoi.o)
 .debug_frame   0x00003484      0x120 c:/program files/microchip/xc32/v1.33/bin/bin/../../lib/gcc/pic32mx/4.5.2/../../../../pic32mx/lib\libc.a(ctypef.o)
 .debug_frame   0x000035a4       0x20 c:/program files/microchip/xc32/v1.33/bin/bin/../../lib/gcc/pic32mx/4.5.2/../../../../pic32mx/lib\libc.a(ungetc.o)
 .debug_frame   0x000035c4       0x30 c:/program files/microchip/xc32/v1.33/bin/bin/../../lib/gcc/pic32mx/4.5.2/../../../../pic32mx/lib\libc.a(filbuf.o)
 .debug_frame   0x000035f4       0x8c c:/program files/microchip/xc32/v1.33/bin/bin/../../lib/gcc/pic32mx/4.5.2/../../../../pic32mx/lib\libpic32.a(sbrk.o)
 .debug_frame   0x00003680       0x2c c:/program files/microchip/xc32/v1.33/bin/bin/../../lib/gcc/pic32mx/4.5.2/../../../../pic32mx/lib\libpic32.a(read.o)
 .debug_frame   0x000036ac       0x28 c:/program files/microchip/xc32/v1.33/bin/bin/../../lib/gcc/pic32mx/4.5.2/../../../../pic32mx/lib\libpic32.a(write.o)
 .debug_frame   0x000036d4       0x20 c:/program files/microchip/xc32/v1.33/bin/bin/../../lib/gcc/pic32mx/4.5.2/../../../../pic32mx/lib\libe.a(_floatdisf.o)
 .debug_frame   0x000036f4       0x2c c:/program files/microchip/xc32/v1.33/bin/bin/../../lib/gcc/pic32mx/4.5.2\libgcc.a(_floatundisf.o)
 .debug_frame   0x00003720       0x20 c:/program files/microchip/xc32/v1.33/bin/bin/../../lib/gcc/pic32mx/4.5.2\libgcc.a(_udivdi3.o)
 .debug_frame   0x00003740       0x20 c:/program files/microchip/xc32/v1.33/bin/bin/../../lib/gcc/pic32mx/4.5.2\libgcc.a(_umoddi3.o)
 .debug_frame   0x00003760       0x28 c:/program files/microchip/xc32/v1.33/bin/bin/../../lib/gcc/pic32mx/4.5.2\libgcc.a(floatunsisf.o)

.debug_str      0x00000000     0x3167
 *(.debug_str)
 .debug_str     0x00000000        0x0 c:/program files/microchip/xc32/v1.33/bin/bin/../../lib/gcc/pic32mx/4.5.2/../../../../pic32mx/lib\software-debug-break.o
 .debug_str     0x00000000      0x242 build/ChaletDuinoV2_775F512H_/debug/Source/ChaletduinoV2Board.o
 .debug_str     0x00000242      0x14a build/ChaletDuinoV2_775F512H_/debug/Source/winc3400/bsp/source/nm_bsp.o
 .debug_str     0x0000038c      0x149 build/ChaletDuinoV2_775F512H_/debug/Source/winc3400/bus_wrapper/source/nm_bus_wrapper.o
 .debug_str     0x000004d5        0xa build/ChaletDuinoV2_775F512H_/debug/Source/winc3400/common/source/nm_common.o
 .debug_str     0x000004df        0x0 build/ChaletDuinoV2_775F512H_/debug/Source/winc3400/driver/source/m2m_ate_mode.o
 .debug_str     0x000004df        0x0 build/ChaletDuinoV2_775F512H_/debug/Source/winc3400/driver/source/m2m_crypto.o
 .debug_str     0x000004df       0x36 build/ChaletDuinoV2_775F512H_/debug/Source/winc3400/driver/source/m2m_hif.o
 .debug_str     0x00000515        0x0 build/ChaletDuinoV2_775F512H_/debug/Source/winc3400/driver/source/m2m_ota.o
 .debug_str     0x00000515        0xa build/ChaletDuinoV2_775F512H_/debug/Source/winc3400/driver/source/m2m_periph.o
 .debug_str     0x0000051f       0x25 build/ChaletDuinoV2_775F512H_/debug/Source/winc3400/driver/source/m2m_ssl.o
 .debug_str     0x00000544      0x178 build/ChaletDuinoV2_775F512H_/debug/Source/winc3400/driver/source/m2m_wifi.o
 .debug_str     0x000006bc       0x2d build/ChaletDuinoV2_775F512H_/debug/Source/winc3400/driver/source/nmasic.o
 .debug_str     0x000006e9       0x31 build/ChaletDuinoV2_775F512H_/debug/Source/winc3400/driver/source/nmbus.o
 .debug_str     0x0000071a       0x12 build/ChaletDuinoV2_775F512H_/debug/Source/winc3400/driver/source/nmdrv.o
 .debug_str     0x0000072c        0x0 build/ChaletDuinoV2_775F512H_/debug/Source/winc3400/driver/source/nmi2c.o
 .debug_str     0x0000072c       0x19 build/ChaletDuinoV2_775F512H_/debug/Source/winc3400/driver/source/nmspi.o
 .debug_str     0x00000745        0x0 build/ChaletDuinoV2_775F512H_/debug/Source/winc3400/driver/source/nmuart.o
 .debug_str     0x00000745      0x168 build/ChaletDuinoV2_775F512H_/debug/Source/winc3400/socket/source/socket.o
 .debug_str     0x000008ad       0x2d build/ChaletDuinoV2_775F512H_/debug/Source/winc3400/spi_flash/source/spi_flash.o
 .debug_str     0x000008da       0x16 build/ChaletDuinoV2_775F512H_/debug/Source/winc3400/winc_init.o
 .debug_str     0x000008f0      0x12f build/ChaletDuinoV2_775F512H_/debug/Source/DigitalIO.o
 .debug_str     0x00000a1f      0x226 build/ChaletDuinoV2_775F512H_/debug/Source/InternalUart.o
 .debug_str     0x00000c45      0x14f build/ChaletDuinoV2_775F512H_/debug/Source/NetworkProtocol.o
 .debug_str     0x00000d94      0x1ac build/ChaletDuinoV2_775F512H_/debug/Source/Terminal.o
 .debug_str     0x00000f40      0x181 build/ChaletDuinoV2_775F512H_/debug/Source/Uart.o
 .debug_str     0x000010c1      0x145 build/ChaletDuinoV2_775F512H_/debug/Source/Util.o
 .debug_str     0x00001206      0x12f build/ChaletDuinoV2_775F512H_/debug/Source/exceptions.o
 .debug_str     0x00001335      0x12f build/ChaletDuinoV2_775F512H_/debug/Source/interrupts.o
 .debug_str     0x00001464      0x14d build/ChaletDuinoV2_775F512H_/debug/Source/main.o
 .debug_str     0x000015b1      0x12f build/ChaletDuinoV2_775F512H_/debug/Source/system.o
 .debug_str     0x000016e0      0x12f build/ChaletDuinoV2_775F512H_/debug/Source/template.o
 .debug_str     0x0000180f      0x17f build/ChaletDuinoV2_775F512H_/debug/Source/timer.o
 .debug_str     0x0000198e      0x281 build/ChaletDuinoV2_775F512H_/debug/Source/WiFiCtrl.o
 .debug_str     0x00001c0f      0x146 build/ChaletDuinoV2_775F512H_/debug/Source/SPI.o
 .debug_str     0x00001d55      0x170 build/ChaletDuinoV2_775F512H_/debug/Source/LoraNetworkInterface.o
 .debug_str     0x00001ec5      0x15b build/ChaletDuinoV2_775F512H_/debug/Source/ChaletPowerRelay.o
 .debug_str     0x00002020      0x138 build/ChaletDuinoV2_775F512H_/debug/Source/HarakiriRelay.o
 .debug_str     0x00002158      0x1ac build/ChaletDuinoV2_775F512H_/debug/Source/BatteryMonitor.o
 .debug_str     0x00002304      0x18b build/ChaletDuinoV2_775F512H_/debug/Source/ina219.o
 .debug_str     0x0000248f      0x17e build/ChaletDuinoV2_775F512H_/debug/Source/I2C.o
 .debug_str     0x0000260d      0x193 build/ChaletDuinoV2_775F512H_/debug/Source/SPI_Flash.o
 .debug_str     0x000027a0      0x14b build/ChaletDuinoV2_775F512H_/debug/Source/Syslog.o
 .debug_str     0x000028eb      0x15e build/ChaletDuinoV2_775F512H_/debug/Source/Watchdog.o
 .debug_str     0x00002a49      0x29e build/ChaletDuinoV2_775F512H_/debug/Source/BootloaderInterface.o
 .debug_str     0x00002ce7      0x13a build/ChaletDuinoV2_775F512H_/debug/Source/TemperatureSensor.o
 .debug_str     0x00002e21      0x159 build/ChaletDuinoV2_775F512H_/debug/Source/TC77.o
 .debug_str     0x00002f7a      0x1ed build/ChaletDuinoV2_775F512H_/debug/Source/BootloaderProtocol.o
 .debug_str     0x00003167        0x0 build/ChaletDuinoV2_775F512H_/debug/Source/crc32.o
 .debug_str     0x00003167        0x0 c:/program files/microchip/xc32/v1.33/bin/bin/../../lib/gcc/pic32mx/4.5.2/../../../../pic32mx/lib\libmchp_peripheral_32MX795F512H.a(soft_reset_lib.o)
 .debug_str     0x00003167        0x0 c:/program files/microchip/xc32/v1.33/bin/bin/../../lib/gcc/pic32mx/4.5.2/../../../../pic32mx/lib\libmchp_peripheral_32MX795F512H.a(pcache.o)
 .debug_str     0x00003167        0x0 c:/program files/microchip/xc32/v1.33/bin/bin/../../lib/gcc/pic32mx/4.5.2/../../../../pic32mx/lib\libmchp_peripheral_32MX795F512H.a(int_configure_system_lib.o)
 .debug_str     0x00003167        0x0 c:/program files/microchip/xc32/v1.33/bin/bin/../../lib/gcc/pic32mx/4.5.2/../../../../pic32mx/lib\libmchp_peripheral_32MX795F512H.a(int_enable_interrupts_lib.o)
 .debug_str     0x00003167        0x0 c:/program files/microchip/xc32/v1.33/bin/bin/../../lib/gcc/pic32mx/4.5.2/../../../../pic32mx/lib\libmchp_peripheral_32MX795F512H.a(int_disable_interrupts_lib.o)
 .debug_str     0x00003167        0x0 c:/program files/microchip/xc32/v1.33/bin/bin/../../lib/gcc/pic32mx/4.5.2/../../../../pic32mx/lib\libmchp_peripheral_32MX795F512H.a(int_restore_interrupts_lib.o)
 .debug_str     0x00003167        0x0 c:/program files/microchip/xc32/v1.33/bin/bin/../../lib/gcc/pic32mx/4.5.2/../../../../pic32mx/lib\libpic32.a(default-bootstrap-exception-handler.o)
 .debug_str     0x00003167        0x0 c:/program files/microchip/xc32/v1.33/bin/bin/../../lib/gcc/pic32mx/4.5.2/../../../../pic32mx/lib\libpic32.a(default-on-reset.o)
 .debug_str     0x00003167        0x0 c:/program files/microchip/xc32/v1.33/bin/bin/../../lib/gcc/pic32mx/4.5.2/../../../../pic32mx/lib\libpic32.a(default-on-bootstrap.o)
 .debug_str     0x00003167        0x0 c:/program files/microchip/xc32/v1.33/bin/bin/../../lib/gcc/pic32mx/4.5.2/../../../../pic32mx/lib\libpic32.a(defaultinterrupt.o)
 .debug_str     0x00003167        0x0 c:/program files/microchip/xc32/v1.33/bin/bin/../../lib/gcc/pic32mx/4.5.2/../../../../pic32mx/lib\libc.a(_iob.o)
 .debug_str     0x00003167        0x0 c:/program files/microchip/xc32/v1.33/bin/bin/../../lib/gcc/pic32mx/4.5.2/../../../../pic32mx/lib\libc.a(fflush.o)
 .debug_str     0x00003167        0x0 c:/program files/microchip/xc32/v1.33/bin/bin/../../lib/gcc/pic32mx/4.5.2/../../../../pic32mx/lib\libc.a(malloc.o)
 .debug_str     0x00003167        0x0 c:/program files/microchip/xc32/v1.33/bin/bin/../../lib/gcc/pic32mx/4.5.2/../../../../pic32mx/lib\libc.a(puts.o)
 .debug_str     0x00003167        0x0 c:/program files/microchip/xc32/v1.33/bin/bin/../../lib/gcc/pic32mx/4.5.2/../../../../pic32mx/lib\libc.a(setbuf.o)
 .debug_str     0x00003167        0x0 c:/program files/microchip/xc32/v1.33/bin/bin/../../lib/gcc/pic32mx/4.5.2/../../../../pic32mx/lib\libc.a(strncmp.o)
 .debug_str     0x00003167        0x0 c:/program files/microchip/xc32/v1.33/bin/bin/../../lib/gcc/pic32mx/4.5.2/../../../../pic32mx/lib\libc.a(printf_cdfFnopsuxX.eo)
 .debug_str     0x00003167        0x0 c:/program files/microchip/xc32/v1.33/bin/bin/../../lib/gcc/pic32mx/4.5.2/../../../../pic32mx/lib\libc.a(sprintf_cdfFnopuxX.eo)
 .debug_str     0x00003167        0x0 c:/program files/microchip/xc32/v1.33/bin/bin/../../lib/gcc/pic32mx/4.5.2/../../../../pic32mx/lib\libc.a(sscanf_s.eo)
 .debug_str     0x00003167        0x0 c:/program files/microchip/xc32/v1.33/bin/bin/../../lib/gcc/pic32mx/4.5.2/../../../../pic32mx/lib\libc.a(_fputc_simple.o)
 .debug_str     0x00003167        0x0 c:/program files/microchip/xc32/v1.33/bin/bin/../../lib/gcc/pic32mx/4.5.2/../../../../pic32mx/lib\libc.a(buf.o)
 .debug_str     0x00003167        0x0 c:/program files/microchip/xc32/v1.33/bin/bin/../../lib/gcc/pic32mx/4.5.2/../../../../pic32mx/lib\libc.a(errno.o)
 .debug_str     0x00003167        0x0 c:/program files/microchip/xc32/v1.33/bin/bin/../../lib/gcc/pic32mx/4.5.2/../../../../pic32mx/lib\libc.a(doprnt_cdfFnopsuxX.eo)
 .debug_str     0x00003167        0x0 c:/program files/microchip/xc32/v1.33/bin/bin/../../lib/gcc/pic32mx/4.5.2/../../../../pic32mx/lib\libc.a(doscan_s.eo)
 .debug_str     0x00003167        0x0 c:/program files/microchip/xc32/v1.33/bin/bin/../../lib/gcc/pic32mx/4.5.2/../../../../pic32mx/lib\libc.a(_flsbuf_simple.o)
 .debug_str     0x00003167        0x0 c:/program files/microchip/xc32/v1.33/bin/bin/../../lib/gcc/pic32mx/4.5.2/../../../../pic32mx/lib\libc.a(fgetc.o)
 .debug_str     0x00003167        0x0 c:/program files/microchip/xc32/v1.33/bin/bin/../../lib/gcc/pic32mx/4.5.2/../../../../pic32mx/lib\libc.a(atoi.o)
 .debug_str     0x00003167        0x0 c:/program files/microchip/xc32/v1.33/bin/bin/../../lib/gcc/pic32mx/4.5.2/../../../../pic32mx/lib\libc.a(ctype.o)
 .debug_str     0x00003167        0x0 c:/program files/microchip/xc32/v1.33/bin/bin/../../lib/gcc/pic32mx/4.5.2/../../../../pic32mx/lib\libc.a(ctypef.o)
 .debug_str     0x00003167        0x0 c:/program files/microchip/xc32/v1.33/bin/bin/../../lib/gcc/pic32mx/4.5.2/../../../../pic32mx/lib\libc.a(powersf.o)
 .debug_str     0x00003167        0x0 c:/program files/microchip/xc32/v1.33/bin/bin/../../lib/gcc/pic32mx/4.5.2/../../../../pic32mx/lib\libc.a(ungetc.o)
 .debug_str     0x00003167        0x0 c:/program files/microchip/xc32/v1.33/bin/bin/../../lib/gcc/pic32mx/4.5.2/../../../../pic32mx/lib\libc.a(filbuf.o)
 .debug_str     0x00003167        0x0 c:/program files/microchip/xc32/v1.33/bin/bin/../../lib/gcc/pic32mx/4.5.2/../../../../pic32mx/lib\libpic32.a(sbrk.o)
 .debug_str     0x00003167        0x0 c:/program files/microchip/xc32/v1.33/bin/bin/../../lib/gcc/pic32mx/4.5.2/../../../../pic32mx/lib\libpic32.a(read.o)
 .debug_str     0x00003167        0x0 c:/program files/microchip/xc32/v1.33/bin/bin/../../lib/gcc/pic32mx/4.5.2/../../../../pic32mx/lib\libpic32.a(write.o)
 .debug_str     0x00003167        0x0 c:/program files/microchip/xc32/v1.33/bin/bin/../../lib/gcc/pic32mx/4.5.2/../../../../pic32mx/lib\libpic32.a(xc32_uart.o)
 .debug_str     0x00003167        0x0 c:/program files/microchip/xc32/v1.33/bin/bin/../../lib/gcc/pic32mx/4.5.2/../../../../pic32mx/lib\libe.a(_floatdisf.o)
 .debug_str     0x00003167        0x0 c:/program files/microchip/xc32/v1.33/bin/bin/../../lib/gcc/pic32mx/4.5.2\libgcc.a(_floatundisf.o)
 .debug_str     0x00003167        0x0 c:/program files/microchip/xc32/v1.33/bin/bin/../../lib/gcc/pic32mx/4.5.2\libgcc.a(_udivdi3.o)
 .debug_str     0x00003167        0x0 c:/program files/microchip/xc32/v1.33/bin/bin/../../lib/gcc/pic32mx/4.5.2\libgcc.a(_umoddi3.o)
 .debug_str     0x00003167        0x0 c:/program files/microchip/xc32/v1.33/bin/bin/../../lib/gcc/pic32mx/4.5.2\libgcc.a(floatunsisf.o)

.debug_loc      0x00000000     0xfec1
 *(.debug_loc)
 .debug_loc     0x00000000      0x130 build/ChaletDuinoV2_775F512H_/debug/Source/ChaletduinoV2Board.o
 .debug_loc     0x00000130      0x168 build/ChaletDuinoV2_775F512H_/debug/Source/winc3400/bsp/source/nm_bsp.o
 .debug_loc     0x00000298      0x4b8 build/ChaletDuinoV2_775F512H_/debug/Source/winc3400/bus_wrapper/source/nm_bus_wrapper.o
 .debug_loc     0x00000750      0x59d build/ChaletDuinoV2_775F512H_/debug/Source/winc3400/common/source/nm_common.o
 .debug_loc     0x00000ced      0xcb3 build/ChaletDuinoV2_775F512H_/debug/Source/winc3400/driver/source/m2m_hif.o
 .debug_loc     0x000019a0      0x48f build/ChaletDuinoV2_775F512H_/debug/Source/winc3400/driver/source/m2m_ota.o
 .debug_loc     0x00001e2f      0x2e2 build/ChaletDuinoV2_775F512H_/debug/Source/winc3400/driver/source/m2m_periph.o
 .debug_loc     0x00002111      0x7ba build/ChaletDuinoV2_775F512H_/debug/Source/winc3400/driver/source/m2m_ssl.o
 .debug_loc     0x000028cb     0x1f19 build/ChaletDuinoV2_775F512H_/debug/Source/winc3400/driver/source/m2m_wifi.o
 .debug_loc     0x000047e4      0xfbb build/ChaletDuinoV2_775F512H_/debug/Source/winc3400/driver/source/nmasic.o
 .debug_loc     0x0000579f      0x5e3 build/ChaletDuinoV2_775F512H_/debug/Source/winc3400/driver/source/nmbus.o
 .debug_loc     0x00005d82      0x685 build/ChaletDuinoV2_775F512H_/debug/Source/winc3400/driver/source/nmdrv.o
 .debug_loc     0x00006407      0xd65 build/ChaletDuinoV2_775F512H_/debug/Source/winc3400/driver/source/nmspi.o
 .debug_loc     0x0000716c     0x12f2 build/ChaletDuinoV2_775F512H_/debug/Source/winc3400/socket/source/socket.o
 .debug_loc     0x0000845e      0xd61 build/ChaletDuinoV2_775F512H_/debug/Source/winc3400/spi_flash/source/spi_flash.o
 .debug_loc     0x000091bf       0x6a build/ChaletDuinoV2_775F512H_/debug/Source/winc3400/winc_init.o
 .debug_loc     0x00009229       0x2c build/ChaletDuinoV2_775F512H_/debug/Source/DigitalIO.o
 .debug_loc     0x00009255      0x5ee build/ChaletDuinoV2_775F512H_/debug/Source/InternalUart.o
 .debug_loc     0x00009843      0x369 build/ChaletDuinoV2_775F512H_/debug/Source/NetworkProtocol.o
 .debug_loc     0x00009bac      0x25f build/ChaletDuinoV2_775F512H_/debug/Source/Terminal.o
 .debug_loc     0x00009e0b      0x72a build/ChaletDuinoV2_775F512H_/debug/Source/Uart.o
 .debug_loc     0x0000a535      0x6a1 build/ChaletDuinoV2_775F512H_/debug/Source/Util.o
 .debug_loc     0x0000abd6       0x4b build/ChaletDuinoV2_775F512H_/debug/Source/exceptions.o
 .debug_loc     0x0000ac21      0x31e build/ChaletDuinoV2_775F512H_/debug/Source/main.o
 .debug_loc     0x0000af3f      0x484 build/ChaletDuinoV2_775F512H_/debug/Source/timer.o
 .debug_loc     0x0000b3c3      0xa0d build/ChaletDuinoV2_775F512H_/debug/Source/WiFiCtrl.o
 .debug_loc     0x0000bdd0       0x56 build/ChaletDuinoV2_775F512H_/debug/Source/SPI.o
 .debug_loc     0x0000be26      0x3e5 build/ChaletDuinoV2_775F512H_/debug/Source/LoraNetworkInterface.o
 .debug_loc     0x0000c20b      0x108 build/ChaletDuinoV2_775F512H_/debug/Source/ChaletPowerRelay.o
 .debug_loc     0x0000c313       0x58 build/ChaletDuinoV2_775F512H_/debug/Source/HarakiriRelay.o
 .debug_loc     0x0000c36b      0x1bf build/ChaletDuinoV2_775F512H_/debug/Source/BatteryMonitor.o
 .debug_loc     0x0000c52a      0x412 build/ChaletDuinoV2_775F512H_/debug/Source/ina219.o
 .debug_loc     0x0000c93c      0x21a build/ChaletDuinoV2_775F512H_/debug/Source/I2C.o
 .debug_loc     0x0000cb56      0x8a5 build/ChaletDuinoV2_775F512H_/debug/Source/SPI_Flash.o
 .debug_loc     0x0000d3fb      0x10e build/ChaletDuinoV2_775F512H_/debug/Source/Syslog.o
 .debug_loc     0x0000d509       0xb0 build/ChaletDuinoV2_775F512H_/debug/Source/Watchdog.o
 .debug_loc     0x0000d5b9      0x7f8 build/ChaletDuinoV2_775F512H_/debug/Source/BootloaderInterface.o
 .debug_loc     0x0000ddb1       0xb0 build/ChaletDuinoV2_775F512H_/debug/Source/TemperatureSensor.o
 .debug_loc     0x0000de61       0xf4 build/ChaletDuinoV2_775F512H_/debug/Source/TC77.o
 .debug_loc     0x0000df55      0x812 build/ChaletDuinoV2_775F512H_/debug/Source/BootloaderProtocol.o
 .debug_loc     0x0000e767      0x2d1 build/ChaletDuinoV2_775F512H_/debug/Source/crc32.o
 .debug_loc     0x0000ea38       0xc9 c:/program files/microchip/xc32/v1.33/bin/bin/../../lib/gcc/pic32mx/4.5.2\libgcc.a(_floatundisf.o)
 .debug_loc     0x0000eb01      0x9c3 c:/program files/microchip/xc32/v1.33/bin/bin/../../lib/gcc/pic32mx/4.5.2\libgcc.a(_udivdi3.o)
 .debug_loc     0x0000f4c4      0x995 c:/program files/microchip/xc32/v1.33/bin/bin/../../lib/gcc/pic32mx/4.5.2\libgcc.a(_umoddi3.o)
 .debug_loc     0x0000fe59       0x68 c:/program files/microchip/xc32/v1.33/bin/bin/../../lib/gcc/pic32mx/4.5.2\libgcc.a(floatunsisf.o)

.debug_macinfo
 *(.debug_macinfo)

.debug_weaknames
 *(.debug_weaknames)

.debug_funcnames
 *(.debug_funcnames)

.debug_typenames
 *(.debug_typenames)

.debug_varnames
 *(.debug_varnames)

.debug_pubtypes
                0x00000000     0x3431
 *(.debug_pubtypes)
 .debug_pubtypes
                0x00000000      0x276 build/ChaletDuinoV2_775F512H_/debug/Source/ChaletduinoV2Board.o
 .debug_pubtypes
                0x00000276      0x149 build/ChaletDuinoV2_775F512H_/debug/Source/winc3400/bsp/source/nm_bsp.o
 .debug_pubtypes
                0x000003bf      0x14c build/ChaletDuinoV2_775F512H_/debug/Source/winc3400/bus_wrapper/source/nm_bus_wrapper.o
 .debug_pubtypes
                0x0000050b       0x3c build/ChaletDuinoV2_775F512H_/debug/Source/winc3400/common/source/nm_common.o
 .debug_pubtypes
                0x00000547       0x12 build/ChaletDuinoV2_775F512H_/debug/Source/winc3400/driver/source/m2m_crypto.o
 .debug_pubtypes
                0x00000559       0x5e build/ChaletDuinoV2_775F512H_/debug/Source/winc3400/driver/source/m2m_hif.o
 .debug_pubtypes
                0x000005b7       0xa2 build/ChaletDuinoV2_775F512H_/debug/Source/winc3400/driver/source/m2m_ota.o
 .debug_pubtypes
                0x00000659       0x48 build/ChaletDuinoV2_775F512H_/debug/Source/winc3400/driver/source/m2m_periph.o
 .debug_pubtypes
                0x000006a1      0x10c build/ChaletDuinoV2_775F512H_/debug/Source/winc3400/driver/source/m2m_ssl.o
 .debug_pubtypes
                0x000007ad      0x41c build/ChaletDuinoV2_775F512H_/debug/Source/winc3400/driver/source/m2m_wifi.o
 .debug_pubtypes
                0x00000bc9       0x40 build/ChaletDuinoV2_775F512H_/debug/Source/winc3400/driver/source/nmasic.o
 .debug_pubtypes
                0x00000c09       0x56 build/ChaletDuinoV2_775F512H_/debug/Source/winc3400/driver/source/nmbus.o
 .debug_pubtypes
                0x00000c5f       0x5a build/ChaletDuinoV2_775F512H_/debug/Source/winc3400/driver/source/nmdrv.o
 .debug_pubtypes
                0x00000cb9       0x12 build/ChaletDuinoV2_775F512H_/debug/Source/winc3400/driver/source/nmi2c.o
 .debug_pubtypes
                0x00000ccb       0x47 build/ChaletDuinoV2_775F512H_/debug/Source/winc3400/driver/source/nmspi.o
 .debug_pubtypes
                0x00000d12       0x12 build/ChaletDuinoV2_775F512H_/debug/Source/winc3400/driver/source/nmuart.o
 .debug_pubtypes
                0x00000d24      0x29d build/ChaletDuinoV2_775F512H_/debug/Source/winc3400/socket/source/socket.o
 .debug_pubtypes
                0x00000fc1       0x3c build/ChaletDuinoV2_775F512H_/debug/Source/winc3400/spi_flash/source/spi_flash.o
 .debug_pubtypes
                0x00000ffd       0xcf build/ChaletDuinoV2_775F512H_/debug/Source/winc3400/winc_init.o
 .debug_pubtypes
                0x000010cc       0xe7 build/ChaletDuinoV2_775F512H_/debug/Source/DigitalIO.o
 .debug_pubtypes
                0x000011b3      0x1f8 build/ChaletDuinoV2_775F512H_/debug/Source/InternalUart.o
 .debug_pubtypes
                0x000013ab      0x136 build/ChaletDuinoV2_775F512H_/debug/Source/NetworkProtocol.o
 .debug_pubtypes
                0x000014e1      0x175 build/ChaletDuinoV2_775F512H_/debug/Source/Terminal.o
 .debug_pubtypes
                0x00001656      0x155 build/ChaletDuinoV2_775F512H_/debug/Source/Uart.o
 .debug_pubtypes
                0x000017ab       0xe7 build/ChaletDuinoV2_775F512H_/debug/Source/Util.o
 .debug_pubtypes
                0x00001892       0xe7 build/ChaletDuinoV2_775F512H_/debug/Source/exceptions.o
 .debug_pubtypes
                0x00001979       0xe7 build/ChaletDuinoV2_775F512H_/debug/Source/interrupts.o
 .debug_pubtypes
                0x00001a60      0x13c build/ChaletDuinoV2_775F512H_/debug/Source/main.o
 .debug_pubtypes
                0x00001b9c       0xe7 build/ChaletDuinoV2_775F512H_/debug/Source/system.o
 .debug_pubtypes
                0x00001c83       0xe7 build/ChaletDuinoV2_775F512H_/debug/Source/template.o
 .debug_pubtypes
                0x00001d6a      0x14e build/ChaletDuinoV2_775F512H_/debug/Source/timer.o
 .debug_pubtypes
                0x00001eb8      0x2dc build/ChaletDuinoV2_775F512H_/debug/Source/WiFiCtrl.o
 .debug_pubtypes
                0x00002194       0xfc build/ChaletDuinoV2_775F512H_/debug/Source/SPI.o
 .debug_pubtypes
                0x00002290      0x17e build/ChaletDuinoV2_775F512H_/debug/Source/LoraNetworkInterface.o
 .debug_pubtypes
                0x0000240e      0x13f build/ChaletDuinoV2_775F512H_/debug/Source/ChaletPowerRelay.o
 .debug_pubtypes
                0x0000254d      0x101 build/ChaletDuinoV2_775F512H_/debug/Source/HarakiriRelay.o
 .debug_pubtypes
                0x0000264e      0x137 build/ChaletDuinoV2_775F512H_/debug/Source/BatteryMonitor.o
 .debug_pubtypes
                0x00002785      0x121 build/ChaletDuinoV2_775F512H_/debug/Source/ina219.o
 .debug_pubtypes
                0x000028a6      0x119 build/ChaletDuinoV2_775F512H_/debug/Source/I2C.o
 .debug_pubtypes
                0x000029bf       0xf8 build/ChaletDuinoV2_775F512H_/debug/Source/SPI_Flash.o
 .debug_pubtypes
                0x00002ab7      0x11a build/ChaletDuinoV2_775F512H_/debug/Source/Syslog.o
 .debug_pubtypes
                0x00002bd1       0xf8 build/ChaletDuinoV2_775F512H_/debug/Source/Watchdog.o
 .debug_pubtypes
                0x00002cc9      0x2d9 build/ChaletDuinoV2_775F512H_/debug/Source/BootloaderInterface.o
 .debug_pubtypes
                0x00002fa2       0xe7 build/ChaletDuinoV2_775F512H_/debug/Source/TemperatureSensor.o
 .debug_pubtypes
                0x00003089      0x10d build/ChaletDuinoV2_775F512H_/debug/Source/TC77.o
 .debug_pubtypes
                0x00003196      0x149 build/ChaletDuinoV2_775F512H_/debug/Source/BootloaderProtocol.o
 .debug_pubtypes
                0x000032df       0x2c build/ChaletDuinoV2_775F512H_/debug/Source/crc32.o
 .debug_pubtypes
                0x0000330b       0x40 c:/program files/microchip/xc32/v1.33/bin/bin/../../lib/gcc/pic32mx/4.5.2\libgcc.a(_floatundisf.o)
 .debug_pubtypes
                0x0000334b       0x59 c:/program files/microchip/xc32/v1.33/bin/bin/../../lib/gcc/pic32mx/4.5.2\libgcc.a(_udivdi3.o)
 .debug_pubtypes
                0x000033a4       0x59 c:/program files/microchip/xc32/v1.33/bin/bin/../../lib/gcc/pic32mx/4.5.2\libgcc.a(_umoddi3.o)
 .debug_pubtypes
                0x000033fd       0x34 c:/program files/microchip/xc32/v1.33/bin/bin/../../lib/gcc/pic32mx/4.5.2\libgcc.a(floatunsisf.o)

.debug_ranges   0x00000000      0x290
 *(.debug_ranges)
 .debug_ranges  0x00000000       0x10 c:/program files/microchip/xc32/v1.33/bin/bin/../../lib/gcc/pic32mx/4.5.2/../../../../pic32mx/lib\software-debug-break.o
 .debug_ranges  0x00000010       0x10 c:/program files/microchip/xc32/v1.33/bin/bin/../../lib/gcc/pic32mx/4.5.2/../../../../pic32mx/lib\libpic32.a(default-bootstrap-exception-handler.o)
 .debug_ranges  0x00000020       0x10 c:/program files/microchip/xc32/v1.33/bin/bin/../../lib/gcc/pic32mx/4.5.2/../../../../pic32mx/lib\libpic32.a(default-on-reset.o)
 .debug_ranges  0x00000030       0x10 c:/program files/microchip/xc32/v1.33/bin/bin/../../lib/gcc/pic32mx/4.5.2/../../../../pic32mx/lib\libpic32.a(default-on-bootstrap.o)
 .debug_ranges  0x00000040       0x10 c:/program files/microchip/xc32/v1.33/bin/bin/../../lib/gcc/pic32mx/4.5.2/../../../../pic32mx/lib\libpic32.a(defaultinterrupt.o)
 .debug_ranges  0x00000050       0x10 c:/program files/microchip/xc32/v1.33/bin/bin/../../lib/gcc/pic32mx/4.5.2/../../../../pic32mx/lib\libc.a(fflush.o)
 .debug_ranges  0x00000060       0x20 c:/program files/microchip/xc32/v1.33/bin/bin/../../lib/gcc/pic32mx/4.5.2/../../../../pic32mx/lib\libc.a(malloc.o)
 .debug_ranges  0x00000080       0x18 c:/program files/microchip/xc32/v1.33/bin/bin/../../lib/gcc/pic32mx/4.5.2/../../../../pic32mx/lib\libc.a(puts.o)
 .debug_ranges  0x00000098       0x18 c:/program files/microchip/xc32/v1.33/bin/bin/../../lib/gcc/pic32mx/4.5.2/../../../../pic32mx/lib\libc.a(setbuf.o)
 .debug_ranges  0x000000b0       0x10 c:/program files/microchip/xc32/v1.33/bin/bin/../../lib/gcc/pic32mx/4.5.2/../../../../pic32mx/lib\libc.a(strncmp.o)
 .debug_ranges  0x000000c0       0x10 c:/program files/microchip/xc32/v1.33/bin/bin/../../lib/gcc/pic32mx/4.5.2/../../../../pic32mx/lib\libc.a(printf_cdfFnopsuxX.eo)
 .debug_ranges  0x000000d0       0x10 c:/program files/microchip/xc32/v1.33/bin/bin/../../lib/gcc/pic32mx/4.5.2/../../../../pic32mx/lib\libc.a(sprintf_cdfFnopuxX.eo)
 .debug_ranges  0x000000e0       0x10 c:/program files/microchip/xc32/v1.33/bin/bin/../../lib/gcc/pic32mx/4.5.2/../../../../pic32mx/lib\libc.a(sscanf_s.eo)
 .debug_ranges  0x000000f0       0x10 c:/program files/microchip/xc32/v1.33/bin/bin/../../lib/gcc/pic32mx/4.5.2/../../../../pic32mx/lib\libc.a(_fputc_simple.o)
 .debug_ranges  0x00000100       0x18 c:/program files/microchip/xc32/v1.33/bin/bin/../../lib/gcc/pic32mx/4.5.2/../../../../pic32mx/lib\libc.a(buf.o)
 .debug_ranges  0x00000118       0x18 c:/program files/microchip/xc32/v1.33/bin/bin/../../lib/gcc/pic32mx/4.5.2/../../../../pic32mx/lib\libc.a(doprnt_cdfFnopsuxX.eo)
 .debug_ranges  0x00000130       0x20 c:/program files/microchip/xc32/v1.33/bin/bin/../../lib/gcc/pic32mx/4.5.2/../../../../pic32mx/lib\libc.a(doscan_s.eo)
 .debug_ranges  0x00000150       0x10 c:/program files/microchip/xc32/v1.33/bin/bin/../../lib/gcc/pic32mx/4.5.2/../../../../pic32mx/lib\libc.a(_flsbuf_simple.o)
 .debug_ranges  0x00000160       0x10 c:/program files/microchip/xc32/v1.33/bin/bin/../../lib/gcc/pic32mx/4.5.2/../../../../pic32mx/lib\libc.a(fgetc.o)
 .debug_ranges  0x00000170       0x10 c:/program files/microchip/xc32/v1.33/bin/bin/../../lib/gcc/pic32mx/4.5.2/../../../../pic32mx/lib\libc.a(atoi.o)
 .debug_ranges  0x00000180       0x90 c:/program files/microchip/xc32/v1.33/bin/bin/../../lib/gcc/pic32mx/4.5.2/../../../../pic32mx/lib\libc.a(ctypef.o)
 .debug_ranges  0x00000210       0x10 c:/program files/microchip/xc32/v1.33/bin/bin/../../lib/gcc/pic32mx/4.5.2/../../../../pic32mx/lib\libc.a(ungetc.o)
 .debug_ranges  0x00000220       0x10 c:/program files/microchip/xc32/v1.33/bin/bin/../../lib/gcc/pic32mx/4.5.2/../../../../pic32mx/lib\libc.a(filbuf.o)
 .debug_ranges  0x00000230       0x30 c:/program files/microchip/xc32/v1.33/bin/bin/../../lib/gcc/pic32mx/4.5.2/../../../../pic32mx/lib\libpic32.a(sbrk.o)
 .debug_ranges  0x00000260       0x10 c:/program files/microchip/xc32/v1.33/bin/bin/../../lib/gcc/pic32mx/4.5.2/../../../../pic32mx/lib\libpic32.a(read.o)
 .debug_ranges  0x00000270       0x10 c:/program files/microchip/xc32/v1.33/bin/bin/../../lib/gcc/pic32mx/4.5.2/../../../../pic32mx/lib\libpic32.a(write.o)
 .debug_ranges  0x00000280       0x10 c:/program files/microchip/xc32/v1.33/bin/bin/../../lib/gcc/pic32mx/4.5.2/../../../../pic32mx/lib\libe.a(_floatdisf.o)

.gnu.attributes
                0x00000000       0x10
 *(.gnu.attributes)
 .gnu.attributes
                0x00000000       0x10 c:/program files/microchip/xc32/v1.33/bin/bin/../../lib/gcc/pic32mx/4.5.2/../../../../pic32mx/lib\software-debug-break.o
 .gnu.attributes
                0x00000010       0x10 build/ChaletDuinoV2_775F512H_/debug/Source/ChaletduinoV2Board.o
 .gnu.attributes
                0x00000020       0x10 build/ChaletDuinoV2_775F512H_/debug/Source/winc3400/bsp/source/nm_bsp.o
 .gnu.attributes
                0x00000030       0x10 build/ChaletDuinoV2_775F512H_/debug/Source/winc3400/bus_wrapper/source/nm_bus_wrapper.o
 .gnu.attributes
                0x00000040       0x10 build/ChaletDuinoV2_775F512H_/debug/Source/winc3400/common/source/nm_common.o
 .gnu.attributes
                0x00000050       0x10 build/ChaletDuinoV2_775F512H_/debug/Source/winc3400/driver/source/m2m_ate_mode.o
 .gnu.attributes
                0x00000060       0x10 build/ChaletDuinoV2_775F512H_/debug/Source/winc3400/driver/source/m2m_crypto.o
 .gnu.attributes
                0x00000070       0x10 build/ChaletDuinoV2_775F512H_/debug/Source/winc3400/driver/source/m2m_hif.o
 .gnu.attributes
                0x00000080       0x10 build/ChaletDuinoV2_775F512H_/debug/Source/winc3400/driver/source/m2m_ota.o
 .gnu.attributes
                0x00000090       0x10 build/ChaletDuinoV2_775F512H_/debug/Source/winc3400/driver/source/m2m_periph.o
 .gnu.attributes
                0x000000a0       0x10 build/ChaletDuinoV2_775F512H_/debug/Source/winc3400/driver/source/m2m_ssl.o
 .gnu.attributes
                0x000000b0       0x10 build/ChaletDuinoV2_775F512H_/debug/Source/winc3400/driver/source/m2m_wifi.o
 .gnu.attributes
                0x000000c0       0x10 build/ChaletDuinoV2_775F512H_/debug/Source/winc3400/driver/source/nmasic.o
 .gnu.attributes
                0x000000d0       0x10 build/ChaletDuinoV2_775F512H_/debug/Source/winc3400/driver/source/nmbus.o
 .gnu.attributes
                0x000000e0       0x10 build/ChaletDuinoV2_775F512H_/debug/Source/winc3400/driver/source/nmdrv.o
 .gnu.attributes
                0x000000f0       0x10 build/ChaletDuinoV2_775F512H_/debug/Source/winc3400/driver/source/nmi2c.o
 .gnu.attributes
                0x00000100       0x10 build/ChaletDuinoV2_775F512H_/debug/Source/winc3400/driver/source/nmspi.o
 .gnu.attributes
                0x00000110       0x10 build/ChaletDuinoV2_775F512H_/debug/Source/winc3400/driver/source/nmuart.o
 .gnu.attributes
                0x00000120       0x10 build/ChaletDuinoV2_775F512H_/debug/Source/winc3400/socket/source/socket.o
 .gnu.attributes
                0x00000130       0x10 build/ChaletDuinoV2_775F512H_/debug/Source/winc3400/spi_flash/source/spi_flash.o
 .gnu.attributes
                0x00000140       0x10 build/ChaletDuinoV2_775F512H_/debug/Source/winc3400/winc_init.o
 .gnu.attributes
                0x00000150       0x10 build/ChaletDuinoV2_775F512H_/debug/Source/DigitalIO.o
 .gnu.attributes
                0x00000160       0x10 build/ChaletDuinoV2_775F512H_/debug/Source/InternalUart.o
 .gnu.attributes
                0x00000170       0x10 build/ChaletDuinoV2_775F512H_/debug/Source/NetworkProtocol.o
 .gnu.attributes
                0x00000180       0x10 build/ChaletDuinoV2_775F512H_/debug/Source/Terminal.o
 .gnu.attributes
                0x00000190       0x10 build/ChaletDuinoV2_775F512H_/debug/Source/Uart.o
 .gnu.attributes
                0x000001a0       0x10 build/ChaletDuinoV2_775F512H_/debug/Source/Util.o
 .gnu.attributes
                0x000001b0       0x10 build/ChaletDuinoV2_775F512H_/debug/Source/exceptions.o
 .gnu.attributes
                0x000001c0       0x10 build/ChaletDuinoV2_775F512H_/debug/Source/interrupts.o
 .gnu.attributes
                0x000001d0       0x10 build/ChaletDuinoV2_775F512H_/debug/Source/main.o
 .gnu.attributes
                0x000001e0       0x10 build/ChaletDuinoV2_775F512H_/debug/Source/system.o
 .gnu.attributes
                0x000001f0       0x10 build/ChaletDuinoV2_775F512H_/debug/Source/template.o
 .gnu.attributes
                0x00000200       0x10 build/ChaletDuinoV2_775F512H_/debug/Source/timer.o
 .gnu.attributes
                0x00000210       0x10 build/ChaletDuinoV2_775F512H_/debug/Source/WiFiCtrl.o
 .gnu.attributes
                0x00000220       0x10 build/ChaletDuinoV2_775F512H_/debug/Source/SPI.o
 .gnu.attributes
                0x00000230       0x10 build/ChaletDuinoV2_775F512H_/debug/Source/LoraNetworkInterface.o
 .gnu.attributes
                0x00000240       0x10 build/ChaletDuinoV2_775F512H_/debug/Source/ChaletPowerRelay.o
 .gnu.attributes
                0x00000250       0x10 build/ChaletDuinoV2_775F512H_/debug/Source/HarakiriRelay.o
 .gnu.attributes
                0x00000260       0x10 build/ChaletDuinoV2_775F512H_/debug/Source/BatteryMonitor.o
 .gnu.attributes
                0x00000270       0x10 build/ChaletDuinoV2_775F512H_/debug/Source/ina219.o
 .gnu.attributes
                0x00000280       0x10 build/ChaletDuinoV2_775F512H_/debug/Source/I2C.o
 .gnu.attributes
                0x00000290       0x10 build/ChaletDuinoV2_775F512H_/debug/Source/SPI_Flash.o
 .gnu.attributes
                0x000002a0       0x10 build/ChaletDuinoV2_775F512H_/debug/Source/Syslog.o
 .gnu.attributes
                0x000002b0       0x10 build/ChaletDuinoV2_775F512H_/debug/Source/Watchdog.o
 .gnu.attributes
                0x000002c0       0x10 build/ChaletDuinoV2_775F512H_/debug/Source/BootloaderInterface.o
 .gnu.attributes
                0x000002d0       0x10 build/ChaletDuinoV2_775F512H_/debug/Source/TemperatureSensor.o
 .gnu.attributes
                0x000002e0       0x10 build/ChaletDuinoV2_775F512H_/debug/Source/TC77.o
 .gnu.attributes
                0x000002f0       0x10 build/ChaletDuinoV2_775F512H_/debug/Source/BootloaderProtocol.o
 .gnu.attributes
                0x00000300       0x10 build/ChaletDuinoV2_775F512H_/debug/Source/crc32.o
 .gnu.attributes
                0x00000310       0x10 c:/program files/microchip/xc32/v1.33/bin/bin/../../lib/gcc/pic32mx/4.5.2/../../../../pic32mx/lib\libmchp_peripheral_32MX795F512H.a(soft_reset_lib.o)
 .gnu.attributes
                0x00000320       0x10 c:/program files/microchip/xc32/v1.33/bin/bin/../../lib/gcc/pic32mx/4.5.2/../../../../pic32mx/lib\libmchp_peripheral_32MX795F512H.a(pcache.o)
 .gnu.attributes
                0x00000330       0x10 c:/program files/microchip/xc32/v1.33/bin/bin/../../lib/gcc/pic32mx/4.5.2/../../../../pic32mx/lib\libmchp_peripheral_32MX795F512H.a(int_configure_system_lib.o)
 .gnu.attributes
                0x00000340       0x10 c:/program files/microchip/xc32/v1.33/bin/bin/../../lib/gcc/pic32mx/4.5.2/../../../../pic32mx/lib\libmchp_peripheral_32MX795F512H.a(int_enable_interrupts_lib.o)
 .gnu.attributes
                0x00000350       0x10 c:/program files/microchip/xc32/v1.33/bin/bin/../../lib/gcc/pic32mx/4.5.2/../../../../pic32mx/lib\libmchp_peripheral_32MX795F512H.a(int_disable_interrupts_lib.o)
 .gnu.attributes
                0x00000360       0x10 c:/program files/microchip/xc32/v1.33/bin/bin/../../lib/gcc/pic32mx/4.5.2/../../../../pic32mx/lib\libmchp_peripheral_32MX795F512H.a(int_restore_interrupts_lib.o)
 .gnu.attributes
                0x00000370       0x10 c:/program files/microchip/xc32/v1.33/bin/bin/../../lib/gcc/pic32mx/4.5.2/../../../../pic32mx/lib\libpic32.a(default-bootstrap-exception-handler.o)
 .gnu.attributes
                0x00000380       0x10 c:/program files/microchip/xc32/v1.33/bin/bin/../../lib/gcc/pic32mx/4.5.2/../../../../pic32mx/lib\libpic32.a(default-on-reset.o)
 .gnu.attributes
                0x00000390       0x10 c:/program files/microchip/xc32/v1.33/bin/bin/../../lib/gcc/pic32mx/4.5.2/../../../../pic32mx/lib\libpic32.a(default-on-bootstrap.o)
 .gnu.attributes
                0x000003a0       0x10 c:/program files/microchip/xc32/v1.33/bin/bin/../../lib/gcc/pic32mx/4.5.2/../../../../pic32mx/lib\libpic32.a(defaultinterrupt.o)
 .gnu.attributes
                0x000003b0       0x10 c:/program files/microchip/xc32/v1.33/bin/bin/../../lib/gcc/pic32mx/4.5.2/../../../../pic32mx/lib\libc.a(_iob.o)
 .gnu.attributes
                0x000003c0       0x10 c:/program files/microchip/xc32/v1.33/bin/bin/../../lib/gcc/pic32mx/4.5.2/../../../../pic32mx/lib\libc.a(fflush.o)
 .gnu.attributes
                0x000003d0       0x10 c:/program files/microchip/xc32/v1.33/bin/bin/../../lib/gcc/pic32mx/4.5.2/../../../../pic32mx/lib\libc.a(malloc.o)
 .gnu.attributes
                0x000003e0       0x10 c:/program files/microchip/xc32/v1.33/bin/bin/../../lib/gcc/pic32mx/4.5.2/../../../../pic32mx/lib\libc.a(puts.o)
 .gnu.attributes
                0x000003f0       0x10 c:/program files/microchip/xc32/v1.33/bin/bin/../../lib/gcc/pic32mx/4.5.2/../../../../pic32mx/lib\libc.a(setbuf.o)
 .gnu.attributes
                0x00000400       0x10 c:/program files/microchip/xc32/v1.33/bin/bin/../../lib/gcc/pic32mx/4.5.2/../../../../pic32mx/lib\libc.a(strncmp.o)
 .gnu.attributes
                0x00000410       0x10 c:/program files/microchip/xc32/v1.33/bin/bin/../../lib/gcc/pic32mx/4.5.2/../../../../pic32mx/lib\libc.a(printf_cdfFnopsuxX.eo)
 .gnu.attributes
                0x00000420       0x10 c:/program files/microchip/xc32/v1.33/bin/bin/../../lib/gcc/pic32mx/4.5.2/../../../../pic32mx/lib\libc.a(sprintf_cdfFnopuxX.eo)
 .gnu.attributes
                0x00000430       0x10 c:/program files/microchip/xc32/v1.33/bin/bin/../../lib/gcc/pic32mx/4.5.2/../../../../pic32mx/lib\libc.a(sscanf_s.eo)
 .gnu.attributes
                0x00000440       0x10 c:/program files/microchip/xc32/v1.33/bin/bin/../../lib/gcc/pic32mx/4.5.2/../../../../pic32mx/lib\libc.a(_fputc_simple.o)
 .gnu.attributes
                0x00000450       0x10 c:/program files/microchip/xc32/v1.33/bin/bin/../../lib/gcc/pic32mx/4.5.2/../../../../pic32mx/lib\libc.a(buf.o)
 .gnu.attributes
                0x00000460       0x10 c:/program files/microchip/xc32/v1.33/bin/bin/../../lib/gcc/pic32mx/4.5.2/../../../../pic32mx/lib\libc.a(errno.o)
 .gnu.attributes
                0x00000470       0x10 c:/program files/microchip/xc32/v1.33/bin/bin/../../lib/gcc/pic32mx/4.5.2/../../../../pic32mx/lib\libc.a(doprnt_cdfFnopsuxX.eo)
 .gnu.attributes
                0x00000480       0x10 c:/program files/microchip/xc32/v1.33/bin/bin/../../lib/gcc/pic32mx/4.5.2/../../../../pic32mx/lib\libc.a(doscan_s.eo)
 .gnu.attributes
                0x00000490       0x10 c:/program files/microchip/xc32/v1.33/bin/bin/../../lib/gcc/pic32mx/4.5.2/../../../../pic32mx/lib\libc.a(_flsbuf_simple.o)
 .gnu.attributes
                0x000004a0       0x10 c:/program files/microchip/xc32/v1.33/bin/bin/../../lib/gcc/pic32mx/4.5.2/../../../../pic32mx/lib\libc.a(fgetc.o)
 .gnu.attributes
                0x000004b0       0x10 c:/program files/microchip/xc32/v1.33/bin/bin/../../lib/gcc/pic32mx/4.5.2/../../../../pic32mx/lib\libc.a(atoi.o)
 .gnu.attributes
                0x000004c0       0x10 c:/program files/microchip/xc32/v1.33/bin/bin/../../lib/gcc/pic32mx/4.5.2/../../../../pic32mx/lib\libc.a(ctype.o)
 .gnu.attributes
                0x000004d0       0x10 c:/program files/microchip/xc32/v1.33/bin/bin/../../lib/gcc/pic32mx/4.5.2/../../../../pic32mx/lib\libc.a(ctypef.o)
 .gnu.attributes
                0x000004e0       0x10 c:/program files/microchip/xc32/v1.33/bin/bin/../../lib/gcc/pic32mx/4.5.2/../../../../pic32mx/lib\libc.a(powersf.o)
 .gnu.attributes
                0x000004f0       0x10 c:/program files/microchip/xc32/v1.33/bin/bin/../../lib/gcc/pic32mx/4.5.2/../../../../pic32mx/lib\libc.a(ungetc.o)
 .gnu.attributes
                0x00000500       0x10 c:/program files/microchip/xc32/v1.33/bin/bin/../../lib/gcc/pic32mx/4.5.2/../../../../pic32mx/lib\libc.a(filbuf.o)
 .gnu.attributes
                0x00000510       0x10 c:/program files/microchip/xc32/v1.33/bin/bin/../../lib/gcc/pic32mx/4.5.2/../../../../pic32mx/lib\libpic32.a(sbrk.o)
 .gnu.attributes
                0x00000520       0x10 c:/program files/microchip/xc32/v1.33/bin/bin/../../lib/gcc/pic32mx/4.5.2/../../../../pic32mx/lib\libpic32.a(read.o)
 .gnu.attributes
                0x00000530       0x10 c:/program files/microchip/xc32/v1.33/bin/bin/../../lib/gcc/pic32mx/4.5.2/../../../../pic32mx/lib\libpic32.a(write.o)
 .gnu.attributes
                0x00000540       0x10 c:/program files/microchip/xc32/v1.33/bin/bin/../../lib/gcc/pic32mx/4.5.2/../../../../pic32mx/lib\libpic32.a(xc32_uart.o)
 .gnu.attributes
                0x00000550       0x10 c:/program files/microchip/xc32/v1.33/bin/bin/../../lib/gcc/pic32mx/4.5.2/../../../../pic32mx/lib\libe.a(_floatdisf.o)
 .gnu.attributes
                0x00000560       0x10 c:/program files/microchip/xc32/v1.33/bin/bin/../../lib/gcc/pic32mx/4.5.2\libgcc.a(_floatundisf.o)
 .gnu.attributes
                0x00000570       0x10 c:/program files/microchip/xc32/v1.33/bin/bin/../../lib/gcc/pic32mx/4.5.2\libgcc.a(_udivdi3.o)
 .gnu.attributes
                0x00000580       0x10 c:/program files/microchip/xc32/v1.33/bin/bin/../../lib/gcc/pic32mx/4.5.2\libgcc.a(_umoddi3.o)
 .gnu.attributes
                0x00000590       0x10 c:/program files/microchip/xc32/v1.33/bin/bin/../../lib/gcc/pic32mx/4.5.2\libgcc.a(floatunsisf.o)
LOAD c:/program files/microchip/xc32/v1.33/bin/bin/../../lib/gcc/pic32mx/4.5.2\libgcc.a
START GROUP
LOAD c:/program files/microchip/xc32/v1.33/bin/bin/../../lib/gcc/pic32mx/4.5.2/../../../../pic32mx/lib\libpic32.a
LOAD c:/program files/microchip/xc32/v1.33/bin/bin/../../lib/gcc/pic32mx/4.5.2/../../../../pic32mx/lib\libdebug.a
LOAD c:/program files/microchip/xc32/v1.33/bin/bin/../../lib/gcc/pic32mx/4.5.2/../../../../pic32mx/lib\libpic32.a
LOAD c:/program files/microchip/xc32/v1.33/bin/bin/../../lib/gcc/pic32mx/4.5.2/../../../../pic32mx/lib\libm.a
LOAD c:/program files/microchip/xc32/v1.33/bin/bin/../../lib/gcc/pic32mx/4.5.2/../../../../pic32mx/lib\libe.a
LOAD c:/program files/microchip/xc32/v1.33/bin/bin/../../lib/gcc/pic32mx/4.5.2/../../../../pic32mx/lib\libdsp.a
LOAD c:/program files/microchip/xc32/v1.33/bin/bin/../../lib/gcc/pic32mx/4.5.2\libgcc.a
LOAD c:/program files/microchip/xc32/v1.33/bin/bin/../../lib/gcc/pic32mx/4.5.2/../../../../pic32mx/lib\libc.a
LOAD c:/program files/microchip/xc32/v1.33/bin/bin/../../lib/gcc/pic32mx/4.5.2/../../../../pic32mx/lib\libpic32.a
END GROUP
LOAD c:/program files/microchip/xc32/v1.33/bin/bin/../../lib/gcc/pic32mx/4.5.2\libgcc.a
OUTPUT(dist/ChaletDuinoV2_775F512H_/debug/ChaletLora.X.debug.elf elf32-tradlittlemips)
LOAD stack
LOAD data_init

.reginfo        0x00000000       0x18
 .reginfo       0x00000000       0x18 c:/program files/microchip/xc32/v1.33/bin/bin/../../lib/gcc/pic32mx/4.5.2/../../../../pic32mx/lib/./proc/32MX795F512H/crt0_mips32r2.o

.stack          0xa0004478      0x400
 .stack         0xa0004478      0x400 stack

.data           0xa0003268      0x4bc
 .data          0xa0003268      0x4bc build/ChaletDuinoV2_775F512H_/debug/Source/Terminal.o

.bss            0xa0003724      0x800
 .bss           0xa0003724      0x400 build/ChaletDuinoV2_775F512H_/debug/Source/WiFiCtrl.o
 .bss           0xa0003b24      0x400 build/ChaletDuinoV2_775F512H_/debug/Source/crc32.o

.data           0xa0003f24      0x2c4
 .data          0xa0003f24       0xa0 c:/program files/microchip/xc32/v1.33/bin/bin/../../lib/gcc/pic32mx/4.5.2/../../../../pic32mx/lib\libc.a(_iob.o)
                0xa0003f24                _iob
 .data          0xa0003fc4       0x6c build/ChaletDuinoV2_775F512H_/debug/Source/WiFiCtrl.o
 .data          0xa0004030       0x58 build/ChaletDuinoV2_775F512H_/debug/Source/main.o
 .data          0xa0004088       0x58 build/ChaletDuinoV2_775F512H_/debug/Source/BatteryMonitor.o
 .data          0xa00040e0       0x58 build/ChaletDuinoV2_775F512H_/debug/Source/Syslog.o
 .data          0xa0004138       0x58 build/ChaletDuinoV2_775F512H_/debug/Source/BootloaderInterface.o
 .data          0xa0004190       0x58 build/ChaletDuinoV2_775F512H_/debug/Source/BootloaderProtocol.o

.bss            0xa00041e8       0x74
 .bss           0xa00041e8       0x40 c:/program files/microchip/xc32/v1.33/bin/bin/../../lib/gcc/pic32mx/4.5.2/../../../../pic32mx/lib\libc.a(_iob.o)
                0xa00041e8                _sibuf
                0xa0004208                _sobuf
 .bss           0xa0004228       0x1c c:/program files/microchip/xc32/v1.33/bin/bin/../../lib/gcc/pic32mx/4.5.2/../../../../pic32mx/lib\libpic32.a(sbrk.o)
 .bss           0xa0004244       0x10 c:/program files/microchip/xc32/v1.33/bin/bin/../../lib/gcc/pic32mx/4.5.2/../../../../pic32mx/lib\libc.a(malloc.o)
                0xa0004244                __allocs
 .bss           0xa0004254        0x4 c:/program files/microchip/xc32/v1.33/bin/bin/../../lib/gcc/pic32mx/4.5.2/../../../../pic32mx/lib\libc.a(buf.o)
 .bss           0xa0004258        0x4 c:/program files/microchip/xc32/v1.33/bin/bin/../../lib/gcc/pic32mx/4.5.2/../../../../pic32mx/lib\libc.a(doscan_s.eo)

.bss%z1         0x00000000        0x0
 .bss           0x00000000        0x0 c:/program files/microchip/xc32/v1.33/bin/bin/../../lib/gcc/pic32mx/4.5.2\libgcc.a(floatunsisf.o)

.data%z2        0x00000000        0x0
 .data          0x00000000        0x0 c:/program files/microchip/xc32/v1.33/bin/bin/../../lib/gcc/pic32mx/4.5.2\libgcc.a(floatunsisf.o)

.bss%z3         0x00000000        0x0
 .bss           0x00000000        0x0 c:/program files/microchip/xc32/v1.33/bin/bin/../../lib/gcc/pic32mx/4.5.2\libgcc.a(_umoddi3.o)

.data%z4        0x00000000        0x0
 .data          0x00000000        0x0 c:/program files/microchip/xc32/v1.33/bin/bin/../../lib/gcc/pic32mx/4.5.2\libgcc.a(_umoddi3.o)

.bss%z5         0x00000000        0x0
 .bss           0x00000000        0x0 c:/program files/microchip/xc32/v1.33/bin/bin/../../lib/gcc/pic32mx/4.5.2\libgcc.a(_udivdi3.o)

.data%z6        0x00000000        0x0
 .data          0x00000000        0x0 c:/program files/microchip/xc32/v1.33/bin/bin/../../lib/gcc/pic32mx/4.5.2\libgcc.a(_udivdi3.o)

.bss%z7         0x00000000        0x0
 .bss           0x00000000        0x0 c:/program files/microchip/xc32/v1.33/bin/bin/../../lib/gcc/pic32mx/4.5.2\libgcc.a(_floatundisf.o)

.data%z8        0x00000000        0x0
 .data          0x00000000        0x0 c:/program files/microchip/xc32/v1.33/bin/bin/../../lib/gcc/pic32mx/4.5.2\libgcc.a(_floatundisf.o)

.bss%z9         0x00000000        0x0
 .bss           0x00000000        0x0 c:/program files/microchip/xc32/v1.33/bin/bin/../../lib/gcc/pic32mx/4.5.2/../../../../pic32mx/lib\libe.a(_floatdisf.o)

.data%z10       0x00000000        0x0
 .data          0x00000000        0x0 c:/program files/microchip/xc32/v1.33/bin/bin/../../lib/gcc/pic32mx/4.5.2/../../../../pic32mx/lib\libe.a(_floatdisf.o)

.bss%z11        0x00000000        0x0
 .bss           0x00000000        0x0 c:/program files/microchip/xc32/v1.33/bin/bin/../../lib/gcc/pic32mx/4.5.2/../../../../pic32mx/lib\libm.a(fptoul.o)

.data%z12       0x00000000        0x0
 .data          0x00000000        0x0 c:/program files/microchip/xc32/v1.33/bin/bin/../../lib/gcc/pic32mx/4.5.2/../../../../pic32mx/lib\libm.a(fptoul.o)

.bss%z13        0x00000000        0x0
 .bss           0x00000000        0x0 c:/program files/microchip/xc32/v1.33/bin/bin/../../lib/gcc/pic32mx/4.5.2/../../../../pic32mx/lib\libm.a(fpfrexp.o)

.data%z14       0x00000000        0x0
 .data          0x00000000        0x0 c:/program files/microchip/xc32/v1.33/bin/bin/../../lib/gcc/pic32mx/4.5.2/../../../../pic32mx/lib\libm.a(fpfrexp.o)

.bss%z15        0x00000000        0x0
 .bss           0x00000000        0x0 c:/program files/microchip/xc32/v1.33/bin/bin/../../lib/gcc/pic32mx/4.5.2/../../../../pic32mx/lib\libm.a(fpcmp.o)

.data%z16       0x00000000        0x0
 .data          0x00000000        0x0 c:/program files/microchip/xc32/v1.33/bin/bin/../../lib/gcc/pic32mx/4.5.2/../../../../pic32mx/lib\libm.a(fpcmp.o)

.bss%z17        0x00000000        0x0
 .bss           0x00000000        0x0 c:/program files/microchip/xc32/v1.33/bin/bin/../../lib/gcc/pic32mx/4.5.2/../../../../pic32mx/lib\libpic32.a(xc32_uart.o)

.data%z18       0x00000000        0x0
 .data          0x00000000        0x0 c:/program files/microchip/xc32/v1.33/bin/bin/../../lib/gcc/pic32mx/4.5.2/../../../../pic32mx/lib\libpic32.a(xc32_uart.o)

.bss%z19        0x00000000        0x0
 .bss           0x00000000        0x0 c:/program files/microchip/xc32/v1.33/bin/bin/../../lib/gcc/pic32mx/4.5.2/../../../../pic32mx/lib\libpic32.a(write.o)

.data%z20       0x00000000        0x0
 .data          0x00000000        0x0 c:/program files/microchip/xc32/v1.33/bin/bin/../../lib/gcc/pic32mx/4.5.2/../../../../pic32mx/lib\libpic32.a(write.o)

.bss%z21        0x00000000        0x0
 .bss           0x00000000        0x0 c:/program files/microchip/xc32/v1.33/bin/bin/../../lib/gcc/pic32mx/4.5.2/../../../../pic32mx/lib\libpic32.a(read.o)

.data%z22       0x00000000        0x0
 .data          0x00000000        0x0 c:/program files/microchip/xc32/v1.33/bin/bin/../../lib/gcc/pic32mx/4.5.2/../../../../pic32mx/lib\libpic32.a(read.o)

.data%z23       0x00000000        0x0
 .data          0x00000000        0x0 c:/program files/microchip/xc32/v1.33/bin/bin/../../lib/gcc/pic32mx/4.5.2/../../../../pic32mx/lib\libpic32.a(sbrk.o)

.bss%z24        0x00000000        0x0
 .bss           0x00000000        0x0 c:/program files/microchip/xc32/v1.33/bin/bin/../../lib/gcc/pic32mx/4.5.2/../../../../pic32mx/lib\libc.a(filbuf.o)

.data%z25       0x00000000        0x0
 .data          0x00000000        0x0 c:/program files/microchip/xc32/v1.33/bin/bin/../../lib/gcc/pic32mx/4.5.2/../../../../pic32mx/lib\libc.a(filbuf.o)

.bss%z26        0x00000000        0x0
 .bss           0x00000000        0x0 c:/program files/microchip/xc32/v1.33/bin/bin/../../lib/gcc/pic32mx/4.5.2/../../../../pic32mx/lib\libc.a(ungetc.o)

.data%z27       0x00000000        0x0
 .data          0x00000000        0x0 c:/program files/microchip/xc32/v1.33/bin/bin/../../lib/gcc/pic32mx/4.5.2/../../../../pic32mx/lib\libc.a(ungetc.o)

.bss%z28        0x00000000        0x0
 .bss           0x00000000        0x0 c:/program files/microchip/xc32/v1.33/bin/bin/../../lib/gcc/pic32mx/4.5.2/../../../../pic32mx/lib\libc.a(powersf.o)

.data%z29       0x00000000        0x0
 .data          0x00000000        0x0 c:/program files/microchip/xc32/v1.33/bin/bin/../../lib/gcc/pic32mx/4.5.2/../../../../pic32mx/lib\libc.a(powersf.o)

.bss%z30        0x00000000        0x0
 .bss           0x00000000        0x0 c:/program files/microchip/xc32/v1.33/bin/bin/../../lib/gcc/pic32mx/4.5.2/../../../../pic32mx/lib\libc.a(ctypef.o)

.data%z31       0x00000000        0x0
 .data          0x00000000        0x0 c:/program files/microchip/xc32/v1.33/bin/bin/../../lib/gcc/pic32mx/4.5.2/../../../../pic32mx/lib\libc.a(ctypef.o)

.bss%z32        0x00000000        0x0
 .bss           0x00000000        0x0 c:/program files/microchip/xc32/v1.33/bin/bin/../../lib/gcc/pic32mx/4.5.2/../../../../pic32mx/lib\libc.a(ctype.o)

.data%z33       0x00000000        0x0
 .data          0x00000000        0x0 c:/program files/microchip/xc32/v1.33/bin/bin/../../lib/gcc/pic32mx/4.5.2/../../../../pic32mx/lib\libc.a(ctype.o)

.bss%z34        0x00000000        0x0
 .bss           0x00000000        0x0 c:/program files/microchip/xc32/v1.33/bin/bin/../../lib/gcc/pic32mx/4.5.2/../../../../pic32mx/lib\libc.a(atoi.o)

.data%z35       0x00000000        0x0
 .data          0x00000000        0x0 c:/program files/microchip/xc32/v1.33/bin/bin/../../lib/gcc/pic32mx/4.5.2/../../../../pic32mx/lib\libc.a(atoi.o)

.bss%z36        0x00000000        0x0
 .bss           0x00000000        0x0 c:/program files/microchip/xc32/v1.33/bin/bin/../../lib/gcc/pic32mx/4.5.2/../../../../pic32mx/lib\libc.a(fgetc.o)

.data%z37       0x00000000        0x0
 .data          0x00000000        0x0 c:/program files/microchip/xc32/v1.33/bin/bin/../../lib/gcc/pic32mx/4.5.2/../../../../pic32mx/lib\libc.a(fgetc.o)

.bss%z38        0x00000000        0x0
 .bss           0x00000000        0x0 c:/program files/microchip/xc32/v1.33/bin/bin/../../lib/gcc/pic32mx/4.5.2/../../../../pic32mx/lib\libc.a(_flsbuf_simple.o)

.data%z39       0x00000000        0x0
 .data          0x00000000        0x0 c:/program files/microchip/xc32/v1.33/bin/bin/../../lib/gcc/pic32mx/4.5.2/../../../../pic32mx/lib\libc.a(_flsbuf_simple.o)

.data%z40       0x00000000        0x0
 .data          0x00000000        0x0 c:/program files/microchip/xc32/v1.33/bin/bin/../../lib/gcc/pic32mx/4.5.2/../../../../pic32mx/lib\libc.a(doscan_s.eo)

.bss%z41        0x00000000        0x0
 .bss           0x00000000        0x0 c:/program files/microchip/xc32/v1.33/bin/bin/../../lib/gcc/pic32mx/4.5.2/../../../../pic32mx/lib\libc.a(doprnt_cdfFnopsuxX.eo)

.data%z42       0x00000000        0x0
 .data          0x00000000        0x0 c:/program files/microchip/xc32/v1.33/bin/bin/../../lib/gcc/pic32mx/4.5.2/../../../../pic32mx/lib\libc.a(doprnt_cdfFnopsuxX.eo)

.bss%z43        0x00000000        0x0
 .bss           0x00000000        0x0 c:/program files/microchip/xc32/v1.33/bin/bin/../../lib/gcc/pic32mx/4.5.2/../../../../pic32mx/lib\libc.a(errno.o)

.data%z44       0x00000000        0x0
 .data          0x00000000        0x0 c:/program files/microchip/xc32/v1.33/bin/bin/../../lib/gcc/pic32mx/4.5.2/../../../../pic32mx/lib\libc.a(errno.o)

.data%z45       0x00000000        0x0
 .data          0x00000000        0x0 c:/program files/microchip/xc32/v1.33/bin/bin/../../lib/gcc/pic32mx/4.5.2/../../../../pic32mx/lib\libc.a(buf.o)

.bss%z46        0x00000000        0x0
 .bss           0x00000000        0x0 c:/program files/microchip/xc32/v1.33/bin/bin/../../lib/gcc/pic32mx/4.5.2/../../../../pic32mx/lib\libc.a(_fputc_simple.o)

.data%z47       0x00000000        0x0
 .data          0x00000000        0x0 c:/program files/microchip/xc32/v1.33/bin/bin/../../lib/gcc/pic32mx/4.5.2/../../../../pic32mx/lib\libc.a(_fputc_simple.o)

.bss%z48        0x00000000        0x0
 .bss           0x00000000        0x0 c:/program files/microchip/xc32/v1.33/bin/bin/../../lib/gcc/pic32mx/4.5.2/../../../../pic32mx/lib\libc.a(sscanf_s.eo)

.data%z49       0x00000000        0x0
 .data          0x00000000        0x0 c:/program files/microchip/xc32/v1.33/bin/bin/../../lib/gcc/pic32mx/4.5.2/../../../../pic32mx/lib\libc.a(sscanf_s.eo)

.bss%z50        0x00000000        0x0
 .bss           0x00000000        0x0 c:/program files/microchip/xc32/v1.33/bin/bin/../../lib/gcc/pic32mx/4.5.2/../../../../pic32mx/lib\libc.a(sprintf_cdfFnopuxX.eo)

.data%z51       0x00000000        0x0
 .data          0x00000000        0x0 c:/program files/microchip/xc32/v1.33/bin/bin/../../lib/gcc/pic32mx/4.5.2/../../../../pic32mx/lib\libc.a(sprintf_cdfFnopuxX.eo)

.bss%z52        0x00000000        0x0
 .bss           0x00000000        0x0 c:/program files/microchip/xc32/v1.33/bin/bin/../../lib/gcc/pic32mx/4.5.2/../../../../pic32mx/lib\libc.a(printf_cdfFnopsuxX.eo)

.data%z53       0x00000000        0x0
 .data          0x00000000        0x0 c:/program files/microchip/xc32/v1.33/bin/bin/../../lib/gcc/pic32mx/4.5.2/../../../../pic32mx/lib\libc.a(printf_cdfFnopsuxX.eo)

.bss%z54        0x00000000        0x0
 .bss           0x00000000        0x0 c:/program files/microchip/xc32/v1.33/bin/bin/../../lib/gcc/pic32mx/4.5.2/../../../../pic32mx/lib\libc.a(strncmp.o)

.data%z55       0x00000000        0x0
 .data          0x00000000        0x0 c:/program files/microchip/xc32/v1.33/bin/bin/../../lib/gcc/pic32mx/4.5.2/../../../../pic32mx/lib\libc.a(strncmp.o)

.bss%z56        0x00000000        0x0
 .bss           0x00000000        0x0 c:/program files/microchip/xc32/v1.33/bin/bin/../../lib/gcc/pic32mx/4.5.2/../../../../pic32mx/lib\libc.a(setbuf.o)

.data%z57       0x00000000        0x0
 .data          0x00000000        0x0 c:/program files/microchip/xc32/v1.33/bin/bin/../../lib/gcc/pic32mx/4.5.2/../../../../pic32mx/lib\libc.a(setbuf.o)

.bss%z58        0x00000000        0x0
 .bss           0x00000000        0x0 c:/program files/microchip/xc32/v1.33/bin/bin/../../lib/gcc/pic32mx/4.5.2/../../../../pic32mx/lib\libc.a(puts.o)

.data%z59       0x00000000        0x0
 .data          0x00000000        0x0 c:/program files/microchip/xc32/v1.33/bin/bin/../../lib/gcc/pic32mx/4.5.2/../../../../pic32mx/lib\libc.a(puts.o)

.data%z60       0x00000000        0x0
 .data          0x00000000        0x0 c:/program files/microchip/xc32/v1.33/bin/bin/../../lib/gcc/pic32mx/4.5.2/../../../../pic32mx/lib\libc.a(malloc.o)

.bss%z61        0x00000000        0x0
 .bss           0x00000000        0x0 c:/program files/microchip/xc32/v1.33/bin/bin/../../lib/gcc/pic32mx/4.5.2/../../../../pic32mx/lib\libc.a(fflush.o)

.data%z62       0x00000000        0x0
 .data          0x00000000        0x0 c:/program files/microchip/xc32/v1.33/bin/bin/../../lib/gcc/pic32mx/4.5.2/../../../../pic32mx/lib\libc.a(fflush.o)

.bss%z63        0x00000000        0x0
 .bss           0x00000000        0x0 c:/program files/microchip/xc32/v1.33/bin/bin/../../lib/gcc/pic32mx/4.5.2/../../../../pic32mx/lib\libm.a(sitofp.o)

.data%z64       0x00000000        0x0
 .data          0x00000000        0x0 c:/program files/microchip/xc32/v1.33/bin/bin/../../lib/gcc/pic32mx/4.5.2/../../../../pic32mx/lib\libm.a(sitofp.o)

.bss%z65        0x00000000        0x0
 .bss           0x00000000        0x0 c:/program files/microchip/xc32/v1.33/bin/bin/../../lib/gcc/pic32mx/4.5.2/../../../../pic32mx/lib\libm.a(fp32subadd.o)

.data%z66       0x00000000        0x0
 .data          0x00000000        0x0 c:/program files/microchip/xc32/v1.33/bin/bin/../../lib/gcc/pic32mx/4.5.2/../../../../pic32mx/lib\libm.a(fp32subadd.o)

.bss%z67        0x00000000        0x0
 .bss           0x00000000        0x0 c:/program files/microchip/xc32/v1.33/bin/bin/../../lib/gcc/pic32mx/4.5.2/../../../../pic32mx/lib\libm.a(fp32mul.o)

.data%z68       0x00000000        0x0
 .data          0x00000000        0x0 c:/program files/microchip/xc32/v1.33/bin/bin/../../lib/gcc/pic32mx/4.5.2/../../../../pic32mx/lib\libm.a(fp32mul.o)

.bss%z69        0x00000000        0x0
 .bss           0x00000000        0x0 c:/program files/microchip/xc32/v1.33/bin/bin/../../lib/gcc/pic32mx/4.5.2/../../../../pic32mx/lib\libm.a(fp32div.o)

.data%z70       0x00000000        0x0
 .data          0x00000000        0x0 c:/program files/microchip/xc32/v1.33/bin/bin/../../lib/gcc/pic32mx/4.5.2/../../../../pic32mx/lib\libm.a(fp32div.o)

.bss%z71        0x00000000        0x0
 .bss           0x00000000        0x0 c:/program files/microchip/xc32/v1.33/bin/bin/../../lib/gcc/pic32mx/4.5.2/../../../../pic32mx/lib\libpic32.a(defaultinterrupt.o)

.data%z72       0x00000000        0x0
 .data          0x00000000        0x0 c:/program files/microchip/xc32/v1.33/bin/bin/../../lib/gcc/pic32mx/4.5.2/../../../../pic32mx/lib\libpic32.a(defaultinterrupt.o)

.bss%z73        0x00000000        0x0
 .bss           0x00000000        0x0 c:/program files/microchip/xc32/v1.33/bin/bin/../../lib/gcc/pic32mx/4.5.2/../../../../pic32mx/lib\libpic32.a(vector63.o)

.data%z74       0x00000000        0x0
 .data          0x00000000        0x0 c:/program files/microchip/xc32/v1.33/bin/bin/../../lib/gcc/pic32mx/4.5.2/../../../../pic32mx/lib\libpic32.a(vector63.o)

.bss%z75        0x00000000        0x0
 .bss           0x00000000        0x0 c:/program files/microchip/xc32/v1.33/bin/bin/../../lib/gcc/pic32mx/4.5.2/../../../../pic32mx/lib\libpic32.a(vector62.o)

.data%z76       0x00000000        0x0
 .data          0x00000000        0x0 c:/program files/microchip/xc32/v1.33/bin/bin/../../lib/gcc/pic32mx/4.5.2/../../../../pic32mx/lib\libpic32.a(vector62.o)

.bss%z77        0x00000000        0x0
 .bss           0x00000000        0x0 c:/program files/microchip/xc32/v1.33/bin/bin/../../lib/gcc/pic32mx/4.5.2/../../../../pic32mx/lib\libpic32.a(vector61.o)

.data%z78       0x00000000        0x0
 .data          0x00000000        0x0 c:/program files/microchip/xc32/v1.33/bin/bin/../../lib/gcc/pic32mx/4.5.2/../../../../pic32mx/lib\libpic32.a(vector61.o)

.bss%z79        0x00000000        0x0
 .bss           0x00000000        0x0 c:/program files/microchip/xc32/v1.33/bin/bin/../../lib/gcc/pic32mx/4.5.2/../../../../pic32mx/lib\libpic32.a(vector60.o)

.data%z80       0x00000000        0x0
 .data          0x00000000        0x0 c:/program files/microchip/xc32/v1.33/bin/bin/../../lib/gcc/pic32mx/4.5.2/../../../../pic32mx/lib\libpic32.a(vector60.o)

.bss%z81        0x00000000        0x0
 .bss           0x00000000        0x0 c:/program files/microchip/xc32/v1.33/bin/bin/../../lib/gcc/pic32mx/4.5.2/../../../../pic32mx/lib\libpic32.a(vector59.o)

.data%z82       0x00000000        0x0
 .data          0x00000000        0x0 c:/program files/microchip/xc32/v1.33/bin/bin/../../lib/gcc/pic32mx/4.5.2/../../../../pic32mx/lib\libpic32.a(vector59.o)

.bss%z83        0x00000000        0x0
 .bss           0x00000000        0x0 c:/program files/microchip/xc32/v1.33/bin/bin/../../lib/gcc/pic32mx/4.5.2/../../../../pic32mx/lib\libpic32.a(vector58.o)

.data%z84       0x00000000        0x0
 .data          0x00000000        0x0 c:/program files/microchip/xc32/v1.33/bin/bin/../../lib/gcc/pic32mx/4.5.2/../../../../pic32mx/lib\libpic32.a(vector58.o)

.bss%z85        0x00000000        0x0
 .bss           0x00000000        0x0 c:/program files/microchip/xc32/v1.33/bin/bin/../../lib/gcc/pic32mx/4.5.2/../../../../pic32mx/lib\libpic32.a(vector57.o)

.data%z86       0x00000000        0x0
 .data          0x00000000        0x0 c:/program files/microchip/xc32/v1.33/bin/bin/../../lib/gcc/pic32mx/4.5.2/../../../../pic32mx/lib\libpic32.a(vector57.o)

.bss%z87        0x00000000        0x0
 .bss           0x00000000        0x0 c:/program files/microchip/xc32/v1.33/bin/bin/../../lib/gcc/pic32mx/4.5.2/../../../../pic32mx/lib\libpic32.a(vector56.o)

.data%z88       0x00000000        0x0
 .data          0x00000000        0x0 c:/program files/microchip/xc32/v1.33/bin/bin/../../lib/gcc/pic32mx/4.5.2/../../../../pic32mx/lib\libpic32.a(vector56.o)

.bss%z89        0x00000000        0x0
 .bss           0x00000000        0x0 c:/program files/microchip/xc32/v1.33/bin/bin/../../lib/gcc/pic32mx/4.5.2/../../../../pic32mx/lib\libpic32.a(vector55.o)

.data%z90       0x00000000        0x0
 .data          0x00000000        0x0 c:/program files/microchip/xc32/v1.33/bin/bin/../../lib/gcc/pic32mx/4.5.2/../../../../pic32mx/lib\libpic32.a(vector55.o)

.bss%z91        0x00000000        0x0
 .bss           0x00000000        0x0 c:/program files/microchip/xc32/v1.33/bin/bin/../../lib/gcc/pic32mx/4.5.2/../../../../pic32mx/lib\libpic32.a(vector54.o)

.data%z92       0x00000000        0x0
 .data          0x00000000        0x0 c:/program files/microchip/xc32/v1.33/bin/bin/../../lib/gcc/pic32mx/4.5.2/../../../../pic32mx/lib\libpic32.a(vector54.o)

.bss%z93        0x00000000        0x0
 .bss           0x00000000        0x0 c:/program files/microchip/xc32/v1.33/bin/bin/../../lib/gcc/pic32mx/4.5.2/../../../../pic32mx/lib\libpic32.a(vector53.o)

.data%z94       0x00000000        0x0
 .data          0x00000000        0x0 c:/program files/microchip/xc32/v1.33/bin/bin/../../lib/gcc/pic32mx/4.5.2/../../../../pic32mx/lib\libpic32.a(vector53.o)

.bss%z95        0x00000000        0x0
 .bss           0x00000000        0x0 c:/program files/microchip/xc32/v1.33/bin/bin/../../lib/gcc/pic32mx/4.5.2/../../../../pic32mx/lib\libpic32.a(vector52.o)

.data%z96       0x00000000        0x0
 .data          0x00000000        0x0 c:/program files/microchip/xc32/v1.33/bin/bin/../../lib/gcc/pic32mx/4.5.2/../../../../pic32mx/lib\libpic32.a(vector52.o)

.bss%z97        0x00000000        0x0
 .bss           0x00000000        0x0 c:/program files/microchip/xc32/v1.33/bin/bin/../../lib/gcc/pic32mx/4.5.2/../../../../pic32mx/lib\libpic32.a(vector51.o)

.data%z98       0x00000000        0x0
 .data          0x00000000        0x0 c:/program files/microchip/xc32/v1.33/bin/bin/../../lib/gcc/pic32mx/4.5.2/../../../../pic32mx/lib\libpic32.a(vector51.o)

.bss%z99        0x00000000        0x0
 .bss           0x00000000        0x0 c:/program files/microchip/xc32/v1.33/bin/bin/../../lib/gcc/pic32mx/4.5.2/../../../../pic32mx/lib\libpic32.a(vector50.o)

.data%z100      0x00000000        0x0
 .data          0x00000000        0x0 c:/program files/microchip/xc32/v1.33/bin/bin/../../lib/gcc/pic32mx/4.5.2/../../../../pic32mx/lib\libpic32.a(vector50.o)

.bss%z101       0x00000000        0x0
 .bss           0x00000000        0x0 c:/program files/microchip/xc32/v1.33/bin/bin/../../lib/gcc/pic32mx/4.5.2/../../../../pic32mx/lib\libpic32.a(vector49.o)

.data%z102      0x00000000        0x0
 .data          0x00000000        0x0 c:/program files/microchip/xc32/v1.33/bin/bin/../../lib/gcc/pic32mx/4.5.2/../../../../pic32mx/lib\libpic32.a(vector49.o)

.bss%z103       0x00000000        0x0
 .bss           0x00000000        0x0 c:/program files/microchip/xc32/v1.33/bin/bin/../../lib/gcc/pic32mx/4.5.2/../../../../pic32mx/lib\libpic32.a(vector48.o)

.data%z104      0x00000000        0x0
 .data          0x00000000        0x0 c:/program files/microchip/xc32/v1.33/bin/bin/../../lib/gcc/pic32mx/4.5.2/../../../../pic32mx/lib\libpic32.a(vector48.o)

.bss%z105       0x00000000        0x0
 .bss           0x00000000        0x0 c:/program files/microchip/xc32/v1.33/bin/bin/../../lib/gcc/pic32mx/4.5.2/../../../../pic32mx/lib\libpic32.a(vector47.o)

.data%z106      0x00000000        0x0
 .data          0x00000000        0x0 c:/program files/microchip/xc32/v1.33/bin/bin/../../lib/gcc/pic32mx/4.5.2/../../../../pic32mx/lib\libpic32.a(vector47.o)

.bss%z107       0x00000000        0x0
 .bss           0x00000000        0x0 c:/program files/microchip/xc32/v1.33/bin/bin/../../lib/gcc/pic32mx/4.5.2/../../../../pic32mx/lib\libpic32.a(vector46.o)

.data%z108      0x00000000        0x0
 .data          0x00000000        0x0 c:/program files/microchip/xc32/v1.33/bin/bin/../../lib/gcc/pic32mx/4.5.2/../../../../pic32mx/lib\libpic32.a(vector46.o)

.bss%z109       0x00000000        0x0
 .bss           0x00000000        0x0 c:/program files/microchip/xc32/v1.33/bin/bin/../../lib/gcc/pic32mx/4.5.2/../../../../pic32mx/lib\libpic32.a(vector45.o)

.data%z110      0x00000000        0x0
 .data          0x00000000        0x0 c:/program files/microchip/xc32/v1.33/bin/bin/../../lib/gcc/pic32mx/4.5.2/../../../../pic32mx/lib\libpic32.a(vector45.o)

.bss%z111       0x00000000        0x0
 .bss           0x00000000        0x0 c:/program files/microchip/xc32/v1.33/bin/bin/../../lib/gcc/pic32mx/4.5.2/../../../../pic32mx/lib\libpic32.a(vector44.o)

.data%z112      0x00000000        0x0
 .data          0x00000000        0x0 c:/program files/microchip/xc32/v1.33/bin/bin/../../lib/gcc/pic32mx/4.5.2/../../../../pic32mx/lib\libpic32.a(vector44.o)

.bss%z113       0x00000000        0x0
 .bss           0x00000000        0x0 c:/program files/microchip/xc32/v1.33/bin/bin/../../lib/gcc/pic32mx/4.5.2/../../../../pic32mx/lib\libpic32.a(vector43.o)

.data%z114      0x00000000        0x0
 .data          0x00000000        0x0 c:/program files/microchip/xc32/v1.33/bin/bin/../../lib/gcc/pic32mx/4.5.2/../../../../pic32mx/lib\libpic32.a(vector43.o)

.bss%z115       0x00000000        0x0
 .bss           0x00000000        0x0 c:/program files/microchip/xc32/v1.33/bin/bin/../../lib/gcc/pic32mx/4.5.2/../../../../pic32mx/lib\libpic32.a(vector42.o)

.data%z116      0x00000000        0x0
 .data          0x00000000        0x0 c:/program files/microchip/xc32/v1.33/bin/bin/../../lib/gcc/pic32mx/4.5.2/../../../../pic32mx/lib\libpic32.a(vector42.o)

.bss%z117       0x00000000        0x0
 .bss           0x00000000        0x0 c:/program files/microchip/xc32/v1.33/bin/bin/../../lib/gcc/pic32mx/4.5.2/../../../../pic32mx/lib\libpic32.a(vector41.o)

.data%z118      0x00000000        0x0
 .data          0x00000000        0x0 c:/program files/microchip/xc32/v1.33/bin/bin/../../lib/gcc/pic32mx/4.5.2/../../../../pic32mx/lib\libpic32.a(vector41.o)

.bss%z119       0x00000000        0x0
 .bss           0x00000000        0x0 c:/program files/microchip/xc32/v1.33/bin/bin/../../lib/gcc/pic32mx/4.5.2/../../../../pic32mx/lib\libpic32.a(vector40.o)

.data%z120      0x00000000        0x0
 .data          0x00000000        0x0 c:/program files/microchip/xc32/v1.33/bin/bin/../../lib/gcc/pic32mx/4.5.2/../../../../pic32mx/lib\libpic32.a(vector40.o)

.bss%z121       0x00000000        0x0
 .bss           0x00000000        0x0 c:/program files/microchip/xc32/v1.33/bin/bin/../../lib/gcc/pic32mx/4.5.2/../../../../pic32mx/lib\libpic32.a(vector39.o)

.data%z122      0x00000000        0x0
 .data          0x00000000        0x0 c:/program files/microchip/xc32/v1.33/bin/bin/../../lib/gcc/pic32mx/4.5.2/../../../../pic32mx/lib\libpic32.a(vector39.o)

.bss%z123       0x00000000        0x0
 .bss           0x00000000        0x0 c:/program files/microchip/xc32/v1.33/bin/bin/../../lib/gcc/pic32mx/4.5.2/../../../../pic32mx/lib\libpic32.a(vector38.o)

.data%z124      0x00000000        0x0
 .data          0x00000000        0x0 c:/program files/microchip/xc32/v1.33/bin/bin/../../lib/gcc/pic32mx/4.5.2/../../../../pic32mx/lib\libpic32.a(vector38.o)

.bss%z125       0x00000000        0x0
 .bss           0x00000000        0x0 c:/program files/microchip/xc32/v1.33/bin/bin/../../lib/gcc/pic32mx/4.5.2/../../../../pic32mx/lib\libpic32.a(vector37.o)

.data%z126      0x00000000        0x0
 .data          0x00000000        0x0 c:/program files/microchip/xc32/v1.33/bin/bin/../../lib/gcc/pic32mx/4.5.2/../../../../pic32mx/lib\libpic32.a(vector37.o)

.bss%z127       0x00000000        0x0
 .bss           0x00000000        0x0 c:/program files/microchip/xc32/v1.33/bin/bin/../../lib/gcc/pic32mx/4.5.2/../../../../pic32mx/lib\libpic32.a(vector36.o)

.data%z128      0x00000000        0x0
 .data          0x00000000        0x0 c:/program files/microchip/xc32/v1.33/bin/bin/../../lib/gcc/pic32mx/4.5.2/../../../../pic32mx/lib\libpic32.a(vector36.o)

.bss%z129       0x00000000        0x0
 .bss           0x00000000        0x0 c:/program files/microchip/xc32/v1.33/bin/bin/../../lib/gcc/pic32mx/4.5.2/../../../../pic32mx/lib\libpic32.a(vector35.o)

.data%z130      0x00000000        0x0
 .data          0x00000000        0x0 c:/program files/microchip/xc32/v1.33/bin/bin/../../lib/gcc/pic32mx/4.5.2/../../../../pic32mx/lib\libpic32.a(vector35.o)

.bss%z131       0x00000000        0x0
 .bss           0x00000000        0x0 c:/program files/microchip/xc32/v1.33/bin/bin/../../lib/gcc/pic32mx/4.5.2/../../../../pic32mx/lib\libpic32.a(vector34.o)

.data%z132      0x00000000        0x0
 .data          0x00000000        0x0 c:/program files/microchip/xc32/v1.33/bin/bin/../../lib/gcc/pic32mx/4.5.2/../../../../pic32mx/lib\libpic32.a(vector34.o)

.bss%z133       0x00000000        0x0
 .bss           0x00000000        0x0 c:/program files/microchip/xc32/v1.33/bin/bin/../../lib/gcc/pic32mx/4.5.2/../../../../pic32mx/lib\libpic32.a(vector33.o)

.data%z134      0x00000000        0x0
 .data          0x00000000        0x0 c:/program files/microchip/xc32/v1.33/bin/bin/../../lib/gcc/pic32mx/4.5.2/../../../../pic32mx/lib\libpic32.a(vector33.o)

.bss%z135       0x00000000        0x0
 .bss           0x00000000        0x0 c:/program files/microchip/xc32/v1.33/bin/bin/../../lib/gcc/pic32mx/4.5.2/../../../../pic32mx/lib\libpic32.a(vector31.o)

.data%z136      0x00000000        0x0
 .data          0x00000000        0x0 c:/program files/microchip/xc32/v1.33/bin/bin/../../lib/gcc/pic32mx/4.5.2/../../../../pic32mx/lib\libpic32.a(vector31.o)

.bss%z137       0x00000000        0x0
 .bss           0x00000000        0x0 c:/program files/microchip/xc32/v1.33/bin/bin/../../lib/gcc/pic32mx/4.5.2/../../../../pic32mx/lib\libpic32.a(vector30.o)

.data%z138      0x00000000        0x0
 .data          0x00000000        0x0 c:/program files/microchip/xc32/v1.33/bin/bin/../../lib/gcc/pic32mx/4.5.2/../../../../pic32mx/lib\libpic32.a(vector30.o)

.bss%z139       0x00000000        0x0
 .bss           0x00000000        0x0 c:/program files/microchip/xc32/v1.33/bin/bin/../../lib/gcc/pic32mx/4.5.2/../../../../pic32mx/lib\libpic32.a(vector29.o)

.data%z140      0x00000000        0x0
 .data          0x00000000        0x0 c:/program files/microchip/xc32/v1.33/bin/bin/../../lib/gcc/pic32mx/4.5.2/../../../../pic32mx/lib\libpic32.a(vector29.o)

.bss%z141       0x00000000        0x0
 .bss           0x00000000        0x0 c:/program files/microchip/xc32/v1.33/bin/bin/../../lib/gcc/pic32mx/4.5.2/../../../../pic32mx/lib\libpic32.a(vector28.o)

.data%z142      0x00000000        0x0
 .data          0x00000000        0x0 c:/program files/microchip/xc32/v1.33/bin/bin/../../lib/gcc/pic32mx/4.5.2/../../../../pic32mx/lib\libpic32.a(vector28.o)

.bss%z143       0x00000000        0x0
 .bss           0x00000000        0x0 c:/program files/microchip/xc32/v1.33/bin/bin/../../lib/gcc/pic32mx/4.5.2/../../../../pic32mx/lib\libpic32.a(vector27.o)

.data%z144      0x00000000        0x0
 .data          0x00000000        0x0 c:/program files/microchip/xc32/v1.33/bin/bin/../../lib/gcc/pic32mx/4.5.2/../../../../pic32mx/lib\libpic32.a(vector27.o)

.bss%z145       0x00000000        0x0
 .bss           0x00000000        0x0 c:/program files/microchip/xc32/v1.33/bin/bin/../../lib/gcc/pic32mx/4.5.2/../../../../pic32mx/lib\libpic32.a(vector26.o)

.data%z146      0x00000000        0x0
 .data          0x00000000        0x0 c:/program files/microchip/xc32/v1.33/bin/bin/../../lib/gcc/pic32mx/4.5.2/../../../../pic32mx/lib\libpic32.a(vector26.o)

.bss%z147       0x00000000        0x0
 .bss           0x00000000        0x0 c:/program files/microchip/xc32/v1.33/bin/bin/../../lib/gcc/pic32mx/4.5.2/../../../../pic32mx/lib\libpic32.a(vector25.o)

.data%z148      0x00000000        0x0
 .data          0x00000000        0x0 c:/program files/microchip/xc32/v1.33/bin/bin/../../lib/gcc/pic32mx/4.5.2/../../../../pic32mx/lib\libpic32.a(vector25.o)

.bss%z149       0x00000000        0x0
 .bss           0x00000000        0x0 c:/program files/microchip/xc32/v1.33/bin/bin/../../lib/gcc/pic32mx/4.5.2/../../../../pic32mx/lib\libpic32.a(vector23.o)

.data%z150      0x00000000        0x0
 .data          0x00000000        0x0 c:/program files/microchip/xc32/v1.33/bin/bin/../../lib/gcc/pic32mx/4.5.2/../../../../pic32mx/lib\libpic32.a(vector23.o)

.bss%z151       0x00000000        0x0
 .bss           0x00000000        0x0 c:/program files/microchip/xc32/v1.33/bin/bin/../../lib/gcc/pic32mx/4.5.2/../../../../pic32mx/lib\libpic32.a(vector22.o)

.data%z152      0x00000000        0x0
 .data          0x00000000        0x0 c:/program files/microchip/xc32/v1.33/bin/bin/../../lib/gcc/pic32mx/4.5.2/../../../../pic32mx/lib\libpic32.a(vector22.o)

.bss%z153       0x00000000        0x0
 .bss           0x00000000        0x0 c:/program files/microchip/xc32/v1.33/bin/bin/../../lib/gcc/pic32mx/4.5.2/../../../../pic32mx/lib\libpic32.a(vector21.o)

.data%z154      0x00000000        0x0
 .data          0x00000000        0x0 c:/program files/microchip/xc32/v1.33/bin/bin/../../lib/gcc/pic32mx/4.5.2/../../../../pic32mx/lib\libpic32.a(vector21.o)

.bss%z155       0x00000000        0x0
 .bss           0x00000000        0x0 c:/program files/microchip/xc32/v1.33/bin/bin/../../lib/gcc/pic32mx/4.5.2/../../../../pic32mx/lib\libpic32.a(vector20.o)

.data%z156      0x00000000        0x0
 .data          0x00000000        0x0 c:/program files/microchip/xc32/v1.33/bin/bin/../../lib/gcc/pic32mx/4.5.2/../../../../pic32mx/lib\libpic32.a(vector20.o)

.bss%z157       0x00000000        0x0
 .bss           0x00000000        0x0 c:/program files/microchip/xc32/v1.33/bin/bin/../../lib/gcc/pic32mx/4.5.2/../../../../pic32mx/lib\libpic32.a(vector19.o)

.data%z158      0x00000000        0x0
 .data          0x00000000        0x0 c:/program files/microchip/xc32/v1.33/bin/bin/../../lib/gcc/pic32mx/4.5.2/../../../../pic32mx/lib\libpic32.a(vector19.o)

.bss%z159       0x00000000        0x0
 .bss           0x00000000        0x0 c:/program files/microchip/xc32/v1.33/bin/bin/../../lib/gcc/pic32mx/4.5.2/../../../../pic32mx/lib\libpic32.a(vector18.o)

.data%z160      0x00000000        0x0
 .data          0x00000000        0x0 c:/program files/microchip/xc32/v1.33/bin/bin/../../lib/gcc/pic32mx/4.5.2/../../../../pic32mx/lib\libpic32.a(vector18.o)

.bss%z161       0x00000000        0x0
 .bss           0x00000000        0x0 c:/program files/microchip/xc32/v1.33/bin/bin/../../lib/gcc/pic32mx/4.5.2/../../../../pic32mx/lib\libpic32.a(vector17.o)

.data%z162      0x00000000        0x0
 .data          0x00000000        0x0 c:/program files/microchip/xc32/v1.33/bin/bin/../../lib/gcc/pic32mx/4.5.2/../../../../pic32mx/lib\libpic32.a(vector17.o)

.bss%z163       0x00000000        0x0
 .bss           0x00000000        0x0 c:/program files/microchip/xc32/v1.33/bin/bin/../../lib/gcc/pic32mx/4.5.2/../../../../pic32mx/lib\libpic32.a(vector16.o)

.data%z164      0x00000000        0x0
 .data          0x00000000        0x0 c:/program files/microchip/xc32/v1.33/bin/bin/../../lib/gcc/pic32mx/4.5.2/../../../../pic32mx/lib\libpic32.a(vector16.o)

.bss%z165       0x00000000        0x0
 .bss           0x00000000        0x0 c:/program files/microchip/xc32/v1.33/bin/bin/../../lib/gcc/pic32mx/4.5.2/../../../../pic32mx/lib\libpic32.a(vector15.o)

.data%z166      0x00000000        0x0
 .data          0x00000000        0x0 c:/program files/microchip/xc32/v1.33/bin/bin/../../lib/gcc/pic32mx/4.5.2/../../../../pic32mx/lib\libpic32.a(vector15.o)

.bss%z167       0x00000000        0x0
 .bss           0x00000000        0x0 c:/program files/microchip/xc32/v1.33/bin/bin/../../lib/gcc/pic32mx/4.5.2/../../../../pic32mx/lib\libpic32.a(vector14.o)

.data%z168      0x00000000        0x0
 .data          0x00000000        0x0 c:/program files/microchip/xc32/v1.33/bin/bin/../../lib/gcc/pic32mx/4.5.2/../../../../pic32mx/lib\libpic32.a(vector14.o)

.bss%z169       0x00000000        0x0
 .bss           0x00000000        0x0 c:/program files/microchip/xc32/v1.33/bin/bin/../../lib/gcc/pic32mx/4.5.2/../../../../pic32mx/lib\libpic32.a(vector13.o)

.data%z170      0x00000000        0x0
 .data          0x00000000        0x0 c:/program files/microchip/xc32/v1.33/bin/bin/../../lib/gcc/pic32mx/4.5.2/../../../../pic32mx/lib\libpic32.a(vector13.o)

.bss%z171       0x00000000        0x0
 .bss           0x00000000        0x0 c:/program files/microchip/xc32/v1.33/bin/bin/../../lib/gcc/pic32mx/4.5.2/../../../../pic32mx/lib\libpic32.a(vector12.o)

.data%z172      0x00000000        0x0
 .data          0x00000000        0x0 c:/program files/microchip/xc32/v1.33/bin/bin/../../lib/gcc/pic32mx/4.5.2/../../../../pic32mx/lib\libpic32.a(vector12.o)

.bss%z173       0x00000000        0x0
 .bss           0x00000000        0x0 c:/program files/microchip/xc32/v1.33/bin/bin/../../lib/gcc/pic32mx/4.5.2/../../../../pic32mx/lib\libpic32.a(vector11.o)

.data%z174      0x00000000        0x0
 .data          0x00000000        0x0 c:/program files/microchip/xc32/v1.33/bin/bin/../../lib/gcc/pic32mx/4.5.2/../../../../pic32mx/lib\libpic32.a(vector11.o)

.bss%z175       0x00000000        0x0
 .bss           0x00000000        0x0 c:/program files/microchip/xc32/v1.33/bin/bin/../../lib/gcc/pic32mx/4.5.2/../../../../pic32mx/lib\libpic32.a(vector10.o)

.data%z176      0x00000000        0x0
 .data          0x00000000        0x0 c:/program files/microchip/xc32/v1.33/bin/bin/../../lib/gcc/pic32mx/4.5.2/../../../../pic32mx/lib\libpic32.a(vector10.o)

.bss%z177       0x00000000        0x0
 .bss           0x00000000        0x0 c:/program files/microchip/xc32/v1.33/bin/bin/../../lib/gcc/pic32mx/4.5.2/../../../../pic32mx/lib\libpic32.a(vector9.o)

.data%z178      0x00000000        0x0
 .data          0x00000000        0x0 c:/program files/microchip/xc32/v1.33/bin/bin/../../lib/gcc/pic32mx/4.5.2/../../../../pic32mx/lib\libpic32.a(vector9.o)

.bss%z179       0x00000000        0x0
 .bss           0x00000000        0x0 c:/program files/microchip/xc32/v1.33/bin/bin/../../lib/gcc/pic32mx/4.5.2/../../../../pic32mx/lib\libpic32.a(vector8.o)

.data%z180      0x00000000        0x0
 .data          0x00000000        0x0 c:/program files/microchip/xc32/v1.33/bin/bin/../../lib/gcc/pic32mx/4.5.2/../../../../pic32mx/lib\libpic32.a(vector8.o)

.bss%z181       0x00000000        0x0
 .bss           0x00000000        0x0 c:/program files/microchip/xc32/v1.33/bin/bin/../../lib/gcc/pic32mx/4.5.2/../../../../pic32mx/lib\libpic32.a(vector7.o)

.data%z182      0x00000000        0x0
 .data          0x00000000        0x0 c:/program files/microchip/xc32/v1.33/bin/bin/../../lib/gcc/pic32mx/4.5.2/../../../../pic32mx/lib\libpic32.a(vector7.o)

.bss%z183       0x00000000        0x0
 .bss           0x00000000        0x0 c:/program files/microchip/xc32/v1.33/bin/bin/../../lib/gcc/pic32mx/4.5.2/../../../../pic32mx/lib\libpic32.a(vector6.o)

.data%z184      0x00000000        0x0
 .data          0x00000000        0x0 c:/program files/microchip/xc32/v1.33/bin/bin/../../lib/gcc/pic32mx/4.5.2/../../../../pic32mx/lib\libpic32.a(vector6.o)

.bss%z185       0x00000000        0x0
 .bss           0x00000000        0x0 c:/program files/microchip/xc32/v1.33/bin/bin/../../lib/gcc/pic32mx/4.5.2/../../../../pic32mx/lib\libpic32.a(vector5.o)

.data%z186      0x00000000        0x0
 .data          0x00000000        0x0 c:/program files/microchip/xc32/v1.33/bin/bin/../../lib/gcc/pic32mx/4.5.2/../../../../pic32mx/lib\libpic32.a(vector5.o)

.bss%z187       0x00000000        0x0
 .bss           0x00000000        0x0 c:/program files/microchip/xc32/v1.33/bin/bin/../../lib/gcc/pic32mx/4.5.2/../../../../pic32mx/lib\libpic32.a(vector2.o)

.data%z188      0x00000000        0x0
 .data          0x00000000        0x0 c:/program files/microchip/xc32/v1.33/bin/bin/../../lib/gcc/pic32mx/4.5.2/../../../../pic32mx/lib\libpic32.a(vector2.o)

.bss%z189       0x00000000        0x0
 .bss           0x00000000        0x0 c:/program files/microchip/xc32/v1.33/bin/bin/../../lib/gcc/pic32mx/4.5.2/../../../../pic32mx/lib\libpic32.a(vector1.o)

.data%z190      0x00000000        0x0
 .data          0x00000000        0x0 c:/program files/microchip/xc32/v1.33/bin/bin/../../lib/gcc/pic32mx/4.5.2/../../../../pic32mx/lib\libpic32.a(vector1.o)

.bss%z191       0x00000000        0x0
 .bss           0x00000000        0x0 c:/program files/microchip/xc32/v1.33/bin/bin/../../lib/gcc/pic32mx/4.5.2/../../../../pic32mx/lib\libpic32.a(vector0.o)

.data%z192      0x00000000        0x0
 .data          0x00000000        0x0 c:/program files/microchip/xc32/v1.33/bin/bin/../../lib/gcc/pic32mx/4.5.2/../../../../pic32mx/lib\libpic32.a(vector0.o)

.bss%z193       0x00000000        0x0
 .bss           0x00000000        0x0 c:/program files/microchip/xc32/v1.33/bin/bin/../../lib/gcc/pic32mx/4.5.2/../../../../pic32mx/lib\libpic32.a(general-exception.o)

.data%z194      0x00000000        0x0
 .data          0x00000000        0x0 c:/program files/microchip/xc32/v1.33/bin/bin/../../lib/gcc/pic32mx/4.5.2/../../../../pic32mx/lib\libpic32.a(general-exception.o)

.bss%z195       0x00000000        0x0
 .bss           0x00000000        0x0 c:/program files/microchip/xc32/v1.33/bin/bin/../../lib/gcc/pic32mx/4.5.2/../../../../pic32mx/lib\libpic32.a(default-nmi-handler.o)

.data%z196      0x00000000        0x0
 .data          0x00000000        0x0 c:/program files/microchip/xc32/v1.33/bin/bin/../../lib/gcc/pic32mx/4.5.2/../../../../pic32mx/lib\libpic32.a(default-nmi-handler.o)

.bss%z197       0x00000000        0x0
 .bss           0x00000000        0x0 c:/program files/microchip/xc32/v1.33/bin/bin/../../lib/gcc/pic32mx/4.5.2/../../../../pic32mx/lib\libpic32.a(default-on-bootstrap.o)

.data%z198      0x00000000        0x0
 .data          0x00000000        0x0 c:/program files/microchip/xc32/v1.33/bin/bin/../../lib/gcc/pic32mx/4.5.2/../../../../pic32mx/lib\libpic32.a(default-on-bootstrap.o)

.bss%z199       0x00000000        0x0
 .bss           0x00000000        0x0 c:/program files/microchip/xc32/v1.33/bin/bin/../../lib/gcc/pic32mx/4.5.2/../../../../pic32mx/lib\libpic32.a(default-on-reset.o)

.data%z200      0x00000000        0x0
 .data          0x00000000        0x0 c:/program files/microchip/xc32/v1.33/bin/bin/../../lib/gcc/pic32mx/4.5.2/../../../../pic32mx/lib\libpic32.a(default-on-reset.o)

.bss%z201       0x00000000        0x0
 .bss           0x00000000        0x0 c:/program files/microchip/xc32/v1.33/bin/bin/../../lib/gcc/pic32mx/4.5.2/../../../../pic32mx/lib\libpic32.a(default-bootstrap-exception-handler.o)

.data%z202      0x00000000        0x0
 .data          0x00000000        0x0 c:/program files/microchip/xc32/v1.33/bin/bin/../../lib/gcc/pic32mx/4.5.2/../../../../pic32mx/lib\libpic32.a(default-bootstrap-exception-handler.o)

.bss%z203       0x00000000        0x0
 .bss           0x00000000        0x0 c:/program files/microchip/xc32/v1.33/bin/bin/../../lib/gcc/pic32mx/4.5.2/../../../../pic32mx/lib\libpic32.a(strlen.o)

.data%z204      0x00000000        0x0
 .data          0x00000000        0x0 c:/program files/microchip/xc32/v1.33/bin/bin/../../lib/gcc/pic32mx/4.5.2/../../../../pic32mx/lib\libpic32.a(strlen.o)

.bss%z205       0x00000000        0x0
 .bss           0x00000000        0x0 c:/program files/microchip/xc32/v1.33/bin/bin/../../lib/gcc/pic32mx/4.5.2/../../../../pic32mx/lib\libpic32.a(strcpy.o)

.data%z206      0x00000000        0x0
 .data          0x00000000        0x0 c:/program files/microchip/xc32/v1.33/bin/bin/../../lib/gcc/pic32mx/4.5.2/../../../../pic32mx/lib\libpic32.a(strcpy.o)

.bss%z207       0x00000000        0x0
 .bss           0x00000000        0x0 c:/program files/microchip/xc32/v1.33/bin/bin/../../lib/gcc/pic32mx/4.5.2/../../../../pic32mx/lib\libpic32.a(memset.o)

.data%z208      0x00000000        0x0
 .data          0x00000000        0x0 c:/program files/microchip/xc32/v1.33/bin/bin/../../lib/gcc/pic32mx/4.5.2/../../../../pic32mx/lib\libpic32.a(memset.o)

.bss%z209       0x00000000        0x0
 .bss           0x00000000        0x0 c:/program files/microchip/xc32/v1.33/bin/bin/../../lib/gcc/pic32mx/4.5.2/../../../../pic32mx/lib\libpic32.a(memcpy.o)

.data%z210      0x00000000        0x0
 .data          0x00000000        0x0 c:/program files/microchip/xc32/v1.33/bin/bin/../../lib/gcc/pic32mx/4.5.2/../../../../pic32mx/lib\libpic32.a(memcpy.o)

.bss%z211       0x00000000        0x0
 .bss           0x00000000        0x0 c:/program files/microchip/xc32/v1.33/bin/bin/../../lib/gcc/pic32mx/4.5.2/../../../../pic32mx/lib\libmchp_peripheral_32MX795F512H.a(int_restore_interrupts_lib.o)

.data%z212      0x00000000        0x0
 .data          0x00000000        0x0 c:/program files/microchip/xc32/v1.33/bin/bin/../../lib/gcc/pic32mx/4.5.2/../../../../pic32mx/lib\libmchp_peripheral_32MX795F512H.a(int_restore_interrupts_lib.o)

.bss%z213       0x00000000        0x0
 .bss           0x00000000        0x0 c:/program files/microchip/xc32/v1.33/bin/bin/../../lib/gcc/pic32mx/4.5.2/../../../../pic32mx/lib\libmchp_peripheral_32MX795F512H.a(int_disable_interrupts_lib.o)

.data%z214      0x00000000        0x0
 .data          0x00000000        0x0 c:/program files/microchip/xc32/v1.33/bin/bin/../../lib/gcc/pic32mx/4.5.2/../../../../pic32mx/lib\libmchp_peripheral_32MX795F512H.a(int_disable_interrupts_lib.o)

.bss%z215       0x00000000        0x0
 .bss           0x00000000        0x0 c:/program files/microchip/xc32/v1.33/bin/bin/../../lib/gcc/pic32mx/4.5.2/../../../../pic32mx/lib\libmchp_peripheral_32MX795F512H.a(int_enable_interrupts_lib.o)

.data%z216      0x00000000        0x0
 .data          0x00000000        0x0 c:/program files/microchip/xc32/v1.33/bin/bin/../../lib/gcc/pic32mx/4.5.2/../../../../pic32mx/lib\libmchp_peripheral_32MX795F512H.a(int_enable_interrupts_lib.o)

.bss%z217       0x00000000        0x0
 .bss           0x00000000        0x0 c:/program files/microchip/xc32/v1.33/bin/bin/../../lib/gcc/pic32mx/4.5.2/../../../../pic32mx/lib\libmchp_peripheral_32MX795F512H.a(int_configure_system_lib.o)

.data%z218      0x00000000        0x0
 .data          0x00000000        0x0 c:/program files/microchip/xc32/v1.33/bin/bin/../../lib/gcc/pic32mx/4.5.2/../../../../pic32mx/lib\libmchp_peripheral_32MX795F512H.a(int_configure_system_lib.o)

.bss%z219       0x00000000        0x0
 .bss           0x00000000        0x0 c:/program files/microchip/xc32/v1.33/bin/bin/../../lib/gcc/pic32mx/4.5.2/../../../../pic32mx/lib\libmchp_peripheral_32MX795F512H.a(pcache.o)

.data%z220      0x00000000        0x0
 .data          0x00000000        0x0 c:/program files/microchip/xc32/v1.33/bin/bin/../../lib/gcc/pic32mx/4.5.2/../../../../pic32mx/lib\libmchp_peripheral_32MX795F512H.a(pcache.o)

.bss%z221       0x00000000        0x0
 .bss           0x00000000        0x0 c:/program files/microchip/xc32/v1.33/bin/bin/../../lib/gcc/pic32mx/4.5.2/../../../../pic32mx/lib\libmchp_peripheral_32MX795F512H.a(soft_reset_lib.o)

.data%z222      0x00000000        0x0
 .data          0x00000000        0x0 c:/program files/microchip/xc32/v1.33/bin/bin/../../lib/gcc/pic32mx/4.5.2/../../../../pic32mx/lib\libmchp_peripheral_32MX795F512H.a(soft_reset_lib.o)

.bss%z223       0x00000000        0x0
 .bss           0x00000000        0x0 c:/program files/microchip/xc32/v1.33/bin/bin/../../lib/gcc/pic32mx/4.5.2/../../../../pic32mx/lib/./proc/32MX795F512H\processor.o

.data%z224      0x00000000        0x0
 .data          0x00000000        0x0 c:/program files/microchip/xc32/v1.33/bin/bin/../../lib/gcc/pic32mx/4.5.2/../../../../pic32mx/lib/./proc/32MX795F512H\processor.o

.bss%z225       0x00000000        0x0
 .bss           0x00000000        0x0 c:/program files/microchip/xc32/v1.33/bin/bin/../../lib/gcc/pic32mx/4.5.2/../../../../pic32mx/lib\pic32_software_reset.o

.data%z226      0x00000000        0x0
 .data          0x00000000        0x0 c:/program files/microchip/xc32/v1.33/bin/bin/../../lib/gcc/pic32mx/4.5.2/../../../../pic32mx/lib\pic32_software_reset.o

.bss%z227       0x00000000        0x0
 .bss           0x00000000        0x0 c:/program files/microchip/xc32/v1.33/bin/bin/../../lib/gcc/pic32mx/4.5.2/../../../../pic32mx/lib/./proc/32MX795F512H\default_isr_vectors.o

.data%z228      0x00000000        0x0
 .data          0x00000000        0x0 c:/program files/microchip/xc32/v1.33/bin/bin/../../lib/gcc/pic32mx/4.5.2/../../../../pic32mx/lib/./proc/32MX795F512H\default_isr_vectors.o

.data%z229      0x00000000        0x0
 .data          0x00000000        0x0 build/ChaletDuinoV2_775F512H_/debug/Source/crc32.o

.bss%z230       0x00000000        0x0
 .bss           0x00000000        0x0 build/ChaletDuinoV2_775F512H_/debug/Source/BootloaderProtocol.o

.bss%z231       0x00000000        0x0
 .bss           0x00000000        0x0 build/ChaletDuinoV2_775F512H_/debug/Source/TC77.o

.data%z232      0x00000000        0x0
 .data          0x00000000        0x0 build/ChaletDuinoV2_775F512H_/debug/Source/TC77.o

.bss%z233       0x00000000        0x0
 .bss           0x00000000        0x0 build/ChaletDuinoV2_775F512H_/debug/Source/TemperatureSensor.o

.data%z234      0x00000000        0x0
 .data          0x00000000        0x0 build/ChaletDuinoV2_775F512H_/debug/Source/TemperatureSensor.o

.bss%z235       0x00000000        0x0
 .bss           0x00000000        0x0 build/ChaletDuinoV2_775F512H_/debug/Source/BootloaderInterface.o

.bss%z236       0x00000000        0x0
 .bss           0x00000000        0x0 build/ChaletDuinoV2_775F512H_/debug/Source/Watchdog.o

.data%z237      0x00000000        0x0
 .data          0x00000000        0x0 build/ChaletDuinoV2_775F512H_/debug/Source/Watchdog.o

.bss%z238       0x00000000        0x0
 .bss           0x00000000        0x0 build/ChaletDuinoV2_775F512H_/debug/Source/Syslog.o

.bss%z239       0x00000000        0x0
 .bss           0x00000000        0x0 build/ChaletDuinoV2_775F512H_/debug/Source/SPI_Flash.o

.data%z240      0x00000000        0x0
 .data          0x00000000        0x0 build/ChaletDuinoV2_775F512H_/debug/Source/SPI_Flash.o

.bss%z241       0x00000000        0x0
 .bss           0x00000000        0x0 build/ChaletDuinoV2_775F512H_/debug/Source/I2C.o

.data%z242      0x00000000        0x0
 .data          0x00000000        0x0 build/ChaletDuinoV2_775F512H_/debug/Source/I2C.o

.bss%z243       0x00000000        0x0
 .bss           0x00000000        0x0 build/ChaletDuinoV2_775F512H_/debug/Source/ina219.o

.data%z244      0x00000000        0x0
 .data          0x00000000        0x0 build/ChaletDuinoV2_775F512H_/debug/Source/ina219.o

.bss%z245       0x00000000        0x0
 .bss           0x00000000        0x0 build/ChaletDuinoV2_775F512H_/debug/Source/BatteryMonitor.o

.bss%z246       0x00000000        0x0
 .bss           0x00000000        0x0 build/ChaletDuinoV2_775F512H_/debug/Source/HarakiriRelay.o

.data%z247      0x00000000        0x0
 .data          0x00000000        0x0 build/ChaletDuinoV2_775F512H_/debug/Source/HarakiriRelay.o

.bss%z248       0x00000000        0x0
 .bss           0x00000000        0x0 build/ChaletDuinoV2_775F512H_/debug/Source/ChaletPowerRelay.o

.data%z249      0x00000000        0x0
 .data          0x00000000        0x0 build/ChaletDuinoV2_775F512H_/debug/Source/ChaletPowerRelay.o

.bss%z250       0x00000000        0x0
 .bss           0x00000000        0x0 build/ChaletDuinoV2_775F512H_/debug/Source/LoraNetworkInterface.o

.data%z251      0x00000000        0x0
 .data          0x00000000        0x0 build/ChaletDuinoV2_775F512H_/debug/Source/LoraNetworkInterface.o

.bss%z252       0x00000000        0x0
 .bss           0x00000000        0x0 build/ChaletDuinoV2_775F512H_/debug/Source/SPI.o

.data%z253      0x00000000        0x0
 .data          0x00000000        0x0 build/ChaletDuinoV2_775F512H_/debug/Source/SPI.o

.bss%z254       0x00000000        0x0
 .bss           0x00000000        0x0 build/ChaletDuinoV2_775F512H_/debug/Source/timer.o

.data%z255      0x00000000        0x0
 .data          0x00000000        0x0 build/ChaletDuinoV2_775F512H_/debug/Source/timer.o

.bss%z256       0x00000000        0x0
 .bss           0x00000000        0x0 build/ChaletDuinoV2_775F512H_/debug/Source/template.o

.data%z257      0x00000000        0x0
 .data          0x00000000        0x0 build/ChaletDuinoV2_775F512H_/debug/Source/template.o

.bss%z258       0x00000000        0x0
 .bss           0x00000000        0x0 build/ChaletDuinoV2_775F512H_/debug/Source/system.o

.data%z259      0x00000000        0x0
 .data          0x00000000        0x0 build/ChaletDuinoV2_775F512H_/debug/Source/system.o

.bss%z260       0x00000000        0x0
 .bss           0x00000000        0x0 build/ChaletDuinoV2_775F512H_/debug/Source/main.o

.bss%z261       0x00000000        0x0
 .bss           0x00000000        0x0 build/ChaletDuinoV2_775F512H_/debug/Source/interrupts.o

.data%z262      0x00000000        0x0
 .data          0x00000000        0x0 build/ChaletDuinoV2_775F512H_/debug/Source/interrupts.o

.bss%z263       0x00000000        0x0
 .bss           0x00000000        0x0 build/ChaletDuinoV2_775F512H_/debug/Source/exceptions.o

.data%z264      0x00000000        0x0
 .data          0x00000000        0x0 build/ChaletDuinoV2_775F512H_/debug/Source/exceptions.o

.bss%z265       0x00000000        0x0
 .bss           0x00000000        0x0 build/ChaletDuinoV2_775F512H_/debug/Source/Util.o

.data%z266      0x00000000        0x0
 .data          0x00000000        0x0 build/ChaletDuinoV2_775F512H_/debug/Source/Util.o

.bss%z267       0x00000000        0x0
 .bss           0x00000000        0x0 build/ChaletDuinoV2_775F512H_/debug/Source/Uart.o

.data%z268      0x00000000        0x0
 .data          0x00000000        0x0 build/ChaletDuinoV2_775F512H_/debug/Source/Uart.o

.bss%z269       0x00000000        0x0
 .bss           0x00000000        0x0 build/ChaletDuinoV2_775F512H_/debug/Source/Terminal.o

.bss%z270       0x00000000        0x0
 .bss           0x00000000        0x0 build/ChaletDuinoV2_775F512H_/debug/Source/NetworkProtocol.o

.data%z271      0x00000000        0x0
 .data          0x00000000        0x0 build/ChaletDuinoV2_775F512H_/debug/Source/NetworkProtocol.o

.bss%z272       0x00000000        0x0
 .bss           0x00000000        0x0 build/ChaletDuinoV2_775F512H_/debug/Source/InternalUart.o

.data%z273      0x00000000        0x0
 .data          0x00000000        0x0 build/ChaletDuinoV2_775F512H_/debug/Source/InternalUart.o

.bss%z274       0x00000000        0x0
 .bss           0x00000000        0x0 build/ChaletDuinoV2_775F512H_/debug/Source/DigitalIO.o

.data%z275      0x00000000        0x0
 .data          0x00000000        0x0 build/ChaletDuinoV2_775F512H_/debug/Source/DigitalIO.o

.bss%z276       0x00000000        0x0
 .bss           0x00000000        0x0 build/ChaletDuinoV2_775F512H_/debug/Source/winc3400/winc_init.o

.data%z277      0x00000000        0x0
 .data          0x00000000        0x0 build/ChaletDuinoV2_775F512H_/debug/Source/winc3400/winc_init.o

.bss%z278       0x00000000        0x0
 .bss           0x00000000        0x0 build/ChaletDuinoV2_775F512H_/debug/Source/winc3400/spi_flash/source/spi_flash.o

.data%z279      0x00000000        0x0
 .data          0x00000000        0x0 build/ChaletDuinoV2_775F512H_/debug/Source/winc3400/spi_flash/source/spi_flash.o

.bss%z280       0x00000000        0x0
 .bss           0x00000000        0x0 build/ChaletDuinoV2_775F512H_/debug/Source/winc3400/socket/source/socket.o

.data%z281      0x00000000        0x0
 .data          0x00000000        0x0 build/ChaletDuinoV2_775F512H_/debug/Source/winc3400/socket/source/socket.o

.bss%z282       0x00000000        0x0
 .bss           0x00000000        0x0 build/ChaletDuinoV2_775F512H_/debug/Source/winc3400/driver/source/nmuart.o

.data%z283      0x00000000        0x0
 .data          0x00000000        0x0 build/ChaletDuinoV2_775F512H_/debug/Source/winc3400/driver/source/nmuart.o

.bss%z284       0x00000000        0x0
 .bss           0x00000000        0x0 build/ChaletDuinoV2_775F512H_/debug/Source/winc3400/driver/source/nmspi.o

.data%z285      0x00000000        0x0
 .data          0x00000000        0x0 build/ChaletDuinoV2_775F512H_/debug/Source/winc3400/driver/source/nmspi.o

.bss%z286       0x00000000        0x0
 .bss           0x00000000        0x0 build/ChaletDuinoV2_775F512H_/debug/Source/winc3400/driver/source/nmi2c.o

.data%z287      0x00000000        0x0
 .data          0x00000000        0x0 build/ChaletDuinoV2_775F512H_/debug/Source/winc3400/driver/source/nmi2c.o

.bss%z288       0x00000000        0x0
 .bss           0x00000000        0x0 build/ChaletDuinoV2_775F512H_/debug/Source/winc3400/driver/source/nmdrv.o

.data%z289      0x00000000        0x0
 .data          0x00000000        0x0 build/ChaletDuinoV2_775F512H_/debug/Source/winc3400/driver/source/nmdrv.o

.bss%z290       0x00000000        0x0
 .bss           0x00000000        0x0 build/ChaletDuinoV2_775F512H_/debug/Source/winc3400/driver/source/nmbus.o

.data%z291      0x00000000        0x0
 .data          0x00000000        0x0 build/ChaletDuinoV2_775F512H_/debug/Source/winc3400/driver/source/nmbus.o

.bss%z292       0x00000000        0x0
 .bss           0x00000000        0x0 build/ChaletDuinoV2_775F512H_/debug/Source/winc3400/driver/source/nmasic.o

.data%z293      0x00000000        0x0
 .data          0x00000000        0x0 build/ChaletDuinoV2_775F512H_/debug/Source/winc3400/driver/source/nmasic.o

.bss%z294       0x00000000        0x0
 .bss           0x00000000        0x0 build/ChaletDuinoV2_775F512H_/debug/Source/winc3400/driver/source/m2m_wifi.o

.data%z295      0x00000000        0x0
 .data          0x00000000        0x0 build/ChaletDuinoV2_775F512H_/debug/Source/winc3400/driver/source/m2m_wifi.o

.bss%z296       0x00000000        0x0
 .bss           0x00000000        0x0 build/ChaletDuinoV2_775F512H_/debug/Source/winc3400/driver/source/m2m_ssl.o

.data%z297      0x00000000        0x0
 .data          0x00000000        0x0 build/ChaletDuinoV2_775F512H_/debug/Source/winc3400/driver/source/m2m_ssl.o

.bss%z298       0x00000000        0x0
 .bss           0x00000000        0x0 build/ChaletDuinoV2_775F512H_/debug/Source/winc3400/driver/source/m2m_periph.o

.data%z299      0x00000000        0x0
 .data          0x00000000        0x0 build/ChaletDuinoV2_775F512H_/debug/Source/winc3400/driver/source/m2m_periph.o

.bss%z300       0x00000000        0x0
 .bss           0x00000000        0x0 build/ChaletDuinoV2_775F512H_/debug/Source/winc3400/driver/source/m2m_ota.o

.data%z301      0x00000000        0x0
 .data          0x00000000        0x0 build/ChaletDuinoV2_775F512H_/debug/Source/winc3400/driver/source/m2m_ota.o

.bss%z302       0x00000000        0x0
 .bss           0x00000000        0x0 build/ChaletDuinoV2_775F512H_/debug/Source/winc3400/driver/source/m2m_hif.o

.data%z303      0x00000000        0x0
 .data          0x00000000        0x0 build/ChaletDuinoV2_775F512H_/debug/Source/winc3400/driver/source/m2m_hif.o

.bss%z304       0x00000000        0x0
 .bss           0x00000000        0x0 build/ChaletDuinoV2_775F512H_/debug/Source/winc3400/driver/source/m2m_crypto.o

.data%z305      0x00000000        0x0
 .data          0x00000000        0x0 build/ChaletDuinoV2_775F512H_/debug/Source/winc3400/driver/source/m2m_crypto.o

.bss%z306       0x00000000        0x0
 .bss           0x00000000        0x0 build/ChaletDuinoV2_775F512H_/debug/Source/winc3400/driver/source/m2m_ate_mode.o

.data%z307      0x00000000        0x0
 .data          0x00000000        0x0 build/ChaletDuinoV2_775F512H_/debug/Source/winc3400/driver/source/m2m_ate_mode.o

.bss%z308       0x00000000        0x0
 .bss           0x00000000        0x0 build/ChaletDuinoV2_775F512H_/debug/Source/winc3400/common/source/nm_common.o

.data%z309      0x00000000        0x0
 .data          0x00000000        0x0 build/ChaletDuinoV2_775F512H_/debug/Source/winc3400/common/source/nm_common.o

.bss%z310       0x00000000        0x0
 .bss           0x00000000        0x0 build/ChaletDuinoV2_775F512H_/debug/Source/winc3400/bus_wrapper/source/nm_bus_wrapper.o

.data%z311      0x00000000        0x0
 .data          0x00000000        0x0 build/ChaletDuinoV2_775F512H_/debug/Source/winc3400/bus_wrapper/source/nm_bus_wrapper.o

.bss%z312       0x00000000        0x0
 .bss           0x00000000        0x0 build/ChaletDuinoV2_775F512H_/debug/Source/winc3400/bsp/source/nm_bsp.o

.data%z313      0x00000000        0x0
 .data          0x00000000        0x0 build/ChaletDuinoV2_775F512H_/debug/Source/winc3400/bsp/source/nm_bsp.o

.bss%z314       0x00000000        0x0
 .bss           0x00000000        0x0 build/ChaletDuinoV2_775F512H_/debug/Source/ChaletduinoV2Board.o

.data%z315      0x00000000        0x0
 .data          0x00000000        0x0 build/ChaletDuinoV2_775F512H_/debug/Source/ChaletduinoV2Board.o

.bss%z316       0x00000000        0x0
 .bss           0x00000000        0x0 c:/program files/microchip/xc32/v1.33/bin/bin/../../lib/gcc/pic32mx/4.5.2/../../../../pic32mx/lib\software-debug-break.o

.data%z317      0x00000000        0x0
 .data          0x00000000        0x0 c:/program files/microchip/xc32/v1.33/bin/bin/../../lib/gcc/pic32mx/4.5.2/../../../../pic32mx/lib\software-debug-break.o

.bss%z318       0x00000000        0x0
 .bss           0x00000000        0x0 c:/program files/microchip/xc32/v1.33/bin/bin/../../lib/gcc/pic32mx/4.5.2/../../../../pic32mx/lib/./proc/32MX795F512H/crt0_mips32r2.o

.data%z319      0x00000000        0x0
 .data          0x00000000        0x0 c:/program files/microchip/xc32/v1.33/bin/bin/../../lib/gcc/pic32mx/4.5.2/../../../../pic32mx/lib/./proc/32MX795F512H/crt0_mips32r2.o

.text           0x9d003800     0xbcd4
 .text          0x9d003800     0x2904 build/ChaletDuinoV2_775F512H_/debug/Source/winc3400/driver/source/m2m_wifi.o
                0x9d003fb4                m2m_wifi_download_mode
                0x9d0042f4                m2m_wifi_ble_set_gain_table
                0x9d004368                m2m_wifi_init_hold
                0x9d0043ac                m2m_wifi_init_start
                0x9d0044f8                m2m_wifi_init
                0x9d004554                m2m_wifi_deinit
                0x9d00459c                m2m_wifi_reinit_hold
                0x9d0045d8                m2m_wifi_reinit_start
                0x9d004610                m2m_wifi_reinit
                0x9d004670                m2m_wifi_yield
                0x9d0046a0                m2m_wifi_handle_events
                0x9d0046d4                m2m_wifi_default_connect
                0x9d004720                m2m_wifi_connect
                0x9d004794                m2m_wifi_connect_sc
                0x9d004bd8                m2m_wifi_disconnect
                0x9d004c24                m2m_wifi_set_mac_address
                0x9d004c90                m2m_wifi_set_static_ip
                0x9d004d24                m2m_wifi_request_dhcp_client
                0x9d004d48                m2m_wifi_request_dhcp_server
                0x9d004d70                m2m_wifi_enable_dhcp
                0x9d004de8                m2m_wifi_set_lsn_int
                0x9d004e3c                m2m_wifi_set_cust_InfoElement
                0x9d004e9c                m2m_wifi_set_scan_options
                0x9d004f14                m2m_wifi_set_scan_region
                0x9d004f84                m2m_wifi_request_scan
                0x9d00502c                m2m_wifi_request_scan_passive
                0x9d0050d4                m2m_wifi_wps
                0x9d005160                m2m_wifi_wps_disable
                0x9d0051b8                m2m_wifi_p2p
                0x9d005264                m2m_wifi_p2p_disconnect
                0x9d0052bc                m2m_wifi_enable_ap
                0x9d005334                m2m_wifi_disable_ap
                0x9d00538c                m2m_wifi_req_curr_rssi
                0x9d0053e4                m2m_wifi_req_restrict_ble
                0x9d00543c                m2m_wifi_req_unrestrict_ble
                0x9d005494                m2m_wifi_send_ethernet_pkt
                0x9d005534                m2m_wifi_get_otp_mac_address
                0x9d0055b0                m2m_wifi_get_mac_address
                0x9d005624                m2m_wifi_req_scan_result
                0x9d005690                m2m_wifi_get_num_ap_found
                0x9d0056b8                m2m_wifi_get_sleep_mode
                0x9d0056e8                m2m_wifi_set_sleep_mode
                0x9d005774                m2m_wifi_request_sleep
                0x9d0057f8                m2m_wifi_set_device_name
                0x9d005894                m2m_wifi_get_chipId
                0x9d0058c4                m2m_wifi_get_firmware_version
                0x9d005928                m2m_wifi_check_ota_rb
                0x9d005994                m2m_ota_get_firmware_version
                0x9d0059f8                m2m_wifi_enable_monitoring_mode
                0x9d005aac                m2m_wifi_disable_monitoring_mode
                0x9d005af8                m2m_wifi_send_wlan_pkt
                0x9d005b94                m2m_wifi_start_provision_mode
                0x9d005c8c                m2m_wifi_stop_provision_mode
                0x9d005cd8                m2m_wifi_get_connection_info
                0x9d005d24                m2m_wifi_set_sytem_time
                0x9d005d78                m2m_wifi_get_sytem_time
                0x9d005dc4                m2m_wifi_enable_sntp
                0x9d005e3c                m2m_wifi_set_power_profile
                0x9d005ea8                m2m_wifi_set_tx_power
                0x9d005f14                m2m_wifi_enable_firmware_logs
                0x9d005f80                m2m_wifi_set_battery_voltage
                0x9d005ff0                m2m_wifi_prng_get_random_bytes
                0x9d006090                m2m_wifi_ble_api_send
 .text          0x9d006104     0x2140 build/ChaletDuinoV2_775F512H_/debug/Source/winc3400/socket/source/socket.o
                0x9d006104                Socket_ReadSocketData
                0x9d006a3c                socketInit
                0x9d006ab0                socketDeinit
                0x9d006b10                registerSocketCallback
                0x9d006b48                socket
                0x9d006dd0                bind
                0x9d006f00                listen
                0x9d006fe8                accept
                0x9d00705c                connect
                0x9d0071d4                send
                0x9d007378                sendto
                0x9d007510                recv
                0x9d0076f8                close
                0x9d007838                recvfrom
                0x9d007a28                nmi_inet_addr
                0x9d007b9c                gethostbyname
                0x9d007fd4                setsockopt
                0x9d008160                getsockopt
                0x9d00819c                m2m_ping_req
 .text          0x9d008244     0x1a7c build/ChaletDuinoV2_775F512H_/debug/Source/Uart.o
                0x9d008244                InitUart
                0x9d0084f4                UartResetPort
                0x9d0087a8                UartOpenComPort
                0x9d008998                UartReceiveData
                0x9d008ae4                UartGetPendingDataSize
                0x9d008bdc                UartTransmitData
                0x9d009320                DataSentNotification
                0x9d0095f4                UartTick
                0x9d009bcc                UartBlockAndTick
                0x9d009c2c                UartBlockUntillBufEmpty
 .text          0x9d009cc0     0x18ac build/ChaletDuinoV2_775F512H_/debug/Source/WiFiCtrl.o
                0x9d00a83c                InitWiFi
                0x9d00ab14                TurnOFFWiFi
                0x9d00aba8                CloseSockets
                0x9d00ac94                GetWiFiSate
                0x9d00acb8                TickWiFi
                0x9d00ada4                OpenTerminalServer
                0x9d00ae60                SendTerminalData
                0x9d00aee8                SentTerminalByte
                0x9d00af64                OpenNetworkServer
                0x9d00b020                SendNetworkData
                0x9d00b0a8                SentNetworkByte
                0x9d00b124                OpenSyslogServer
                0x9d00b1e0                SendSyslogData
                0x9d00b258                SendSyslogByte
                0x9d00b2d4                IsSyslogClientConnected
                0x9d00b314                OpenBootloaderServer
                0x9d00b3d0                CloseBootloaderServer
                0x9d00b438                SendBootloaderData
                0x9d00b4b0                SendSBootloaderByte
                0x9d00b52c                IsBootloaderClientConnected
 .text          0x9d00b56c     0x15c0 build/ChaletDuinoV2_775F512H_/debug/Source/BootloaderInterface.o
                0x9d00b56c                BootloaderInterfaceInit
                0x9d00b5c0                BootloaderInterfaceTick
                0x9d00b5f8                BootloaderExecuteCmd
                0x9d00b834                BootloaderCRCError
                0x9d00b89c                BootloaderInterfaceStateMachine
                0x9d00c100                BootloaderResetStateMachine
                0x9d00c15c                BootloaderActivateBootloader
                0x9d00c19c                BootloaderDeactivateBootloader
                0x9d00c1cc                BootloaderFlashEraseStateMachine
                0x9d00c400                ResetBootloaderFlashEraseStateMachine
                0x9d00c434                BootloaderFlashWriteStateMachine
                0x9d00c660                BootloaderPrintFlashData
                0x9d00c680                BootloaderCheckFlashBootloaderData
                0x9d00ca34                ResetBootloaderFlashWriteStateMachine
                0x9d00ca74                BootloaderBytesToInt
 .text          0x9d00cb2c     0x1584 build/ChaletDuinoV2_775F512H_/debug/Source/winc3400/driver/source/nmasic.o
                0x9d00cb2c                chip_apply_conf
                0x9d00cbe0                nm_clkless_wake
                0x9d00ce20                chip_idle
                0x9d00ce94                enable_rf_blocks
                0x9d00cf34                enable_interrupts
                0x9d00d03c                cpu_start
                0x9d00d1b8                nmi_get_chipid
                0x9d00d3d0                nmi_get_rfrevid
                0x9d00d428                restore_pmu_settings_after_global_reset
                0x9d00d47c                nmi_update_pll
                0x9d00d4f0                nmi_set_sys_clk_src_to_xo
                0x9d00d54c                chip_wake
                0x9d00d5a0                chip_reset_and_cpu_halt
                0x9d00d734                chip_reset
                0x9d00d79c                wait_for_bootrom
                0x9d00d928                wait_for_firmware_start
                0x9d00da48                chip_deinit
                0x9d00db64                set_gpio_dir
                0x9d00dc38                set_gpio_val
                0x9d00dd0c                get_gpio_val
                0x9d00dd98                pullup_ctrl
                0x9d00de50                nmi_get_otp_mac_address
                0x9d00dfb0                nmi_get_mac_address
 .text          0x9d00e0b0     0x1424 build/ChaletDuinoV2_775F512H_/debug/Source/winc3400/driver/source/m2m_hif.o
                0x9d00e1e8                hif_chip_wake
                0x9d00e2b4                hif_set_sleep_mode
                0x9d00e2e4                hif_get_sleep_mode
                0x9d00e30c                hif_chip_sleep
                0x9d00e430                hif_init
                0x9d00e49c                hif_deinit
                0x9d00e4fc                hif_check_compatibility
                0x9d00e574                hif_enable_access
                0x9d00e694                hif_check_code
                0x9d00e784                hif_send
                0x9d00f09c                hif_yield
                0x9d00f0c4                hif_handle_isr
                0x9d00f190                hif_receive
                0x9d00f3ec                hif_register_cb

.text._vfprintf_cdfFnopsuxX
                0x9d00f4d4     0x13d4
 .text._vfprintf_cdfFnopsuxX
                0x9d00f4d4     0x13d4 c:/program files/microchip/xc32/v1.33/bin/bin/../../lib/gcc/pic32mx/4.5.2/../../../../pic32mx/lib\libc.a(doprnt_cdfFnopsuxX.eo)
                0x9d00f4d4                _vfprintf_cdfFnopsuxX
                0x9d00f4d4                _vfprintf_cdfFnopuxX
                0x9d00f4d4                _vfprintf_cdnopsuxX
                0x9d00f4d4                _vfprintf_fF
                0x9d00f4d4                _vfprintf_cdnopuxX

.text           0x9d0108a8     0x7248
 .text          0x9d0108a8     0x117c build/ChaletDuinoV2_775F512H_/debug/Source/winc3400/spi_flash/source/spi_flash.o
                0x9d0115a8                spi_flash_read
                0x9d011680                spi_flash_write
                0x9d011858                spi_flash_erase
                0x9d0119a4                spi_flash_get_size
 .text          0x9d011a24     0x1108 build/ChaletDuinoV2_775F512H_/debug/Source/winc3400/driver/source/nmspi.o
                0x9d0124c0                nm_spi_write_reg
                0x9d012598                nm_spi_write_block
                0x9d0126a0                nm_spi_read_reg_with_ret
                0x9d0127ec                nm_spi_read_block
                0x9d0129a8                nm_spi_init
                0x9d012ac0                nm_spi_deinit
                0x9d012ae8                nm_spi_read_reg
 .text          0x9d012b2c      0xf40 build/ChaletDuinoV2_775F512H_/debug/Source/InternalUart.o
                0x9d012b2c                InternalUartInit
                0x9d012d04                OpenInternalPort
                0x9d012f24                SendInternalUartData
                0x9d013240                SendInternalUartDataBlocking
                0x9d013318                TickInternalUart
                0x9d0133f0                InternalUart1AInterrupt
                0x9d01362c                InternalUart2Interrupt
                0x9d01384c                ResetUart1
                0x9d013954                ResetUart2
                0x9d013a4c                process
 .text          0x9d013a6c      0xe68 build/ChaletDuinoV2_775F512H_/debug/Source/Terminal.o
                0x9d013a6c                InitTerminal
                0x9d013aec                TickTerminal
                0x9d013b48                RxTerminalBuf
                0x9d013bd4                RxTerminalData
                0x9d013d24                ParseNewBuffer
                0x9d014820                TerminalPrintString
                0x9d014874                TerminalPrintChar
                0x9d0148b4                TerminalStateMachine
 .text          0x9d0148d4      0xda8 build/ChaletDuinoV2_775F512H_/debug/Source/SPI_Flash.o
                0x9d0148d4                InitSPIFlash
                0x9d014a48                SPIFlashCheckAndConfigure
                0x9d014b18                SPIFlashWriteEnable
                0x9d014b7c                SPIFlashReadStatusReg
                0x9d014c24                SPIFlashCheckBusy
                0x9d014c80                SPIFlashCheckChipID
                0x9d014dbc                SPIFlashReadBuffer
                0x9d014f3c                SPIFlashEraseSector
                0x9d015064                SPIFlashErase64KSector
                0x9d0151b8                SPIFlashWriteSectorWorkingBuffer
                0x9d015374                SPIFlashWriteByte
                0x9d0154c8                SPIFlashWriteBuffer
 .text          0x9d01567c      0xce8 build/ChaletDuinoV2_775F512H_/debug/Source/Util.o
                0x9d01567c                SwapEndianShort
                0x9d0156c8                SwapEndianInt
                0x9d015724                ConvertIntToStrLeadingZero
                0x9d015b48                ConvertIntToStr
                0x9d015e9c                ConvertCharToStrLeadingZero
                0x9d016004                ConvertStrToValue
                0x9d0161f0                ConvertCharToStr
                0x9d0162a8                Crc8
                0x9d016340                Delay
 .text          0x9d016364      0xbf4 build/ChaletDuinoV2_775F512H_/debug/Source/winc3400/driver/source/m2m_ssl.o
                0x9d016670                m2m_ssl_handshake_rsp
                0x9d0166e8                m2m_ssl_send_certs_to_winc
                0x9d016a30                m2m_ssl_retrieve_cert
                0x9d016d6c                m2m_ssl_retrieve_hash
                0x9d016e2c                m2m_ssl_stop_processing_certs
                0x9d016e6c                m2m_ssl_ecc_process_done
                0x9d016e90                m2m_ssl_set_active_ciphersuites
                0x9d016ef8                m2m_ssl_init
 .text          0x9d016f58      0xb98 build/ChaletDuinoV2_775F512H_/debug/Source/timer.o
                0x9d016f58                TimerInit
                0x9d017028                IsMilliSecTimerExpired
                0x9d017190                IsSecTimerExpired
                0x9d0172f4                IsTimerExpired
                0x9d0176a8                TimerStart
                0x9d0177d0                TimerStartSeconds
                0x9d017874                TimerReset
                0x9d0178f8                IsTimerRunning
                0x9d01793c                TimerStop
                0x9d017980                Sleep
                0x9d0179dc                Timer1MilliSecInterrupt

.dinit          0x9d017af0      0xb50
 .dinit         0x9d017af0      0xb50 data_init

.text           0x9d018640      0xb04
 .text          0x9d018640      0xb04 build/ChaletDuinoV2_775F512H_/debug/Source/BootloaderProtocol.o
                0x9d018640                BootloaderProtocolInit
                0x9d018670                BootloaderProtocolStateMachine
                0x9d018a74                BootloaderProtocolProtocolAnalyzeNewData
                0x9d018af0                BootloaderProtocolResetStateMachine
                0x9d018b3c                BootloaderProtocolSendFrame
                0x9d018cb4                BootloaderProtocolGetDataBufferPtr
                0x9d018cd8                BootloaderProtocolSendHeartbeat
                0x9d018d20                BootloaderProtocolSendACK
                0x9d018d74                BootloaderProtocolSendNACK
                0x9d018dc4                BootloaderProtocolSendInitUploadResponse
                0x9d018f24                BootloaderProtocolSendDataChunkResult
                0x9d019018                BootloaderProtocolSendBootloaderState
                0x9d01907c                BootloaderProtocolSendFirmwareUploadResult
                0x9d0190e0                BootloaderProtocolSendFlashCheckResult

.rodata         0x9d019144      0x990
 .rodata        0x9d019144      0x990 build/ChaletDuinoV2_775F512H_/debug/Source/BootloaderInterface.o

.text           0x9d019ad4      0x974
 .text          0x9d019ad4      0x974 build/ChaletDuinoV2_775F512H_/debug/Source/NetworkProtocol.o
                0x9d019ad4                ProtocolInit
                0x9d019b04                StateMachine
                0x9d01a080                ProtocolAnalyzeNewData
                0x9d01a0c0                ResetStateMachine
                0x9d01a108                ProtocolExecCmd
                0x9d01a144                ProtocolAcknowledge
                0x9d01a1a8                ProtocolCalcCrc
                0x9d01a224                ProtocolIsReceiving
                0x9d01a264                ProtocolGetFrame
                0x9d01a420                ProtocolMsgDataPtr

.text._vfscanf_s
                0x9d01a448      0x868
 .text._vfscanf_s
                0x9d01a448      0x868 c:/program files/microchip/xc32/v1.33/bin/bin/../../lib/gcc/pic32mx/4.5.2/../../../../pic32mx/lib\libc.a(doscan_s.eo)
                0x9d01a448                _vfscanf_s
                0x9d01a448                _vfscanf_0

.text           0x9d01acb0     0x2a84
 .text          0x9d01acb0      0x740 build/ChaletDuinoV2_775F512H_/debug/Source/winc3400/driver/source/nmdrv.o
                0x9d01acb0                nm_get_hif_info
                0x9d01ad50                nm_get_firmware_full_info
                0x9d01aee4                nm_get_ota_firmware_info
                0x9d01b078                nm_drv_init_download_mode
                0x9d01b0f4                nm_drv_init_hold
                0x9d01b1a0                nm_drv_init_start
                0x9d01b2d4                nm_drv_init
                0x9d01b338                nm_drv_deinit
                0x9d01b3b8                nm_cpu_start
 .text          0x9d01b3f0      0x6fc build/ChaletDuinoV2_775F512H_/debug/Source/ChaletduinoV2Board.o
                0x9d01b3f0                InitBoard
 .text          0x9d01baec      0x674 build/ChaletDuinoV2_775F512H_/debug/Source/LoraNetworkInterface.o
                0x9d01baec                ExecuteMasterCommand
                0x9d01c070                SendLoraNetworkCommand
                0x9d01c118                TestTx
 .text          0x9d01c160      0x654 build/ChaletDuinoV2_775F512H_/debug/Source/ina219.o
                0x9d01c368                ina219SetCalibration_13V_10A
                0x9d01c3cc                ina219SetCalibration_32V_2A
                0x9d01c430                ina219SetCalibration_32V_1A
                0x9d01c494                ina219SetCalibration_16V_500mA
                0x9d01c4f8                ina219SetCalibration_16V_200mA
                0x9d01c55c                ina219Init
                0x9d01c5dc                ina219GetShuntVoltage
                0x9d01c620                ina219GetBusVoltage
                0x9d01c674                ina219GetPower
                0x9d01c6b8                ina219GetPower_mW
                0x9d01c714                ina219GetCurrent
                0x9d01c758                ina219GetCurrent_mA
 .text          0x9d01c7b4      0x574 build/ChaletDuinoV2_775F512H_/debug/Source/I2C.o
                0x9d01c7b4                I2CInit
                0x9d01c820                I2CWrite
                0x9d01c9e4                I2CTransmitByte
                0x9d01ca10                I2CRead
                0x9d01cd04                I2CWasLastTransactionOK
 .text          0x9d01cd28      0x51c build/ChaletDuinoV2_775F512H_/debug/Source/main.o
                0x9d01cd28                main
                0x9d01d204                _mon_putc
 .text          0x9d01d244      0x4f0 build/ChaletDuinoV2_775F512H_/debug/Source/winc3400/driver/source/m2m_ota.o
                0x9d01d37c                m2m_ota_init
                0x9d01d3f0                m2m_ota_notif_set_url
                0x9d01d464                m2m_ota_notif_check_for_update
                0x9d01d4bc                m2m_ota_notif_sched
                0x9d01d518                m2m_ota_start_update
                0x9d01d58c                m2m_ota_rollback
                0x9d01d634                m2m_ota_abort
                0x9d01d68c                m2m_ota_switch_firmware

.rodata         0x9d01d734      0x494
 .rodata        0x9d01d734      0x494 build/ChaletDuinoV2_775F512H_/debug/Source/Terminal.o

.text           0x9d01dbc8     0x1108
 .text          0x9d01dbc8      0x45c c:/program files/microchip/xc32/v1.33/bin/bin/../../lib/gcc/pic32mx/4.5.2\libgcc.a(_umoddi3.o)
                0x9d01dbc8                __umoddi3
 .text          0x9d01e024      0x454 build/ChaletDuinoV2_775F512H_/debug/Source/winc3400/driver/source/nmbus.o
                0x9d01e024                nm_bus_iface_init
                0x9d01e070                nm_bus_iface_deinit
                0x9d01e0ac                nm_bus_iface_reconfigure
                0x9d01e0d8                nm_read_reg
                0x9d01e110                nm_read_reg_with_ret
                0x9d01e150                nm_write_reg
                0x9d01e1e0                nm_read_block
                0x9d01e354                nm_write_block
 .text          0x9d01e478      0x44c c:/program files/microchip/xc32/v1.33/bin/bin/../../lib/gcc/pic32mx/4.5.2\libgcc.a(_udivdi3.o)
                0x9d01e478                __udivdi3
 .text          0x9d01e8c4      0x40c build/ChaletDuinoV2_775F512H_/debug/Source/winc3400/common/source/nm_common.o
                0x9d01e8c4                m2m_memcpy
                0x9d01e948                m2m_checksum
                0x9d01e9b8                m2m_memset
                0x9d01ea30                m2m_strlen
                0x9d01ea8c                m2m_strncmp
                0x9d01eb60                m2m_strstr
                0x9d01ec38                m2m_memcmp

.rodata         0x9d01ecd0      0x404
 .rodata        0x9d01ecd0      0x404 build/ChaletDuinoV2_775F512H_/debug/Source/Util.o
                0x9d01ecd4                CRC8_TABLE

.text           0x9d01f0d4     0x1048
 .text          0x9d01f0d4      0x390 build/ChaletDuinoV2_775F512H_/debug/Source/winc3400/bus_wrapper/source/nm_bus_wrapper.o
                0x9d01f0d4                nm_spi_rw
                0x9d01f294                nm_bus_init
                0x9d01f380                nm_bus_ioctl
                0x9d01f414                nm_bus_deinit
                0x9d01f43c                nm_bus_reinit
 .text          0x9d01f464      0x380 build/ChaletDuinoV2_775F512H_/debug/Source/winc3400/driver/source/m2m_periph.o
                0x9d01f674                m2m_periph_init
                0x9d01f69c                m2m_periph_gpio_set_dir
                0x9d01f6f4                m2m_periph_gpio_set_val
                0x9d01f74c                m2m_periph_gpio_get_val
                0x9d01f79c                m2m_periph_pullup_ctrl
 .text          0x9d01f7e4      0x378 build/ChaletDuinoV2_775F512H_/debug/Source/TC77.o
                0x9d01f7e4                TC77Configure
                0x9d01fa34                TC77GetActualTemp
                0x9d01fb38                TC77GetDeviceID
 .text          0x9d01fb5c      0x2f8 build/ChaletDuinoV2_775F512H_/debug/Source/BatteryMonitor.o
                0x9d01fb5c                InitBatteryMonitor
                0x9d01fbcc                BatteryMonitorTick
                0x9d01fd40                GetBatteryVoltage
                0x9d01fda8                GetSolarPanelCurrent
                0x9d01fdcc                GetBatterySOC
                0x9d01fdf0                SendNetworkBatteryData
                0x9d01fe30                GetCurrentModuleOK
 .text          0x9d01fe54      0x2c8 build/ChaletDuinoV2_775F512H_/debug/Source/winc3400/bsp/source/nm_bsp.o
                0x9d01fe54                chip_isr
                0x9d01ff84                nm_bsp_init
                0x9d01ffac                nm_bsp_deinit
                0x9d01ffd0                nm_bsp_reset
                0x9d020058                nm_bsp_sleep
                0x9d020090                nm_bsp_register_isr
                0x9d0200bc                nm_bsp_interrupt_ctrl

.text.scale     0x9d02011c      0x2a0
 .text.scale    0x9d02011c      0x2a0 c:/program files/microchip/xc32/v1.33/bin/bin/../../lib/gcc/pic32mx/4.5.2/../../../../pic32mx/lib\libc.a(doprnt_cdfFnopsuxX.eo)

.text.fpsubadd  0x9d0203bc      0x278
 .text.fpsubadd
                0x9d0203bc      0x278 c:/program files/microchip/xc32/v1.33/bin/bin/../../lib/gcc/pic32mx/4.5.2/../../../../pic32mx/lib\libm.a(fp32subadd.o)
                0x9d0203bc                __subsf3
                0x9d0203bc                fpsub
                0x9d0203c4                __addsf3
                0x9d0203c4                fpadd

.text.malloc    0x9d020634      0x278
 .text.malloc   0x9d020634      0x278 c:/program files/microchip/xc32/v1.33/bin/bin/../../lib/gcc/pic32mx/4.5.2/../../../../pic32mx/lib\libc.a(malloc.o)
                0x9d020634                malloc

.text           0x9d0208ac      0x26c
 .text          0x9d0208ac      0x26c build/ChaletDuinoV2_775F512H_/debug/Source/crc32.o
                0x9d0208ac                crc_32
                0x9d0209a4                update_crc_32

.rodata         0x9d020b18      0x268
 .rodata        0x9d020b18      0x268 build/ChaletDuinoV2_775F512H_/debug/Source/WiFiCtrl.o

.text           0x9d020d80      0x4a8
 .text          0x9d020d80      0x260 build/ChaletDuinoV2_775F512H_/debug/Source/ChaletPowerRelay.o
                0x9d020d80                InitChaletPowerRelay
                0x9d020ddc                ChaletPowerRelayTick
                0x9d020ee0                ChaletPowerRelayKickTimer
                0x9d020f18                ChaletPowerRelayTurnOn
                0x9d020f68                ChaletPowerRelayTurnOff
                0x9d020fb8                GetChaletPowerRelayState
 .text          0x9d020fe0      0x248 build/ChaletDuinoV2_775F512H_/debug/Source/Syslog.o
                0x9d020fe0                InitSyslog
                0x9d021034                SyslogTick
                0x9d0210d0                SyslogNewByte
                0x9d021174                SyslogNewString
                0x9d0211ec                SyslogIsBufferEmpty

.text.fp32div   0x9d021228      0x230
 .text.fp32div  0x9d021228      0x230 c:/program files/microchip/xc32/v1.33/bin/bin/../../lib/gcc/pic32mx/4.5.2/../../../../pic32mx/lib\libm.a(fp32div.o)
                0x9d021228                fpdiv
                0x9d021228                __divsf3

.text.__floatdisf
                0x9d021458      0x220
 .text.__floatdisf
                0x9d021458      0x220 c:/program files/microchip/xc32/v1.33/bin/bin/../../lib/gcc/pic32mx/4.5.2/../../../../pic32mx/lib\libe.a(_floatdisf.o)
                0x9d021458                __floatdisf

.text.fp32mul   0x9d021678      0x1bc
 .text.fp32mul  0x9d021678      0x1bc c:/program files/microchip/xc32/v1.33/bin/bin/../../lib/gcc/pic32mx/4.5.2/../../../../pic32mx/lib\libm.a(fp32mul.o)
                0x9d021678                __mulsf3
                0x9d021678                fpmul

.text           0x9d021834      0x1a0
 .text          0x9d021834      0x1a0 c:/program files/microchip/xc32/v1.33/bin/bin/../../lib/gcc/pic32mx/4.5.2/../../../../pic32mx/lib\libpic32.a(strcpy.o)
                0x9d021834                strcpy

.text.realloc   0x9d0219d4      0x194
 .text.realloc  0x9d0219d4      0x194 c:/program files/microchip/xc32/v1.33/bin/bin/../../lib/gcc/pic32mx/4.5.2/../../../../pic32mx/lib\libc.a(malloc.o)
                0x9d0219d4                realloc

.text._sbrk_init
                0x9d021b68      0x194
 .text._sbrk_init
                0x9d021b68      0x194 c:/program files/microchip/xc32/v1.33/bin/bin/../../lib/gcc/pic32mx/4.5.2/../../../../pic32mx/lib\libpic32.a(sbrk.o)
                0x9d021b68                _sbrk_init

.text._filbuf   0x9d021cfc      0x188
 .text._filbuf  0x9d021cfc      0x188 c:/program files/microchip/xc32/v1.33/bin/bin/../../lib/gcc/pic32mx/4.5.2/../../../../pic32mx/lib\libc.a(filbuf.o)
                0x9d021cfc                _filbuf

.text.read      0x9d021e84      0x174
 .text.read     0x9d021e84      0x174 c:/program files/microchip/xc32/v1.33/bin/bin/../../lib/gcc/pic32mx/4.5.2/../../../../pic32mx/lib\libpic32.a(read.o)
                0x9d021e84                read

.text           0x9d021ff8      0x2d0
 .text          0x9d021ff8      0x168 c:/program files/microchip/xc32/v1.33/bin/bin/../../lib/gcc/pic32mx/4.5.2/../../../../pic32mx/lib\libpic32.a(memcpy.o)
                0x9d021ff8                memcpy
 .text          0x9d022160      0x168 c:/program files/microchip/xc32/v1.33/bin/bin/../../lib/gcc/pic32mx/4.5.2/../../../../pic32mx/lib\libpic32.a(strlen.o)
                0x9d022160                strlen

.text.fputc     0x9d0222c8      0x15c
 .text.fputc    0x9d0222c8      0x15c c:/program files/microchip/xc32/v1.33/bin/bin/../../lib/gcc/pic32mx/4.5.2/../../../../pic32mx/lib\libc.a(_fputc_simple.o)
                0x9d0222c8                fputc

.text._flsbuf   0x9d022424      0x12c
 .text._flsbuf  0x9d022424      0x12c c:/program files/microchip/xc32/v1.33/bin/bin/../../lib/gcc/pic32mx/4.5.2/../../../../pic32mx/lib\libc.a(_flsbuf_simple.o)
                0x9d022424                _flsbuf

.text           0x9d022550      0x11c
 .text          0x9d022550      0x11c build/ChaletDuinoV2_775F512H_/debug/Source/TemperatureSensor.o
                0x9d022550                InitTempSensor
                0x9d022594                TempSensorCheckAndConfigure
                0x9d0225f0                TempSensorGetTemp
                0x9d022614                TickTempSensor

.text.fgetc     0x9d02266c      0x108
 .text.fgetc    0x9d02266c      0x108 c:/program files/microchip/xc32/v1.33/bin/bin/../../lib/gcc/pic32mx/4.5.2/../../../../pic32mx/lib\libc.a(fgetc.o)
                0x9d02266c                fgetc

.rodata         0x9d022774      0x204
 .rodata        0x9d022774      0x104 c:/program files/microchip/xc32/v1.33/bin/bin/../../lib/gcc/pic32mx/4.5.2/../../../../pic32mx/lib\libc.a(ctype.o)
                0x9d022774                _ctype
 .rodata        0x9d022878      0x100 build/ChaletDuinoV2_775F512H_/debug/Source/winc3400/driver/source/nmspi.o

.text.setvbuf   0x9d022978       0xfc
 .text.setvbuf  0x9d022978       0xfc c:/program files/microchip/xc32/v1.33/bin/bin/../../lib/gcc/pic32mx/4.5.2/../../../../pic32mx/lib\libc.a(setbuf.o)
                0x9d022978                setvbuf

.rodata         0x9d022a78       0xe0
 .rodata        0x9d022a78       0xe0 c:/program files/microchip/xc32/v1.33/bin/bin/../../lib/gcc/pic32mx/4.5.2/../../../../pic32mx/lib\libc.a(doprnt_cdfFnopsuxX.eo)

.text.general_exception
                0x9d022b58       0xdc
 .text.general_exception
                0x9d022b58       0xdc c:/program files/microchip/xc32/v1.33/bin/bin/../../lib/gcc/pic32mx/4.5.2/../../../../pic32mx/lib\libpic32.a(general-exception.o)
                0x9d022b58                _general_exception_context

.text           0x9d022c34      0x1ac
 .text          0x9d022c34       0xd8 build/ChaletDuinoV2_775F512H_/debug/Source/Watchdog.o
                0x9d022c34                InitWatchdog
                0x9d022c88                EnableWatchdog
                0x9d022cb4                DisableWatchdog
                0x9d022ce0                KickWatchdog
 .text          0x9d022d0c       0xd4 c:/program files/microchip/xc32/v1.33/bin/bin/../../lib/gcc/pic32mx/4.5.2\libgcc.a(_floatundisf.o)
                0x9d022d0c                __floatundisf

.rodata         0x9d022de0       0xc8
 .rodata        0x9d022de0       0xc8 build/ChaletDuinoV2_775F512H_/debug/Source/SPI_Flash.o

.text._sbrk     0x9d022ea8       0xc4
 .text._sbrk    0x9d022ea8       0xc4 c:/program files/microchip/xc32/v1.33/bin/bin/../../lib/gcc/pic32mx/4.5.2/../../../../pic32mx/lib\libpic32.a(sbrk.o)
                0x9d022ea8                _sbrk

.text           0x9d022f6c       0xa8
 .text          0x9d022f6c       0xa8 c:/program files/microchip/xc32/v1.33/bin/bin/../../lib/gcc/pic32mx/4.5.2/../../../../pic32mx/lib\libpic32.a(memset.o)
                0x9d022f6c                memset

.text.atoi      0x9d023014       0xa8
 .text.atoi     0x9d023014       0xa8 c:/program files/microchip/xc32/v1.33/bin/bin/../../lib/gcc/pic32mx/4.5.2/../../../../pic32mx/lib\libc.a(atoi.o)
                0x9d023014                atoi

.text.range     0x9d0230bc       0xa0
 .text.range    0x9d0230bc       0xa0 c:/program files/microchip/xc32/v1.33/bin/bin/../../lib/gcc/pic32mx/4.5.2/../../../../pic32mx/lib\libc.a(doscan_s.eo)

.text.fpcmp     0x9d02315c       0x9c
 .text.fpcmp    0x9d02315c       0x9c c:/program files/microchip/xc32/v1.33/bin/bin/../../lib/gcc/pic32mx/4.5.2/../../../../pic32mx/lib\libm.a(fpcmp.o)
                0x9d02315c                __eqsf2
                0x9d02315c                __lesf2
                0x9d02315c                __gtsf2
                0x9d02315c                __nesf2
                0x9d02315c                fpcmp
                0x9d02315c                __gesf2
                0x9d02315c                __ltsf2

.text.fflush    0x9d0231f8       0x94
 .text.fflush   0x9d0231f8       0x94 c:/program files/microchip/xc32/v1.33/bin/bin/../../lib/gcc/pic32mx/4.5.2/../../../../pic32mx/lib\libc.a(fflush.o)
                0x9d0231f8                fflush

.text.write     0x9d02328c       0x94
 .text.write    0x9d02328c       0x94 c:/program files/microchip/xc32/v1.33/bin/bin/../../lib/gcc/pic32mx/4.5.2/../../../../pic32mx/lib\libpic32.a(write.o)
                0x9d02328c                write

.text.libm      0x9d023320       0x88
 .text.libm     0x9d023320       0x88 c:/program files/microchip/xc32/v1.33/bin/bin/../../lib/gcc/pic32mx/4.5.2/../../../../pic32mx/lib\libm.a(fpfrexp.o)
                0x9d023320                frexpf
                0x9d023320                fpfrexp

.text           0x9d0233a8       0x80
 .text          0x9d0233a8       0x80 build/ChaletDuinoV2_775F512H_/debug/Source/winc3400/winc_init.o
                0x9d0233a8                wifi_init

.text.fptoul    0x9d023428       0x7c
 .text.fptoul   0x9d023428       0x7c c:/program files/microchip/xc32/v1.33/bin/bin/../../lib/gcc/pic32mx/4.5.2/../../../../pic32mx/lib\libm.a(fptoul.o)
                0x9d023428                fptoul
                0x9d023428                fptoui
                0x9d023428                __fixunssfsi

.text.SoftReset
                0x9d0234a4       0x78
 .text.SoftReset
                0x9d0234a4       0x78 c:/program files/microchip/xc32/v1.33/bin/bin/../../lib/gcc/pic32mx/4.5.2/../../../../pic32mx/lib\libmchp_peripheral_32MX795F512H.a(soft_reset_lib.o)
                0x9d0234a4                SoftReset

.text.fputs     0x9d02351c       0x78
 .text.fputs    0x9d02351c       0x78 c:/program files/microchip/xc32/v1.33/bin/bin/../../lib/gcc/pic32mx/4.5.2/../../../../pic32mx/lib\libc.a(puts.o)
                0x9d02351c                fputs

.text.strncmp   0x9d023594       0x78
 .text.strncmp  0x9d023594       0x78 c:/program files/microchip/xc32/v1.33/bin/bin/../../lib/gcc/pic32mx/4.5.2/../../../../pic32mx/lib\libc.a(strncmp.o)
                0x9d023594                strncmp

.text.ungetc    0x9d02360c       0x74
 .text.ungetc   0x9d02360c       0x74 c:/program files/microchip/xc32/v1.33/bin/bin/../../lib/gcc/pic32mx/4.5.2/../../../../pic32mx/lib\libc.a(ungetc.o)
                0x9d02360c                ungetc

.text           0x9d023680       0xd8
 .text          0x9d023680       0x70 build/ChaletDuinoV2_775F512H_/debug/Source/SPI.o
                0x9d023680                SPITransaction
 .text          0x9d0236f0       0x68 build/ChaletDuinoV2_775F512H_/debug/Source/HarakiriRelay.o
                0x9d0236f0                InitHarakiriRelay
                0x9d023720                HarakiriRelayTurnOff

.text._sprintf_cdfFnopuxX
                0x9d023758       0x68
 .text._sprintf_cdfFnopuxX
                0x9d023758       0x68 c:/program files/microchip/xc32/v1.33/bin/bin/../../lib/gcc/pic32mx/4.5.2/../../../../pic32mx/lib\libc.a(sprintf_cdfFnopuxX.eo)
                0x9d023758                _sprintf_cdnopuxX
                0x9d023758                _sprintf_cdfFnopuxX

.rodata         0x9d0237c0       0x68
 .rodata        0x9d0237c0       0x68 c:/program files/microchip/xc32/v1.33/bin/bin/../../lib/gcc/pic32mx/4.5.2/../../../../pic32mx/lib\libc.a(powersf.o)
                0x9d0237c0                _powers_f
                0x9d0237f4                _npowers_f

.text.sitofp    0x9d023828       0x60
 .text.sitofp   0x9d023828       0x60 c:/program files/microchip/xc32/v1.33/bin/bin/../../lib/gcc/pic32mx/4.5.2/../../../../pic32mx/lib\libm.a(sitofp.o)
                0x9d023828                sitofp
                0x9d023828                litofp
                0x9d023828                __floatsisf

.text.wspace    0x9d023888       0x60
 .text.wspace   0x9d023888       0x60 c:/program files/microchip/xc32/v1.33/bin/bin/../../lib/gcc/pic32mx/4.5.2/../../../../pic32mx/lib\libc.a(doscan_s.eo)

.text           0x9d0238e8       0x58
 .text          0x9d0238e8       0x58 build/ChaletDuinoV2_775F512H_/debug/Source/exceptions.o
                0x9d0238e8                _general_exception_handler

.text._sscanf_s
                0x9d023940       0x54
 .text._sscanf_s
                0x9d023940       0x54 c:/program files/microchip/xc32/v1.33/bin/bin/../../lib/gcc/pic32mx/4.5.2/../../../../pic32mx/lib\libc.a(sscanf_s.eo)
                0x9d023940                _sscanf_s
                0x9d023940                _sscanf_0

.text._bufallo  0x9d023994       0x54
 .text._bufallo
                0x9d023994       0x54 c:/program files/microchip/xc32/v1.33/bin/bin/../../lib/gcc/pic32mx/4.5.2/../../../../pic32mx/lib\libc.a(buf.o)
                0x9d023994                _bufallo

.text.sbrk      0x9d0239e8       0x50
 .text.sbrk     0x9d0239e8       0x50 c:/program files/microchip/xc32/v1.33/bin/bin/../../lib/gcc/pic32mx/4.5.2/../../../../pic32mx/lib\libpic32.a(sbrk.o)
                0x9d0239e8                sbrk

.text.main_entry
                0x9d023a38       0x4c
 .text.main_entry
                0x9d023a38       0x4c c:/program files/microchip/xc32/v1.33/bin/bin/../../lib/gcc/pic32mx/4.5.2/../../../../pic32mx/lib/./proc/32MX795F512H/crt0_mips32r2.o
                0x9d023a64                __crt0_exit

.text           0x9d023a84       0x4c
 .text          0x9d023a84       0x4c c:/program files/microchip/xc32/v1.33/bin/bin/../../lib/gcc/pic32mx/4.5.2\libgcc.a(floatunsisf.o)
                0x9d023a84                __floatunsisf

.text._bootstrap_exception_handler
                0x9d023ad0       0x48
 .text._bootstrap_exception_handler
                0x9d023ad0       0x48 c:/program files/microchip/xc32/v1.33/bin/bin/../../lib/gcc/pic32mx/4.5.2/../../../../pic32mx/lib\libpic32.a(default-bootstrap-exception-handler.o)
                0x9d023ad0                _bootstrap_exception_handler

.text           0x9d023b18       0x44
 .text          0x9d023b18       0x44 c:/program files/microchip/xc32/v1.33/bin/bin/../../lib/gcc/pic32mx/4.5.2/../../../../pic32mx/lib\pic32_software_reset.o
                0x9d023b18                __pic32_software_reset

.text.puts      0x9d023b5c       0x44
 .text.puts     0x9d023b5c       0x44 c:/program files/microchip/xc32/v1.33/bin/bin/../../lib/gcc/pic32mx/4.5.2/../../../../pic32mx/lib\libc.a(puts.o)
                0x9d023b5c                puts

.text._printf_cdfFnopsuxX
                0x9d023ba0       0x40
 .text._printf_cdfFnopsuxX
                0x9d023ba0       0x40 c:/program files/microchip/xc32/v1.33/bin/bin/../../lib/gcc/pic32mx/4.5.2/../../../../pic32mx/lib\libc.a(printf_cdfFnopsuxX.eo)
                0x9d023ba0                _printf_cdnopsuxX
                0x9d023ba0                _printf_cdnopuxX
                0x9d023ba0                _printf_cdfFnopsuxX
                0x9d023ba0                _printf_fF

.vector_default
                0x9d023be0       0x38
 .vector_default
                0x9d023be0       0x38 c:/program files/microchip/xc32/v1.33/bin/bin/../../lib/gcc/pic32mx/4.5.2/../../../../pic32mx/lib\libpic32.a(defaultinterrupt.o)
                0x9d023be0                _DefaultInterrupt

.rodata         0x9d023c18       0x30
 .rodata        0x9d023c18       0x30 build/ChaletDuinoV2_775F512H_/debug/Source/main.o

.text.INTConfigureSystem
                0x9d023c48       0x30
 .text.INTConfigureSystem
                0x9d023c48       0x30 c:/program files/microchip/xc32/v1.33/bin/bin/../../lib/gcc/pic32mx/4.5.2/../../../../pic32mx/lib\libmchp_peripheral_32MX795F512H.a(int_configure_system_lib.o)
                0x9d023c48                INTConfigureSystem

.text.free      0x9d023c78       0x30
 .text.free     0x9d023c78       0x30 c:/program files/microchip/xc32/v1.33/bin/bin/../../lib/gcc/pic32mx/4.5.2/../../../../pic32mx/lib\libc.a(malloc.o)
                0x9d023c78                free

.rodata         0x9d023ca8       0x2c
 .rodata        0x9d023ca8       0x2c build/ChaletDuinoV2_775F512H_/debug/Source/BatteryMonitor.o

.text._stub_sbd_memlayout
                0x9d023cd4       0x2c
 .text._stub_sbd_memlayout
                0x9d023cd4       0x2c c:/program files/microchip/xc32/v1.33/bin/bin/../../lib/gcc/pic32mx/4.5.2/../../../../pic32mx/lib\libpic32.a(sbrk.o)
                0x9d023cd4                _sbd_memlayout
                0x9d023cd4                _stub_sbd_memlayout

.rodata         0x9d023d00       0x28
 .rodata        0x9d023d00       0x28 build/ChaletDuinoV2_775F512H_/debug/Source/ChaletPowerRelay.o

.text.tolower   0x9d023d28       0x24
 .text.tolower  0x9d023d28       0x24 c:/program files/microchip/xc32/v1.33/bin/bin/../../lib/gcc/pic32mx/4.5.2/../../../../pic32mx/lib\libc.a(ctypef.o)
                0x9d023d28                tolower

.text.toupper   0x9d023d4c       0x24
 .text.toupper  0x9d023d4c       0x24 c:/program files/microchip/xc32/v1.33/bin/bin/../../lib/gcc/pic32mx/4.5.2/../../../../pic32mx/lib\libc.a(ctypef.o)
                0x9d023d4c                toupper

.text           0x9d023d70       0x20
 .text          0x9d023d70       0x20 build/ChaletDuinoV2_775F512H_/debug/Source/DigitalIO.o
                0x9d023d70                InitDigitalIO

.rodata         0x9d023d90       0x1c
 .rodata        0x9d023d90       0x1c build/ChaletDuinoV2_775F512H_/debug/Source/Uart.o

.text.INTRestoreInterrupts
                0x9d023dac       0x1c
 .text.INTRestoreInterrupts
                0x9d023dac       0x1c c:/program files/microchip/xc32/v1.33/bin/bin/../../lib/gcc/pic32mx/4.5.2/../../../../pic32mx/lib\libmchp_peripheral_32MX795F512H.a(int_restore_interrupts_lib.o)
                0x9d023dac                INTRestoreInterrupts

.text.setbuf    0x9d023dc8       0x1c
 .text.setbuf   0x9d023dc8       0x1c c:/program files/microchip/xc32/v1.33/bin/bin/../../lib/gcc/pic32mx/4.5.2/../../../../pic32mx/lib\libc.a(setbuf.o)
                0x9d023dc8                setbuf

.rodata         0x9d023de4       0x18
 .rodata        0x9d023de4       0x18 build/ChaletDuinoV2_775F512H_/debug/Source/Watchdog.o

.text.CheKseg0CacheOff
                0x9d023dfc       0x18
 .text.CheKseg0CacheOff
                0x9d023dfc       0x18 c:/program files/microchip/xc32/v1.33/bin/bin/../../lib/gcc/pic32mx/4.5.2/../../../../pic32mx/lib\libmchp_peripheral_32MX795F512H.a(pcache.o)
                0x9d023dfc                CheKseg0CacheOff

.text.CheKseg0CacheOn
                0x9d023e14       0x18
 .text.CheKseg0CacheOn
                0x9d023e14       0x18 c:/program files/microchip/xc32/v1.33/bin/bin/../../lib/gcc/pic32mx/4.5.2/../../../../pic32mx/lib\libmchp_peripheral_32MX795F512H.a(pcache.o)
                0x9d023e14                CheKseg0CacheOn

.text           0x9d023e2c       0x18
 .text          0x9d023e2c       0x18 c:/program files/microchip/xc32/v1.33/bin/bin/../../lib/gcc/pic32mx/4.5.2/../../../../pic32mx/lib\libpic32.a(default-nmi-handler.o)
                0x9d023e2c                _nmi_handler

.text.isalnum   0x9d023e44       0x18
 .text.isalnum  0x9d023e44       0x18 c:/program files/microchip/xc32/v1.33/bin/bin/../../lib/gcc/pic32mx/4.5.2/../../../../pic32mx/lib\libc.a(ctypef.o)
                0x9d023e44                isalnum

.text.isalpha   0x9d023e5c       0x18
 .text.isalpha  0x9d023e5c       0x18 c:/program files/microchip/xc32/v1.33/bin/bin/../../lib/gcc/pic32mx/4.5.2/../../../../pic32mx/lib\libc.a(ctypef.o)
                0x9d023e5c                isalpha

.text.iscntrl   0x9d023e74       0x18
 .text.iscntrl  0x9d023e74       0x18 c:/program files/microchip/xc32/v1.33/bin/bin/../../lib/gcc/pic32mx/4.5.2/../../../../pic32mx/lib\libc.a(ctypef.o)
                0x9d023e74                iscntrl

.text.isdigit   0x9d023e8c       0x18
 .text.isdigit  0x9d023e8c       0x18 c:/program files/microchip/xc32/v1.33/bin/bin/../../lib/gcc/pic32mx/4.5.2/../../../../pic32mx/lib\libc.a(ctypef.o)
                0x9d023e8c                isdigit

.text.isgraph   0x9d023ea4       0x18
 .text.isgraph  0x9d023ea4       0x18 c:/program files/microchip/xc32/v1.33/bin/bin/../../lib/gcc/pic32mx/4.5.2/../../../../pic32mx/lib\libc.a(ctypef.o)
                0x9d023ea4                isgraph

.text.islower   0x9d023ebc       0x18
 .text.islower  0x9d023ebc       0x18 c:/program files/microchip/xc32/v1.33/bin/bin/../../lib/gcc/pic32mx/4.5.2/../../../../pic32mx/lib\libc.a(ctypef.o)
                0x9d023ebc                islower

.text.isprint   0x9d023ed4       0x18
 .text.isprint  0x9d023ed4       0x18 c:/program files/microchip/xc32/v1.33/bin/bin/../../lib/gcc/pic32mx/4.5.2/../../../../pic32mx/lib\libc.a(ctypef.o)
                0x9d023ed4                isprint

.text.ispunct   0x9d023eec       0x18
 .text.ispunct  0x9d023eec       0x18 c:/program files/microchip/xc32/v1.33/bin/bin/../../lib/gcc/pic32mx/4.5.2/../../../../pic32mx/lib\libc.a(ctypef.o)
                0x9d023eec                ispunct

.text.isspace   0x9d023f04       0x18
 .text.isspace  0x9d023f04       0x18 c:/program files/microchip/xc32/v1.33/bin/bin/../../lib/gcc/pic32mx/4.5.2/../../../../pic32mx/lib\libc.a(ctypef.o)
                0x9d023f04                isspace

.text.isupper   0x9d023f1c       0x18
 .text.isupper  0x9d023f1c       0x18 c:/program files/microchip/xc32/v1.33/bin/bin/../../lib/gcc/pic32mx/4.5.2/../../../../pic32mx/lib\libc.a(ctypef.o)
                0x9d023f1c                isupper

.text.isxdigit  0x9d023f34       0x18
 .text.isxdigit
                0x9d023f34       0x18 c:/program files/microchip/xc32/v1.33/bin/bin/../../lib/gcc/pic32mx/4.5.2/../../../../pic32mx/lib\libc.a(ctypef.o)
                0x9d023f34                isxdigit

.text._buffree  0x9d023f4c       0x14
 .text._buffree
                0x9d023f4c       0x14 c:/program files/microchip/xc32/v1.33/bin/bin/../../lib/gcc/pic32mx/4.5.2/../../../../pic32mx/lib\libc.a(buf.o)
                0x9d023f4c                _buffree

.text.__exception_handler_break
                0x9d023f60        0xc
 .text.__exception_handler_break
                0x9d023f60        0xc c:/program files/microchip/xc32/v1.33/bin/bin/../../lib/gcc/pic32mx/4.5.2/../../../../pic32mx/lib\software-debug-break.o
                0x9d023f60                __exception_handler_break

.rodata         0x9d023f6c       0x1c
 .rodata        0x9d023f6c        0xc build/ChaletDuinoV2_775F512H_/debug/Source/InternalUart.o
 .rodata        0x9d023f78        0x8 build/ChaletDuinoV2_775F512H_/debug/Source/Syslog.o
 .rodata        0x9d023f80        0x8 build/ChaletDuinoV2_775F512H_/debug/Source/BootloaderProtocol.o

.text.INTEnableInterrupts
                0x9d023f88        0x8
 .text.INTEnableInterrupts
                0x9d023f88        0x8 c:/program files/microchip/xc32/v1.33/bin/bin/../../lib/gcc/pic32mx/4.5.2/../../../../pic32mx/lib\libmchp_peripheral_32MX795F512H.a(int_enable_interrupts_lib.o)
                0x9d023f88                INTEnableInterrupts

.text.INTDisableInterrupts
                0x9d023f90        0x8
 .text.INTDisableInterrupts
                0x9d023f90        0x8 c:/program files/microchip/xc32/v1.33/bin/bin/../../lib/gcc/pic32mx/4.5.2/../../../../pic32mx/lib\libmchp_peripheral_32MX795F512H.a(int_disable_interrupts_lib.o)
                0x9d023f90                INTDisableInterrupts

.text._on_reset
                0x9d023f98        0x8
 .text._on_reset
                0x9d023f98        0x8 c:/program files/microchip/xc32/v1.33/bin/bin/../../lib/gcc/pic32mx/4.5.2/../../../../pic32mx/lib\libpic32.a(default-on-reset.o)
                0x9d023f98                _on_reset

.text._on_bootstrap
                0x9d023fa0        0x8
 .text._on_bootstrap
                0x9d023fa0        0x8 c:/program files/microchip/xc32/v1.33/bin/bin/../../lib/gcc/pic32mx/4.5.2/../../../../pic32mx/lib\libpic32.a(default-on-bootstrap.o)
                0x9d023fa0                _on_bootstrap

.text.isascii   0x9d023fa8        0x8
 .text.isascii  0x9d023fa8        0x8 c:/program files/microchip/xc32/v1.33/bin/bin/../../lib/gcc/pic32mx/4.5.2/../../../../pic32mx/lib\libc.a(ctypef.o)
                0x9d023fa8                isascii

.text.toascii   0x9d023fb0        0x8
 .text.toascii  0x9d023fb0        0x8 c:/program files/microchip/xc32/v1.33/bin/bin/../../lib/gcc/pic32mx/4.5.2/../../../../pic32mx/lib\libc.a(ctypef.o)
                0x9d023fb0                toascii

.text._tolower  0x9d023fb8        0x8
 .text._tolower
                0x9d023fb8        0x8 c:/program files/microchip/xc32/v1.33/bin/bin/../../lib/gcc/pic32mx/4.5.2/../../../../pic32mx/lib\libc.a(ctypef.o)
                0x9d023fb8                _tolower

.text._toupper  0x9d023fc0        0x8
 .text._toupper
                0x9d023fc0        0x8 c:/program files/microchip/xc32/v1.33/bin/bin/../../lib/gcc/pic32mx/4.5.2/../../../../pic32mx/lib\libc.a(ctypef.o)
                0x9d023fc0                _toupper

.text.getpagesize
                0x9d023fc8        0x8
 .text.getpagesize
                0x9d023fc8        0x8 c:/program files/microchip/xc32/v1.33/bin/bin/../../lib/gcc/pic32mx/4.5.2/../../../../pic32mx/lib\libpic32.a(sbrk.o)
                0x9d023fc8                getpagesize

.rodata         0x9d023fd0        0x8
 .rodata        0x9d023fd0        0x8 c:/program files/microchip/xc32/v1.33/bin/bin/../../lib/gcc/pic32mx/4.5.2\libgcc.a(_floatundisf.o)

.rodata         0x9d022a74        0x4
 .rodata        0x9d022a74        0x4 build/ChaletDuinoV2_775F512H_/debug/Source/TemperatureSensor.o

.rodata         0x9d023fd8        0x4
 .rodata        0x9d023fd8        0x4 build/ChaletDuinoV2_775F512H_/debug/Source/TC77.o

.text%z320      0x00000000        0x0
 .text          0x00000000        0x0 c:/program files/microchip/xc32/v1.33/bin/bin/../../lib/gcc/pic32mx/4.5.2/../../../../pic32mx/lib\libe.a(_floatdisf.o)

.text%z321      0x00000000        0x0
 .text          0x00000000        0x0 c:/program files/microchip/xc32/v1.33/bin/bin/../../lib/gcc/pic32mx/4.5.2/../../../../pic32mx/lib\libm.a(fptoul.o)

.text%z322      0x00000000        0x0
 .text          0x00000000        0x0 c:/program files/microchip/xc32/v1.33/bin/bin/../../lib/gcc/pic32mx/4.5.2/../../../../pic32mx/lib\libm.a(fpfrexp.o)

.text%z323      0x00000000        0x0
 .text          0x00000000        0x0 c:/program files/microchip/xc32/v1.33/bin/bin/../../lib/gcc/pic32mx/4.5.2/../../../../pic32mx/lib\libm.a(fpcmp.o)

.text%z324      0x00000000        0x0
 .text          0x00000000        0x0 c:/program files/microchip/xc32/v1.33/bin/bin/../../lib/gcc/pic32mx/4.5.2/../../../../pic32mx/lib\libpic32.a(xc32_uart.o)

.text%z325      0x00000000        0x0
 .text          0x00000000        0x0 c:/program files/microchip/xc32/v1.33/bin/bin/../../lib/gcc/pic32mx/4.5.2/../../../../pic32mx/lib\libpic32.a(write.o)

.text%z326      0x00000000        0x0
 .text          0x00000000        0x0 c:/program files/microchip/xc32/v1.33/bin/bin/../../lib/gcc/pic32mx/4.5.2/../../../../pic32mx/lib\libpic32.a(read.o)

.text%z327      0x00000000        0x0
 .text          0x00000000        0x0 c:/program files/microchip/xc32/v1.33/bin/bin/../../lib/gcc/pic32mx/4.5.2/../../../../pic32mx/lib\libpic32.a(sbrk.o)

.text%z328      0x00000000        0x0
 .text          0x00000000        0x0 c:/program files/microchip/xc32/v1.33/bin/bin/../../lib/gcc/pic32mx/4.5.2/../../../../pic32mx/lib\libc.a(filbuf.o)

.text%z329      0x00000000        0x0
 .text          0x00000000        0x0 c:/program files/microchip/xc32/v1.33/bin/bin/../../lib/gcc/pic32mx/4.5.2/../../../../pic32mx/lib\libc.a(ungetc.o)

.text%z330      0x00000000        0x0
 .text          0x00000000        0x0 c:/program files/microchip/xc32/v1.33/bin/bin/../../lib/gcc/pic32mx/4.5.2/../../../../pic32mx/lib\libc.a(powersf.o)

.text%z331      0x00000000        0x0
 .text          0x00000000        0x0 c:/program files/microchip/xc32/v1.33/bin/bin/../../lib/gcc/pic32mx/4.5.2/../../../../pic32mx/lib\libc.a(ctypef.o)

.text%z332      0x00000000        0x0
 .text          0x00000000        0x0 c:/program files/microchip/xc32/v1.33/bin/bin/../../lib/gcc/pic32mx/4.5.2/../../../../pic32mx/lib\libc.a(ctype.o)

.text%z333      0x00000000        0x0
 .text          0x00000000        0x0 c:/program files/microchip/xc32/v1.33/bin/bin/../../lib/gcc/pic32mx/4.5.2/../../../../pic32mx/lib\libc.a(atoi.o)

.text%z334      0x00000000        0x0
 .text          0x00000000        0x0 c:/program files/microchip/xc32/v1.33/bin/bin/../../lib/gcc/pic32mx/4.5.2/../../../../pic32mx/lib\libc.a(fgetc.o)

.text%z335      0x00000000        0x0
 .text          0x00000000        0x0 c:/program files/microchip/xc32/v1.33/bin/bin/../../lib/gcc/pic32mx/4.5.2/../../../../pic32mx/lib\libc.a(_flsbuf_simple.o)

.text%z336      0x00000000        0x0
 .text          0x00000000        0x0 c:/program files/microchip/xc32/v1.33/bin/bin/../../lib/gcc/pic32mx/4.5.2/../../../../pic32mx/lib\libc.a(doscan_s.eo)

.text%z337      0x00000000        0x0
 .text          0x00000000        0x0 c:/program files/microchip/xc32/v1.33/bin/bin/../../lib/gcc/pic32mx/4.5.2/../../../../pic32mx/lib\libc.a(doprnt_cdfFnopsuxX.eo)

.text%z338      0x00000000        0x0
 .text          0x00000000        0x0 c:/program files/microchip/xc32/v1.33/bin/bin/../../lib/gcc/pic32mx/4.5.2/../../../../pic32mx/lib\libc.a(errno.o)

.text%z339      0x00000000        0x0
 .text          0x00000000        0x0 c:/program files/microchip/xc32/v1.33/bin/bin/../../lib/gcc/pic32mx/4.5.2/../../../../pic32mx/lib\libc.a(buf.o)

.text%z340      0x00000000        0x0
 .text          0x00000000        0x0 c:/program files/microchip/xc32/v1.33/bin/bin/../../lib/gcc/pic32mx/4.5.2/../../../../pic32mx/lib\libc.a(_fputc_simple.o)

.text%z341      0x00000000        0x0
 .text          0x00000000        0x0 c:/program files/microchip/xc32/v1.33/bin/bin/../../lib/gcc/pic32mx/4.5.2/../../../../pic32mx/lib\libc.a(sscanf_s.eo)

.text%z342      0x00000000        0x0
 .text          0x00000000        0x0 c:/program files/microchip/xc32/v1.33/bin/bin/../../lib/gcc/pic32mx/4.5.2/../../../../pic32mx/lib\libc.a(sprintf_cdfFnopuxX.eo)

.text%z343      0x00000000        0x0
 .text          0x00000000        0x0 c:/program files/microchip/xc32/v1.33/bin/bin/../../lib/gcc/pic32mx/4.5.2/../../../../pic32mx/lib\libc.a(printf_cdfFnopsuxX.eo)

.text%z344      0x00000000        0x0
 .text          0x00000000        0x0 c:/program files/microchip/xc32/v1.33/bin/bin/../../lib/gcc/pic32mx/4.5.2/../../../../pic32mx/lib\libc.a(strncmp.o)

.text%z345      0x00000000        0x0
 .text          0x00000000        0x0 c:/program files/microchip/xc32/v1.33/bin/bin/../../lib/gcc/pic32mx/4.5.2/../../../../pic32mx/lib\libc.a(setbuf.o)

.text%z346      0x00000000        0x0
 .text          0x00000000        0x0 c:/program files/microchip/xc32/v1.33/bin/bin/../../lib/gcc/pic32mx/4.5.2/../../../../pic32mx/lib\libc.a(puts.o)

.text%z347      0x00000000        0x0
 .text          0x00000000        0x0 c:/program files/microchip/xc32/v1.33/bin/bin/../../lib/gcc/pic32mx/4.5.2/../../../../pic32mx/lib\libc.a(malloc.o)

.text%z348      0x00000000        0x0
 .text          0x00000000        0x0 c:/program files/microchip/xc32/v1.33/bin/bin/../../lib/gcc/pic32mx/4.5.2/../../../../pic32mx/lib\libc.a(fflush.o)

.text%z349      0x00000000        0x0
 .text          0x00000000        0x0 c:/program files/microchip/xc32/v1.33/bin/bin/../../lib/gcc/pic32mx/4.5.2/../../../../pic32mx/lib\libc.a(_iob.o)

.text%z350      0x00000000        0x0
 .text          0x00000000        0x0 c:/program files/microchip/xc32/v1.33/bin/bin/../../lib/gcc/pic32mx/4.5.2/../../../../pic32mx/lib\libm.a(sitofp.o)

.text%z351      0x00000000        0x0
 .text          0x00000000        0x0 c:/program files/microchip/xc32/v1.33/bin/bin/../../lib/gcc/pic32mx/4.5.2/../../../../pic32mx/lib\libm.a(fp32subadd.o)

.text%z352      0x00000000        0x0
 .text          0x00000000        0x0 c:/program files/microchip/xc32/v1.33/bin/bin/../../lib/gcc/pic32mx/4.5.2/../../../../pic32mx/lib\libm.a(fp32mul.o)

.text%z353      0x00000000        0x0
 .text          0x00000000        0x0 c:/program files/microchip/xc32/v1.33/bin/bin/../../lib/gcc/pic32mx/4.5.2/../../../../pic32mx/lib\libm.a(fp32div.o)

.text%z354      0x00000000        0x0
 .text          0x00000000        0x0 c:/program files/microchip/xc32/v1.33/bin/bin/../../lib/gcc/pic32mx/4.5.2/../../../../pic32mx/lib\libpic32.a(defaultinterrupt.o)

.text%z355      0x00000000        0x0
 .text          0x00000000        0x0 c:/program files/microchip/xc32/v1.33/bin/bin/../../lib/gcc/pic32mx/4.5.2/../../../../pic32mx/lib\libpic32.a(vector63.o)

.text%z356      0x00000000        0x0
 .text          0x00000000        0x0 c:/program files/microchip/xc32/v1.33/bin/bin/../../lib/gcc/pic32mx/4.5.2/../../../../pic32mx/lib\libpic32.a(vector62.o)

.text%z357      0x00000000        0x0
 .text          0x00000000        0x0 c:/program files/microchip/xc32/v1.33/bin/bin/../../lib/gcc/pic32mx/4.5.2/../../../../pic32mx/lib\libpic32.a(vector61.o)

.text%z358      0x00000000        0x0
 .text          0x00000000        0x0 c:/program files/microchip/xc32/v1.33/bin/bin/../../lib/gcc/pic32mx/4.5.2/../../../../pic32mx/lib\libpic32.a(vector60.o)

.text%z359      0x00000000        0x0
 .text          0x00000000        0x0 c:/program files/microchip/xc32/v1.33/bin/bin/../../lib/gcc/pic32mx/4.5.2/../../../../pic32mx/lib\libpic32.a(vector59.o)

.text%z360      0x00000000        0x0
 .text          0x00000000        0x0 c:/program files/microchip/xc32/v1.33/bin/bin/../../lib/gcc/pic32mx/4.5.2/../../../../pic32mx/lib\libpic32.a(vector58.o)

.text%z361      0x00000000        0x0
 .text          0x00000000        0x0 c:/program files/microchip/xc32/v1.33/bin/bin/../../lib/gcc/pic32mx/4.5.2/../../../../pic32mx/lib\libpic32.a(vector57.o)

.text%z362      0x00000000        0x0
 .text          0x00000000        0x0 c:/program files/microchip/xc32/v1.33/bin/bin/../../lib/gcc/pic32mx/4.5.2/../../../../pic32mx/lib\libpic32.a(vector56.o)

.text%z363      0x00000000        0x0
 .text          0x00000000        0x0 c:/program files/microchip/xc32/v1.33/bin/bin/../../lib/gcc/pic32mx/4.5.2/../../../../pic32mx/lib\libpic32.a(vector55.o)

.text%z364      0x00000000        0x0
 .text          0x00000000        0x0 c:/program files/microchip/xc32/v1.33/bin/bin/../../lib/gcc/pic32mx/4.5.2/../../../../pic32mx/lib\libpic32.a(vector54.o)

.text%z365      0x00000000        0x0
 .text          0x00000000        0x0 c:/program files/microchip/xc32/v1.33/bin/bin/../../lib/gcc/pic32mx/4.5.2/../../../../pic32mx/lib\libpic32.a(vector53.o)

.text%z366      0x00000000        0x0
 .text          0x00000000        0x0 c:/program files/microchip/xc32/v1.33/bin/bin/../../lib/gcc/pic32mx/4.5.2/../../../../pic32mx/lib\libpic32.a(vector52.o)

.text%z367      0x00000000        0x0
 .text          0x00000000        0x0 c:/program files/microchip/xc32/v1.33/bin/bin/../../lib/gcc/pic32mx/4.5.2/../../../../pic32mx/lib\libpic32.a(vector51.o)

.text%z368      0x00000000        0x0
 .text          0x00000000        0x0 c:/program files/microchip/xc32/v1.33/bin/bin/../../lib/gcc/pic32mx/4.5.2/../../../../pic32mx/lib\libpic32.a(vector50.o)

.text%z369      0x00000000        0x0
 .text          0x00000000        0x0 c:/program files/microchip/xc32/v1.33/bin/bin/../../lib/gcc/pic32mx/4.5.2/../../../../pic32mx/lib\libpic32.a(vector49.o)

.text%z370      0x00000000        0x0
 .text          0x00000000        0x0 c:/program files/microchip/xc32/v1.33/bin/bin/../../lib/gcc/pic32mx/4.5.2/../../../../pic32mx/lib\libpic32.a(vector48.o)

.text%z371      0x00000000        0x0
 .text          0x00000000        0x0 c:/program files/microchip/xc32/v1.33/bin/bin/../../lib/gcc/pic32mx/4.5.2/../../../../pic32mx/lib\libpic32.a(vector47.o)

.text%z372      0x00000000        0x0
 .text          0x00000000        0x0 c:/program files/microchip/xc32/v1.33/bin/bin/../../lib/gcc/pic32mx/4.5.2/../../../../pic32mx/lib\libpic32.a(vector46.o)

.text%z373      0x00000000        0x0
 .text          0x00000000        0x0 c:/program files/microchip/xc32/v1.33/bin/bin/../../lib/gcc/pic32mx/4.5.2/../../../../pic32mx/lib\libpic32.a(vector45.o)

.text%z374      0x00000000        0x0
 .text          0x00000000        0x0 c:/program files/microchip/xc32/v1.33/bin/bin/../../lib/gcc/pic32mx/4.5.2/../../../../pic32mx/lib\libpic32.a(vector44.o)

.text%z375      0x00000000        0x0
 .text          0x00000000        0x0 c:/program files/microchip/xc32/v1.33/bin/bin/../../lib/gcc/pic32mx/4.5.2/../../../../pic32mx/lib\libpic32.a(vector43.o)

.text%z376      0x00000000        0x0
 .text          0x00000000        0x0 c:/program files/microchip/xc32/v1.33/bin/bin/../../lib/gcc/pic32mx/4.5.2/../../../../pic32mx/lib\libpic32.a(vector42.o)

.text%z377      0x00000000        0x0
 .text          0x00000000        0x0 c:/program files/microchip/xc32/v1.33/bin/bin/../../lib/gcc/pic32mx/4.5.2/../../../../pic32mx/lib\libpic32.a(vector41.o)

.text%z378      0x00000000        0x0
 .text          0x00000000        0x0 c:/program files/microchip/xc32/v1.33/bin/bin/../../lib/gcc/pic32mx/4.5.2/../../../../pic32mx/lib\libpic32.a(vector40.o)

.text%z379      0x00000000        0x0
 .text          0x00000000        0x0 c:/program files/microchip/xc32/v1.33/bin/bin/../../lib/gcc/pic32mx/4.5.2/../../../../pic32mx/lib\libpic32.a(vector39.o)

.text%z380      0x00000000        0x0
 .text          0x00000000        0x0 c:/program files/microchip/xc32/v1.33/bin/bin/../../lib/gcc/pic32mx/4.5.2/../../../../pic32mx/lib\libpic32.a(vector38.o)

.text%z381      0x00000000        0x0
 .text          0x00000000        0x0 c:/program files/microchip/xc32/v1.33/bin/bin/../../lib/gcc/pic32mx/4.5.2/../../../../pic32mx/lib\libpic32.a(vector37.o)

.text%z382      0x00000000        0x0
 .text          0x00000000        0x0 c:/program files/microchip/xc32/v1.33/bin/bin/../../lib/gcc/pic32mx/4.5.2/../../../../pic32mx/lib\libpic32.a(vector36.o)

.text%z383      0x00000000        0x0
 .text          0x00000000        0x0 c:/program files/microchip/xc32/v1.33/bin/bin/../../lib/gcc/pic32mx/4.5.2/../../../../pic32mx/lib\libpic32.a(vector35.o)

.text%z384      0x00000000        0x0
 .text          0x00000000        0x0 c:/program files/microchip/xc32/v1.33/bin/bin/../../lib/gcc/pic32mx/4.5.2/../../../../pic32mx/lib\libpic32.a(vector34.o)

.text%z385      0x00000000        0x0
 .text          0x00000000        0x0 c:/program files/microchip/xc32/v1.33/bin/bin/../../lib/gcc/pic32mx/4.5.2/../../../../pic32mx/lib\libpic32.a(vector33.o)

.text%z386      0x00000000        0x0
 .text          0x00000000        0x0 c:/program files/microchip/xc32/v1.33/bin/bin/../../lib/gcc/pic32mx/4.5.2/../../../../pic32mx/lib\libpic32.a(vector31.o)

.text%z387      0x00000000        0x0
 .text          0x00000000        0x0 c:/program files/microchip/xc32/v1.33/bin/bin/../../lib/gcc/pic32mx/4.5.2/../../../../pic32mx/lib\libpic32.a(vector30.o)

.text%z388      0x00000000        0x0
 .text          0x00000000        0x0 c:/program files/microchip/xc32/v1.33/bin/bin/../../lib/gcc/pic32mx/4.5.2/../../../../pic32mx/lib\libpic32.a(vector29.o)

.text%z389      0x00000000        0x0
 .text          0x00000000        0x0 c:/program files/microchip/xc32/v1.33/bin/bin/../../lib/gcc/pic32mx/4.5.2/../../../../pic32mx/lib\libpic32.a(vector28.o)

.text%z390      0x00000000        0x0
 .text          0x00000000        0x0 c:/program files/microchip/xc32/v1.33/bin/bin/../../lib/gcc/pic32mx/4.5.2/../../../../pic32mx/lib\libpic32.a(vector27.o)

.text%z391      0x00000000        0x0
 .text          0x00000000        0x0 c:/program files/microchip/xc32/v1.33/bin/bin/../../lib/gcc/pic32mx/4.5.2/../../../../pic32mx/lib\libpic32.a(vector26.o)

.text%z392      0x00000000        0x0
 .text          0x00000000        0x0 c:/program files/microchip/xc32/v1.33/bin/bin/../../lib/gcc/pic32mx/4.5.2/../../../../pic32mx/lib\libpic32.a(vector25.o)

.text%z393      0x00000000        0x0
 .text          0x00000000        0x0 c:/program files/microchip/xc32/v1.33/bin/bin/../../lib/gcc/pic32mx/4.5.2/../../../../pic32mx/lib\libpic32.a(vector23.o)

.text%z394      0x00000000        0x0
 .text          0x00000000        0x0 c:/program files/microchip/xc32/v1.33/bin/bin/../../lib/gcc/pic32mx/4.5.2/../../../../pic32mx/lib\libpic32.a(vector22.o)

.text%z395      0x00000000        0x0
 .text          0x00000000        0x0 c:/program files/microchip/xc32/v1.33/bin/bin/../../lib/gcc/pic32mx/4.5.2/../../../../pic32mx/lib\libpic32.a(vector21.o)

.text%z396      0x00000000        0x0
 .text          0x00000000        0x0 c:/program files/microchip/xc32/v1.33/bin/bin/../../lib/gcc/pic32mx/4.5.2/../../../../pic32mx/lib\libpic32.a(vector20.o)

.text%z397      0x00000000        0x0
 .text          0x00000000        0x0 c:/program files/microchip/xc32/v1.33/bin/bin/../../lib/gcc/pic32mx/4.5.2/../../../../pic32mx/lib\libpic32.a(vector19.o)

.text%z398      0x00000000        0x0
 .text          0x00000000        0x0 c:/program files/microchip/xc32/v1.33/bin/bin/../../lib/gcc/pic32mx/4.5.2/../../../../pic32mx/lib\libpic32.a(vector18.o)

.text%z399      0x00000000        0x0
 .text          0x00000000        0x0 c:/program files/microchip/xc32/v1.33/bin/bin/../../lib/gcc/pic32mx/4.5.2/../../../../pic32mx/lib\libpic32.a(vector17.o)

.text%z400      0x00000000        0x0
 .text          0x00000000        0x0 c:/program files/microchip/xc32/v1.33/bin/bin/../../lib/gcc/pic32mx/4.5.2/../../../../pic32mx/lib\libpic32.a(vector16.o)

.text%z401      0x00000000        0x0
 .text          0x00000000        0x0 c:/program files/microchip/xc32/v1.33/bin/bin/../../lib/gcc/pic32mx/4.5.2/../../../../pic32mx/lib\libpic32.a(vector15.o)

.text%z402      0x00000000        0x0
 .text          0x00000000        0x0 c:/program files/microchip/xc32/v1.33/bin/bin/../../lib/gcc/pic32mx/4.5.2/../../../../pic32mx/lib\libpic32.a(vector14.o)

.text%z403      0x00000000        0x0
 .text          0x00000000        0x0 c:/program files/microchip/xc32/v1.33/bin/bin/../../lib/gcc/pic32mx/4.5.2/../../../../pic32mx/lib\libpic32.a(vector13.o)

.text%z404      0x00000000        0x0
 .text          0x00000000        0x0 c:/program files/microchip/xc32/v1.33/bin/bin/../../lib/gcc/pic32mx/4.5.2/../../../../pic32mx/lib\libpic32.a(vector12.o)

.text%z405      0x00000000        0x0
 .text          0x00000000        0x0 c:/program files/microchip/xc32/v1.33/bin/bin/../../lib/gcc/pic32mx/4.5.2/../../../../pic32mx/lib\libpic32.a(vector11.o)

.text%z406      0x00000000        0x0
 .text          0x00000000        0x0 c:/program files/microchip/xc32/v1.33/bin/bin/../../lib/gcc/pic32mx/4.5.2/../../../../pic32mx/lib\libpic32.a(vector10.o)

.text%z407      0x00000000        0x0
 .text          0x00000000        0x0 c:/program files/microchip/xc32/v1.33/bin/bin/../../lib/gcc/pic32mx/4.5.2/../../../../pic32mx/lib\libpic32.a(vector9.o)

.text%z408      0x00000000        0x0
 .text          0x00000000        0x0 c:/program files/microchip/xc32/v1.33/bin/bin/../../lib/gcc/pic32mx/4.5.2/../../../../pic32mx/lib\libpic32.a(vector8.o)

.text%z409      0x00000000        0x0
 .text          0x00000000        0x0 c:/program files/microchip/xc32/v1.33/bin/bin/../../lib/gcc/pic32mx/4.5.2/../../../../pic32mx/lib\libpic32.a(vector7.o)

.text%z410      0x00000000        0x0
 .text          0x00000000        0x0 c:/program files/microchip/xc32/v1.33/bin/bin/../../lib/gcc/pic32mx/4.5.2/../../../../pic32mx/lib\libpic32.a(vector6.o)

.text%z411      0x00000000        0x0
 .text          0x00000000        0x0 c:/program files/microchip/xc32/v1.33/bin/bin/../../lib/gcc/pic32mx/4.5.2/../../../../pic32mx/lib\libpic32.a(vector5.o)

.text%z412      0x00000000        0x0
 .text          0x00000000        0x0 c:/program files/microchip/xc32/v1.33/bin/bin/../../lib/gcc/pic32mx/4.5.2/../../../../pic32mx/lib\libpic32.a(vector2.o)

.text%z413      0x00000000        0x0
 .text          0x00000000        0x0 c:/program files/microchip/xc32/v1.33/bin/bin/../../lib/gcc/pic32mx/4.5.2/../../../../pic32mx/lib\libpic32.a(vector1.o)

.text%z414      0x00000000        0x0
 .text          0x00000000        0x0 c:/program files/microchip/xc32/v1.33/bin/bin/../../lib/gcc/pic32mx/4.5.2/../../../../pic32mx/lib\libpic32.a(vector0.o)

.text%z415      0x00000000        0x0
 .text          0x00000000        0x0 c:/program files/microchip/xc32/v1.33/bin/bin/../../lib/gcc/pic32mx/4.5.2/../../../../pic32mx/lib\libpic32.a(general-exception.o)

.text%z416      0x00000000        0x0
 .text          0x00000000        0x0 c:/program files/microchip/xc32/v1.33/bin/bin/../../lib/gcc/pic32mx/4.5.2/../../../../pic32mx/lib\libpic32.a(default-on-bootstrap.o)

.text%z417      0x00000000        0x0
 .text          0x00000000        0x0 c:/program files/microchip/xc32/v1.33/bin/bin/../../lib/gcc/pic32mx/4.5.2/../../../../pic32mx/lib\libpic32.a(default-on-reset.o)

.text%z418      0x00000000        0x0
 .text          0x00000000        0x0 c:/program files/microchip/xc32/v1.33/bin/bin/../../lib/gcc/pic32mx/4.5.2/../../../../pic32mx/lib\libpic32.a(default-bootstrap-exception-handler.o)

.text%z419      0x00000000        0x0
 .text          0x00000000        0x0 c:/program files/microchip/xc32/v1.33/bin/bin/../../lib/gcc/pic32mx/4.5.2/../../../../pic32mx/lib\libmchp_peripheral_32MX795F512H.a(int_restore_interrupts_lib.o)

.text%z420      0x00000000        0x0
 .text          0x00000000        0x0 c:/program files/microchip/xc32/v1.33/bin/bin/../../lib/gcc/pic32mx/4.5.2/../../../../pic32mx/lib\libmchp_peripheral_32MX795F512H.a(int_disable_interrupts_lib.o)

.text%z421      0x00000000        0x0
 .text          0x00000000        0x0 c:/program files/microchip/xc32/v1.33/bin/bin/../../lib/gcc/pic32mx/4.5.2/../../../../pic32mx/lib\libmchp_peripheral_32MX795F512H.a(int_enable_interrupts_lib.o)

.text%z422      0x00000000        0x0
 .text          0x00000000        0x0 c:/program files/microchip/xc32/v1.33/bin/bin/../../lib/gcc/pic32mx/4.5.2/../../../../pic32mx/lib\libmchp_peripheral_32MX795F512H.a(int_configure_system_lib.o)

.text%z423      0x00000000        0x0
 .text          0x00000000        0x0 c:/program files/microchip/xc32/v1.33/bin/bin/../../lib/gcc/pic32mx/4.5.2/../../../../pic32mx/lib\libmchp_peripheral_32MX795F512H.a(pcache.o)

.text%z424      0x00000000        0x0
 .text          0x00000000        0x0 c:/program files/microchip/xc32/v1.33/bin/bin/../../lib/gcc/pic32mx/4.5.2/../../../../pic32mx/lib\libmchp_peripheral_32MX795F512H.a(soft_reset_lib.o)

.text%z425      0x00000000        0x0
 .text          0x00000000        0x0 c:/program files/microchip/xc32/v1.33/bin/bin/../../lib/gcc/pic32mx/4.5.2/../../../../pic32mx/lib/./proc/32MX795F512H\processor.o

.text%z426      0x00000000        0x0
 .text          0x00000000        0x0 c:/program files/microchip/xc32/v1.33/bin/bin/../../lib/gcc/pic32mx/4.5.2/../../../../pic32mx/lib/./proc/32MX795F512H\default_isr_vectors.o

.text%z427      0x00000000        0x0
 .text          0x00000000        0x0 build/ChaletDuinoV2_775F512H_/debug/Source/template.o

.text%z428      0x00000000        0x0
 .text          0x00000000        0x0 build/ChaletDuinoV2_775F512H_/debug/Source/system.o

.text%z429      0x00000000        0x0
 .text          0x00000000        0x0 build/ChaletDuinoV2_775F512H_/debug/Source/interrupts.o

.text%z430      0x00000000        0x0
 .text          0x00000000        0x0 build/ChaletDuinoV2_775F512H_/debug/Source/winc3400/driver/source/nmuart.o

.text%z431      0x00000000        0x0
 .text          0x00000000        0x0 build/ChaletDuinoV2_775F512H_/debug/Source/winc3400/driver/source/nmi2c.o

.text%z432      0x00000000        0x0
 .text          0x00000000        0x0 build/ChaletDuinoV2_775F512H_/debug/Source/winc3400/driver/source/m2m_crypto.o

.text%z433      0x00000000        0x0
 .text          0x00000000        0x0 build/ChaletDuinoV2_775F512H_/debug/Source/winc3400/driver/source/m2m_ate_mode.o

.text%z434      0x00000000        0x0
 .text          0x00000000        0x0 c:/program files/microchip/xc32/v1.33/bin/bin/../../lib/gcc/pic32mx/4.5.2/../../../../pic32mx/lib\software-debug-break.o

.text%z435      0x00000000        0x0
 .text          0x00000000        0x0 c:/program files/microchip/xc32/v1.33/bin/bin/../../lib/gcc/pic32mx/4.5.2/../../../../pic32mx/lib/./proc/32MX795F512H/crt0_mips32r2.o
